Archive member included because of file (symbol)

c:/program files/microchip/mplabc32/v2.02/bin/../lib/gcc/pic32mx/4.5.1/speed\libgcc.a(_udivdi3.o)
                              output\FSIO.o (__udivdi3)
c:/program files/microchip/mplabc32/v2.02/bin/../lib/gcc/pic32mx/4.5.1/speed\libgcc.a(_umoddi3.o)
                              output\FSIO.o (__umoddi3)
c:/program files/microchip/mplabc32/v2.02/bin/../lib/gcc/pic32mx/4.5.1/speed\libgcc.a(floatunsisf.o)
                              output\DstaDPlusClientUDP.o (__floatunsisf)
c:/program files/microchip/mplabc32/v2.02/bin/../lib/gcc/pic32mx/4.5.1/../../../../pic32mx/lib/speed\libc.a(memcmp.o)
                              output\prvTaskTCPIP.o (memcmp)
c:/program files/microchip/mplabc32/v2.02/bin/../lib/gcc/pic32mx/4.5.1/../../../../pic32mx/lib/speed\libc.a(memcpy.o)
                              output\main.o (memcpy)
c:/program files/microchip/mplabc32/v2.02/bin/../lib/gcc/pic32mx/4.5.1/../../../../pic32mx/lib/speed\libc.a(memset.o)
                              output\main.o (memset)
c:/program files/microchip/mplabc32/v2.02/bin/../lib/gcc/pic32mx/4.5.1/../../../../pic32mx/lib/speed\libc.a(strcmp.o)
                              output\CustomHTTPApp.o (strcmp)
c:/program files/microchip/mplabc32/v2.02/bin/../lib/gcc/pic32mx/4.5.1/../../../../pic32mx/lib/speed\libc.a(strcpy.o)
                              output\FSIO.o (strcpy)
c:/program files/microchip/mplabc32/v2.02/bin/../lib/gcc/pic32mx/4.5.1/../../../../pic32mx/lib/speed\libc.a(strlen.o)
                              output\prvTaskTCPIP.o (strlen)
c:/program files/microchip/mplabc32/v2.02/bin/../lib/gcc/pic32mx/4.5.1/../../../../pic32mx/lib/speed\libc.a(general-exception.o)
                              c:/program files/microchip/mplabc32/v2.02/bin/../lib/gcc/pic32mx/4.5.1/../../../../pic32mx/lib/speed/crt0.o (_general_exception_context)
c:/program files/microchip/mplabc32/v2.02/bin/../lib/gcc/pic32mx/4.5.1/../../../../pic32mx/lib/speed\libc.a(atoi.o)
                              output\CustomHTTPApp.o (atoi)
c:/program files/microchip/mplabc32/v2.02/bin/../lib/gcc/pic32mx/4.5.1/../../../../pic32mx/lib/speed\libc.a(atol.o)
                              output\DstaDPlusClientUDP.o (atol)
c:/program files/microchip/mplabc32/v2.02/bin/../lib/gcc/pic32mx/4.5.1/../../../../pic32mx/lib/speed\libc.a(ctime.o)
                              output\SNTP.o (localtime)
c:/program files/microchip/mplabc32/v2.02/bin/../lib/gcc/pic32mx/4.5.1/../../../../pic32mx/lib/speed\libc.a(ctype.o)
                              output\FSIO.o (_ctype)
c:/program files/microchip/mplabc32/v2.02/bin/../lib/gcc/pic32mx/4.5.1/../../../../pic32mx/lib/speed\libc.a(ctypef.o)
                              output\FSIO.o (tolower)
c:/program files/microchip/mplabc32/v2.02/bin/../lib/gcc/pic32mx/4.5.1/../../../../pic32mx/lib/speed\libc.a(strcat.o)
                              output\FTP.o (strcat)
c:/program files/microchip/mplabc32/v2.02/bin/../lib/gcc/pic32mx/4.5.1/../../../../pic32mx/lib/speed\libc.a(strchr.o)
                              output\DstaDPlusClientUDP.o (strchr)
c:/program files/microchip/mplabc32/v2.02/bin/../lib/gcc/pic32mx/4.5.1/../../../../pic32mx/lib/speed\libc.a(strncpy.o)
                              output\tasks.o (strncpy)
c:/program files/microchip/mplabc32/v2.02/bin/../lib/gcc/pic32mx/4.5.1/../../../../pic32mx/lib/speed\libc.a(strstr.o)
                              output\DstaDPlusClientUDP.o (strstr)
c:/program files/microchip/mplabc32/v2.02/bin/../lib/gcc/pic32mx/4.5.1/../../../../pic32mx/lib/speed\libc.a(atof.o)
                              output\CustomHTTPApp.o (atof)
c:/program files/microchip/mplabc32/v2.02/bin/../lib/gcc/pic32mx/4.5.1/../../../../pic32mx/lib/speed\libc.a(sprintf_cdnopsuxX.eo)
                              output\CustomHTTPApp.o (_sprintf_cdnopsuxX)
c:/program files/microchip/mplabc32/v2.02/bin/../lib/gcc/pic32mx/4.5.1/../../../../pic32mx/lib/speed\libc.a(sprintf_cdnopuxX.eo)
                              output\FTP.o (_sprintf_cdnopuxX)
c:/program files/microchip/mplabc32/v2.02/bin/../lib/gcc/pic32mx/4.5.1/../../../../pic32mx/lib/speed\libc.a(sprintf_s.eo)
                              output\main.o (_sprintf_s)
c:/program files/microchip/mplabc32/v2.02/bin/../lib/gcc/pic32mx/4.5.1/../../../../pic32mx/lib/speed\libc.a(default-bootstrap-exception-handler.o)
                              c:/program files/microchip/mplabc32/v2.02/bin/../lib/gcc/pic32mx/4.5.1/../../../../pic32mx/lib/speed/crt0.o (_bootstrap_exception_handler)
c:/program files/microchip/mplabc32/v2.02/bin/../lib/gcc/pic32mx/4.5.1/../../../../pic32mx/lib/speed\libc.a(default-on-reset.o)
                              c:/program files/microchip/mplabc32/v2.02/bin/../lib/gcc/pic32mx/4.5.1/../../../../pic32mx/lib/speed/crt0.o (_on_reset)
c:/program files/microchip/mplabc32/v2.02/bin/../lib/gcc/pic32mx/4.5.1/../../../../pic32mx/lib/speed\libc.a(default-on-bootstrap.o)
                              c:/program files/microchip/mplabc32/v2.02/bin/../lib/gcc/pic32mx/4.5.1/../../../../pic32mx/lib/speed/crt0.o (_on_bootstrap)
c:/program files/microchip/mplabc32/v2.02/bin/../lib/gcc/pic32mx/4.5.1/../../../../pic32mx/lib/speed\libc.a(default-nmi-handler.o)
                              c:/program files/microchip/mplabc32/v2.02/bin/../lib/gcc/pic32mx/4.5.1/../../../../pic32mx/lib/speed/crt0.o (_nmi_handler)
c:/program files/microchip/mplabc32/v2.02/bin/../lib/gcc/pic32mx/4.5.1/../../../../pic32mx/lib/speed\libc.a(strncmp.o)
                              c:/program files/microchip/mplabc32/v2.02/bin/../lib/gcc/pic32mx/4.5.1/../../../../pic32mx/lib/speed\libc.a(strstr.o) (strncmp)
c:/program files/microchip/mplabc32/v2.02/bin/../lib/gcc/pic32mx/4.5.1/../../../../pic32mx/lib/speed\libc.a(strtod.o)
                              c:/program files/microchip/mplabc32/v2.02/bin/../lib/gcc/pic32mx/4.5.1/../../../../pic32mx/lib/speed\libc.a(atof.o) (_dstrtod)
c:/program files/microchip/mplabc32/v2.02/bin/../lib/gcc/pic32mx/4.5.1/../../../../pic32mx/lib/speed\libc.a(doprnt_cdnopsuxX.eo)
                              c:/program files/microchip/mplabc32/v2.02/bin/../lib/gcc/pic32mx/4.5.1/../../../../pic32mx/lib/speed\libc.a(sprintf_cdnopsuxX.eo) (_vfprintf_cdnopsuxX)
c:/program files/microchip/mplabc32/v2.02/bin/../lib/gcc/pic32mx/4.5.1/../../../../pic32mx/lib/speed\libc.a(doprnt_cdnopuxX.eo)
                              c:/program files/microchip/mplabc32/v2.02/bin/../lib/gcc/pic32mx/4.5.1/../../../../pic32mx/lib/speed\libc.a(sprintf_cdnopuxX.eo) (_vfprintf_cdnopuxX)
c:/program files/microchip/mplabc32/v2.02/bin/../lib/gcc/pic32mx/4.5.1/../../../../pic32mx/lib/speed\libc.a(doprnt_s.eo)
                              c:/program files/microchip/mplabc32/v2.02/bin/../lib/gcc/pic32mx/4.5.1/../../../../pic32mx/lib/speed\libc.a(sprintf_s.eo) (_vfprintf_s)
c:/program files/microchip/mplabc32/v2.02/bin/../lib/gcc/pic32mx/4.5.1/../../../../pic32mx/lib/speed\libc.a(_fputc_simple.o)
                              c:/program files/microchip/mplabc32/v2.02/bin/../lib/gcc/pic32mx/4.5.1/../../../../pic32mx/lib/speed\libc.a(doprnt_cdnopsuxX.eo) (fputc)
c:/program files/microchip/mplabc32/v2.02/bin/../lib/gcc/pic32mx/4.5.1/../../../../pic32mx/lib/speed\libc.a(write.o)
                              c:/program files/microchip/mplabc32/v2.02/bin/../lib/gcc/pic32mx/4.5.1/../../../../pic32mx/lib/speed\libc.a(_fputc_simple.o) (write)
c:/program files/microchip/mplabc32/v2.02/bin/../lib/gcc/pic32mx/4.5.1/../../../../pic32mx/lib/speed\libc.a(_iob.o)
                              c:/program files/microchip/mplabc32/v2.02/bin/../lib/gcc/pic32mx/4.5.1/../../../../pic32mx/lib/speed\libc.a(_fputc_simple.o) (_outdone)
c:/program files/microchip/mplabc32/v2.02/bin/../lib/gcc/pic32mx/4.5.1/../../../../pic32mx/lib/speed\libc.a(_flsbuf_simple.o)
                              c:/program files/microchip/mplabc32/v2.02/bin/../lib/gcc/pic32mx/4.5.1/../../../../pic32mx/lib/speed\libc.a(_fputc_simple.o) (_flsbuf)
c:/program files/microchip/mplabc32/v2.02/bin/../lib/gcc/pic32mx/4.5.1/../../../../pic32mx/lib/speed\libc.a(_mon_putc.o)
                              c:/program files/microchip/mplabc32/v2.02/bin/../lib/gcc/pic32mx/4.5.1/../../../../pic32mx/lib/speed\libc.a(write.o) (_mon_putc)
c:/program files/microchip/mplabc32/v2.02/bin/../lib/gcc/pic32mx/4.5.1/../../../../pic32mx/lib/speed\libc.a(c32_uart.o)
                              c:/program files/microchip/mplabc32/v2.02/bin/../lib/gcc/pic32mx/4.5.1/../../../../pic32mx/lib/speed\libc.a(_mon_putc.o) (__C32_UART)
c:/program files/microchip/mplabc32/v2.02/bin/../lib/gcc/pic32mx/4.5.1/../../../../pic32mx/lib/speed\libm.a(dp32.o)
                              c:/program files/microchip/mplabc32/v2.02/bin/../lib/gcc/pic32mx/4.5.1/../../../../pic32mx/lib/speed\libc.a(atof.o) (dptofp)
c:/program files/microchip/mplabc32/v2.02/bin/../lib/gcc/pic32mx/4.5.1/../../../../pic32mx/lib/speed\libm.a(fp32.o)
                              output\serial.o (fpsub)
c:/program files/microchip/mplabc32/v2.02/bin/../lib/gcc/pic32mx/4.5.1/../../../../pic32mx/lib/speed\libe.a(_strtod.o)
                              c:/program files/microchip/mplabc32/v2.02/bin/../lib/gcc/pic32mx/4.5.1/../../../../pic32mx/lib/speed\libc.a(strtod.o) (__strtod)
c:/program files/microchip/mplabc32/v2.02/bin/../lib/gcc/pic32mx/4.5.1/../../../../pic32mx/lib/speed\libe.a(_ldexp.o)
                              c:/program files/microchip/mplabc32/v2.02/bin/../lib/gcc/pic32mx/4.5.1/../../../../pic32mx/lib/speed\libe.a(_strtod.o) (__ldexp)
c:/program files/microchip/mplabc32/v2.02/bin/../lib/gcc/pic32mx/4.5.1/../../../../pic32mx/lib/speed\libmchp_peripheral.a(read_core_timer_lib.o)
                              output\CustomHTTPApp.o (ReadCoreTimer)
c:/program files/microchip/mplabc32/v2.02/bin/../lib/gcc/pic32mx/4.5.1/../../../../pic32mx/lib/speed\libmchp_peripheral.a(write_core_timer_lib.o)
                              output\CustomHTTPApp.o (WriteCoreTimer)
c:/program files/microchip/mplabc32/v2.02/bin/../lib/gcc/pic32mx/4.5.1/../../../../pic32mx/lib/speed\libmchp_peripheral_32MX795F512L.a(eth_ack_packet_lib.o)
                              output\ETHPIC32IntMac.o (EthRxAcknowledgeBuffer)
c:/program files/microchip/mplabc32/v2.02/bin/../lib/gcc/pic32mx/4.5.1/../../../../pic32mx/lib/speed\libmchp_peripheral_32MX795F512L.a(eth_descriptors_add_lib.o)
                              output\ETHPIC32IntMac.o (EthDescriptorsPoolAdd)
c:/program files/microchip/mplabc32/v2.02/bin/../lib/gcc/pic32mx/4.5.1/../../../../pic32mx/lib/speed\libmchp_peripheral_32MX795F512L.a(eth_init_lib.o)
                              output\ETHPIC32IntMac.o (EthInit)
c:/program files/microchip/mplabc32/v2.02/bin/../lib/gcc/pic32mx/4.5.1/../../../../pic32mx/lib/speed\libmchp_peripheral_32MX795F512L.a(eth_mac_open_lib.o)
                              output\ETHPIC32IntMac.o (EthMACOpen)
c:/program files/microchip/mplabc32/v2.02/bin/../lib/gcc/pic32mx/4.5.1/../../../../pic32mx/lib/speed\libmchp_peripheral_32MX795F512L.a(eth_mac_set_address_max_lib.o)
                              output\ETHPIC32IntMac.o (EthMACSetAddress)
c:/program files/microchip/mplabc32/v2.02/bin/../lib/gcc/pic32mx/4.5.1/../../../../pic32mx/lib/speed\libmchp_peripheral_32MX795F512L.a(eth_rx_buffers_append_lib.o)
                              output\ETHPIC32IntMac.o (EthRxBuffersAppend)
c:/program files/microchip/mplabc32/v2.02/bin/../lib/gcc/pic32mx/4.5.1/../../../../pic32mx/lib/speed\libmchp_peripheral_32MX795F512L.a(eth_rx_filters_lib.o)
                              output\ETHPIC32IntMac.o (EthRxFiltersSet)
c:/program files/microchip/mplabc32/v2.02/bin/../lib/gcc/pic32mx/4.5.1/../../../../pic32mx/lib/speed\libmchp_peripheral_32MX795F512L.a(eth_rx_get_packet_lib.o)
                              output\ETHPIC32IntMac.o (EthRxGetBuffer)
c:/program files/microchip/mplabc32/v2.02/bin/../lib/gcc/pic32mx/4.5.1/../../../../pic32mx/lib/speed\libmchp_peripheral_32MX795F512L.a(eth_rx_set_buffer_size_lib.o)
                              output\ETHPIC32IntMac.o (EthRxSetBufferSize)
c:/program files/microchip/mplabc32/v2.02/bin/../lib/gcc/pic32mx/4.5.1/../../../../pic32mx/lib/speed\libmchp_peripheral_32MX795F512L.a(eth_tx_packet_lib.o)
                              output\ETHPIC32IntMac.o (EthTxSendBuffer)
c:/program files/microchip/mplabc32/v2.02/bin/../lib/gcc/pic32mx/4.5.1/../../../../pic32mx/lib/speed\libmchp_peripheral_32MX795F512L.a(_eth_append_busy_list_lib.o)
                              c:/program files/microchip/mplabc32/v2.02/bin/../lib/gcc/pic32mx/4.5.1/../../../../pic32mx/lib/speed\libmchp_peripheral_32MX795F512L.a(eth_ack_packet_lib.o) (_EthAppendBusyList)
c:/program files/microchip/mplabc32/v2.02/bin/../lib/gcc/pic32mx/4.5.1/../../../../pic32mx/lib/speed\libmchp_peripheral_32MX795F512L.a(eth_miim_access.o)
                              output\ETHPIC32ExtPhy.o (EthMIIMReadStart)
c:/program files/microchip/mplabc32/v2.02/bin/../lib/gcc/pic32mx/4.5.1/../../../../pic32mx/lib/speed\libmchp_peripheral_32MX795F512L.a(soft_reset_lib.o)
                              output\prvTaskTCPIP.o (SoftReset)
c:/program files/microchip/mplabc32/v2.02/bin/../lib/gcc/pic32mx/4.5.1/../../../../pic32mx/lib/speed\libmchp_peripheral_32MX795F512L.a(pcache.o)
                              output\main.o (CheKseg0CacheOn)
c:/program files/microchip/mplabc32/v2.02/bin/../lib/gcc/pic32mx/4.5.1/../../../../pic32mx/lib/speed\libmchp_peripheral_32MX795F512L.a(set_core_sw0_leg_lib.o)
                              output\port.o (SetCoreSW0)
c:/program files/microchip/mplabc32/v2.02/bin/../lib/gcc/pic32mx/4.5.1/../../../../pic32mx/lib/speed\libmchp_peripheral_32MX795F512L.a(int_disable_interrupts_lib.o)
                              output\main.o (INTDisableInterrupts)
c:/program files/microchip/mplabc32/v2.02/bin/../lib/gcc/pic32mx/4.5.1/../../../../pic32mx/lib/speed\libmchp_peripheral_32MX795F512L.a(int_restore_interrupts_lib.o)
                              output\main.o (INTRestoreInterrupts)
c:/program files/microchip/mplabc32/v2.02/bin/../lib/gcc/pic32mx/4.5.1/../../../../pic32mx/lib/speed\libmchp_peripheral_32MX795F512L.a(int_enable_mv_int_lib.o)
                              output\main.o (INTEnableSystemMultiVectoredInt)
c:/program files/microchip/mplabc32/v2.02/bin/../lib/gcc/pic32mx/4.5.1/../../../../pic32mx/lib/speed\libmchp_peripheral_32MX795F512L.a(int_tbl_lib.o)
                              c:/program files/microchip/mplabc32/v2.02/bin/../lib/gcc/pic32mx/4.5.1/../../../../pic32mx/lib/speed\libmchp_peripheral_32MX795F512L.a(eth_init_lib.o) (INTClearFlag)
c:/program files/microchip/mplabc32/v2.02/bin/../lib/gcc/pic32mx/4.5.1/../../../../pic32mx/lib/speed\libmchp_peripheral_32MX795F512L.a(rtcc_init_lib.o)
                              output\main.o (RtccInit)
c:/program files/microchip/mplabc32/v2.02/bin/../lib/gcc/pic32mx/4.5.1/../../../../pic32mx/lib/speed\libmchp_peripheral_32MX795F512L.a(rtcc_set_time_date_lib.o)
                              output\SNTP.o (RtccSetTimeDate)
c:/program files/microchip/mplabc32/v2.02/bin/../lib/gcc/pic32mx/4.5.1/../../../../pic32mx/lib/speed\libmchp_peripheral_32MX795F512L.a(rtcc_open_lib.o)
                              output\main.o (RtccOpen)
c:/program files/microchip/mplabc32/v2.02/bin/../lib/gcc/pic32mx/4.5.1/../../../../pic32mx/lib/speed\libmchp_peripheral_32MX795F512L.a(spi_getc_spi1_lib_legacy.o)
                              output\SD-SPI.o (getcSPI1)
c:/program files/microchip/mplabc32/v2.02/bin/../lib/gcc/pic32mx/4.5.1/../../../../pic32mx/lib/speed\libmchp_peripheral_32MX795F512L.a(spi_open_spi1_lib_legacy.o)
                              output\SD-SPI.o (OpenSPI1)
c:/program files/microchip/mplabc32/v2.02/bin/../lib/gcc/pic32mx/4.5.1/../../../../pic32mx/lib/speed\libmchp_peripheral_32MX795F512L.a(spi_brg_tbl_lib_legacy.o)
                              c:/program files/microchip/mplabc32/v2.02/bin/../lib/gcc/pic32mx/4.5.1/../../../../pic32mx/lib/speed\libmchp_peripheral_32MX795F512L.a(spi_open_spi1_lib_legacy.o) (_SpiBrgConvTbl)
c:/program files/microchip/mplabc32/v2.02/bin/../lib/gcc/pic32mx/4.5.1/../../../../pic32mx/lib/speed\libmchp_peripheral_32MX795F512L.a(port_set_pins_digital_in_lib.o)
                              output\ETHPIC32ExtPhy.o (PORTSetPinsDigitalIn)
c:/program files/microchip/mplabc32/v2.02/bin/../lib/gcc/pic32mx/4.5.1/../../../../pic32mx/lib/speed\libmchp_peripheral_32MX795F512L.a(port_set_pins_digital_out_lib.o)
                              output\ETHPIC32ExtPhy.o (PORTSetPinsDigitalOut)
c:/program files/microchip/mplabc32/v2.02/bin/../lib/gcc/pic32mx/4.5.1/../../../../pic32mx/lib/speed\libmchp_peripheral_32MX795F512L.a(_ports_tbl_libp.o)
                              c:/program files/microchip/mplabc32/v2.02/bin/../lib/gcc/pic32mx/4.5.1/../../../../pic32mx/lib/speed\libmchp_peripheral_32MX795F512L.a(port_set_pins_digital_in_lib.o) (PortRegTbl)
c:/program files/microchip/mplabc32/v2.02/bin/../lib/gcc/pic32mx/4.5.1/../../../../pic32mx/lib/speed\libmchp_peripheral_32MX795F512L.a(int_enable_interrupts_lib.o)
                              c:/program files/microchip/mplabc32/v2.02/bin/../lib/gcc/pic32mx/4.5.1/../../../../pic32mx/lib/speed\libmchp_peripheral_32MX795F512L.a(int_enable_mv_int_lib.o) (INTEnableInterrupts)
c:/program files/microchip/mplabc32/v2.02/bin/../lib/gcc/pic32mx/4.5.1/../../../../pic32mx/lib/speed\libmchp_peripheral_32MX795F512L.a(_rtcc_set_time_and_date_lib.o)
                              c:/program files/microchip/mplabc32/v2.02/bin/../lib/gcc/pic32mx/4.5.1/../../../../pic32mx/lib/speed\libmchp_peripheral_32MX795F512L.a(rtcc_set_time_date_lib.o) (_RtccSetTimeAndDate)
c:/program files/microchip/mplabc32/v2.02/bin/../lib/gcc/pic32mx/4.5.1/../../../../pic32mx/lib/speed\libmchp_peripheral_32MX795F512L.a(_rtcc_wait_clock_off_lib.o)
                              c:/program files/microchip/mplabc32/v2.02/bin/../lib/gcc/pic32mx/4.5.1/../../../../pic32mx/lib/speed\libmchp_peripheral_32MX795F512L.a(rtcc_init_lib.o) (_RtccWaitClockOff)
c:/program files/microchip/mplabc32/v2.02/bin/../lib/gcc/pic32mx/4.5.1/../../../../pic32mx/lib/speed\libc.a(calloc.o)
                              c:/program files/microchip/mplabc32/v2.02/bin/../lib/gcc/pic32mx/4.5.1/../../../../pic32mx/lib/speed\libmchp_peripheral_32MX795F512L.a(eth_descriptors_add_lib.o) (calloc)
c:/program files/microchip/mplabc32/v2.02/bin/../lib/gcc/pic32mx/4.5.1/../../../../pic32mx/lib/speed\libc.a(errno.o)
                              c:/program files/microchip/mplabc32/v2.02/bin/../lib/gcc/pic32mx/4.5.1/../../../../pic32mx/lib/speed\libe.a(_strtod.o) (errno)
c:/program files/microchip/mplabc32/v2.02/bin/../lib/gcc/pic32mx/4.5.1/../../../../pic32mx/lib/speed\libc.a(malloc.o)
                              c:/program files/microchip/mplabc32/v2.02/bin/../lib/gcc/pic32mx/4.5.1/../../../../pic32mx/lib/speed\libc.a(calloc.o) (malloc)
c:/program files/microchip/mplabc32/v2.02/bin/../lib/gcc/pic32mx/4.5.1/../../../../pic32mx/lib/speed\libc.a(sbrk.o)
                              c:/program files/microchip/mplabc32/v2.02/bin/../lib/gcc/pic32mx/4.5.1/../../../../pic32mx/lib/speed\libc.a(malloc.o) (sbrk)
c:/program files/microchip/mplabc32/v2.02/bin/../lib/gcc/pic32mx/4.5.1/speed\libgcc.a(_lshrdi3.o)
                              c:/program files/microchip/mplabc32/v2.02/bin/../lib/gcc/pic32mx/4.5.1/../../../../pic32mx/lib/speed\libe.a(_ldexp.o) (__lshrdi3)
c:/program files/microchip/mplabc32/v2.02/bin/../lib/gcc/pic32mx/4.5.1/speed\libgcc.a(_ashldi3.o)
                              c:/program files/microchip/mplabc32/v2.02/bin/../lib/gcc/pic32mx/4.5.1/../../../../pic32mx/lib/speed\libe.a(_ldexp.o) (__ashldi3)

Allocating common symbols
Common symbol       size              file

AdParam             0x4e              output\main.o
Radio_GPS_A_Msg_send
                    0x4               output\DstaDPlusClientUDP.o
xHighestPriorityTask
                    0x4               output\QPeek.o
SSN                 0x2               output\main.o
tempCWDobj          0x44              output\FSIO.o
header              0x29              output\main.o
gMediaSectorSize    0x2               output\SD-SPI.o
RadioSpeed          0x3               output\DstaDPlusClientUDP.o
RadioLong           0x9               output\DstaDPlusClientUDP.o
gSDMode             0x1               output\SD-SPI.o
RadioDprsSend       0x4               output\DstaDPlusClientUDP.o
xDstarHttpQueue     0x4               output\main.o
xMessage            0x8               output\main.o
VoiceMsg            0x4               output\prvTaskUSB.o
activeUDPSocket     0x1               output\UDP.o
Text                0x20              output\main.o
utf16Filename       0x4               output\FSIO.o
MACReadWriteSW      0x1               output\MACread.o
curHTTP             0x8c              output\HTTP2.o
Msg                 0x1               output\DstaDPlusClientUDP.o
MDD_SDSPI_finalLBA  0x4               output\SD-SPI.o
CurUser             0x8               output\CustomHTTPApp.o
recordSearchLength  0x2               output\FSIO.o
AprsSeq             0x4               output\CustomHTTPApp.o
DPRS                0x94              output\main.o
MyCallSign          0x8               output\DstaDPlusClientUDP.o
TempClusterCalc     0x4               output\FSIO.o
COS_On              0x4               output\main.o
LCDHandle           0x4               output\lcd.o
gTimeCrtTime        0x2               output\FSIO.o
AprsMsgTX           0x3               output\DstaDPlusClientUDP.o
xHighPriorityNormallyFullTask2
                    0x4               output\IntQueue.o
rig_buffer          0x20              output\main.o
UDPTxCount          0x2               output\UDP.o
SMTPClient          0x2c              output\SMTP.o
PTT_On              0x4               output\main.o
xDstarDprsMsgQueue  0x4               output\main.o
FWUpdate            0x4               output\main.o
DprsMsgDstCallSign  0xa               output\prvTaskFS.o
deviceAddress       0x1               output\DstaDPlusClientUDP.o
fileFoundString     0x20a             output\FSIO.o
PicVer              0x2               output\main.o
ReqRefList          0x4               output\CustomHTTPApp.o
lfnData             0x606             output\FSIO.o
xDstarDprsEmailMsgQueue
                    0x4               output\main.o
gFileSlotOpen       0x3               output\FSIO.o
xDstarRcvQueue      0x4               output\main.o
RefSkipSW           0x1               output\DstaDPlusClientUDP.o
EmailAddress        0x30              output\DstaDPlusClientUDP.o
curHTTPID           0x1               output\HTTP2.o
xHighPriorityNormallyEmptyTask1
                    0x4               output\IntQueue.o
REF_IP_address      0x10              output\CustomHTTPApp.o
gDiskData           0x26              output\FSIO.o
xDstarDprsAccQueue  0x4               output\main.o
AprsDest            0x9               output\CustomHTTPApp.o
xHighPriorityTask   0x4               output\QPeek.o
gFATBuffer          0x200             output\FSIO.o
newAppConfig        0xa8              output\CustomHTTPApp.o
xDstarAccQueue      0x4               output\main.o
gc_DevData          0x10              output\usb_host_generic.o
InetDirection       0x3               output\DstaDPlusClientUDP.o
cwd                 0x44              output\FSIO.o
gTimeAccDate        0x2               output\FSIO.o
RadioAtitude        0x6               output\DstaDPlusClientUDP.o
xDstarLogQueue      0x4               output\main.o
TimeDate            0x14              output\main.o
voice_pnt           0x2               output\main.o
left_byte           0x2               output\main.o
gTimeCrtDate        0x2               output\FSIO.o
xMediumPriorityTask
                    0x4               output\QPeek.o
InetAtitude         0x6               output\DstaDPlusClientUDP.o
AccessFileReadSW    0x4               output\main.o
KeepAliveTimer      0x4               output\DstaDPlusClientUDP.o
_PhyAdd             0x4               output\ETHPIC32ExtPhy.o
asciiFilename       0x4               output\FSIO.o
xHighPriorityNormallyEmptyTask2
                    0x4               output\IntQueue.o
FSHandle            0x4               output\main.o
ReqConvertLocalRefFile
                    0x4               output\main.o
USBHandle           0x4               output\main.o
RadioCall           0x8               output\DstaDPlusClientUDP.o
InetCall            0x8               output\DstaDPlusClientUDP.o
ReqRefDomainName    0x4               output\main.o
FSerrno             0x1               output\FSIO.o
RefNameSet          0x1               output\DstaDPlusClientUDP.o
Inet_GPS_A_Msg_send
                    0x4               output\DstaDPlusClientUDP.o
gDataBuffer         0x200             output\FSIO.o
FirstTable          0x14              output\DstaDPlusClientUDP.o
fileNameLength      0x2               output\FSIO.o
InetLong            0x9               output\DstaDPlusClientUDP.o
dirCleared          0x1               output\FSIO.o
UDPSocketInfo       0x280             output\UDP.o
xDstarRefQueue      0x4               output\main.o
gTimeWrtTime        0x2               output\FSIO.o
EmailTemp           0x8a              output\DprsSMTP.o
InetSpeed           0x3               output\DstaDPlusClientUDP.o
recordFoundName     0x202             output\FSIO.o
Radio_Callsign_Check_String
                    0x9               output\prvTaskFS.o
RDateTime           0xa               output\DstaDPlusClientUDP.o
remoteNode          0xa               output\StackTsk.o
Radio_GPS_A_MSG     0x78              output\DstaDPlusClientUDP.o
RefNameTemp         0x8               output\DstaDPlusClientUDP.o
xLCDQueue           0x4               output\lcd.o
MyMACAddr           0x6               output\main.o
gFileArray          0xcc              output\FSIO.o
xDstarSndQueue      0x4               output\main.o
DprsMyCall          0x9               output\prvTaskUSB.o
recordSearchName    0x202             output\FSIO.o
FSInitSW            0x4               output\main.o
InetLat             0x8               output\DstaDPlusClientUDP.o
DPRS_SW             0x1               output\main.o
UDPRxCount          0x2               output\UDP.o
Inet_GPS_A_MSG      0x78              output\DstaDPlusClientUDP.o
AprsSenderCall      0xa               output\CustomHTTPApp.o
RadioMsg            0x14              output\DstaDPlusClientUDP.o
headerRead          0x4               output\prvTaskUSB.o
TCPHandle           0x4               output\main.o
FatRootDirClusterValue
                    0x4               output\FSIO.o
httpStubs           0x8               output\HTTP2.o
gTimeCrtMS          0x1               output\FSIO.o
RadioDirection      0x3               output\DstaDPlusClientUDP.o
ReqLoadAprsCallCheck
                    0x4               output\prvTaskFS.o
gFileTemp           0x44              output\FSIO.o
CurServerName       0x14              output\DstaDPlusClientUDP.o
DprsMsgDstCallSignSave
                    0x9               output\DstaDPlusClientUDP.o
RefDomainName       0x6e              output\DstaDPlusClientUDP.o
tempDirectoryString
                    0x20a             output\FSIO.o
DprsMsgSrcCallSign  0xa               output\prvTaskFS.o
RadioLat            0x8               output\DstaDPlusClientUDP.o
AppConfig           0xa8              output\main.o
InetMsg             0x14              output\DstaDPlusClientUDP.o
defaultArray        0xa               output\FSIO.o
CallCheck_Skip      0x4               output\prvTaskFS.o
gTimeWrtDate        0x2               output\FSIO.o
AprsMessage         0x46              output\CustomHTTPApp.o
Inet_Callsign_Check_String
                    0x9               output\prvTaskFS.o
InetDprsSend        0x4               output\DstaDPlusClientUDP.o
xHighPriorityNormallyFullTask1
                    0x4               output\IntQueue.o
voice               0xc               output\main.o
DCS_recv            0x63              output\DstaDPlusClientUDP.o
RefNameSave         0x8               output\DstaDPlusClientUDP.o
DprsAccessFileReadSW
                    0x4               output\prvTaskFS.o

Microchip PIC32 Memory-Usage Report

kseg0 Program-Memory Usage
section                    address  length [bytes]      (dec)  Description
-------                 ----------  -------------------------  -----------
.rodata                 0x9d007e00           0x48          72  Read-only const 
.text                   0x9d007e50        0x102ec       66284  App's exec code 
.rodata                 0x9d01813c         0xb764       46948  Read-only const 
.text                   0x9d0238a0        0x40be0      265184  App's exec code 
.dinit                  0x9d064480         0x1024        4132   
.text                   0x9d0654a4         0x2920       10528  App's exec code 
.text._vfprintf_cdnopsu 0x9d067dc4          0xc7c        3196   
.rodata                 0x9d068a40          0xbcc        3020  Read-only const 
.text                   0x9d06960c          0xb90        2960  App's exec code 
.rodata                 0x9d06a19c          0xa58        2648  Read-only const 
.text                   0x9d06abf4         0x21d4        8660  App's exec code 
.rodata                 0x9d06cdc8          0x7d4        2004  Read-only const 
.text                   0x9d06d59c         0x1fe8        8168  App's exec code 
.rodata                 0x9d06f584          0x9c4        2500  Read-only const 
.text                   0x9d06ff48          0xd20        3360  App's exec code 
.text.EthRxBuffersAppen 0x9d070c68          0x448        1096   
.text                   0x9d0710b0          0x850        2128  App's exec code 
.text.__strtod          0x9d071900          0x3f0        1008   
.text                   0x9d071cf0          0xa68        2664  App's exec code 
.rodata                 0x9d072758          0x338         824  Read-only const 
.text                   0x9d072a90          0x330         816  App's exec code 
.rodata                 0x9d072dc0          0x2f0         752  Read-only const 
.text                   0x9d0730b0          0xb14        2836  App's exec code 
.text.gmtime            0x9d073bc4          0x2a4         676   
.text                   0x9d073e68          0x254         596  App's exec code 
.text._RtccSetTimeAndDa 0x9d0740bc          0x23c         572   
.text                   0x9d0742f8          0x230         560  App's exec code 
.text.RtccOpen          0x9d074528          0x1ec         492   
.text._EthAckPacket     0x9d074714          0x1dc         476   
.text.__ldexp           0x9d0748f0          0x1d4         468   
.text.RtccInit          0x9d074ac4          0x1ac         428   
.text                   0x9d074c70          0x1a8         424  App's exec code 
.text.EthTxSendBuffer   0x9d074e18          0x1a4         420   
.text                   0x9d074fbc          0x1a0         416  App's exec code 
.text._EthAppendBusyLis 0x9d07515c          0x19c         412   
.text._EthRxAckBuffer   0x9d0752f8          0x184         388   
.text.EthRxGetPacket    0x9d07547c          0x180         384   
.text                   0x9d0755fc          0x5a4        1444  App's exec code 
.text.fputc             0x9d075ba0          0x140         320   
.text.EthMIIMConfig     0x9d075ce0          0x13c         316   
.text.EthDescriptorsPoo 0x9d075e1c          0x134         308   
.text._flsbuf           0x9d075f50          0x12c         300   
.text                   0x9d07607c          0x120         288  App's exec code 
.rodata                 0x9d07619c          0x104         260  Read-only const 
.text._RtccWaitClockOff 0x9d0762a0           0xf8         248   
.rodata                 0x9d076398           0xf0         240  Read-only const 
.text.strncpy           0x9d076488           0xe8         232   
.rodata                 0x9d076570           0xe0         224  Read-only const 
.text                   0x9d076650           0xd4         212  App's exec code 
.text.general_exception 0x9d076724           0xd0         208   
.rodata                 0x9d0767f4            0x4           4  Read-only const 
.rodata                 0x9d0767f8          0x188         392  Read-only const 
.text._mon_putc         0x9d076980           0xb4         180   
.text.EthInit           0x9d076a34           0xb4         180   
.text.EthMACOpen        0x9d076ae8           0xb4         180   
.text                   0x9d076b9c           0xa8         168  App's exec code 
.text.atoi              0x9d076c44           0xa4         164   
.text.atol              0x9d076ce8           0xa4         164   
.text.strstr            0x9d076d8c           0xa4         164   
.rodata                 0x9d076e30           0x98         152  Read-only const 
.text                   0x9d076ec8           0x98         152  App's exec code 
.rodata                 0x9d076f60           0x90         144  Read-only const 
.text.write             0x9d076ff0           0x88         136   
.rodata                 0x9d077078           0x80         128  Read-only const 
.text.SoftReset         0x9d0770f8           0x78         120   
.text.strncmp           0x9d077170           0x70         112   
.text._sprintf_cdnopsux 0x9d0771e0           0x68         104   
.rodata                 0x9d077248           0x60          96  Read-only const 
.text.OpenSPI1          0x9d0772a8           0x60          96   
.text.INTEnable         0x9d077308           0x58          88   
.rodata                 0x9d077360           0x54          84  Read-only const 
.text                   0x9d0773b4           0x4c          76  App's exec code 
.rodata                 0x9d077400           0x4c          76  Read-only const 
.text.EthMACSetAddress  0x9d07744c           0x48          72   
.text                   0x9d077494           0x88         136  App's exec code 
.text.EthMIIMReadStart  0x9d07751c           0x40          64   
.text.PORTSetPinsDigita 0x9d07755c           0x40          64   
.text.PORTSetPinsDigita 0x9d07759c           0x40          64   
.text.localtime         0x9d0775dc           0x3c          60   
.text.EthRxGetBuffer    0x9d077618           0x3c          60   
.text.strcat            0x9d077654           0x38          56   
.text.EthMIIMWriteStart 0x9d07768c           0x38          56   
.text.EthMIIMScanStart  0x9d0776c4           0x34          52   
.text.INTEnableSystemMu 0x9d0776f8           0x34          52   
.text.EthTxAcknowledgeB 0x9d07772c           0x30          48   
.text.EthRxSetBufferSiz 0x9d07775c           0x30          48   
.text.INTClearFlag      0x9d07778c           0x2c          44   
.rodata                 0x9d0777b8           0x28          40  Read-only const 
.text.strchr            0x9d0777e0           0x28          40   
.text.atof              0x9d077808           0x28          40   
.text.EthMIIMReadResult 0x9d077830           0x28          40   
.text.RtccSetTimeDate   0x9d077858           0x28          40   
.rodata                 0x9d077880           0x24          36  Read-only const 
.text.tolower           0x9d0778a4           0x24          36   
.text.toupper           0x9d0778c8           0x24          36   
.rodata                 0x9d0778ec           0x60          96  Read-only const 
.text.EthMIIMScanResult 0x9d07794c           0x20          32   
.text.getcSPI1          0x9d07796c           0x20          32   
.text._dstrtod          0x9d07798c           0x1c          28   
.text.EthRxAcknowledgeB 0x9d0779a8           0x1c          28   
.text.INTRestoreInterru 0x9d0779c4           0x1c          28   
.text                   0x9d0779e0           0x18          24  App's exec code 
.text.CheKseg0CacheOn   0x9d0779f8           0x18          24   
.text                   0x9d077a10           0x10          16  App's exec code 
.rodata                 0x9d077a20           0x40          64  Read-only const 
.text.EthRxFiltersSet   0x9d077a60           0x10          16   
.text.EthRxFiltersClr   0x9d077a70           0x10          16   
.text.SetCoreSW0        0x9d077a80           0x10          16   
.rodata                 0x9d077a90            0xc          12  Read-only const 
.text._bootstrap_except 0x9d077a9c            0xc          12   
.rodata                 0x9d077aa8           0x18          24  Read-only const 
.text._on_reset         0x9d077ac0            0x8           8   
.text._on_bootstrap     0x9d077ac8            0x8           8   
.text.ReadCoreTimer     0x9d077ad0            0x8           8   
.text.WriteCoreTimer    0x9d077ad8            0x8           8   
.text.INTDisableInterru 0x9d077ae0            0x8           8   
.text.INTEnableInterrup 0x9d077ae8            0x8           8   
.rodata                 0x9d077af0            0x2           2  Read-only const 
      Total kseg0_program_mem used  :     0x6fcea      457962  88.6% of 0x7e200

kseg0 Boot-Memory Usage
section                    address  length [bytes]      (dec)  Description
-------                 ----------  -------------------------  -----------
         Total kseg0_boot_mem used  :           0           0  <1% of 0x970

Exception-Memory Usage 
section                    address  length [bytes]      (dec)  Description
-------                 ----------  -------------------------  -----------
.app_excpt              0x9d006180           0x10          16  General-Exception 
.vector_1               0x9d006220            0x8           8  Interrupt Vector 1 
.vector_4               0x9d006280            0x8           8  Interrupt Vector 4 
.vector_12              0x9d006380            0x8           8  Interrupt Vector 12 
.vector_16              0x9d006400            0x8           8  Interrupt Vector 16 
.vector_20              0x9d006480            0x8           8  Interrupt Vector 20 
.vector_32              0x9d006600            0x8           8  Interrupt Vector 32 
.vector_45              0x9d0067a0           0x10          16  Interrupt Vector 45 
          Total exception_mem used  :        0x50          80  2.0% of 0x1000

kseg1 Boot-Memory Usage
section                    address  length [bytes]      (dec)  Description
-------                 ----------  -------------------------  -----------
.reset                  0x9d007970          0x1f4         500  Reset handler 
.bev_excpt              0x9d007cf0           0x10          16  BEV-Exception 
         Total kseg1_boot_mem used  :       0x204         516  44.2% of 0x490
        --------------------------------------------------------------------------
         Total Program Memory used  :     0x6ff3e      458558  87.5% of 0x80000
        --------------------------------------------------------------------------


kseg1 Data-Memory Usage
section                    address  length [bytes]      (dec)  Description
-------                 ----------  -------------------------  -----------
.eh_frame               0xa0000000           0x3c          60   
.sdata                  0xa000003c           0xc0         192  Small init data 
.sbss                   0xa00000fc          0x875        2165  Small uninit data 
.bss                    0xa0000974         0x1db4        7604  Uninitialized data 
.bss                    0xa000273c        0x17cf4       97524  Uninitialized data 
.data                   0xa001a430          0x85c        2140  Initialized data 
.bss                    0xa001ac8c         0x1298        4760  Uninitialized data 
.data                   0xa001bf24           0xcc         204  Initialized data 
.data                   0xa001bff0           0x10          16  Initialized data 
.bss                    0xa001c000          0x754        1876  Uninitialized data 
.bss                    0xa001c754          0x18c         396  Uninitialized data 
.data                   0xa001c8e0           0x98         152  Initialized data 
.bss                    0xa001c978          0x214         532  Uninitialized data 
.bss                    0xa001cb90           0xac         172  Uninitialized data 
.data                   0xa001cc3c           0x28          40  Initialized data 
.bss                    0xa001cc64           0x6c         108  Uninitialized data 
.data                   0xa001ccd0           0x10          16  Initialized data 
.bss                    0xa001cce0           0x1c          28  Uninitialized data 
         Total kseg1_data_mem used  :     0x1cce1      117985  90.0% of 0x20000
        --------------------------------------------------------------------------
            Total Data Memory used  :     0x1cce1      117985  90.0% of 0x20000
        --------------------------------------------------------------------------


Dynamic Data-Memory Reservation
section                    address  length [bytes]      (dec)  Description
-------                 ----------  -------------------------  -----------
heap                    0xa001cd00              0           0  Reserved for heap 
stack                   0xa001cd18         0x32d8       13016  Reserved for stack 

        --------------------------------------------------------------------------

Discarded input sections

 .data          0x00000000        0x0 c:/program files/microchip/mplabc32/v2.02/bin/../lib/gcc/pic32mx/4.5.1/../../../../pic32mx/lib/speed/crt0.o
 .bss           0x00000000        0x0 c:/program files/microchip/mplabc32/v2.02/bin/../lib/gcc/pic32mx/4.5.1/../../../../pic32mx/lib/speed/crt0.o
 .reginfo       0x00000000       0x18 c:/program files/microchip/mplabc32/v2.02/bin/../lib/gcc/pic32mx/4.5.1/../../../../pic32mx/lib/speed/crt0.o
 .pdr           0x00000000       0xa0 c:/program files/microchip/mplabc32/v2.02/bin/../lib/gcc/pic32mx/4.5.1/../../../../pic32mx/lib/speed/crt0.o
 .data          0x00000000        0x0 output\main.o
 .reginfo       0x00000000       0x18 output\main.o
 .pdr           0x00000000       0xa0 output\main.o
 .mdebug.abi32  0x00000000        0x0 output\main.o
 .data          0x00000000        0x0 output\IntQueueTimer.o
 .bss           0x00000000        0x0 output\IntQueueTimer.o
 .reginfo       0x00000000       0x18 output\IntQueueTimer.o
 .pdr           0x00000000       0xa0 output\IntQueueTimer.o
 .mdebug.abi32  0x00000000        0x0 output\IntQueueTimer.o
 .data          0x00000000        0x0 output\IntQueueTimer_isr.o
 .bss           0x00000000        0x0 output\IntQueueTimer_isr.o
 .reginfo       0x00000000       0x18 output\IntQueueTimer_isr.o
 .pdr           0x00000000       0x40 output\IntQueueTimer_isr.o
 .data          0x00000000        0x0 output\port.o
 .reginfo       0x00000000       0x18 output\port.o
 .pdr           0x00000000      0x120 output\port.o
 .mdebug.abi32  0x00000000        0x0 output\port.o
 .data          0x00000000        0x0 output\port_asm.o
 .bss           0x00000000        0x0 output\port_asm.o
 .reginfo       0x00000000       0x18 output\port_asm.o
 .pdr           0x00000000       0x60 output\port_asm.o
 .data          0x00000000        0x0 output\queue.o
 .bss           0x00000000        0x0 output\queue.o
 .reginfo       0x00000000       0x18 output\queue.o
 .pdr           0x00000000      0x1e0 output\queue.o
 .mdebug.abi32  0x00000000        0x0 output\queue.o
 .data          0x00000000        0x0 output\tasks.o
 .reginfo       0x00000000       0x18 output\tasks.o
 .pdr           0x00000000      0x420 output\tasks.o
 .mdebug.abi32  0x00000000        0x0 output\tasks.o
 .data          0x00000000        0x0 output\list.o
 .bss           0x00000000        0x0 output\list.o
 .reginfo       0x00000000       0x18 output\list.o
 .pdr           0x00000000       0xa0 output\list.o
 .mdebug.abi32  0x00000000        0x0 output\list.o
 .data          0x00000000        0x0 output\IntQueue.o
 .reginfo       0x00000000       0x18 output\IntQueue.o
 .pdr           0x00000000      0x180 output\IntQueue.o
 .mdebug.abi32  0x00000000        0x0 output\IntQueue.o
 .data          0x00000000        0x0 output\QPeek.o
 .bss           0x00000000        0x0 output\QPeek.o
 .reginfo       0x00000000       0x18 output\QPeek.o
 .pdr           0x00000000       0xc0 output\QPeek.o
 .mdebug.abi32  0x00000000        0x0 output\QPeek.o
 .data          0x00000000        0x0 output\lcd.o
 .bss           0x00000000        0x0 output\lcd.o
 .reginfo       0x00000000       0x18 output\lcd.o
 .pdr           0x00000000       0xe0 output\lcd.o
 .mdebug.abi32  0x00000000        0x0 output\lcd.o
 .data          0x00000000        0x0 output\prvTaskTCPIP.o
 .reginfo       0x00000000       0x18 output\prvTaskTCPIP.o
 .pdr           0x00000000       0x60 output\prvTaskTCPIP.o
 .mdebug.abi32  0x00000000        0x0 output\prvTaskTCPIP.o
 .data          0x00000000        0x0 output\heap_2.o
 .reginfo       0x00000000       0x18 output\heap_2.o
 .pdr           0x00000000       0x80 output\heap_2.o
 .mdebug.abi32  0x00000000        0x0 output\heap_2.o
 .data          0x00000000        0x0 output\usb_host.o
 .reginfo       0x00000000       0x18 output\usb_host.o
 .pdr           0x00000000      0x4c0 output\usb_host.o
 .mdebug.abi32  0x00000000        0x0 output\usb_host.o
 .text          0x00000000        0x0 output\usb_config.o
 .bss           0x00000000        0x0 output\usb_config.o
 .reginfo       0x00000000       0x18 output\usb_config.o
 .pdr           0x00000000        0x0 output\usb_config.o
 .mdebug.abi32  0x00000000        0x0 output\usb_config.o
 .reginfo       0x00000000       0x18 output\CustomHTTPApp.o
 .pdr           0x00000000     0x1160 output\CustomHTTPApp.o
 .mdebug.abi32  0x00000000        0x0 output\CustomHTTPApp.o
 .data          0x00000000        0x0 output\usb_host_generic.o
 .bss           0x00000000        0x0 output\usb_host_generic.o
 .reginfo       0x00000000       0x18 output\usb_host_generic.o
 .pdr           0x00000000       0xa0 output\usb_host_generic.o
 .mdebug.abi32  0x00000000        0x0 output\usb_host_generic.o
 .data          0x00000000        0x0 output\FSIO.o
 .bss           0x00000000        0x0 output\FSIO.o
 .reginfo       0x00000000       0x18 output\FSIO.o
 .pdr           0x00000000      0x920 output\FSIO.o
 .mdebug.abi32  0x00000000        0x0 output\FSIO.o
 .data          0x00000000        0x0 output\UDP.o
 .bss           0x00000000        0x0 output\UDP.o
 .reginfo       0x00000000       0x18 output\UDP.o
 .pdr           0x00000000      0x240 output\UDP.o
 .mdebug.abi32  0x00000000        0x0 output\UDP.o
 .data          0x00000000        0x0 output\ARP.o
 .reginfo       0x00000000       0x18 output\ARP.o
 .pdr           0x00000000       0xc0 output\ARP.o
 .mdebug.abi32  0x00000000        0x0 output\ARP.o
 .data          0x00000000        0x0 output\Delay.o
 .bss           0x00000000        0x0 output\Delay.o
 .reginfo       0x00000000       0x18 output\Delay.o
 .pdr           0x00000000       0x40 output\Delay.o
 .mdebug.abi32  0x00000000        0x0 output\Delay.o
 .data          0x00000000        0x0 output\DHCP.o
 .reginfo       0x00000000       0x18 output\DHCP.o
 .pdr           0x00000000      0x140 output\DHCP.o
 .mdebug.abi32  0x00000000        0x0 output\DHCP.o
 .data          0x00000000        0x0 output\DNS.o
 .reginfo       0x00000000       0x18 output\DNS.o
 .pdr           0x00000000       0xc0 output\DNS.o
 .mdebug.abi32  0x00000000        0x0 output\DNS.o
 .reginfo       0x00000000       0x18 output\DstaDPlusClientUDP.o
 .pdr           0x00000000      0x3c0 output\DstaDPlusClientUDP.o
 .mdebug.abi32  0x00000000        0x0 output\DstaDPlusClientUDP.o
 .data          0x00000000        0x0 output\ETHPIC32ExtPhy.o
 .bss           0x00000000        0x0 output\ETHPIC32ExtPhy.o
 .reginfo       0x00000000       0x18 output\ETHPIC32ExtPhy.o
 .pdr           0x00000000      0x180 output\ETHPIC32ExtPhy.o
 .mdebug.abi32  0x00000000        0x0 output\ETHPIC32ExtPhy.o
 .data          0x00000000        0x0 output\ETHPIC32ExtPhyDP83848.o
 .bss           0x00000000        0x0 output\ETHPIC32ExtPhyDP83848.o
 .reginfo       0x00000000       0x18 output\ETHPIC32ExtPhyDP83848.o
 .pdr           0x00000000       0x80 output\ETHPIC32ExtPhyDP83848.o
 .mdebug.abi32  0x00000000        0x0 output\ETHPIC32ExtPhyDP83848.o
 .data          0x00000000        0x0 output\ETHPIC32IntMac.o
 .reginfo       0x00000000       0x18 output\ETHPIC32IntMac.o
 .pdr           0x00000000      0x320 output\ETHPIC32IntMac.o
 .mdebug.abi32  0x00000000        0x0 output\ETHPIC32IntMac.o
 .text          0x00000000        0x0 output\FileSystem.o
 .data          0x00000000        0x0 output\FileSystem.o
 .bss           0x00000000        0x0 output\FileSystem.o
 .reginfo       0x00000000       0x18 output\FileSystem.o
 .pdr           0x00000000        0x0 output\FileSystem.o
 .mdebug.abi32  0x00000000        0x0 output\FileSystem.o
 .reginfo       0x00000000       0x18 output\FTP.o
 .pdr           0x00000000      0x2a0 output\FTP.o
 .mdebug.abi32  0x00000000        0x0 output\FTP.o
 .text          0x00000000        0x0 output\Hashes.o
 .data          0x00000000        0x0 output\Hashes.o
 .bss           0x00000000        0x0 output\Hashes.o
 .reginfo       0x00000000       0x18 output\Hashes.o
 .pdr           0x00000000        0x0 output\Hashes.o
 .mdebug.abi32  0x00000000        0x0 output\Hashes.o
 .data          0x00000000        0x0 output\Helpers.o
 .bss           0x00000000        0x0 output\Helpers.o
 .reginfo       0x00000000       0x18 output\Helpers.o
 .pdr           0x00000000      0x220 output\Helpers.o
 .mdebug.abi32  0x00000000        0x0 output\Helpers.o
 .data          0x00000000        0x0 output\HTTP2.o
 .reginfo       0x00000000       0x18 output\HTTP2.o
 .pdr           0x00000000      0x220 output\HTTP2.o
 .mdebug.abi32  0x00000000        0x0 output\HTTP2.o
 .data          0x00000000        0x0 output\ICMP.o
 .bss           0x00000000        0x0 output\ICMP.o
 .reginfo       0x00000000       0x18 output\ICMP.o
 .pdr           0x00000000       0x20 output\ICMP.o
 .mdebug.abi32  0x00000000        0x0 output\ICMP.o
 .data          0x00000000        0x0 output\IP.o
 .bss           0x00000000        0x0 output\IP.o
 .reginfo       0x00000000       0x18 output\IP.o
 .pdr           0x00000000       0x80 output\IP.o
 .mdebug.abi32  0x00000000        0x0 output\IP.o
 .data          0x00000000        0x0 output\MPFS2.o
 .reginfo       0x00000000       0x18 output\MPFS2.o
 .pdr           0x00000000      0x280 output\MPFS2.o
 .mdebug.abi32  0x00000000        0x0 output\MPFS2.o
 .text          0x00000000        0x0 output\Random.o
 .data          0x00000000        0x0 output\Random.o
 .bss           0x00000000        0x0 output\Random.o
 .reginfo       0x00000000       0x18 output\Random.o
 .pdr           0x00000000        0x0 output\Random.o
 .mdebug.abi32  0x00000000        0x0 output\Random.o
 .data          0x00000000        0x0 output\SNTP.o
 .reginfo       0x00000000       0x18 output\SNTP.o
 .pdr           0x00000000       0x40 output\SNTP.o
 .mdebug.abi32  0x00000000        0x0 output\SNTP.o
 .data          0x00000000        0x0 output\StackTsk.o
 .bss           0x00000000        0x0 output\StackTsk.o
 .reginfo       0x00000000       0x18 output\StackTsk.o
 .pdr           0x00000000       0x60 output\StackTsk.o
 .mdebug.abi32  0x00000000        0x0 output\StackTsk.o
 .data          0x00000000        0x0 output\TCP.o
 .reginfo       0x00000000       0x18 output\TCP.o
 .pdr           0x00000000      0x420 output\TCP.o
 .mdebug.abi32  0x00000000        0x0 output\TCP.o
 .data          0x00000000        0x0 output\Tick.o
 .bss           0x00000000        0x0 output\Tick.o
 .reginfo       0x00000000       0x18 output\Tick.o
 .pdr           0x00000000      0x100 output\Tick.o
 .mdebug.abi32  0x00000000        0x0 output\Tick.o
 .text          0x00000000        0x0 output\MPFSImg2.o
 .data          0x00000000        0x0 output\MPFSImg2.o
 .bss           0x00000000        0x0 output\MPFSImg2.o
 .reginfo       0x00000000       0x18 output\MPFSImg2.o
 .pdr           0x00000000        0x0 output\MPFSImg2.o
 .mdebug.abi32  0x00000000        0x0 output\MPFSImg2.o
 .data          0x00000000        0x0 output\SD-SPI.o
 .reginfo       0x00000000       0x18 output\SD-SPI.o
 .pdr           0x00000000      0x220 output\SD-SPI.o
 .mdebug.abi32  0x00000000        0x0 output\SD-SPI.o
 .reginfo       0x00000000       0x18 output\prvTaskUSB.o
 .pdr           0x00000000      0x4a0 output\prvTaskUSB.o
 .mdebug.abi32  0x00000000        0x0 output\prvTaskUSB.o
 .reginfo       0x00000000       0x18 output\prvTaskFS.o
 .pdr           0x00000000      0x200 output\prvTaskFS.o
 .mdebug.abi32  0x00000000        0x0 output\prvTaskFS.o
 .data          0x00000000        0x0 output\MACread.o
 .reginfo       0x00000000       0x18 output\MACread.o
 .pdr           0x00000000      0x180 output\MACread.o
 .mdebug.abi32  0x00000000        0x0 output\MACread.o
 .data          0x00000000        0x0 output\SMTP.o
 .bss           0x00000000        0x0 output\SMTP.o
 .reginfo       0x00000000       0x18 output\SMTP.o
 .pdr           0x00000000      0x1a0 output\SMTP.o
 .mdebug.abi32  0x00000000        0x0 output\SMTP.o
 .data          0x00000000        0x0 output\DprsSMTP.o
 .reginfo       0x00000000       0x18 output\DprsSMTP.o
 .pdr           0x00000000       0x20 output\DprsSMTP.o
 .mdebug.abi32  0x00000000        0x0 output\DprsSMTP.o
 .data          0x00000000        0x0 output\serial.o
 .bss           0x00000000        0x0 output\serial.o
 .reginfo       0x00000000       0x18 output\serial.o
 .pdr           0x00000000       0xc0 output\serial.o
 .mdebug.abi32  0x00000000        0x0 output\serial.o
 .data          0x00000000        0x0 output\serial_isr.o
 .bss           0x00000000        0x0 output\serial_isr.o
 .reginfo       0x00000000       0x18 output\serial_isr.o
 .pdr           0x00000000       0x20 output\serial_isr.o
 .data          0x00000000        0x0 output\comtest.o
 .bss           0x00000000        0x0 output\comtest.o
 .reginfo       0x00000000       0x18 output\comtest.o
 .pdr           0x00000000       0x80 output\comtest.o
 .mdebug.abi32  0x00000000        0x0 output\comtest.o
 .data          0x00000000        0x0 output\DHCPs.o
 .reginfo       0x00000000       0x18 output\DHCPs.o
 .pdr           0x00000000       0x60 output\DHCPs.o
 .mdebug.abi32  0x00000000        0x0 output\DHCPs.o
 .data          0x00000000        0x0 output\NBNS.o
 .reginfo       0x00000000       0x18 output\NBNS.o
 .pdr           0x00000000       0x60 output\NBNS.o
 .mdebug.abi32  0x00000000        0x0 output\NBNS.o
 .text          0x00000000        0x0 c:/program files/microchip/mplabc32/v2.02/bin/../lib/gcc/pic32mx/4.5.1/../../../../pic32mx/lib/./proc/32MX795F512L\processor.o
 .data          0x00000000        0x0 c:/program files/microchip/mplabc32/v2.02/bin/../lib/gcc/pic32mx/4.5.1/../../../../pic32mx/lib/./proc/32MX795F512L\processor.o
 .bss           0x00000000        0x0 c:/program files/microchip/mplabc32/v2.02/bin/../lib/gcc/pic32mx/4.5.1/../../../../pic32mx/lib/./proc/32MX795F512L\processor.o
 .reginfo       0x00000000       0x18 c:/program files/microchip/mplabc32/v2.02/bin/../lib/gcc/pic32mx/4.5.1/../../../../pic32mx/lib/./proc/32MX795F512L\processor.o
 .pdr           0x00000000        0x0 c:/program files/microchip/mplabc32/v2.02/bin/../lib/gcc/pic32mx/4.5.1/../../../../pic32mx/lib/./proc/32MX795F512L\processor.o
 .data          0x00000000        0x0 c:/program files/microchip/mplabc32/v2.02/bin/../lib/gcc/pic32mx/4.5.1/speed\libgcc.a(_udivdi3.o)
 .bss           0x00000000        0x0 c:/program files/microchip/mplabc32/v2.02/bin/../lib/gcc/pic32mx/4.5.1/speed\libgcc.a(_udivdi3.o)
 .reginfo       0x00000000       0x18 c:/program files/microchip/mplabc32/v2.02/bin/../lib/gcc/pic32mx/4.5.1/speed\libgcc.a(_udivdi3.o)
 .pdr           0x00000000       0x20 c:/program files/microchip/mplabc32/v2.02/bin/../lib/gcc/pic32mx/4.5.1/speed\libgcc.a(_udivdi3.o)
 .mdebug.abi32  0x00000000        0x0 c:/program files/microchip/mplabc32/v2.02/bin/../lib/gcc/pic32mx/4.5.1/speed\libgcc.a(_udivdi3.o)
 .data          0x00000000        0x0 c:/program files/microchip/mplabc32/v2.02/bin/../lib/gcc/pic32mx/4.5.1/speed\libgcc.a(_umoddi3.o)
 .bss           0x00000000        0x0 c:/program files/microchip/mplabc32/v2.02/bin/../lib/gcc/pic32mx/4.5.1/speed\libgcc.a(_umoddi3.o)
 .reginfo       0x00000000       0x18 c:/program files/microchip/mplabc32/v2.02/bin/../lib/gcc/pic32mx/4.5.1/speed\libgcc.a(_umoddi3.o)
 .pdr           0x00000000       0x20 c:/program files/microchip/mplabc32/v2.02/bin/../lib/gcc/pic32mx/4.5.1/speed\libgcc.a(_umoddi3.o)
 .mdebug.abi32  0x00000000        0x0 c:/program files/microchip/mplabc32/v2.02/bin/../lib/gcc/pic32mx/4.5.1/speed\libgcc.a(_umoddi3.o)
 .data          0x00000000        0x0 c:/program files/microchip/mplabc32/v2.02/bin/../lib/gcc/pic32mx/4.5.1/speed\libgcc.a(floatunsisf.o)
 .bss           0x00000000        0x0 c:/program files/microchip/mplabc32/v2.02/bin/../lib/gcc/pic32mx/4.5.1/speed\libgcc.a(floatunsisf.o)
 .reginfo       0x00000000       0x18 c:/program files/microchip/mplabc32/v2.02/bin/../lib/gcc/pic32mx/4.5.1/speed\libgcc.a(floatunsisf.o)
 .pdr           0x00000000       0x20 c:/program files/microchip/mplabc32/v2.02/bin/../lib/gcc/pic32mx/4.5.1/speed\libgcc.a(floatunsisf.o)
 .mdebug.abi32  0x00000000        0x0 c:/program files/microchip/mplabc32/v2.02/bin/../lib/gcc/pic32mx/4.5.1/speed\libgcc.a(floatunsisf.o)
 .data          0x00000000        0x0 c:/program files/microchip/mplabc32/v2.02/bin/../lib/gcc/pic32mx/4.5.1/../../../../pic32mx/lib/speed\libc.a(memcmp.o)
 .bss           0x00000000        0x0 c:/program files/microchip/mplabc32/v2.02/bin/../lib/gcc/pic32mx/4.5.1/../../../../pic32mx/lib/speed\libc.a(memcmp.o)
 .reginfo       0x00000000       0x18 c:/program files/microchip/mplabc32/v2.02/bin/../lib/gcc/pic32mx/4.5.1/../../../../pic32mx/lib/speed\libc.a(memcmp.o)
 .pdr           0x00000000       0x20 c:/program files/microchip/mplabc32/v2.02/bin/../lib/gcc/pic32mx/4.5.1/../../../../pic32mx/lib/speed\libc.a(memcmp.o)
 .data          0x00000000        0x0 c:/program files/microchip/mplabc32/v2.02/bin/../lib/gcc/pic32mx/4.5.1/../../../../pic32mx/lib/speed\libc.a(memcpy.o)
 .bss           0x00000000        0x0 c:/program files/microchip/mplabc32/v2.02/bin/../lib/gcc/pic32mx/4.5.1/../../../../pic32mx/lib/speed\libc.a(memcpy.o)
 .reginfo       0x00000000       0x18 c:/program files/microchip/mplabc32/v2.02/bin/../lib/gcc/pic32mx/4.5.1/../../../../pic32mx/lib/speed\libc.a(memcpy.o)
 .pdr           0x00000000       0x20 c:/program files/microchip/mplabc32/v2.02/bin/../lib/gcc/pic32mx/4.5.1/../../../../pic32mx/lib/speed\libc.a(memcpy.o)
 .data          0x00000000        0x0 c:/program files/microchip/mplabc32/v2.02/bin/../lib/gcc/pic32mx/4.5.1/../../../../pic32mx/lib/speed\libc.a(memset.o)
 .bss           0x00000000        0x0 c:/program files/microchip/mplabc32/v2.02/bin/../lib/gcc/pic32mx/4.5.1/../../../../pic32mx/lib/speed\libc.a(memset.o)
 .reginfo       0x00000000       0x18 c:/program files/microchip/mplabc32/v2.02/bin/../lib/gcc/pic32mx/4.5.1/../../../../pic32mx/lib/speed\libc.a(memset.o)
 .pdr           0x00000000       0x20 c:/program files/microchip/mplabc32/v2.02/bin/../lib/gcc/pic32mx/4.5.1/../../../../pic32mx/lib/speed\libc.a(memset.o)
 .data          0x00000000        0x0 c:/program files/microchip/mplabc32/v2.02/bin/../lib/gcc/pic32mx/4.5.1/../../../../pic32mx/lib/speed\libc.a(strcmp.o)
 .bss           0x00000000        0x0 c:/program files/microchip/mplabc32/v2.02/bin/../lib/gcc/pic32mx/4.5.1/../../../../pic32mx/lib/speed\libc.a(strcmp.o)
 .reginfo       0x00000000       0x18 c:/program files/microchip/mplabc32/v2.02/bin/../lib/gcc/pic32mx/4.5.1/../../../../pic32mx/lib/speed\libc.a(strcmp.o)
 .pdr           0x00000000       0x20 c:/program files/microchip/mplabc32/v2.02/bin/../lib/gcc/pic32mx/4.5.1/../../../../pic32mx/lib/speed\libc.a(strcmp.o)
 .data          0x00000000        0x0 c:/program files/microchip/mplabc32/v2.02/bin/../lib/gcc/pic32mx/4.5.1/../../../../pic32mx/lib/speed\libc.a(strcpy.o)
 .bss           0x00000000        0x0 c:/program files/microchip/mplabc32/v2.02/bin/../lib/gcc/pic32mx/4.5.1/../../../../pic32mx/lib/speed\libc.a(strcpy.o)
 .reginfo       0x00000000       0x18 c:/program files/microchip/mplabc32/v2.02/bin/../lib/gcc/pic32mx/4.5.1/../../../../pic32mx/lib/speed\libc.a(strcpy.o)
 .pdr           0x00000000       0x20 c:/program files/microchip/mplabc32/v2.02/bin/../lib/gcc/pic32mx/4.5.1/../../../../pic32mx/lib/speed\libc.a(strcpy.o)
 .data          0x00000000        0x0 c:/program files/microchip/mplabc32/v2.02/bin/../lib/gcc/pic32mx/4.5.1/../../../../pic32mx/lib/speed\libc.a(strlen.o)
 .bss           0x00000000        0x0 c:/program files/microchip/mplabc32/v2.02/bin/../lib/gcc/pic32mx/4.5.1/../../../../pic32mx/lib/speed\libc.a(strlen.o)
 .reginfo       0x00000000       0x18 c:/program files/microchip/mplabc32/v2.02/bin/../lib/gcc/pic32mx/4.5.1/../../../../pic32mx/lib/speed\libc.a(strlen.o)
 .pdr           0x00000000       0x20 c:/program files/microchip/mplabc32/v2.02/bin/../lib/gcc/pic32mx/4.5.1/../../../../pic32mx/lib/speed\libc.a(strlen.o)
 .text          0x00000000        0x0 c:/program files/microchip/mplabc32/v2.02/bin/../lib/gcc/pic32mx/4.5.1/../../../../pic32mx/lib/speed\libc.a(general-exception.o)
 .data          0x00000000        0x0 c:/program files/microchip/mplabc32/v2.02/bin/../lib/gcc/pic32mx/4.5.1/../../../../pic32mx/lib/speed\libc.a(general-exception.o)
 .bss           0x00000000        0x0 c:/program files/microchip/mplabc32/v2.02/bin/../lib/gcc/pic32mx/4.5.1/../../../../pic32mx/lib/speed\libc.a(general-exception.o)
 .reginfo       0x00000000       0x18 c:/program files/microchip/mplabc32/v2.02/bin/../lib/gcc/pic32mx/4.5.1/../../../../pic32mx/lib/speed\libc.a(general-exception.o)
 .pdr           0x00000000       0x20 c:/program files/microchip/mplabc32/v2.02/bin/../lib/gcc/pic32mx/4.5.1/../../../../pic32mx/lib/speed\libc.a(general-exception.o)
 .text          0x00000000        0x0 c:/program files/microchip/mplabc32/v2.02/bin/../lib/gcc/pic32mx/4.5.1/../../../../pic32mx/lib/speed\libc.a(atoi.o)
 .data          0x00000000        0x0 c:/program files/microchip/mplabc32/v2.02/bin/../lib/gcc/pic32mx/4.5.1/../../../../pic32mx/lib/speed\libc.a(atoi.o)
 .bss           0x00000000        0x0 c:/program files/microchip/mplabc32/v2.02/bin/../lib/gcc/pic32mx/4.5.1/../../../../pic32mx/lib/speed\libc.a(atoi.o)
 .reginfo       0x00000000       0x18 c:/program files/microchip/mplabc32/v2.02/bin/../lib/gcc/pic32mx/4.5.1/../../../../pic32mx/lib/speed\libc.a(atoi.o)
 .pdr           0x00000000       0x20 c:/program files/microchip/mplabc32/v2.02/bin/../lib/gcc/pic32mx/4.5.1/../../../../pic32mx/lib/speed\libc.a(atoi.o)
 .mdebug.abi32  0x00000000        0x0 c:/program files/microchip/mplabc32/v2.02/bin/../lib/gcc/pic32mx/4.5.1/../../../../pic32mx/lib/speed\libc.a(atoi.o)
 .text          0x00000000        0x0 c:/program files/microchip/mplabc32/v2.02/bin/../lib/gcc/pic32mx/4.5.1/../../../../pic32mx/lib/speed\libc.a(atol.o)
 .data          0x00000000        0x0 c:/program files/microchip/mplabc32/v2.02/bin/../lib/gcc/pic32mx/4.5.1/../../../../pic32mx/lib/speed\libc.a(atol.o)
 .bss           0x00000000        0x0 c:/program files/microchip/mplabc32/v2.02/bin/../lib/gcc/pic32mx/4.5.1/../../../../pic32mx/lib/speed\libc.a(atol.o)
 .reginfo       0x00000000       0x18 c:/program files/microchip/mplabc32/v2.02/bin/../lib/gcc/pic32mx/4.5.1/../../../../pic32mx/lib/speed\libc.a(atol.o)
 .pdr           0x00000000       0x20 c:/program files/microchip/mplabc32/v2.02/bin/../lib/gcc/pic32mx/4.5.1/../../../../pic32mx/lib/speed\libc.a(atol.o)
 .mdebug.abi32  0x00000000        0x0 c:/program files/microchip/mplabc32/v2.02/bin/../lib/gcc/pic32mx/4.5.1/../../../../pic32mx/lib/speed\libc.a(atol.o)
 .text          0x00000000        0x0 c:/program files/microchip/mplabc32/v2.02/bin/../lib/gcc/pic32mx/4.5.1/../../../../pic32mx/lib/speed\libc.a(ctime.o)
 .data          0x00000000        0x0 c:/program files/microchip/mplabc32/v2.02/bin/../lib/gcc/pic32mx/4.5.1/../../../../pic32mx/lib/speed\libc.a(ctime.o)
 .reginfo       0x00000000       0x18 c:/program files/microchip/mplabc32/v2.02/bin/../lib/gcc/pic32mx/4.5.1/../../../../pic32mx/lib/speed\libc.a(ctime.o)
 .pdr           0x00000000       0x80 c:/program files/microchip/mplabc32/v2.02/bin/../lib/gcc/pic32mx/4.5.1/../../../../pic32mx/lib/speed\libc.a(ctime.o)
 .mdebug.abi32  0x00000000        0x0 c:/program files/microchip/mplabc32/v2.02/bin/../lib/gcc/pic32mx/4.5.1/../../../../pic32mx/lib/speed\libc.a(ctime.o)
 .text.asctime  0x00000000      0x2f0 c:/program files/microchip/mplabc32/v2.02/bin/../lib/gcc/pic32mx/4.5.1/../../../../pic32mx/lib/speed\libc.a(ctime.o)
 .text.ctime    0x00000000       0x20 c:/program files/microchip/mplabc32/v2.02/bin/../lib/gcc/pic32mx/4.5.1/../../../../pic32mx/lib/speed\libc.a(ctime.o)
 .text          0x00000000        0x0 c:/program files/microchip/mplabc32/v2.02/bin/../lib/gcc/pic32mx/4.5.1/../../../../pic32mx/lib/speed\libc.a(ctype.o)
 .data          0x00000000        0x0 c:/program files/microchip/mplabc32/v2.02/bin/../lib/gcc/pic32mx/4.5.1/../../../../pic32mx/lib/speed\libc.a(ctype.o)
 .bss           0x00000000        0x0 c:/program files/microchip/mplabc32/v2.02/bin/../lib/gcc/pic32mx/4.5.1/../../../../pic32mx/lib/speed\libc.a(ctype.o)
 .reginfo       0x00000000       0x18 c:/program files/microchip/mplabc32/v2.02/bin/../lib/gcc/pic32mx/4.5.1/../../../../pic32mx/lib/speed\libc.a(ctype.o)
 .pdr           0x00000000        0x0 c:/program files/microchip/mplabc32/v2.02/bin/../lib/gcc/pic32mx/4.5.1/../../../../pic32mx/lib/speed\libc.a(ctype.o)
 .mdebug.abi32  0x00000000        0x0 c:/program files/microchip/mplabc32/v2.02/bin/../lib/gcc/pic32mx/4.5.1/../../../../pic32mx/lib/speed\libc.a(ctype.o)
 .text          0x00000000        0x0 c:/program files/microchip/mplabc32/v2.02/bin/../lib/gcc/pic32mx/4.5.1/../../../../pic32mx/lib/speed\libc.a(ctypef.o)
 .data          0x00000000        0x0 c:/program files/microchip/mplabc32/v2.02/bin/../lib/gcc/pic32mx/4.5.1/../../../../pic32mx/lib/speed\libc.a(ctypef.o)
 .bss           0x00000000        0x0 c:/program files/microchip/mplabc32/v2.02/bin/../lib/gcc/pic32mx/4.5.1/../../../../pic32mx/lib/speed\libc.a(ctypef.o)
 .reginfo       0x00000000       0x18 c:/program files/microchip/mplabc32/v2.02/bin/../lib/gcc/pic32mx/4.5.1/../../../../pic32mx/lib/speed\libc.a(ctypef.o)
 .pdr           0x00000000      0x220 c:/program files/microchip/mplabc32/v2.02/bin/../lib/gcc/pic32mx/4.5.1/../../../../pic32mx/lib/speed\libc.a(ctypef.o)
 .mdebug.abi32  0x00000000        0x0 c:/program files/microchip/mplabc32/v2.02/bin/../lib/gcc/pic32mx/4.5.1/../../../../pic32mx/lib/speed\libc.a(ctypef.o)
 .text.isalnum  0x00000000       0x18 c:/program files/microchip/mplabc32/v2.02/bin/../lib/gcc/pic32mx/4.5.1/../../../../pic32mx/lib/speed\libc.a(ctypef.o)
 .text.isalpha  0x00000000       0x18 c:/program files/microchip/mplabc32/v2.02/bin/../lib/gcc/pic32mx/4.5.1/../../../../pic32mx/lib/speed\libc.a(ctypef.o)
 .text.isascii  0x00000000        0x8 c:/program files/microchip/mplabc32/v2.02/bin/../lib/gcc/pic32mx/4.5.1/../../../../pic32mx/lib/speed\libc.a(ctypef.o)
 .text.iscntrl  0x00000000       0x18 c:/program files/microchip/mplabc32/v2.02/bin/../lib/gcc/pic32mx/4.5.1/../../../../pic32mx/lib/speed\libc.a(ctypef.o)
 .text.isdigit  0x00000000       0x18 c:/program files/microchip/mplabc32/v2.02/bin/../lib/gcc/pic32mx/4.5.1/../../../../pic32mx/lib/speed\libc.a(ctypef.o)
 .text.isgraph  0x00000000       0x18 c:/program files/microchip/mplabc32/v2.02/bin/../lib/gcc/pic32mx/4.5.1/../../../../pic32mx/lib/speed\libc.a(ctypef.o)
 .text.islower  0x00000000       0x18 c:/program files/microchip/mplabc32/v2.02/bin/../lib/gcc/pic32mx/4.5.1/../../../../pic32mx/lib/speed\libc.a(ctypef.o)
 .text.isprint  0x00000000       0x18 c:/program files/microchip/mplabc32/v2.02/bin/../lib/gcc/pic32mx/4.5.1/../../../../pic32mx/lib/speed\libc.a(ctypef.o)
 .text.ispunct  0x00000000       0x18 c:/program files/microchip/mplabc32/v2.02/bin/../lib/gcc/pic32mx/4.5.1/../../../../pic32mx/lib/speed\libc.a(ctypef.o)
 .text.isspace  0x00000000       0x18 c:/program files/microchip/mplabc32/v2.02/bin/../lib/gcc/pic32mx/4.5.1/../../../../pic32mx/lib/speed\libc.a(ctypef.o)
 .text.isupper  0x00000000       0x18 c:/program files/microchip/mplabc32/v2.02/bin/../lib/gcc/pic32mx/4.5.1/../../../../pic32mx/lib/speed\libc.a(ctypef.o)
 .text.isxdigit
                0x00000000       0x18 c:/program files/microchip/mplabc32/v2.02/bin/../lib/gcc/pic32mx/4.5.1/../../../../pic32mx/lib/speed\libc.a(ctypef.o)
 .text.toascii  0x00000000        0x8 c:/program files/microchip/mplabc32/v2.02/bin/../lib/gcc/pic32mx/4.5.1/../../../../pic32mx/lib/speed\libc.a(ctypef.o)
 .text._tolower
                0x00000000        0x8 c:/program files/microchip/mplabc32/v2.02/bin/../lib/gcc/pic32mx/4.5.1/../../../../pic32mx/lib/speed\libc.a(ctypef.o)
 .text._toupper
                0x00000000        0x8 c:/program files/microchip/mplabc32/v2.02/bin/../lib/gcc/pic32mx/4.5.1/../../../../pic32mx/lib/speed\libc.a(ctypef.o)
 .text          0x00000000        0x0 c:/program files/microchip/mplabc32/v2.02/bin/../lib/gcc/pic32mx/4.5.1/../../../../pic32mx/lib/speed\libc.a(strcat.o)
 .data          0x00000000        0x0 c:/program files/microchip/mplabc32/v2.02/bin/../lib/gcc/pic32mx/4.5.1/../../../../pic32mx/lib/speed\libc.a(strcat.o)
 .bss           0x00000000        0x0 c:/program files/microchip/mplabc32/v2.02/bin/../lib/gcc/pic32mx/4.5.1/../../../../pic32mx/lib/speed\libc.a(strcat.o)
 .reginfo       0x00000000       0x18 c:/program files/microchip/mplabc32/v2.02/bin/../lib/gcc/pic32mx/4.5.1/../../../../pic32mx/lib/speed\libc.a(strcat.o)
 .pdr           0x00000000       0x20 c:/program files/microchip/mplabc32/v2.02/bin/../lib/gcc/pic32mx/4.5.1/../../../../pic32mx/lib/speed\libc.a(strcat.o)
 .mdebug.abi32  0x00000000        0x0 c:/program files/microchip/mplabc32/v2.02/bin/../lib/gcc/pic32mx/4.5.1/../../../../pic32mx/lib/speed\libc.a(strcat.o)
 .text          0x00000000        0x0 c:/program files/microchip/mplabc32/v2.02/bin/../lib/gcc/pic32mx/4.5.1/../../../../pic32mx/lib/speed\libc.a(strchr.o)
 .data          0x00000000        0x0 c:/program files/microchip/mplabc32/v2.02/bin/../lib/gcc/pic32mx/4.5.1/../../../../pic32mx/lib/speed\libc.a(strchr.o)
 .bss           0x00000000        0x0 c:/program files/microchip/mplabc32/v2.02/bin/../lib/gcc/pic32mx/4.5.1/../../../../pic32mx/lib/speed\libc.a(strchr.o)
 .reginfo       0x00000000       0x18 c:/program files/microchip/mplabc32/v2.02/bin/../lib/gcc/pic32mx/4.5.1/../../../../pic32mx/lib/speed\libc.a(strchr.o)
 .pdr           0x00000000       0x20 c:/program files/microchip/mplabc32/v2.02/bin/../lib/gcc/pic32mx/4.5.1/../../../../pic32mx/lib/speed\libc.a(strchr.o)
 .mdebug.abi32  0x00000000        0x0 c:/program files/microchip/mplabc32/v2.02/bin/../lib/gcc/pic32mx/4.5.1/../../../../pic32mx/lib/speed\libc.a(strchr.o)
 .text          0x00000000        0x0 c:/program files/microchip/mplabc32/v2.02/bin/../lib/gcc/pic32mx/4.5.1/../../../../pic32mx/lib/speed\libc.a(strncpy.o)
 .data          0x00000000        0x0 c:/program files/microchip/mplabc32/v2.02/bin/../lib/gcc/pic32mx/4.5.1/../../../../pic32mx/lib/speed\libc.a(strncpy.o)
 .bss           0x00000000        0x0 c:/program files/microchip/mplabc32/v2.02/bin/../lib/gcc/pic32mx/4.5.1/../../../../pic32mx/lib/speed\libc.a(strncpy.o)
 .reginfo       0x00000000       0x18 c:/program files/microchip/mplabc32/v2.02/bin/../lib/gcc/pic32mx/4.5.1/../../../../pic32mx/lib/speed\libc.a(strncpy.o)
 .pdr           0x00000000       0x20 c:/program files/microchip/mplabc32/v2.02/bin/../lib/gcc/pic32mx/4.5.1/../../../../pic32mx/lib/speed\libc.a(strncpy.o)
 .mdebug.abi32  0x00000000        0x0 c:/program files/microchip/mplabc32/v2.02/bin/../lib/gcc/pic32mx/4.5.1/../../../../pic32mx/lib/speed\libc.a(strncpy.o)
 .text          0x00000000        0x0 c:/program files/microchip/mplabc32/v2.02/bin/../lib/gcc/pic32mx/4.5.1/../../../../pic32mx/lib/speed\libc.a(strstr.o)
 .data          0x00000000        0x0 c:/program files/microchip/mplabc32/v2.02/bin/../lib/gcc/pic32mx/4.5.1/../../../../pic32mx/lib/speed\libc.a(strstr.o)
 .bss           0x00000000        0x0 c:/program files/microchip/mplabc32/v2.02/bin/../lib/gcc/pic32mx/4.5.1/../../../../pic32mx/lib/speed\libc.a(strstr.o)
 .reginfo       0x00000000       0x18 c:/program files/microchip/mplabc32/v2.02/bin/../lib/gcc/pic32mx/4.5.1/../../../../pic32mx/lib/speed\libc.a(strstr.o)
 .pdr           0x00000000       0x20 c:/program files/microchip/mplabc32/v2.02/bin/../lib/gcc/pic32mx/4.5.1/../../../../pic32mx/lib/speed\libc.a(strstr.o)
 .mdebug.abi32  0x00000000        0x0 c:/program files/microchip/mplabc32/v2.02/bin/../lib/gcc/pic32mx/4.5.1/../../../../pic32mx/lib/speed\libc.a(strstr.o)
 .text          0x00000000        0x0 c:/program files/microchip/mplabc32/v2.02/bin/../lib/gcc/pic32mx/4.5.1/../../../../pic32mx/lib/speed\libc.a(atof.o)
 .data          0x00000000        0x0 c:/program files/microchip/mplabc32/v2.02/bin/../lib/gcc/pic32mx/4.5.1/../../../../pic32mx/lib/speed\libc.a(atof.o)
 .bss           0x00000000        0x0 c:/program files/microchip/mplabc32/v2.02/bin/../lib/gcc/pic32mx/4.5.1/../../../../pic32mx/lib/speed\libc.a(atof.o)
 .reginfo       0x00000000       0x18 c:/program files/microchip/mplabc32/v2.02/bin/../lib/gcc/pic32mx/4.5.1/../../../../pic32mx/lib/speed\libc.a(atof.o)
 .pdr           0x00000000       0x20 c:/program files/microchip/mplabc32/v2.02/bin/../lib/gcc/pic32mx/4.5.1/../../../../pic32mx/lib/speed\libc.a(atof.o)
 .mdebug.abi32  0x00000000        0x0 c:/program files/microchip/mplabc32/v2.02/bin/../lib/gcc/pic32mx/4.5.1/../../../../pic32mx/lib/speed\libc.a(atof.o)
 .text          0x00000000        0x0 c:/program files/microchip/mplabc32/v2.02/bin/../lib/gcc/pic32mx/4.5.1/../../../../pic32mx/lib/speed\libc.a(sprintf_cdnopsuxX.eo)
 .data          0x00000000        0x0 c:/program files/microchip/mplabc32/v2.02/bin/../lib/gcc/pic32mx/4.5.1/../../../../pic32mx/lib/speed\libc.a(sprintf_cdnopsuxX.eo)
 .bss           0x00000000        0x0 c:/program files/microchip/mplabc32/v2.02/bin/../lib/gcc/pic32mx/4.5.1/../../../../pic32mx/lib/speed\libc.a(sprintf_cdnopsuxX.eo)
 .reginfo       0x00000000       0x18 c:/program files/microchip/mplabc32/v2.02/bin/../lib/gcc/pic32mx/4.5.1/../../../../pic32mx/lib/speed\libc.a(sprintf_cdnopsuxX.eo)
 .pdr           0x00000000       0x20 c:/program files/microchip/mplabc32/v2.02/bin/../lib/gcc/pic32mx/4.5.1/../../../../pic32mx/lib/speed\libc.a(sprintf_cdnopsuxX.eo)
 .mdebug.abi32  0x00000000        0x0 c:/program files/microchip/mplabc32/v2.02/bin/../lib/gcc/pic32mx/4.5.1/../../../../pic32mx/lib/speed\libc.a(sprintf_cdnopsuxX.eo)
 .text          0x00000000        0x0 c:/program files/microchip/mplabc32/v2.02/bin/../lib/gcc/pic32mx/4.5.1/../../../../pic32mx/lib/speed\libc.a(default-bootstrap-exception-handler.o)
 .data          0x00000000        0x0 c:/program files/microchip/mplabc32/v2.02/bin/../lib/gcc/pic32mx/4.5.1/../../../../pic32mx/lib/speed\libc.a(default-bootstrap-exception-handler.o)
 .bss           0x00000000        0x0 c:/program files/microchip/mplabc32/v2.02/bin/../lib/gcc/pic32mx/4.5.1/../../../../pic32mx/lib/speed\libc.a(default-bootstrap-exception-handler.o)
 .reginfo       0x00000000       0x18 c:/program files/microchip/mplabc32/v2.02/bin/../lib/gcc/pic32mx/4.5.1/../../../../pic32mx/lib/speed\libc.a(default-bootstrap-exception-handler.o)
 .pdr           0x00000000       0x20 c:/program files/microchip/mplabc32/v2.02/bin/../lib/gcc/pic32mx/4.5.1/../../../../pic32mx/lib/speed\libc.a(default-bootstrap-exception-handler.o)
 .mdebug.abi32  0x00000000        0x0 c:/program files/microchip/mplabc32/v2.02/bin/../lib/gcc/pic32mx/4.5.1/../../../../pic32mx/lib/speed\libc.a(default-bootstrap-exception-handler.o)
 .text          0x00000000        0x0 c:/program files/microchip/mplabc32/v2.02/bin/../lib/gcc/pic32mx/4.5.1/../../../../pic32mx/lib/speed\libc.a(default-on-reset.o)
 .data          0x00000000        0x0 c:/program files/microchip/mplabc32/v2.02/bin/../lib/gcc/pic32mx/4.5.1/../../../../pic32mx/lib/speed\libc.a(default-on-reset.o)
 .bss           0x00000000        0x0 c:/program files/microchip/mplabc32/v2.02/bin/../lib/gcc/pic32mx/4.5.1/../../../../pic32mx/lib/speed\libc.a(default-on-reset.o)
 .reginfo       0x00000000       0x18 c:/program files/microchip/mplabc32/v2.02/bin/../lib/gcc/pic32mx/4.5.1/../../../../pic32mx/lib/speed\libc.a(default-on-reset.o)
 .pdr           0x00000000       0x20 c:/program files/microchip/mplabc32/v2.02/bin/../lib/gcc/pic32mx/4.5.1/../../../../pic32mx/lib/speed\libc.a(default-on-reset.o)
 .mdebug.abi32  0x00000000        0x0 c:/program files/microchip/mplabc32/v2.02/bin/../lib/gcc/pic32mx/4.5.1/../../../../pic32mx/lib/speed\libc.a(default-on-reset.o)
 .text          0x00000000        0x0 c:/program files/microchip/mplabc32/v2.02/bin/../lib/gcc/pic32mx/4.5.1/../../../../pic32mx/lib/speed\libc.a(default-on-bootstrap.o)
 .data          0x00000000        0x0 c:/program files/microchip/mplabc32/v2.02/bin/../lib/gcc/pic32mx/4.5.1/../../../../pic32mx/lib/speed\libc.a(default-on-bootstrap.o)
 .bss           0x00000000        0x0 c:/program files/microchip/mplabc32/v2.02/bin/../lib/gcc/pic32mx/4.5.1/../../../../pic32mx/lib/speed\libc.a(default-on-bootstrap.o)
 .reginfo       0x00000000       0x18 c:/program files/microchip/mplabc32/v2.02/bin/../lib/gcc/pic32mx/4.5.1/../../../../pic32mx/lib/speed\libc.a(default-on-bootstrap.o)
 .pdr           0x00000000       0x20 c:/program files/microchip/mplabc32/v2.02/bin/../lib/gcc/pic32mx/4.5.1/../../../../pic32mx/lib/speed\libc.a(default-on-bootstrap.o)
 .mdebug.abi32  0x00000000        0x0 c:/program files/microchip/mplabc32/v2.02/bin/../lib/gcc/pic32mx/4.5.1/../../../../pic32mx/lib/speed\libc.a(default-on-bootstrap.o)
 .data          0x00000000        0x0 c:/program files/microchip/mplabc32/v2.02/bin/../lib/gcc/pic32mx/4.5.1/../../../../pic32mx/lib/speed\libc.a(default-nmi-handler.o)
 .bss           0x00000000        0x0 c:/program files/microchip/mplabc32/v2.02/bin/../lib/gcc/pic32mx/4.5.1/../../../../pic32mx/lib/speed\libc.a(default-nmi-handler.o)
 .reginfo       0x00000000       0x18 c:/program files/microchip/mplabc32/v2.02/bin/../lib/gcc/pic32mx/4.5.1/../../../../pic32mx/lib/speed\libc.a(default-nmi-handler.o)
 .pdr           0x00000000       0x20 c:/program files/microchip/mplabc32/v2.02/bin/../lib/gcc/pic32mx/4.5.1/../../../../pic32mx/lib/speed\libc.a(default-nmi-handler.o)
 .text          0x00000000        0x0 c:/program files/microchip/mplabc32/v2.02/bin/../lib/gcc/pic32mx/4.5.1/../../../../pic32mx/lib/speed\libc.a(strncmp.o)
 .data          0x00000000        0x0 c:/program files/microchip/mplabc32/v2.02/bin/../lib/gcc/pic32mx/4.5.1/../../../../pic32mx/lib/speed\libc.a(strncmp.o)
 .bss           0x00000000        0x0 c:/program files/microchip/mplabc32/v2.02/bin/../lib/gcc/pic32mx/4.5.1/../../../../pic32mx/lib/speed\libc.a(strncmp.o)
 .reginfo       0x00000000       0x18 c:/program files/microchip/mplabc32/v2.02/bin/../lib/gcc/pic32mx/4.5.1/../../../../pic32mx/lib/speed\libc.a(strncmp.o)
 .pdr           0x00000000       0x20 c:/program files/microchip/mplabc32/v2.02/bin/../lib/gcc/pic32mx/4.5.1/../../../../pic32mx/lib/speed\libc.a(strncmp.o)
 .mdebug.abi32  0x00000000        0x0 c:/program files/microchip/mplabc32/v2.02/bin/../lib/gcc/pic32mx/4.5.1/../../../../pic32mx/lib/speed\libc.a(strncmp.o)
 .text          0x00000000        0x0 c:/program files/microchip/mplabc32/v2.02/bin/../lib/gcc/pic32mx/4.5.1/../../../../pic32mx/lib/speed\libc.a(strtod.o)
 .data          0x00000000        0x0 c:/program files/microchip/mplabc32/v2.02/bin/../lib/gcc/pic32mx/4.5.1/../../../../pic32mx/lib/speed\libc.a(strtod.o)
 .bss           0x00000000        0x0 c:/program files/microchip/mplabc32/v2.02/bin/../lib/gcc/pic32mx/4.5.1/../../../../pic32mx/lib/speed\libc.a(strtod.o)
 .reginfo       0x00000000       0x18 c:/program files/microchip/mplabc32/v2.02/bin/../lib/gcc/pic32mx/4.5.1/../../../../pic32mx/lib/speed\libc.a(strtod.o)
 .pdr           0x00000000       0x40 c:/program files/microchip/mplabc32/v2.02/bin/../lib/gcc/pic32mx/4.5.1/../../../../pic32mx/lib/speed\libc.a(strtod.o)
 .mdebug.abi32  0x00000000        0x0 c:/program files/microchip/mplabc32/v2.02/bin/../lib/gcc/pic32mx/4.5.1/../../../../pic32mx/lib/speed\libc.a(strtod.o)
 .text.strtod   0x00000000       0x1c c:/program files/microchip/mplabc32/v2.02/bin/../lib/gcc/pic32mx/4.5.1/../../../../pic32mx/lib/speed\libc.a(strtod.o)
 .text          0x00000000        0x0 c:/program files/microchip/mplabc32/v2.02/bin/../lib/gcc/pic32mx/4.5.1/../../../../pic32mx/lib/speed\libc.a(doprnt_cdnopsuxX.eo)
 .data          0x00000000        0x0 c:/program files/microchip/mplabc32/v2.02/bin/../lib/gcc/pic32mx/4.5.1/../../../../pic32mx/lib/speed\libc.a(doprnt_cdnopsuxX.eo)
 .bss           0x00000000        0x0 c:/program files/microchip/mplabc32/v2.02/bin/../lib/gcc/pic32mx/4.5.1/../../../../pic32mx/lib/speed\libc.a(doprnt_cdnopsuxX.eo)
 .reginfo       0x00000000       0x18 c:/program files/microchip/mplabc32/v2.02/bin/../lib/gcc/pic32mx/4.5.1/../../../../pic32mx/lib/speed\libc.a(doprnt_cdnopsuxX.eo)
 .pdr           0x00000000       0x20 c:/program files/microchip/mplabc32/v2.02/bin/../lib/gcc/pic32mx/4.5.1/../../../../pic32mx/lib/speed\libc.a(doprnt_cdnopsuxX.eo)
 .mdebug.abi32  0x00000000        0x0 c:/program files/microchip/mplabc32/v2.02/bin/../lib/gcc/pic32mx/4.5.1/../../../../pic32mx/lib/speed\libc.a(doprnt_cdnopsuxX.eo)
 .text          0x00000000        0x0 c:/program files/microchip/mplabc32/v2.02/bin/../lib/gcc/pic32mx/4.5.1/../../../../pic32mx/lib/speed\libc.a(_fputc_simple.o)
 .data          0x00000000        0x0 c:/program files/microchip/mplabc32/v2.02/bin/../lib/gcc/pic32mx/4.5.1/../../../../pic32mx/lib/speed\libc.a(_fputc_simple.o)
 .bss           0x00000000        0x0 c:/program files/microchip/mplabc32/v2.02/bin/../lib/gcc/pic32mx/4.5.1/../../../../pic32mx/lib/speed\libc.a(_fputc_simple.o)
 .reginfo       0x00000000       0x18 c:/program files/microchip/mplabc32/v2.02/bin/../lib/gcc/pic32mx/4.5.1/../../../../pic32mx/lib/speed\libc.a(_fputc_simple.o)
 .pdr           0x00000000       0x20 c:/program files/microchip/mplabc32/v2.02/bin/../lib/gcc/pic32mx/4.5.1/../../../../pic32mx/lib/speed\libc.a(_fputc_simple.o)
 .mdebug.abi32  0x00000000        0x0 c:/program files/microchip/mplabc32/v2.02/bin/../lib/gcc/pic32mx/4.5.1/../../../../pic32mx/lib/speed\libc.a(_fputc_simple.o)
 .text          0x00000000        0x0 c:/program files/microchip/mplabc32/v2.02/bin/../lib/gcc/pic32mx/4.5.1/../../../../pic32mx/lib/speed\libc.a(write.o)
 .data          0x00000000        0x0 c:/program files/microchip/mplabc32/v2.02/bin/../lib/gcc/pic32mx/4.5.1/../../../../pic32mx/lib/speed\libc.a(write.o)
 .bss           0x00000000        0x0 c:/program files/microchip/mplabc32/v2.02/bin/../lib/gcc/pic32mx/4.5.1/../../../../pic32mx/lib/speed\libc.a(write.o)
 .reginfo       0x00000000       0x18 c:/program files/microchip/mplabc32/v2.02/bin/../lib/gcc/pic32mx/4.5.1/../../../../pic32mx/lib/speed\libc.a(write.o)
 .pdr           0x00000000       0x20 c:/program files/microchip/mplabc32/v2.02/bin/../lib/gcc/pic32mx/4.5.1/../../../../pic32mx/lib/speed\libc.a(write.o)
 .mdebug.abi32  0x00000000        0x0 c:/program files/microchip/mplabc32/v2.02/bin/../lib/gcc/pic32mx/4.5.1/../../../../pic32mx/lib/speed\libc.a(write.o)
 .text          0x00000000        0x0 c:/program files/microchip/mplabc32/v2.02/bin/../lib/gcc/pic32mx/4.5.1/../../../../pic32mx/lib/speed\libc.a(_iob.o)
 .data          0x00000000       0xa0 c:/program files/microchip/mplabc32/v2.02/bin/../lib/gcc/pic32mx/4.5.1/../../../../pic32mx/lib/speed\libc.a(_iob.o)
 .reginfo       0x00000000       0x18 c:/program files/microchip/mplabc32/v2.02/bin/../lib/gcc/pic32mx/4.5.1/../../../../pic32mx/lib/speed\libc.a(_iob.o)
 .pdr           0x00000000        0x0 c:/program files/microchip/mplabc32/v2.02/bin/../lib/gcc/pic32mx/4.5.1/../../../../pic32mx/lib/speed\libc.a(_iob.o)
 .mdebug.abi32  0x00000000        0x0 c:/program files/microchip/mplabc32/v2.02/bin/../lib/gcc/pic32mx/4.5.1/../../../../pic32mx/lib/speed\libc.a(_iob.o)
 .sdata         0x00000000        0x4 c:/program files/microchip/mplabc32/v2.02/bin/../lib/gcc/pic32mx/4.5.1/../../../../pic32mx/lib/speed\libc.a(_iob.o)
 .text          0x00000000        0x0 c:/program files/microchip/mplabc32/v2.02/bin/../lib/gcc/pic32mx/4.5.1/../../../../pic32mx/lib/speed\libc.a(_flsbuf_simple.o)
 .data          0x00000000        0x0 c:/program files/microchip/mplabc32/v2.02/bin/../lib/gcc/pic32mx/4.5.1/../../../../pic32mx/lib/speed\libc.a(_flsbuf_simple.o)
 .bss           0x00000000        0x0 c:/program files/microchip/mplabc32/v2.02/bin/../lib/gcc/pic32mx/4.5.1/../../../../pic32mx/lib/speed\libc.a(_flsbuf_simple.o)
 .reginfo       0x00000000       0x18 c:/program files/microchip/mplabc32/v2.02/bin/../lib/gcc/pic32mx/4.5.1/../../../../pic32mx/lib/speed\libc.a(_flsbuf_simple.o)
 .pdr           0x00000000       0x20 c:/program files/microchip/mplabc32/v2.02/bin/../lib/gcc/pic32mx/4.5.1/../../../../pic32mx/lib/speed\libc.a(_flsbuf_simple.o)
 .mdebug.abi32  0x00000000        0x0 c:/program files/microchip/mplabc32/v2.02/bin/../lib/gcc/pic32mx/4.5.1/../../../../pic32mx/lib/speed\libc.a(_flsbuf_simple.o)
 .text          0x00000000        0x0 c:/program files/microchip/mplabc32/v2.02/bin/../lib/gcc/pic32mx/4.5.1/../../../../pic32mx/lib/speed\libc.a(_mon_putc.o)
 .data          0x00000000        0x0 c:/program files/microchip/mplabc32/v2.02/bin/../lib/gcc/pic32mx/4.5.1/../../../../pic32mx/lib/speed\libc.a(_mon_putc.o)
 .bss           0x00000000        0x0 c:/program files/microchip/mplabc32/v2.02/bin/../lib/gcc/pic32mx/4.5.1/../../../../pic32mx/lib/speed\libc.a(_mon_putc.o)
 .reginfo       0x00000000       0x18 c:/program files/microchip/mplabc32/v2.02/bin/../lib/gcc/pic32mx/4.5.1/../../../../pic32mx/lib/speed\libc.a(_mon_putc.o)
 .pdr           0x00000000       0x20 c:/program files/microchip/mplabc32/v2.02/bin/../lib/gcc/pic32mx/4.5.1/../../../../pic32mx/lib/speed\libc.a(_mon_putc.o)
 .mdebug.abi32  0x00000000        0x0 c:/program files/microchip/mplabc32/v2.02/bin/../lib/gcc/pic32mx/4.5.1/../../../../pic32mx/lib/speed\libc.a(_mon_putc.o)
 .text          0x00000000        0x0 c:/program files/microchip/mplabc32/v2.02/bin/../lib/gcc/pic32mx/4.5.1/../../../../pic32mx/lib/speed\libc.a(c32_uart.o)
 .data          0x00000000        0x0 c:/program files/microchip/mplabc32/v2.02/bin/../lib/gcc/pic32mx/4.5.1/../../../../pic32mx/lib/speed\libc.a(c32_uart.o)
 .bss           0x00000000        0x0 c:/program files/microchip/mplabc32/v2.02/bin/../lib/gcc/pic32mx/4.5.1/../../../../pic32mx/lib/speed\libc.a(c32_uart.o)
 .reginfo       0x00000000       0x18 c:/program files/microchip/mplabc32/v2.02/bin/../lib/gcc/pic32mx/4.5.1/../../../../pic32mx/lib/speed\libc.a(c32_uart.o)
 .pdr           0x00000000        0x0 c:/program files/microchip/mplabc32/v2.02/bin/../lib/gcc/pic32mx/4.5.1/../../../../pic32mx/lib/speed\libc.a(c32_uart.o)
 .mdebug.abi32  0x00000000        0x0 c:/program files/microchip/mplabc32/v2.02/bin/../lib/gcc/pic32mx/4.5.1/../../../../pic32mx/lib/speed\libc.a(c32_uart.o)
 .data          0x00000000        0x0 c:/program files/microchip/mplabc32/v2.02/bin/../lib/gcc/pic32mx/4.5.1/../../../../pic32mx/lib/speed\libm.a(dp32.o)
 .bss           0x00000000        0x0 c:/program files/microchip/mplabc32/v2.02/bin/../lib/gcc/pic32mx/4.5.1/../../../../pic32mx/lib/speed\libm.a(dp32.o)
 .reginfo       0x00000000       0x18 c:/program files/microchip/mplabc32/v2.02/bin/../lib/gcc/pic32mx/4.5.1/../../../../pic32mx/lib/speed\libm.a(dp32.o)
 .pdr           0x00000000        0x0 c:/program files/microchip/mplabc32/v2.02/bin/../lib/gcc/pic32mx/4.5.1/../../../../pic32mx/lib/speed\libm.a(dp32.o)
 .data          0x00000000        0x0 c:/program files/microchip/mplabc32/v2.02/bin/../lib/gcc/pic32mx/4.5.1/../../../../pic32mx/lib/speed\libm.a(fp32.o)
 .bss           0x00000000        0x0 c:/program files/microchip/mplabc32/v2.02/bin/../lib/gcc/pic32mx/4.5.1/../../../../pic32mx/lib/speed\libm.a(fp32.o)
 .reginfo       0x00000000       0x18 c:/program files/microchip/mplabc32/v2.02/bin/../lib/gcc/pic32mx/4.5.1/../../../../pic32mx/lib/speed\libm.a(fp32.o)
 .pdr           0x00000000        0x0 c:/program files/microchip/mplabc32/v2.02/bin/../lib/gcc/pic32mx/4.5.1/../../../../pic32mx/lib/speed\libm.a(fp32.o)
 .text          0x00000000        0x0 c:/program files/microchip/mplabc32/v2.02/bin/../lib/gcc/pic32mx/4.5.1/../../../../pic32mx/lib/speed\libe.a(_strtod.o)
 .data          0x00000000        0x0 c:/program files/microchip/mplabc32/v2.02/bin/../lib/gcc/pic32mx/4.5.1/../../../../pic32mx/lib/speed\libe.a(_strtod.o)
 .bss           0x00000000        0x0 c:/program files/microchip/mplabc32/v2.02/bin/../lib/gcc/pic32mx/4.5.1/../../../../pic32mx/lib/speed\libe.a(_strtod.o)
 .reginfo       0x00000000       0x18 c:/program files/microchip/mplabc32/v2.02/bin/../lib/gcc/pic32mx/4.5.1/../../../../pic32mx/lib/speed\libe.a(_strtod.o)
 .pdr           0x00000000       0x20 c:/program files/microchip/mplabc32/v2.02/bin/../lib/gcc/pic32mx/4.5.1/../../../../pic32mx/lib/speed\libe.a(_strtod.o)
 .mdebug.abi32  0x00000000        0x0 c:/program files/microchip/mplabc32/v2.02/bin/../lib/gcc/pic32mx/4.5.1/../../../../pic32mx/lib/speed\libe.a(_strtod.o)
 .text          0x00000000        0x0 c:/program files/microchip/mplabc32/v2.02/bin/../lib/gcc/pic32mx/4.5.1/../../../../pic32mx/lib/speed\libe.a(_ldexp.o)
 .data          0x00000000        0x0 c:/program files/microchip/mplabc32/v2.02/bin/../lib/gcc/pic32mx/4.5.1/../../../../pic32mx/lib/speed\libe.a(_ldexp.o)
 .bss           0x00000000        0x0 c:/program files/microchip/mplabc32/v2.02/bin/../lib/gcc/pic32mx/4.5.1/../../../../pic32mx/lib/speed\libe.a(_ldexp.o)
 .reginfo       0x00000000       0x18 c:/program files/microchip/mplabc32/v2.02/bin/../lib/gcc/pic32mx/4.5.1/../../../../pic32mx/lib/speed\libe.a(_ldexp.o)
 .pdr           0x00000000       0x20 c:/program files/microchip/mplabc32/v2.02/bin/../lib/gcc/pic32mx/4.5.1/../../../../pic32mx/lib/speed\libe.a(_ldexp.o)
 .mdebug.abi32  0x00000000        0x0 c:/program files/microchip/mplabc32/v2.02/bin/../lib/gcc/pic32mx/4.5.1/../../../../pic32mx/lib/speed\libe.a(_ldexp.o)
 .text          0x00000000        0x0 c:/program files/microchip/mplabc32/v2.02/bin/../lib/gcc/pic32mx/4.5.1/../../../../pic32mx/lib/speed\libmchp_peripheral.a(read_core_timer_lib.o)
 .data          0x00000000        0x0 c:/program files/microchip/mplabc32/v2.02/bin/../lib/gcc/pic32mx/4.5.1/../../../../pic32mx/lib/speed\libmchp_peripheral.a(read_core_timer_lib.o)
 .bss           0x00000000        0x0 c:/program files/microchip/mplabc32/v2.02/bin/../lib/gcc/pic32mx/4.5.1/../../../../pic32mx/lib/speed\libmchp_peripheral.a(read_core_timer_lib.o)
 .reginfo       0x00000000       0x18 c:/program files/microchip/mplabc32/v2.02/bin/../lib/gcc/pic32mx/4.5.1/../../../../pic32mx/lib/speed\libmchp_peripheral.a(read_core_timer_lib.o)
 .pdr           0x00000000       0x20 c:/program files/microchip/mplabc32/v2.02/bin/../lib/gcc/pic32mx/4.5.1/../../../../pic32mx/lib/speed\libmchp_peripheral.a(read_core_timer_lib.o)
 .mdebug.abi32  0x00000000        0x0 c:/program files/microchip/mplabc32/v2.02/bin/../lib/gcc/pic32mx/4.5.1/../../../../pic32mx/lib/speed\libmchp_peripheral.a(read_core_timer_lib.o)
 .text          0x00000000        0x0 c:/program files/microchip/mplabc32/v2.02/bin/../lib/gcc/pic32mx/4.5.1/../../../../pic32mx/lib/speed\libmchp_peripheral.a(write_core_timer_lib.o)
 .data          0x00000000        0x0 c:/program files/microchip/mplabc32/v2.02/bin/../lib/gcc/pic32mx/4.5.1/../../../../pic32mx/lib/speed\libmchp_peripheral.a(write_core_timer_lib.o)
 .bss           0x00000000        0x0 c:/program files/microchip/mplabc32/v2.02/bin/../lib/gcc/pic32mx/4.5.1/../../../../pic32mx/lib/speed\libmchp_peripheral.a(write_core_timer_lib.o)
 .reginfo       0x00000000       0x18 c:/program files/microchip/mplabc32/v2.02/bin/../lib/gcc/pic32mx/4.5.1/../../../../pic32mx/lib/speed\libmchp_peripheral.a(write_core_timer_lib.o)
 .pdr           0x00000000       0x20 c:/program files/microchip/mplabc32/v2.02/bin/../lib/gcc/pic32mx/4.5.1/../../../../pic32mx/lib/speed\libmchp_peripheral.a(write_core_timer_lib.o)
 .mdebug.abi32  0x00000000        0x0 c:/program files/microchip/mplabc32/v2.02/bin/../lib/gcc/pic32mx/4.5.1/../../../../pic32mx/lib/speed\libmchp_peripheral.a(write_core_timer_lib.o)
 .text          0x00000000        0x0 c:/program files/microchip/mplabc32/v2.02/bin/../lib/gcc/pic32mx/4.5.1/../../../../pic32mx/lib/speed\libmchp_peripheral_32MX795F512L.a(eth_ack_packet_lib.o)
 .data          0x00000000        0x0 c:/program files/microchip/mplabc32/v2.02/bin/../lib/gcc/pic32mx/4.5.1/../../../../pic32mx/lib/speed\libmchp_peripheral_32MX795F512L.a(eth_ack_packet_lib.o)
 .bss           0x00000000        0x0 c:/program files/microchip/mplabc32/v2.02/bin/../lib/gcc/pic32mx/4.5.1/../../../../pic32mx/lib/speed\libmchp_peripheral_32MX795F512L.a(eth_ack_packet_lib.o)
 .reginfo       0x00000000       0x18 c:/program files/microchip/mplabc32/v2.02/bin/../lib/gcc/pic32mx/4.5.1/../../../../pic32mx/lib/speed\libmchp_peripheral_32MX795F512L.a(eth_ack_packet_lib.o)
 .pdr           0x00000000       0xc0 c:/program files/microchip/mplabc32/v2.02/bin/../lib/gcc/pic32mx/4.5.1/../../../../pic32mx/lib/speed\libmchp_peripheral_32MX795F512L.a(eth_ack_packet_lib.o)
 .mdebug.abi32  0x00000000        0x0 c:/program files/microchip/mplabc32/v2.02/bin/../lib/gcc/pic32mx/4.5.1/../../../../pic32mx/lib/speed\libmchp_peripheral_32MX795F512L.a(eth_ack_packet_lib.o)
 .text.EthRxAckBuffer
                0x00000000       0x1c c:/program files/microchip/mplabc32/v2.02/bin/../lib/gcc/pic32mx/4.5.1/../../../../pic32mx/lib/speed\libmchp_peripheral_32MX795F512L.a(eth_ack_packet_lib.o)
 .text.EthTxAckBuffer
                0x00000000       0x30 c:/program files/microchip/mplabc32/v2.02/bin/../lib/gcc/pic32mx/4.5.1/../../../../pic32mx/lib/speed\libmchp_peripheral_32MX795F512L.a(eth_ack_packet_lib.o)
 .text          0x00000000        0x0 c:/program files/microchip/mplabc32/v2.02/bin/../lib/gcc/pic32mx/4.5.1/../../../../pic32mx/lib/speed\libmchp_peripheral_32MX795F512L.a(eth_descriptors_add_lib.o)
 .data          0x00000000        0x0 c:/program files/microchip/mplabc32/v2.02/bin/../lib/gcc/pic32mx/4.5.1/../../../../pic32mx/lib/speed\libmchp_peripheral_32MX795F512L.a(eth_descriptors_add_lib.o)
 .bss           0x00000000        0x0 c:/program files/microchip/mplabc32/v2.02/bin/../lib/gcc/pic32mx/4.5.1/../../../../pic32mx/lib/speed\libmchp_peripheral_32MX795F512L.a(eth_descriptors_add_lib.o)
 .reginfo       0x00000000       0x18 c:/program files/microchip/mplabc32/v2.02/bin/../lib/gcc/pic32mx/4.5.1/../../../../pic32mx/lib/speed\libmchp_peripheral_32MX795F512L.a(eth_descriptors_add_lib.o)
 .pdr           0x00000000       0x40 c:/program files/microchip/mplabc32/v2.02/bin/../lib/gcc/pic32mx/4.5.1/../../../../pic32mx/lib/speed\libmchp_peripheral_32MX795F512L.a(eth_descriptors_add_lib.o)
 .mdebug.abi32  0x00000000        0x0 c:/program files/microchip/mplabc32/v2.02/bin/../lib/gcc/pic32mx/4.5.1/../../../../pic32mx/lib/speed\libmchp_peripheral_32MX795F512L.a(eth_descriptors_add_lib.o)
 .text.EthDescriptorsAdd
                0x00000000      0x12c c:/program files/microchip/mplabc32/v2.02/bin/../lib/gcc/pic32mx/4.5.1/../../../../pic32mx/lib/speed\libmchp_peripheral_32MX795F512L.a(eth_descriptors_add_lib.o)
 .text          0x00000000        0x0 c:/program files/microchip/mplabc32/v2.02/bin/../lib/gcc/pic32mx/4.5.1/../../../../pic32mx/lib/speed\libmchp_peripheral_32MX795F512L.a(eth_init_lib.o)
 .data          0x00000000        0x0 c:/program files/microchip/mplabc32/v2.02/bin/../lib/gcc/pic32mx/4.5.1/../../../../pic32mx/lib/speed\libmchp_peripheral_32MX795F512L.a(eth_init_lib.o)
 .bss           0x00000000        0x0 c:/program files/microchip/mplabc32/v2.02/bin/../lib/gcc/pic32mx/4.5.1/../../../../pic32mx/lib/speed\libmchp_peripheral_32MX795F512L.a(eth_init_lib.o)
 .reginfo       0x00000000       0x18 c:/program files/microchip/mplabc32/v2.02/bin/../lib/gcc/pic32mx/4.5.1/../../../../pic32mx/lib/speed\libmchp_peripheral_32MX795F512L.a(eth_init_lib.o)
 .pdr           0x00000000       0x20 c:/program files/microchip/mplabc32/v2.02/bin/../lib/gcc/pic32mx/4.5.1/../../../../pic32mx/lib/speed\libmchp_peripheral_32MX795F512L.a(eth_init_lib.o)
 .mdebug.abi32  0x00000000        0x0 c:/program files/microchip/mplabc32/v2.02/bin/../lib/gcc/pic32mx/4.5.1/../../../../pic32mx/lib/speed\libmchp_peripheral_32MX795F512L.a(eth_init_lib.o)
 .text          0x00000000        0x0 c:/program files/microchip/mplabc32/v2.02/bin/../lib/gcc/pic32mx/4.5.1/../../../../pic32mx/lib/speed\libmchp_peripheral_32MX795F512L.a(eth_mac_open_lib.o)
 .data          0x00000000        0x0 c:/program files/microchip/mplabc32/v2.02/bin/../lib/gcc/pic32mx/4.5.1/../../../../pic32mx/lib/speed\libmchp_peripheral_32MX795F512L.a(eth_mac_open_lib.o)
 .bss           0x00000000        0x0 c:/program files/microchip/mplabc32/v2.02/bin/../lib/gcc/pic32mx/4.5.1/../../../../pic32mx/lib/speed\libmchp_peripheral_32MX795F512L.a(eth_mac_open_lib.o)
 .reginfo       0x00000000       0x18 c:/program files/microchip/mplabc32/v2.02/bin/../lib/gcc/pic32mx/4.5.1/../../../../pic32mx/lib/speed\libmchp_peripheral_32MX795F512L.a(eth_mac_open_lib.o)
 .pdr           0x00000000       0x20 c:/program files/microchip/mplabc32/v2.02/bin/../lib/gcc/pic32mx/4.5.1/../../../../pic32mx/lib/speed\libmchp_peripheral_32MX795F512L.a(eth_mac_open_lib.o)
 .mdebug.abi32  0x00000000        0x0 c:/program files/microchip/mplabc32/v2.02/bin/../lib/gcc/pic32mx/4.5.1/../../../../pic32mx/lib/speed\libmchp_peripheral_32MX795F512L.a(eth_mac_open_lib.o)
 .text          0x00000000        0x0 c:/program files/microchip/mplabc32/v2.02/bin/../lib/gcc/pic32mx/4.5.1/../../../../pic32mx/lib/speed\libmchp_peripheral_32MX795F512L.a(eth_mac_set_address_max_lib.o)
 .data          0x00000000        0x0 c:/program files/microchip/mplabc32/v2.02/bin/../lib/gcc/pic32mx/4.5.1/../../../../pic32mx/lib/speed\libmchp_peripheral_32MX795F512L.a(eth_mac_set_address_max_lib.o)
 .bss           0x00000000        0x0 c:/program files/microchip/mplabc32/v2.02/bin/../lib/gcc/pic32mx/4.5.1/../../../../pic32mx/lib/speed\libmchp_peripheral_32MX795F512L.a(eth_mac_set_address_max_lib.o)
 .reginfo       0x00000000       0x18 c:/program files/microchip/mplabc32/v2.02/bin/../lib/gcc/pic32mx/4.5.1/../../../../pic32mx/lib/speed\libmchp_peripheral_32MX795F512L.a(eth_mac_set_address_max_lib.o)
 .pdr           0x00000000       0x60 c:/program files/microchip/mplabc32/v2.02/bin/../lib/gcc/pic32mx/4.5.1/../../../../pic32mx/lib/speed\libmchp_peripheral_32MX795F512L.a(eth_mac_set_address_max_lib.o)
 .mdebug.abi32  0x00000000        0x0 c:/program files/microchip/mplabc32/v2.02/bin/../lib/gcc/pic32mx/4.5.1/../../../../pic32mx/lib/speed\libmchp_peripheral_32MX795F512L.a(eth_mac_set_address_max_lib.o)
 .text.EthMACGetAddress
                0x00000000       0x44 c:/program files/microchip/mplabc32/v2.02/bin/../lib/gcc/pic32mx/4.5.1/../../../../pic32mx/lib/speed\libmchp_peripheral_32MX795F512L.a(eth_mac_set_address_max_lib.o)
 .text.EthMACSetMaxFrame
                0x00000000       0x14 c:/program files/microchip/mplabc32/v2.02/bin/../lib/gcc/pic32mx/4.5.1/../../../../pic32mx/lib/speed\libmchp_peripheral_32MX795F512L.a(eth_mac_set_address_max_lib.o)
 .text          0x00000000        0x0 c:/program files/microchip/mplabc32/v2.02/bin/../lib/gcc/pic32mx/4.5.1/../../../../pic32mx/lib/speed\libmchp_peripheral_32MX795F512L.a(eth_rx_buffers_append_lib.o)
 .data          0x00000000        0x0 c:/program files/microchip/mplabc32/v2.02/bin/../lib/gcc/pic32mx/4.5.1/../../../../pic32mx/lib/speed\libmchp_peripheral_32MX795F512L.a(eth_rx_buffers_append_lib.o)
 .bss           0x00000000        0x0 c:/program files/microchip/mplabc32/v2.02/bin/../lib/gcc/pic32mx/4.5.1/../../../../pic32mx/lib/speed\libmchp_peripheral_32MX795F512L.a(eth_rx_buffers_append_lib.o)
 .reginfo       0x00000000       0x18 c:/program files/microchip/mplabc32/v2.02/bin/../lib/gcc/pic32mx/4.5.1/../../../../pic32mx/lib/speed\libmchp_peripheral_32MX795F512L.a(eth_rx_buffers_append_lib.o)
 .pdr           0x00000000       0x20 c:/program files/microchip/mplabc32/v2.02/bin/../lib/gcc/pic32mx/4.5.1/../../../../pic32mx/lib/speed\libmchp_peripheral_32MX795F512L.a(eth_rx_buffers_append_lib.o)
 .mdebug.abi32  0x00000000        0x0 c:/program files/microchip/mplabc32/v2.02/bin/../lib/gcc/pic32mx/4.5.1/../../../../pic32mx/lib/speed\libmchp_peripheral_32MX795F512L.a(eth_rx_buffers_append_lib.o)
 .text          0x00000000        0x0 c:/program files/microchip/mplabc32/v2.02/bin/../lib/gcc/pic32mx/4.5.1/../../../../pic32mx/lib/speed\libmchp_peripheral_32MX795F512L.a(eth_rx_filters_lib.o)
 .data          0x00000000        0x0 c:/program files/microchip/mplabc32/v2.02/bin/../lib/gcc/pic32mx/4.5.1/../../../../pic32mx/lib/speed\libmchp_peripheral_32MX795F512L.a(eth_rx_filters_lib.o)
 .bss           0x00000000        0x0 c:/program files/microchip/mplabc32/v2.02/bin/../lib/gcc/pic32mx/4.5.1/../../../../pic32mx/lib/speed\libmchp_peripheral_32MX795F512L.a(eth_rx_filters_lib.o)
 .reginfo       0x00000000       0x18 c:/program files/microchip/mplabc32/v2.02/bin/../lib/gcc/pic32mx/4.5.1/../../../../pic32mx/lib/speed\libmchp_peripheral_32MX795F512L.a(eth_rx_filters_lib.o)
 .pdr           0x00000000       0xc0 c:/program files/microchip/mplabc32/v2.02/bin/../lib/gcc/pic32mx/4.5.1/../../../../pic32mx/lib/speed\libmchp_peripheral_32MX795F512L.a(eth_rx_filters_lib.o)
 .mdebug.abi32  0x00000000        0x0 c:/program files/microchip/mplabc32/v2.02/bin/../lib/gcc/pic32mx/4.5.1/../../../../pic32mx/lib/speed\libmchp_peripheral_32MX795F512L.a(eth_rx_filters_lib.o)
 .text.EthRxFiltersWrite
                0x00000000       0x10 c:/program files/microchip/mplabc32/v2.02/bin/../lib/gcc/pic32mx/4.5.1/../../../../pic32mx/lib/speed\libmchp_peripheral_32MX795F512L.a(eth_rx_filters_lib.o)
 .text.EthRxFiltersHTSet
                0x00000000       0x18 c:/program files/microchip/mplabc32/v2.02/bin/../lib/gcc/pic32mx/4.5.1/../../../../pic32mx/lib/speed\libmchp_peripheral_32MX795F512L.a(eth_rx_filters_lib.o)
 .text.EthRxFiltersPMSet
                0x00000000       0x6c c:/program files/microchip/mplabc32/v2.02/bin/../lib/gcc/pic32mx/4.5.1/../../../../pic32mx/lib/speed\libmchp_peripheral_32MX795F512L.a(eth_rx_filters_lib.o)
 .text.EthRxFiltersPMClr
                0x00000000       0x14 c:/program files/microchip/mplabc32/v2.02/bin/../lib/gcc/pic32mx/4.5.1/../../../../pic32mx/lib/speed\libmchp_peripheral_32MX795F512L.a(eth_rx_filters_lib.o)
 .text          0x00000000        0x0 c:/program files/microchip/mplabc32/v2.02/bin/../lib/gcc/pic32mx/4.5.1/../../../../pic32mx/lib/speed\libmchp_peripheral_32MX795F512L.a(eth_rx_get_packet_lib.o)
 .data          0x00000000        0x0 c:/program files/microchip/mplabc32/v2.02/bin/../lib/gcc/pic32mx/4.5.1/../../../../pic32mx/lib/speed\libmchp_peripheral_32MX795F512L.a(eth_rx_get_packet_lib.o)
 .bss           0x00000000        0x0 c:/program files/microchip/mplabc32/v2.02/bin/../lib/gcc/pic32mx/4.5.1/../../../../pic32mx/lib/speed\libmchp_peripheral_32MX795F512L.a(eth_rx_get_packet_lib.o)
 .reginfo       0x00000000       0x18 c:/program files/microchip/mplabc32/v2.02/bin/../lib/gcc/pic32mx/4.5.1/../../../../pic32mx/lib/speed\libmchp_peripheral_32MX795F512L.a(eth_rx_get_packet_lib.o)
 .pdr           0x00000000       0x40 c:/program files/microchip/mplabc32/v2.02/bin/../lib/gcc/pic32mx/4.5.1/../../../../pic32mx/lib/speed\libmchp_peripheral_32MX795F512L.a(eth_rx_get_packet_lib.o)
 .mdebug.abi32  0x00000000        0x0 c:/program files/microchip/mplabc32/v2.02/bin/../lib/gcc/pic32mx/4.5.1/../../../../pic32mx/lib/speed\libmchp_peripheral_32MX795F512L.a(eth_rx_get_packet_lib.o)
 .text          0x00000000        0x0 c:/program files/microchip/mplabc32/v2.02/bin/../lib/gcc/pic32mx/4.5.1/../../../../pic32mx/lib/speed\libmchp_peripheral_32MX795F512L.a(eth_rx_set_buffer_size_lib.o)
 .data          0x00000000        0x0 c:/program files/microchip/mplabc32/v2.02/bin/../lib/gcc/pic32mx/4.5.1/../../../../pic32mx/lib/speed\libmchp_peripheral_32MX795F512L.a(eth_rx_set_buffer_size_lib.o)
 .bss           0x00000000        0x0 c:/program files/microchip/mplabc32/v2.02/bin/../lib/gcc/pic32mx/4.5.1/../../../../pic32mx/lib/speed\libmchp_peripheral_32MX795F512L.a(eth_rx_set_buffer_size_lib.o)
 .reginfo       0x00000000       0x18 c:/program files/microchip/mplabc32/v2.02/bin/../lib/gcc/pic32mx/4.5.1/../../../../pic32mx/lib/speed\libmchp_peripheral_32MX795F512L.a(eth_rx_set_buffer_size_lib.o)
 .pdr           0x00000000       0x20 c:/program files/microchip/mplabc32/v2.02/bin/../lib/gcc/pic32mx/4.5.1/../../../../pic32mx/lib/speed\libmchp_peripheral_32MX795F512L.a(eth_rx_set_buffer_size_lib.o)
 .mdebug.abi32  0x00000000        0x0 c:/program files/microchip/mplabc32/v2.02/bin/../lib/gcc/pic32mx/4.5.1/../../../../pic32mx/lib/speed\libmchp_peripheral_32MX795F512L.a(eth_rx_set_buffer_size_lib.o)
 .text          0x00000000        0x0 c:/program files/microchip/mplabc32/v2.02/bin/../lib/gcc/pic32mx/4.5.1/../../../../pic32mx/lib/speed\libmchp_peripheral_32MX795F512L.a(eth_tx_packet_lib.o)
 .data          0x00000000        0x0 c:/program files/microchip/mplabc32/v2.02/bin/../lib/gcc/pic32mx/4.5.1/../../../../pic32mx/lib/speed\libmchp_peripheral_32MX795F512L.a(eth_tx_packet_lib.o)
 .bss           0x00000000        0x0 c:/program files/microchip/mplabc32/v2.02/bin/../lib/gcc/pic32mx/4.5.1/../../../../pic32mx/lib/speed\libmchp_peripheral_32MX795F512L.a(eth_tx_packet_lib.o)
 .reginfo       0x00000000       0x18 c:/program files/microchip/mplabc32/v2.02/bin/../lib/gcc/pic32mx/4.5.1/../../../../pic32mx/lib/speed\libmchp_peripheral_32MX795F512L.a(eth_tx_packet_lib.o)
 .pdr           0x00000000       0x80 c:/program files/microchip/mplabc32/v2.02/bin/../lib/gcc/pic32mx/4.5.1/../../../../pic32mx/lib/speed\libmchp_peripheral_32MX795F512L.a(eth_tx_packet_lib.o)
 .mdebug.abi32  0x00000000        0x0 c:/program files/microchip/mplabc32/v2.02/bin/../lib/gcc/pic32mx/4.5.1/../../../../pic32mx/lib/speed\libmchp_peripheral_32MX795F512L.a(eth_tx_packet_lib.o)
 .text.EthTxSendPacket
                0x00000000      0x278 c:/program files/microchip/mplabc32/v2.02/bin/../lib/gcc/pic32mx/4.5.1/../../../../pic32mx/lib/speed\libmchp_peripheral_32MX795F512L.a(eth_tx_packet_lib.o)
 .text.EthTxGetBufferStatus
                0x00000000       0x70 c:/program files/microchip/mplabc32/v2.02/bin/../lib/gcc/pic32mx/4.5.1/../../../../pic32mx/lib/speed\libmchp_peripheral_32MX795F512L.a(eth_tx_packet_lib.o)
 .text._EthFindPacket
                0x00000000       0x38 c:/program files/microchip/mplabc32/v2.02/bin/../lib/gcc/pic32mx/4.5.1/../../../../pic32mx/lib/speed\libmchp_peripheral_32MX795F512L.a(eth_tx_packet_lib.o)
 .text          0x00000000        0x0 c:/program files/microchip/mplabc32/v2.02/bin/../lib/gcc/pic32mx/4.5.1/../../../../pic32mx/lib/speed\libmchp_peripheral_32MX795F512L.a(_eth_append_busy_list_lib.o)
 .data          0x00000000        0x0 c:/program files/microchip/mplabc32/v2.02/bin/../lib/gcc/pic32mx/4.5.1/../../../../pic32mx/lib/speed\libmchp_peripheral_32MX795F512L.a(_eth_append_busy_list_lib.o)
 .bss           0x00000000        0x0 c:/program files/microchip/mplabc32/v2.02/bin/../lib/gcc/pic32mx/4.5.1/../../../../pic32mx/lib/speed\libmchp_peripheral_32MX795F512L.a(_eth_append_busy_list_lib.o)
 .reginfo       0x00000000       0x18 c:/program files/microchip/mplabc32/v2.02/bin/../lib/gcc/pic32mx/4.5.1/../../../../pic32mx/lib/speed\libmchp_peripheral_32MX795F512L.a(_eth_append_busy_list_lib.o)
 .pdr           0x00000000       0x20 c:/program files/microchip/mplabc32/v2.02/bin/../lib/gcc/pic32mx/4.5.1/../../../../pic32mx/lib/speed\libmchp_peripheral_32MX795F512L.a(_eth_append_busy_list_lib.o)
 .mdebug.abi32  0x00000000        0x0 c:/program files/microchip/mplabc32/v2.02/bin/../lib/gcc/pic32mx/4.5.1/../../../../pic32mx/lib/speed\libmchp_peripheral_32MX795F512L.a(_eth_append_busy_list_lib.o)
 .text          0x00000000        0x0 c:/program files/microchip/mplabc32/v2.02/bin/../lib/gcc/pic32mx/4.5.1/../../../../pic32mx/lib/speed\libmchp_peripheral_32MX795F512L.a(eth_miim_access.o)
 .data          0x00000000        0x0 c:/program files/microchip/mplabc32/v2.02/bin/../lib/gcc/pic32mx/4.5.1/../../../../pic32mx/lib/speed\libmchp_peripheral_32MX795F512L.a(eth_miim_access.o)
 .bss           0x00000000        0x0 c:/program files/microchip/mplabc32/v2.02/bin/../lib/gcc/pic32mx/4.5.1/../../../../pic32mx/lib/speed\libmchp_peripheral_32MX795F512L.a(eth_miim_access.o)
 .reginfo       0x00000000       0x18 c:/program files/microchip/mplabc32/v2.02/bin/../lib/gcc/pic32mx/4.5.1/../../../../pic32mx/lib/speed\libmchp_peripheral_32MX795F512L.a(eth_miim_access.o)
 .pdr           0x00000000       0xc0 c:/program files/microchip/mplabc32/v2.02/bin/../lib/gcc/pic32mx/4.5.1/../../../../pic32mx/lib/speed\libmchp_peripheral_32MX795F512L.a(eth_miim_access.o)
 .mdebug.abi32  0x00000000        0x0 c:/program files/microchip/mplabc32/v2.02/bin/../lib/gcc/pic32mx/4.5.1/../../../../pic32mx/lib/speed\libmchp_peripheral_32MX795F512L.a(eth_miim_access.o)
 .text          0x00000000        0x0 c:/program files/microchip/mplabc32/v2.02/bin/../lib/gcc/pic32mx/4.5.1/../../../../pic32mx/lib/speed\libmchp_peripheral_32MX795F512L.a(soft_reset_lib.o)
 .data          0x00000000        0x0 c:/program files/microchip/mplabc32/v2.02/bin/../lib/gcc/pic32mx/4.5.1/../../../../pic32mx/lib/speed\libmchp_peripheral_32MX795F512L.a(soft_reset_lib.o)
 .bss           0x00000000        0x0 c:/program files/microchip/mplabc32/v2.02/bin/../lib/gcc/pic32mx/4.5.1/../../../../pic32mx/lib/speed\libmchp_peripheral_32MX795F512L.a(soft_reset_lib.o)
 .reginfo       0x00000000       0x18 c:/program files/microchip/mplabc32/v2.02/bin/../lib/gcc/pic32mx/4.5.1/../../../../pic32mx/lib/speed\libmchp_peripheral_32MX795F512L.a(soft_reset_lib.o)
 .pdr           0x00000000       0x20 c:/program files/microchip/mplabc32/v2.02/bin/../lib/gcc/pic32mx/4.5.1/../../../../pic32mx/lib/speed\libmchp_peripheral_32MX795F512L.a(soft_reset_lib.o)
 .mdebug.abi32  0x00000000        0x0 c:/program files/microchip/mplabc32/v2.02/bin/../lib/gcc/pic32mx/4.5.1/../../../../pic32mx/lib/speed\libmchp_peripheral_32MX795F512L.a(soft_reset_lib.o)
 .text          0x00000000        0x0 c:/program files/microchip/mplabc32/v2.02/bin/../lib/gcc/pic32mx/4.5.1/../../../../pic32mx/lib/speed\libmchp_peripheral_32MX795F512L.a(pcache.o)
 .data          0x00000000        0x0 c:/program files/microchip/mplabc32/v2.02/bin/../lib/gcc/pic32mx/4.5.1/../../../../pic32mx/lib/speed\libmchp_peripheral_32MX795F512L.a(pcache.o)
 .bss           0x00000000        0x0 c:/program files/microchip/mplabc32/v2.02/bin/../lib/gcc/pic32mx/4.5.1/../../../../pic32mx/lib/speed\libmchp_peripheral_32MX795F512L.a(pcache.o)
 .reginfo       0x00000000       0x18 c:/program files/microchip/mplabc32/v2.02/bin/../lib/gcc/pic32mx/4.5.1/../../../../pic32mx/lib/speed\libmchp_peripheral_32MX795F512L.a(pcache.o)
 .pdr           0x00000000       0x40 c:/program files/microchip/mplabc32/v2.02/bin/../lib/gcc/pic32mx/4.5.1/../../../../pic32mx/lib/speed\libmchp_peripheral_32MX795F512L.a(pcache.o)
 .mdebug.abi32  0x00000000        0x0 c:/program files/microchip/mplabc32/v2.02/bin/../lib/gcc/pic32mx/4.5.1/../../../../pic32mx/lib/speed\libmchp_peripheral_32MX795F512L.a(pcache.o)
 .text.CheKseg0CacheOff
                0x00000000       0x18 c:/program files/microchip/mplabc32/v2.02/bin/../lib/gcc/pic32mx/4.5.1/../../../../pic32mx/lib/speed\libmchp_peripheral_32MX795F512L.a(pcache.o)
 .text          0x00000000        0x0 c:/program files/microchip/mplabc32/v2.02/bin/../lib/gcc/pic32mx/4.5.1/../../../../pic32mx/lib/speed\libmchp_peripheral_32MX795F512L.a(set_core_sw0_leg_lib.o)
 .data          0x00000000        0x0 c:/program files/microchip/mplabc32/v2.02/bin/../lib/gcc/pic32mx/4.5.1/../../../../pic32mx/lib/speed\libmchp_peripheral_32MX795F512L.a(set_core_sw0_leg_lib.o)
 .bss           0x00000000        0x0 c:/program files/microchip/mplabc32/v2.02/bin/../lib/gcc/pic32mx/4.5.1/../../../../pic32mx/lib/speed\libmchp_peripheral_32MX795F512L.a(set_core_sw0_leg_lib.o)
 .reginfo       0x00000000       0x18 c:/program files/microchip/mplabc32/v2.02/bin/../lib/gcc/pic32mx/4.5.1/../../../../pic32mx/lib/speed\libmchp_peripheral_32MX795F512L.a(set_core_sw0_leg_lib.o)
 .pdr           0x00000000       0x20 c:/program files/microchip/mplabc32/v2.02/bin/../lib/gcc/pic32mx/4.5.1/../../../../pic32mx/lib/speed\libmchp_peripheral_32MX795F512L.a(set_core_sw0_leg_lib.o)
 .mdebug.abi32  0x00000000        0x0 c:/program files/microchip/mplabc32/v2.02/bin/../lib/gcc/pic32mx/4.5.1/../../../../pic32mx/lib/speed\libmchp_peripheral_32MX795F512L.a(set_core_sw0_leg_lib.o)
 .text          0x00000000        0x0 c:/program files/microchip/mplabc32/v2.02/bin/../lib/gcc/pic32mx/4.5.1/../../../../pic32mx/lib/speed\libmchp_peripheral_32MX795F512L.a(int_disable_interrupts_lib.o)
 .data          0x00000000        0x0 c:/program files/microchip/mplabc32/v2.02/bin/../lib/gcc/pic32mx/4.5.1/../../../../pic32mx/lib/speed\libmchp_peripheral_32MX795F512L.a(int_disable_interrupts_lib.o)
 .bss           0x00000000        0x0 c:/program files/microchip/mplabc32/v2.02/bin/../lib/gcc/pic32mx/4.5.1/../../../../pic32mx/lib/speed\libmchp_peripheral_32MX795F512L.a(int_disable_interrupts_lib.o)
 .reginfo       0x00000000       0x18 c:/program files/microchip/mplabc32/v2.02/bin/../lib/gcc/pic32mx/4.5.1/../../../../pic32mx/lib/speed\libmchp_peripheral_32MX795F512L.a(int_disable_interrupts_lib.o)
 .pdr           0x00000000       0x20 c:/program files/microchip/mplabc32/v2.02/bin/../lib/gcc/pic32mx/4.5.1/../../../../pic32mx/lib/speed\libmchp_peripheral_32MX795F512L.a(int_disable_interrupts_lib.o)
 .mdebug.abi32  0x00000000        0x0 c:/program files/microchip/mplabc32/v2.02/bin/../lib/gcc/pic32mx/4.5.1/../../../../pic32mx/lib/speed\libmchp_peripheral_32MX795F512L.a(int_disable_interrupts_lib.o)
 .text          0x00000000        0x0 c:/program files/microchip/mplabc32/v2.02/bin/../lib/gcc/pic32mx/4.5.1/../../../../pic32mx/lib/speed\libmchp_peripheral_32MX795F512L.a(int_restore_interrupts_lib.o)
 .data          0x00000000        0x0 c:/program files/microchip/mplabc32/v2.02/bin/../lib/gcc/pic32mx/4.5.1/../../../../pic32mx/lib/speed\libmchp_peripheral_32MX795F512L.a(int_restore_interrupts_lib.o)
 .bss           0x00000000        0x0 c:/program files/microchip/mplabc32/v2.02/bin/../lib/gcc/pic32mx/4.5.1/../../../../pic32mx/lib/speed\libmchp_peripheral_32MX795F512L.a(int_restore_interrupts_lib.o)
 .reginfo       0x00000000       0x18 c:/program files/microchip/mplabc32/v2.02/bin/../lib/gcc/pic32mx/4.5.1/../../../../pic32mx/lib/speed\libmchp_peripheral_32MX795F512L.a(int_restore_interrupts_lib.o)
 .pdr           0x00000000       0x20 c:/program files/microchip/mplabc32/v2.02/bin/../lib/gcc/pic32mx/4.5.1/../../../../pic32mx/lib/speed\libmchp_peripheral_32MX795F512L.a(int_restore_interrupts_lib.o)
 .mdebug.abi32  0x00000000        0x0 c:/program files/microchip/mplabc32/v2.02/bin/../lib/gcc/pic32mx/4.5.1/../../../../pic32mx/lib/speed\libmchp_peripheral_32MX795F512L.a(int_restore_interrupts_lib.o)
 .text          0x00000000        0x0 c:/program files/microchip/mplabc32/v2.02/bin/../lib/gcc/pic32mx/4.5.1/../../../../pic32mx/lib/speed\libmchp_peripheral_32MX795F512L.a(int_enable_mv_int_lib.o)
 .data          0x00000000        0x0 c:/program files/microchip/mplabc32/v2.02/bin/../lib/gcc/pic32mx/4.5.1/../../../../pic32mx/lib/speed\libmchp_peripheral_32MX795F512L.a(int_enable_mv_int_lib.o)
 .bss           0x00000000        0x0 c:/program files/microchip/mplabc32/v2.02/bin/../lib/gcc/pic32mx/4.5.1/../../../../pic32mx/lib/speed\libmchp_peripheral_32MX795F512L.a(int_enable_mv_int_lib.o)
 .reginfo       0x00000000       0x18 c:/program files/microchip/mplabc32/v2.02/bin/../lib/gcc/pic32mx/4.5.1/../../../../pic32mx/lib/speed\libmchp_peripheral_32MX795F512L.a(int_enable_mv_int_lib.o)
 .pdr           0x00000000       0x20 c:/program files/microchip/mplabc32/v2.02/bin/../lib/gcc/pic32mx/4.5.1/../../../../pic32mx/lib/speed\libmchp_peripheral_32MX795F512L.a(int_enable_mv_int_lib.o)
 .mdebug.abi32  0x00000000        0x0 c:/program files/microchip/mplabc32/v2.02/bin/../lib/gcc/pic32mx/4.5.1/../../../../pic32mx/lib/speed\libmchp_peripheral_32MX795F512L.a(int_enable_mv_int_lib.o)
 .text          0x00000000        0x0 c:/program files/microchip/mplabc32/v2.02/bin/../lib/gcc/pic32mx/4.5.1/../../../../pic32mx/lib/speed\libmchp_peripheral_32MX795F512L.a(int_tbl_lib.o)
 .data          0x00000000        0x0 c:/program files/microchip/mplabc32/v2.02/bin/../lib/gcc/pic32mx/4.5.1/../../../../pic32mx/lib/speed\libmchp_peripheral_32MX795F512L.a(int_tbl_lib.o)
 .bss           0x00000000        0x0 c:/program files/microchip/mplabc32/v2.02/bin/../lib/gcc/pic32mx/4.5.1/../../../../pic32mx/lib/speed\libmchp_peripheral_32MX795F512L.a(int_tbl_lib.o)
 .reginfo       0x00000000       0x18 c:/program files/microchip/mplabc32/v2.02/bin/../lib/gcc/pic32mx/4.5.1/../../../../pic32mx/lib/speed\libmchp_peripheral_32MX795F512L.a(int_tbl_lib.o)
 .pdr           0x00000000      0x120 c:/program files/microchip/mplabc32/v2.02/bin/../lib/gcc/pic32mx/4.5.1/../../../../pic32mx/lib/speed\libmchp_peripheral_32MX795F512L.a(int_tbl_lib.o)
 .mdebug.abi32  0x00000000        0x0 c:/program files/microchip/mplabc32/v2.02/bin/../lib/gcc/pic32mx/4.5.1/../../../../pic32mx/lib/speed\libmchp_peripheral_32MX795F512L.a(int_tbl_lib.o)
 .text.INTSetFlag
                0x00000000       0x2c c:/program files/microchip/mplabc32/v2.02/bin/../lib/gcc/pic32mx/4.5.1/../../../../pic32mx/lib/speed\libmchp_peripheral_32MX795F512L.a(int_tbl_lib.o)
 .text.INTGetFlag
                0x00000000       0x2c c:/program files/microchip/mplabc32/v2.02/bin/../lib/gcc/pic32mx/4.5.1/../../../../pic32mx/lib/speed\libmchp_peripheral_32MX795F512L.a(int_tbl_lib.o)
 .text.INTGetEnable
                0x00000000       0x2c c:/program files/microchip/mplabc32/v2.02/bin/../lib/gcc/pic32mx/4.5.1/../../../../pic32mx/lib/speed\libmchp_peripheral_32MX795F512L.a(int_tbl_lib.o)
 .text.INTSetVectorPriority
                0x00000000       0x3c c:/program files/microchip/mplabc32/v2.02/bin/../lib/gcc/pic32mx/4.5.1/../../../../pic32mx/lib/speed\libmchp_peripheral_32MX795F512L.a(int_tbl_lib.o)
 .text.INTGetVectorPriority
                0x00000000       0x30 c:/program files/microchip/mplabc32/v2.02/bin/../lib/gcc/pic32mx/4.5.1/../../../../pic32mx/lib/speed\libmchp_peripheral_32MX795F512L.a(int_tbl_lib.o)
 .text.INTSetVectorSubPriority
                0x00000000       0x3c c:/program files/microchip/mplabc32/v2.02/bin/../lib/gcc/pic32mx/4.5.1/../../../../pic32mx/lib/speed\libmchp_peripheral_32MX795F512L.a(int_tbl_lib.o)
 .text.INTGetVectorSubPriority
                0x00000000       0x30 c:/program files/microchip/mplabc32/v2.02/bin/../lib/gcc/pic32mx/4.5.1/../../../../pic32mx/lib/speed\libmchp_peripheral_32MX795F512L.a(int_tbl_lib.o)
 .text          0x00000000        0x0 c:/program files/microchip/mplabc32/v2.02/bin/../lib/gcc/pic32mx/4.5.1/../../../../pic32mx/lib/speed\libmchp_peripheral_32MX795F512L.a(rtcc_init_lib.o)
 .data          0x00000000        0x0 c:/program files/microchip/mplabc32/v2.02/bin/../lib/gcc/pic32mx/4.5.1/../../../../pic32mx/lib/speed\libmchp_peripheral_32MX795F512L.a(rtcc_init_lib.o)
 .bss           0x00000000        0x0 c:/program files/microchip/mplabc32/v2.02/bin/../lib/gcc/pic32mx/4.5.1/../../../../pic32mx/lib/speed\libmchp_peripheral_32MX795F512L.a(rtcc_init_lib.o)
 .reginfo       0x00000000       0x18 c:/program files/microchip/mplabc32/v2.02/bin/../lib/gcc/pic32mx/4.5.1/../../../../pic32mx/lib/speed\libmchp_peripheral_32MX795F512L.a(rtcc_init_lib.o)
 .pdr           0x00000000       0x20 c:/program files/microchip/mplabc32/v2.02/bin/../lib/gcc/pic32mx/4.5.1/../../../../pic32mx/lib/speed\libmchp_peripheral_32MX795F512L.a(rtcc_init_lib.o)
 .mdebug.abi32  0x00000000        0x0 c:/program files/microchip/mplabc32/v2.02/bin/../lib/gcc/pic32mx/4.5.1/../../../../pic32mx/lib/speed\libmchp_peripheral_32MX795F512L.a(rtcc_init_lib.o)
 .text          0x00000000        0x0 c:/program files/microchip/mplabc32/v2.02/bin/../lib/gcc/pic32mx/4.5.1/../../../../pic32mx/lib/speed\libmchp_peripheral_32MX795F512L.a(rtcc_set_time_date_lib.o)
 .data          0x00000000        0x0 c:/program files/microchip/mplabc32/v2.02/bin/../lib/gcc/pic32mx/4.5.1/../../../../pic32mx/lib/speed\libmchp_peripheral_32MX795F512L.a(rtcc_set_time_date_lib.o)
 .bss           0x00000000        0x0 c:/program files/microchip/mplabc32/v2.02/bin/../lib/gcc/pic32mx/4.5.1/../../../../pic32mx/lib/speed\libmchp_peripheral_32MX795F512L.a(rtcc_set_time_date_lib.o)
 .reginfo       0x00000000       0x18 c:/program files/microchip/mplabc32/v2.02/bin/../lib/gcc/pic32mx/4.5.1/../../../../pic32mx/lib/speed\libmchp_peripheral_32MX795F512L.a(rtcc_set_time_date_lib.o)
 .pdr           0x00000000       0x20 c:/program files/microchip/mplabc32/v2.02/bin/../lib/gcc/pic32mx/4.5.1/../../../../pic32mx/lib/speed\libmchp_peripheral_32MX795F512L.a(rtcc_set_time_date_lib.o)
 .mdebug.abi32  0x00000000        0x0 c:/program files/microchip/mplabc32/v2.02/bin/../lib/gcc/pic32mx/4.5.1/../../../../pic32mx/lib/speed\libmchp_peripheral_32MX795F512L.a(rtcc_set_time_date_lib.o)
 .text          0x00000000        0x0 c:/program files/microchip/mplabc32/v2.02/bin/../lib/gcc/pic32mx/4.5.1/../../../../pic32mx/lib/speed\libmchp_peripheral_32MX795F512L.a(rtcc_open_lib.o)
 .data          0x00000000        0x0 c:/program files/microchip/mplabc32/v2.02/bin/../lib/gcc/pic32mx/4.5.1/../../../../pic32mx/lib/speed\libmchp_peripheral_32MX795F512L.a(rtcc_open_lib.o)
 .bss           0x00000000        0x0 c:/program files/microchip/mplabc32/v2.02/bin/../lib/gcc/pic32mx/4.5.1/../../../../pic32mx/lib/speed\libmchp_peripheral_32MX795F512L.a(rtcc_open_lib.o)
 .reginfo       0x00000000       0x18 c:/program files/microchip/mplabc32/v2.02/bin/../lib/gcc/pic32mx/4.5.1/../../../../pic32mx/lib/speed\libmchp_peripheral_32MX795F512L.a(rtcc_open_lib.o)
 .pdr           0x00000000       0x20 c:/program files/microchip/mplabc32/v2.02/bin/../lib/gcc/pic32mx/4.5.1/../../../../pic32mx/lib/speed\libmchp_peripheral_32MX795F512L.a(rtcc_open_lib.o)
 .mdebug.abi32  0x00000000        0x0 c:/program files/microchip/mplabc32/v2.02/bin/../lib/gcc/pic32mx/4.5.1/../../../../pic32mx/lib/speed\libmchp_peripheral_32MX795F512L.a(rtcc_open_lib.o)
 .text          0x00000000        0x0 c:/program files/microchip/mplabc32/v2.02/bin/../lib/gcc/pic32mx/4.5.1/../../../../pic32mx/lib/speed\libmchp_peripheral_32MX795F512L.a(spi_getc_spi1_lib_legacy.o)
 .data          0x00000000        0x0 c:/program files/microchip/mplabc32/v2.02/bin/../lib/gcc/pic32mx/4.5.1/../../../../pic32mx/lib/speed\libmchp_peripheral_32MX795F512L.a(spi_getc_spi1_lib_legacy.o)
 .bss           0x00000000        0x0 c:/program files/microchip/mplabc32/v2.02/bin/../lib/gcc/pic32mx/4.5.1/../../../../pic32mx/lib/speed\libmchp_peripheral_32MX795F512L.a(spi_getc_spi1_lib_legacy.o)
 .reginfo       0x00000000       0x18 c:/program files/microchip/mplabc32/v2.02/bin/../lib/gcc/pic32mx/4.5.1/../../../../pic32mx/lib/speed\libmchp_peripheral_32MX795F512L.a(spi_getc_spi1_lib_legacy.o)
 .pdr           0x00000000       0x20 c:/program files/microchip/mplabc32/v2.02/bin/../lib/gcc/pic32mx/4.5.1/../../../../pic32mx/lib/speed\libmchp_peripheral_32MX795F512L.a(spi_getc_spi1_lib_legacy.o)
 .mdebug.abi32  0x00000000        0x0 c:/program files/microchip/mplabc32/v2.02/bin/../lib/gcc/pic32mx/4.5.1/../../../../pic32mx/lib/speed\libmchp_peripheral_32MX795F512L.a(spi_getc_spi1_lib_legacy.o)
 .text          0x00000000        0x0 c:/program files/microchip/mplabc32/v2.02/bin/../lib/gcc/pic32mx/4.5.1/../../../../pic32mx/lib/speed\libmchp_peripheral_32MX795F512L.a(spi_open_spi1_lib_legacy.o)
 .data          0x00000000        0x0 c:/program files/microchip/mplabc32/v2.02/bin/../lib/gcc/pic32mx/4.5.1/../../../../pic32mx/lib/speed\libmchp_peripheral_32MX795F512L.a(spi_open_spi1_lib_legacy.o)
 .bss           0x00000000        0x0 c:/program files/microchip/mplabc32/v2.02/bin/../lib/gcc/pic32mx/4.5.1/../../../../pic32mx/lib/speed\libmchp_peripheral_32MX795F512L.a(spi_open_spi1_lib_legacy.o)
 .reginfo       0x00000000       0x18 c:/program files/microchip/mplabc32/v2.02/bin/../lib/gcc/pic32mx/4.5.1/../../../../pic32mx/lib/speed\libmchp_peripheral_32MX795F512L.a(spi_open_spi1_lib_legacy.o)
 .pdr           0x00000000       0x20 c:/program files/microchip/mplabc32/v2.02/bin/../lib/gcc/pic32mx/4.5.1/../../../../pic32mx/lib/speed\libmchp_peripheral_32MX795F512L.a(spi_open_spi1_lib_legacy.o)
 .mdebug.abi32  0x00000000        0x0 c:/program files/microchip/mplabc32/v2.02/bin/../lib/gcc/pic32mx/4.5.1/../../../../pic32mx/lib/speed\libmchp_peripheral_32MX795F512L.a(spi_open_spi1_lib_legacy.o)
 .text          0x00000000        0x0 c:/program files/microchip/mplabc32/v2.02/bin/../lib/gcc/pic32mx/4.5.1/../../../../pic32mx/lib/speed\libmchp_peripheral_32MX795F512L.a(spi_brg_tbl_lib_legacy.o)
 .data          0x00000000        0x0 c:/program files/microchip/mplabc32/v2.02/bin/../lib/gcc/pic32mx/4.5.1/../../../../pic32mx/lib/speed\libmchp_peripheral_32MX795F512L.a(spi_brg_tbl_lib_legacy.o)
 .bss           0x00000000        0x0 c:/program files/microchip/mplabc32/v2.02/bin/../lib/gcc/pic32mx/4.5.1/../../../../pic32mx/lib/speed\libmchp_peripheral_32MX795F512L.a(spi_brg_tbl_lib_legacy.o)
 .reginfo       0x00000000       0x18 c:/program files/microchip/mplabc32/v2.02/bin/../lib/gcc/pic32mx/4.5.1/../../../../pic32mx/lib/speed\libmchp_peripheral_32MX795F512L.a(spi_brg_tbl_lib_legacy.o)
 .pdr           0x00000000        0x0 c:/program files/microchip/mplabc32/v2.02/bin/../lib/gcc/pic32mx/4.5.1/../../../../pic32mx/lib/speed\libmchp_peripheral_32MX795F512L.a(spi_brg_tbl_lib_legacy.o)
 .mdebug.abi32  0x00000000        0x0 c:/program files/microchip/mplabc32/v2.02/bin/../lib/gcc/pic32mx/4.5.1/../../../../pic32mx/lib/speed\libmchp_peripheral_32MX795F512L.a(spi_brg_tbl_lib_legacy.o)
 .text          0x00000000        0x0 c:/program files/microchip/mplabc32/v2.02/bin/../lib/gcc/pic32mx/4.5.1/../../../../pic32mx/lib/speed\libmchp_peripheral_32MX795F512L.a(port_set_pins_digital_in_lib.o)
 .data          0x00000000        0x0 c:/program files/microchip/mplabc32/v2.02/bin/../lib/gcc/pic32mx/4.5.1/../../../../pic32mx/lib/speed\libmchp_peripheral_32MX795F512L.a(port_set_pins_digital_in_lib.o)
 .bss           0x00000000        0x0 c:/program files/microchip/mplabc32/v2.02/bin/../lib/gcc/pic32mx/4.5.1/../../../../pic32mx/lib/speed\libmchp_peripheral_32MX795F512L.a(port_set_pins_digital_in_lib.o)
 .reginfo       0x00000000       0x18 c:/program files/microchip/mplabc32/v2.02/bin/../lib/gcc/pic32mx/4.5.1/../../../../pic32mx/lib/speed\libmchp_peripheral_32MX795F512L.a(port_set_pins_digital_in_lib.o)
 .pdr           0x00000000       0x20 c:/program files/microchip/mplabc32/v2.02/bin/../lib/gcc/pic32mx/4.5.1/../../../../pic32mx/lib/speed\libmchp_peripheral_32MX795F512L.a(port_set_pins_digital_in_lib.o)
 .mdebug.abi32  0x00000000        0x0 c:/program files/microchip/mplabc32/v2.02/bin/../lib/gcc/pic32mx/4.5.1/../../../../pic32mx/lib/speed\libmchp_peripheral_32MX795F512L.a(port_set_pins_digital_in_lib.o)
 .text          0x00000000        0x0 c:/program files/microchip/mplabc32/v2.02/bin/../lib/gcc/pic32mx/4.5.1/../../../../pic32mx/lib/speed\libmchp_peripheral_32MX795F512L.a(port_set_pins_digital_out_lib.o)
 .data          0x00000000        0x0 c:/program files/microchip/mplabc32/v2.02/bin/../lib/gcc/pic32mx/4.5.1/../../../../pic32mx/lib/speed\libmchp_peripheral_32MX795F512L.a(port_set_pins_digital_out_lib.o)
 .bss           0x00000000        0x0 c:/program files/microchip/mplabc32/v2.02/bin/../lib/gcc/pic32mx/4.5.1/../../../../pic32mx/lib/speed\libmchp_peripheral_32MX795F512L.a(port_set_pins_digital_out_lib.o)
 .reginfo       0x00000000       0x18 c:/program files/microchip/mplabc32/v2.02/bin/../lib/gcc/pic32mx/4.5.1/../../../../pic32mx/lib/speed\libmchp_peripheral_32MX795F512L.a(port_set_pins_digital_out_lib.o)
 .pdr           0x00000000       0x20 c:/program files/microchip/mplabc32/v2.02/bin/../lib/gcc/pic32mx/4.5.1/../../../../pic32mx/lib/speed\libmchp_peripheral_32MX795F512L.a(port_set_pins_digital_out_lib.o)
 .mdebug.abi32  0x00000000        0x0 c:/program files/microchip/mplabc32/v2.02/bin/../lib/gcc/pic32mx/4.5.1/../../../../pic32mx/lib/speed\libmchp_peripheral_32MX795F512L.a(port_set_pins_digital_out_lib.o)
 .text          0x00000000        0x0 c:/program files/microchip/mplabc32/v2.02/bin/../lib/gcc/pic32mx/4.5.1/../../../../pic32mx/lib/speed\libmchp_peripheral_32MX795F512L.a(_ports_tbl_libp.o)
 .data          0x00000000        0x0 c:/program files/microchip/mplabc32/v2.02/bin/../lib/gcc/pic32mx/4.5.1/../../../../pic32mx/lib/speed\libmchp_peripheral_32MX795F512L.a(_ports_tbl_libp.o)
 .bss           0x00000000        0x0 c:/program files/microchip/mplabc32/v2.02/bin/../lib/gcc/pic32mx/4.5.1/../../../../pic32mx/lib/speed\libmchp_peripheral_32MX795F512L.a(_ports_tbl_libp.o)
 .reginfo       0x00000000       0x18 c:/program files/microchip/mplabc32/v2.02/bin/../lib/gcc/pic32mx/4.5.1/../../../../pic32mx/lib/speed\libmchp_peripheral_32MX795F512L.a(_ports_tbl_libp.o)
 .pdr           0x00000000        0x0 c:/program files/microchip/mplabc32/v2.02/bin/../lib/gcc/pic32mx/4.5.1/../../../../pic32mx/lib/speed\libmchp_peripheral_32MX795F512L.a(_ports_tbl_libp.o)
 .mdebug.abi32  0x00000000        0x0 c:/program files/microchip/mplabc32/v2.02/bin/../lib/gcc/pic32mx/4.5.1/../../../../pic32mx/lib/speed\libmchp_peripheral_32MX795F512L.a(_ports_tbl_libp.o)
 .text          0x00000000        0x0 c:/program files/microchip/mplabc32/v2.02/bin/../lib/gcc/pic32mx/4.5.1/../../../../pic32mx/lib/speed\libmchp_peripheral_32MX795F512L.a(int_enable_interrupts_lib.o)
 .data          0x00000000        0x0 c:/program files/microchip/mplabc32/v2.02/bin/../lib/gcc/pic32mx/4.5.1/../../../../pic32mx/lib/speed\libmchp_peripheral_32MX795F512L.a(int_enable_interrupts_lib.o)
 .bss           0x00000000        0x0 c:/program files/microchip/mplabc32/v2.02/bin/../lib/gcc/pic32mx/4.5.1/../../../../pic32mx/lib/speed\libmchp_peripheral_32MX795F512L.a(int_enable_interrupts_lib.o)
 .reginfo       0x00000000       0x18 c:/program files/microchip/mplabc32/v2.02/bin/../lib/gcc/pic32mx/4.5.1/../../../../pic32mx/lib/speed\libmchp_peripheral_32MX795F512L.a(int_enable_interrupts_lib.o)
 .pdr           0x00000000       0x20 c:/program files/microchip/mplabc32/v2.02/bin/../lib/gcc/pic32mx/4.5.1/../../../../pic32mx/lib/speed\libmchp_peripheral_32MX795F512L.a(int_enable_interrupts_lib.o)
 .mdebug.abi32  0x00000000        0x0 c:/program files/microchip/mplabc32/v2.02/bin/../lib/gcc/pic32mx/4.5.1/../../../../pic32mx/lib/speed\libmchp_peripheral_32MX795F512L.a(int_enable_interrupts_lib.o)
 .text          0x00000000        0x0 c:/program files/microchip/mplabc32/v2.02/bin/../lib/gcc/pic32mx/4.5.1/../../../../pic32mx/lib/speed\libmchp_peripheral_32MX795F512L.a(_rtcc_set_time_and_date_lib.o)
 .data          0x00000000        0x0 c:/program files/microchip/mplabc32/v2.02/bin/../lib/gcc/pic32mx/4.5.1/../../../../pic32mx/lib/speed\libmchp_peripheral_32MX795F512L.a(_rtcc_set_time_and_date_lib.o)
 .bss           0x00000000        0x0 c:/program files/microchip/mplabc32/v2.02/bin/../lib/gcc/pic32mx/4.5.1/../../../../pic32mx/lib/speed\libmchp_peripheral_32MX795F512L.a(_rtcc_set_time_and_date_lib.o)
 .reginfo       0x00000000       0x18 c:/program files/microchip/mplabc32/v2.02/bin/../lib/gcc/pic32mx/4.5.1/../../../../pic32mx/lib/speed\libmchp_peripheral_32MX795F512L.a(_rtcc_set_time_and_date_lib.o)
 .pdr           0x00000000       0x20 c:/program files/microchip/mplabc32/v2.02/bin/../lib/gcc/pic32mx/4.5.1/../../../../pic32mx/lib/speed\libmchp_peripheral_32MX795F512L.a(_rtcc_set_time_and_date_lib.o)
 .mdebug.abi32  0x00000000        0x0 c:/program files/microchip/mplabc32/v2.02/bin/../lib/gcc/pic32mx/4.5.1/../../../../pic32mx/lib/speed\libmchp_peripheral_32MX795F512L.a(_rtcc_set_time_and_date_lib.o)
 .text          0x00000000        0x0 c:/program files/microchip/mplabc32/v2.02/bin/../lib/gcc/pic32mx/4.5.1/../../../../pic32mx/lib/speed\libmchp_peripheral_32MX795F512L.a(_rtcc_wait_clock_off_lib.o)
 .data          0x00000000        0x0 c:/program files/microchip/mplabc32/v2.02/bin/../lib/gcc/pic32mx/4.5.1/../../../../pic32mx/lib/speed\libmchp_peripheral_32MX795F512L.a(_rtcc_wait_clock_off_lib.o)
 .bss           0x00000000        0x0 c:/program files/microchip/mplabc32/v2.02/bin/../lib/gcc/pic32mx/4.5.1/../../../../pic32mx/lib/speed\libmchp_peripheral_32MX795F512L.a(_rtcc_wait_clock_off_lib.o)
 .reginfo       0x00000000       0x18 c:/program files/microchip/mplabc32/v2.02/bin/../lib/gcc/pic32mx/4.5.1/../../../../pic32mx/lib/speed\libmchp_peripheral_32MX795F512L.a(_rtcc_wait_clock_off_lib.o)
 .pdr           0x00000000       0x40 c:/program files/microchip/mplabc32/v2.02/bin/../lib/gcc/pic32mx/4.5.1/../../../../pic32mx/lib/speed\libmchp_peripheral_32MX795F512L.a(_rtcc_wait_clock_off_lib.o)
 .mdebug.abi32  0x00000000        0x0 c:/program files/microchip/mplabc32/v2.02/bin/../lib/gcc/pic32mx/4.5.1/../../../../pic32mx/lib/speed\libmchp_peripheral_32MX795F512L.a(_rtcc_wait_clock_off_lib.o)
 .text._RtccSetClockWait
                0x00000000       0x14 c:/program files/microchip/mplabc32/v2.02/bin/../lib/gcc/pic32mx/4.5.1/../../../../pic32mx/lib/speed\libmchp_peripheral_32MX795F512L.a(_rtcc_wait_clock_off_lib.o)
 .text          0x00000000        0x0 c:/program files/microchip/mplabc32/v2.02/bin/../lib/gcc/pic32mx/4.5.1/../../../../pic32mx/lib/speed\libc.a(calloc.o)
 .data          0x00000000        0x0 c:/program files/microchip/mplabc32/v2.02/bin/../lib/gcc/pic32mx/4.5.1/../../../../pic32mx/lib/speed\libc.a(calloc.o)
 .bss           0x00000000        0x0 c:/program files/microchip/mplabc32/v2.02/bin/../lib/gcc/pic32mx/4.5.1/../../../../pic32mx/lib/speed\libc.a(calloc.o)
 .reginfo       0x00000000       0x18 c:/program files/microchip/mplabc32/v2.02/bin/../lib/gcc/pic32mx/4.5.1/../../../../pic32mx/lib/speed\libc.a(calloc.o)
 .pdr           0x00000000       0x20 c:/program files/microchip/mplabc32/v2.02/bin/../lib/gcc/pic32mx/4.5.1/../../../../pic32mx/lib/speed\libc.a(calloc.o)
 .mdebug.abi32  0x00000000        0x0 c:/program files/microchip/mplabc32/v2.02/bin/../lib/gcc/pic32mx/4.5.1/../../../../pic32mx/lib/speed\libc.a(calloc.o)
 .text.calloc   0x00000000       0xdc c:/program files/microchip/mplabc32/v2.02/bin/../lib/gcc/pic32mx/4.5.1/../../../../pic32mx/lib/speed\libc.a(calloc.o)
 .text          0x00000000        0x0 c:/program files/microchip/mplabc32/v2.02/bin/../lib/gcc/pic32mx/4.5.1/../../../../pic32mx/lib/speed\libc.a(errno.o)
 .data          0x00000000        0x0 c:/program files/microchip/mplabc32/v2.02/bin/../lib/gcc/pic32mx/4.5.1/../../../../pic32mx/lib/speed\libc.a(errno.o)
 .bss           0x00000000        0x0 c:/program files/microchip/mplabc32/v2.02/bin/../lib/gcc/pic32mx/4.5.1/../../../../pic32mx/lib/speed\libc.a(errno.o)
 .reginfo       0x00000000       0x18 c:/program files/microchip/mplabc32/v2.02/bin/../lib/gcc/pic32mx/4.5.1/../../../../pic32mx/lib/speed\libc.a(errno.o)
 .pdr           0x00000000        0x0 c:/program files/microchip/mplabc32/v2.02/bin/../lib/gcc/pic32mx/4.5.1/../../../../pic32mx/lib/speed\libc.a(errno.o)
 .mdebug.abi32  0x00000000        0x0 c:/program files/microchip/mplabc32/v2.02/bin/../lib/gcc/pic32mx/4.5.1/../../../../pic32mx/lib/speed\libc.a(errno.o)
 .text          0x00000000        0x0 c:/program files/microchip/mplabc32/v2.02/bin/../lib/gcc/pic32mx/4.5.1/../../../../pic32mx/lib/speed\libc.a(malloc.o)
 .data          0x00000000        0x0 c:/program files/microchip/mplabc32/v2.02/bin/../lib/gcc/pic32mx/4.5.1/../../../../pic32mx/lib/speed\libc.a(malloc.o)
 .bss           0x00000000       0x20 c:/program files/microchip/mplabc32/v2.02/bin/../lib/gcc/pic32mx/4.5.1/../../../../pic32mx/lib/speed\libc.a(malloc.o)
 .reginfo       0x00000000       0x18 c:/program files/microchip/mplabc32/v2.02/bin/../lib/gcc/pic32mx/4.5.1/../../../../pic32mx/lib/speed\libc.a(malloc.o)
 .pdr           0x00000000       0x60 c:/program files/microchip/mplabc32/v2.02/bin/../lib/gcc/pic32mx/4.5.1/../../../../pic32mx/lib/speed\libc.a(malloc.o)
 .mdebug.abi32  0x00000000        0x0 c:/program files/microchip/mplabc32/v2.02/bin/../lib/gcc/pic32mx/4.5.1/../../../../pic32mx/lib/speed\libc.a(malloc.o)
 .text.malloc   0x00000000      0x274 c:/program files/microchip/mplabc32/v2.02/bin/../lib/gcc/pic32mx/4.5.1/../../../../pic32mx/lib/speed\libc.a(malloc.o)
 .text.free     0x00000000       0x24 c:/program files/microchip/mplabc32/v2.02/bin/../lib/gcc/pic32mx/4.5.1/../../../../pic32mx/lib/speed\libc.a(malloc.o)
 .text.realloc  0x00000000      0x220 c:/program files/microchip/mplabc32/v2.02/bin/../lib/gcc/pic32mx/4.5.1/../../../../pic32mx/lib/speed\libc.a(malloc.o)
 .text          0x00000000        0x0 c:/program files/microchip/mplabc32/v2.02/bin/../lib/gcc/pic32mx/4.5.1/../../../../pic32mx/lib/speed\libc.a(sbrk.o)
 .data          0x00000000        0x0 c:/program files/microchip/mplabc32/v2.02/bin/../lib/gcc/pic32mx/4.5.1/../../../../pic32mx/lib/speed\libc.a(sbrk.o)
 .bss           0x00000000       0x1c c:/program files/microchip/mplabc32/v2.02/bin/../lib/gcc/pic32mx/4.5.1/../../../../pic32mx/lib/speed\libc.a(sbrk.o)
 .reginfo       0x00000000       0x18 c:/program files/microchip/mplabc32/v2.02/bin/../lib/gcc/pic32mx/4.5.1/../../../../pic32mx/lib/speed\libc.a(sbrk.o)
 .pdr           0x00000000       0xa0 c:/program files/microchip/mplabc32/v2.02/bin/../lib/gcc/pic32mx/4.5.1/../../../../pic32mx/lib/speed\libc.a(sbrk.o)
 .mdebug.abi32  0x00000000        0x0 c:/program files/microchip/mplabc32/v2.02/bin/../lib/gcc/pic32mx/4.5.1/../../../../pic32mx/lib/speed\libc.a(sbrk.o)
 .text.getpagesize
                0x00000000        0x8 c:/program files/microchip/mplabc32/v2.02/bin/../lib/gcc/pic32mx/4.5.1/../../../../pic32mx/lib/speed\libc.a(sbrk.o)
 .text._stub_sbd_memlayout
                0x00000000       0x2c c:/program files/microchip/mplabc32/v2.02/bin/../lib/gcc/pic32mx/4.5.1/../../../../pic32mx/lib/speed\libc.a(sbrk.o)
 .text._sbrk_init
                0x00000000      0x194 c:/program files/microchip/mplabc32/v2.02/bin/../lib/gcc/pic32mx/4.5.1/../../../../pic32mx/lib/speed\libc.a(sbrk.o)
 .text._sbrk    0x00000000       0xc4 c:/program files/microchip/mplabc32/v2.02/bin/../lib/gcc/pic32mx/4.5.1/../../../../pic32mx/lib/speed\libc.a(sbrk.o)
 .text.sbrk     0x00000000       0x50 c:/program files/microchip/mplabc32/v2.02/bin/../lib/gcc/pic32mx/4.5.1/../../../../pic32mx/lib/speed\libc.a(sbrk.o)
 .sbss          0x00000000        0x8 c:/program files/microchip/mplabc32/v2.02/bin/../lib/gcc/pic32mx/4.5.1/../../../../pic32mx/lib/speed\libc.a(sbrk.o)
 .data          0x00000000        0x0 c:/program files/microchip/mplabc32/v2.02/bin/../lib/gcc/pic32mx/4.5.1/speed\libgcc.a(_lshrdi3.o)
 .bss           0x00000000        0x0 c:/program files/microchip/mplabc32/v2.02/bin/../lib/gcc/pic32mx/4.5.1/speed\libgcc.a(_lshrdi3.o)
 .reginfo       0x00000000       0x18 c:/program files/microchip/mplabc32/v2.02/bin/../lib/gcc/pic32mx/4.5.1/speed\libgcc.a(_lshrdi3.o)
 .pdr           0x00000000       0x20 c:/program files/microchip/mplabc32/v2.02/bin/../lib/gcc/pic32mx/4.5.1/speed\libgcc.a(_lshrdi3.o)
 .mdebug.abi32  0x00000000        0x0 c:/program files/microchip/mplabc32/v2.02/bin/../lib/gcc/pic32mx/4.5.1/speed\libgcc.a(_lshrdi3.o)
 .data          0x00000000        0x0 c:/program files/microchip/mplabc32/v2.02/bin/../lib/gcc/pic32mx/4.5.1/speed\libgcc.a(_ashldi3.o)
 .bss           0x00000000        0x0 c:/program files/microchip/mplabc32/v2.02/bin/../lib/gcc/pic32mx/4.5.1/speed\libgcc.a(_ashldi3.o)
 .reginfo       0x00000000       0x18 c:/program files/microchip/mplabc32/v2.02/bin/../lib/gcc/pic32mx/4.5.1/speed\libgcc.a(_ashldi3.o)
 .pdr           0x00000000       0x20 c:/program files/microchip/mplabc32/v2.02/bin/../lib/gcc/pic32mx/4.5.1/speed\libgcc.a(_ashldi3.o)
 .mdebug.abi32  0x00000000        0x0 c:/program files/microchip/mplabc32/v2.02/bin/../lib/gcc/pic32mx/4.5.1/speed\libgcc.a(_ashldi3.o)

Memory Configuration

Name             Origin             Length             Attributes
kseg0_program_mem 0x9d007e00         0x0007e200         xr
kseg0_boot_mem   0x9d007000         0x00000970
exception_mem    0x9d006000         0x00001000
kseg1_boot_mem   0x9d007970         0x00000490
debug_exec_mem   0xbfc02000         0x00000ff0
config3          0xbfc02ff0         0x00000004
config2          0xbfc02ff4         0x00000004
config1          0xbfc02ff8         0x00000004
config0          0xbfc02ffc         0x00000004
kseg1_data_mem   0xa0000000         0x00020000         w !x
sfrs             0xbf800000         0x00100000
configsfrs       0xbfc02ff0         0x00000010
*default*        0x00000000         0xffffffff

Linker script and memory map

LOAD c:/program files/microchip/mplabc32/v2.02/bin/../lib/gcc/pic32mx/4.5.1/../../../../pic32mx/lib/speed/crt0.o
LOAD output\main.o
LOAD output\IntQueueTimer.o
LOAD output\IntQueueTimer_isr.o
LOAD output\port.o
LOAD output\port_asm.o
LOAD output\queue.o
LOAD output\tasks.o
LOAD output\list.o
LOAD output\IntQueue.o
LOAD output\QPeek.o
LOAD output\lcd.o
LOAD output\prvTaskTCPIP.o
LOAD output\heap_2.o
LOAD output\usb_host.o
LOAD output\usb_config.o
LOAD output\CustomHTTPApp.o
LOAD output\usb_host_generic.o
LOAD output\FSIO.o
LOAD output\UDP.o
LOAD output\ARP.o
LOAD output\Delay.o
LOAD output\DHCP.o
LOAD output\DNS.o
LOAD output\DstaDPlusClientUDP.o
LOAD output\ETHPIC32ExtPhy.o
LOAD output\ETHPIC32ExtPhyDP83848.o
LOAD output\ETHPIC32IntMac.o
LOAD output\FileSystem.o
LOAD output\FTP.o
LOAD output\Hashes.o
LOAD output\Helpers.o
LOAD output\HTTP2.o
LOAD output\ICMP.o
LOAD output\IP.o
LOAD output\MPFS2.o
LOAD output\Random.o
LOAD output\SNTP.o
LOAD output\StackTsk.o
LOAD output\TCP.o
LOAD output\Tick.o
LOAD output\MPFSImg2.o
LOAD output\SD-SPI.o
LOAD output\prvTaskUSB.o
LOAD output\prvTaskFS.o
LOAD output\MACread.o
LOAD output\SMTP.o
LOAD output\DprsSMTP.o
LOAD output\serial.o
LOAD output\serial_isr.o
LOAD output\comtest.o
LOAD output\DHCPs.o
LOAD output\NBNS.o
                0x00000400                PROVIDE (_min_stack_size, 0x400)
                0x00000000                PROVIDE (_min_heap_size, 0x0)
LOAD c:/program files/microchip/mplabc32/v2.02/bin/../lib/gcc/pic32mx/4.5.1/../../../../pic32mx/lib/./proc/32MX795F512L\processor.o
                0x00000001                PROVIDE (_vector_spacing, 0x1)
                0x9d006000                _ebase_address = 0x9d006000
                0x9d007970                _RESET_ADDR = 0x9d007970
                0x9d007cf0                _BEV_EXCPT_ADDR = 0x9d007cf0
                0x9d007df0                _DBG_EXCPT_ADDR = 0x9d007df0
                0xbfc02000                _DBG_CODE_ADDR = 0xbfc02000
                0x00000ff0                _DBG_CODE_SIZE = 0xff0
                0x9d006180                _GEN_EXCPT_ADDR = (_ebase_address + 0x180)

.config_BFC02FF0
                0xbfc02ff0        0x4
 *(.config_BFC02FF0)
 .config_BFC02FF0
                0xbfc02ff0        0x4 output\main.o

.config_BFC02FF4
                0xbfc02ff4        0x4
 *(.config_BFC02FF4)
 .config_BFC02FF4
                0xbfc02ff4        0x4 output\main.o

.config_BFC02FF8
                0xbfc02ff8        0x4
 *(.config_BFC02FF8)
 .config_BFC02FF8
                0xbfc02ff8        0x4 output\main.o

.config_BFC02FFC
 *(.config_BFC02FFC)
                0xbfc02000                PROVIDE (_DBG_CODE_ADDR, 0xbfc02000)
                0x00000ff0                PROVIDE (_DBG_CODE_SIZE, 0xff0)

.reset          0x9d007970      0x1f4
 *(.reset)
 .reset         0x9d007970       0x10 c:/program files/microchip/mplabc32/v2.02/bin/../lib/gcc/pic32mx/4.5.1/../../../../pic32mx/lib/speed/crt0.o
                0x9d007970                _reset
 *(.reset.startup)
 .reset.startup
                0x9d007980      0x1e4 c:/program files/microchip/mplabc32/v2.02/bin/../lib/gcc/pic32mx/4.5.1/../../../../pic32mx/lib/speed/crt0.o

.bev_excpt      0x9d007cf0       0x10
 *(.bev_handler)
 .bev_handler   0x9d007cf0       0x10 c:/program files/microchip/mplabc32/v2.02/bin/../lib/gcc/pic32mx/4.5.1/../../../../pic32mx/lib/speed/crt0.o

.dbg_excpt      0x9d007df0        0x0
                0x9d007df0                . = (. + DEFINED (_DEBUGGER)?0x8:0x0)

.dbg_code       0xbfc02000        0x0
                0xbfc02000                . = (. + DEFINED (_DEBUGGER)?_DBG_CODE_SIZE:0x0)

.app_excpt      0x9d006180       0x10
 *(.gen_handler)
 .gen_handler   0x9d006180       0x10 c:/program files/microchip/mplabc32/v2.02/bin/../lib/gcc/pic32mx/4.5.1/../../../../pic32mx/lib/speed/crt0.o

.vector_0       0x9d006200        0x0
 *(.vector_0)
                0x00000001                ASSERT (((_vector_spacing == 0x0) || (SIZEOF (.vector_0) <= (_vector_spacing << 0x5))), function at exception vector 0 too large)

.vector_1       0x9d006220        0x8
 *(.vector_1)
 .vector_1      0x9d006220        0x8 output\port.o
                0x00000001                ASSERT (((_vector_spacing == 0x0) || (SIZEOF (.vector_1) <= (_vector_spacing << 0x5))), function at exception vector 1 too large)

.vector_2       0x9d006240        0x0
 *(.vector_2)
                0x00000001                ASSERT (((_vector_spacing == 0x0) || (SIZEOF (.vector_2) <= (_vector_spacing << 0x5))), function at exception vector 2 too large)

.vector_3       0x9d006260        0x0
 *(.vector_3)
                0x00000001                ASSERT (((_vector_spacing == 0x0) || (SIZEOF (.vector_3) <= (_vector_spacing << 0x5))), function at exception vector 3 too large)

.vector_4       0x9d006280        0x8
 *(.vector_4)
 .vector_4      0x9d006280        0x8 output\Tick.o
                0x00000001                ASSERT (((_vector_spacing == 0x0) || (SIZEOF (.vector_4) <= (_vector_spacing << 0x5))), function at exception vector 4 too large)

.vector_5       0x9d0062a0        0x0
 *(.vector_5)
                0x00000001                ASSERT (((_vector_spacing == 0x0) || (SIZEOF (.vector_5) <= (_vector_spacing << 0x5))), function at exception vector 5 too large)

.vector_6       0x9d0062c0        0x0
 *(.vector_6)
                0x00000001                ASSERT (((_vector_spacing == 0x0) || (SIZEOF (.vector_6) <= (_vector_spacing << 0x5))), function at exception vector 6 too large)

.vector_7       0x9d0062e0        0x0
 *(.vector_7)
                0x00000001                ASSERT (((_vector_spacing == 0x0) || (SIZEOF (.vector_7) <= (_vector_spacing << 0x5))), function at exception vector 7 too large)

.vector_8       0x9d006300        0x0
 *(.vector_8)
                0x00000001                ASSERT (((_vector_spacing == 0x0) || (SIZEOF (.vector_8) <= (_vector_spacing << 0x5))), function at exception vector 8 too large)

.vector_9       0x9d006320        0x0
 *(.vector_9)
                0x00000001                ASSERT (((_vector_spacing == 0x0) || (SIZEOF (.vector_9) <= (_vector_spacing << 0x5))), function at exception vector 9 too large)

.vector_10      0x9d006340        0x0
 *(.vector_10)
                0x00000001                ASSERT (((_vector_spacing == 0x0) || (SIZEOF (.vector_10) <= (_vector_spacing << 0x5))), function at exception vector 10 too large)

.vector_11      0x9d006360        0x0
 *(.vector_11)
                0x00000001                ASSERT (((_vector_spacing == 0x0) || (SIZEOF (.vector_11) <= (_vector_spacing << 0x5))), function at exception vector 11 too large)

.vector_12      0x9d006380        0x8
 *(.vector_12)
 .vector_12     0x9d006380        0x8 output\IntQueueTimer.o
                0x00000001                ASSERT (((_vector_spacing == 0x0) || (SIZEOF (.vector_12) <= (_vector_spacing << 0x5))), function at exception vector 12 too large)

.vector_13      0x9d0063a0        0x0
 *(.vector_13)
                0x00000001                ASSERT (((_vector_spacing == 0x0) || (SIZEOF (.vector_13) <= (_vector_spacing << 0x5))), function at exception vector 13 too large)

.vector_14      0x9d0063c0        0x0
 *(.vector_14)
                0x00000001                ASSERT (((_vector_spacing == 0x0) || (SIZEOF (.vector_14) <= (_vector_spacing << 0x5))), function at exception vector 14 too large)

.vector_15      0x9d0063e0        0x0
 *(.vector_15)
                0x00000001                ASSERT (((_vector_spacing == 0x0) || (SIZEOF (.vector_15) <= (_vector_spacing << 0x5))), function at exception vector 15 too large)

.vector_16      0x9d006400        0x8
 *(.vector_16)
 .vector_16     0x9d006400        0x8 output\IntQueueTimer.o
                0x00000001                ASSERT (((_vector_spacing == 0x0) || (SIZEOF (.vector_16) <= (_vector_spacing << 0x5))), function at exception vector 16 too large)

.vector_17      0x9d006420        0x0
 *(.vector_17)
                0x00000001                ASSERT (((_vector_spacing == 0x0) || (SIZEOF (.vector_17) <= (_vector_spacing << 0x5))), function at exception vector 17 too large)

.vector_18      0x9d006440        0x0
 *(.vector_18)
                0x00000001                ASSERT (((_vector_spacing == 0x0) || (SIZEOF (.vector_18) <= (_vector_spacing << 0x5))), function at exception vector 18 too large)

.vector_19      0x9d006460        0x0
 *(.vector_19)
                0x00000001                ASSERT (((_vector_spacing == 0x0) || (SIZEOF (.vector_19) <= (_vector_spacing << 0x5))), function at exception vector 19 too large)

.vector_20      0x9d006480        0x8
 *(.vector_20)
 .vector_20     0x9d006480        0x8 output\port.o
                0x00000001                ASSERT (((_vector_spacing == 0x0) || (SIZEOF (.vector_20) <= (_vector_spacing << 0x5))), function at exception vector 20 too large)

.vector_21      0x9d0064a0        0x0
 *(.vector_21)
                0x00000001                ASSERT (((_vector_spacing == 0x0) || (SIZEOF (.vector_21) <= (_vector_spacing << 0x5))), function at exception vector 21 too large)

.vector_22      0x9d0064c0        0x0
 *(.vector_22)
                0x00000001                ASSERT (((_vector_spacing == 0x0) || (SIZEOF (.vector_22) <= (_vector_spacing << 0x5))), function at exception vector 22 too large)

.vector_23      0x9d0064e0        0x0
 *(.vector_23)
                0x00000001                ASSERT (((_vector_spacing == 0x0) || (SIZEOF (.vector_23) <= (_vector_spacing << 0x5))), function at exception vector 23 too large)

.vector_24      0x9d006500        0x0
 *(.vector_24)
                0x00000001                ASSERT (((_vector_spacing == 0x0) || (SIZEOF (.vector_24) <= (_vector_spacing << 0x5))), function at exception vector 24 too large)

.vector_25      0x9d006520        0x0
 *(.vector_25)
                0x00000001                ASSERT (((_vector_spacing == 0x0) || (SIZEOF (.vector_25) <= (_vector_spacing << 0x5))), function at exception vector 25 too large)

.vector_26      0x9d006540        0x0
 *(.vector_26)
                0x00000001                ASSERT (((_vector_spacing == 0x0) || (SIZEOF (.vector_26) <= (_vector_spacing << 0x5))), function at exception vector 26 too large)

.vector_27      0x9d006560        0x0
 *(.vector_27)
                0x00000001                ASSERT (((_vector_spacing == 0x0) || (SIZEOF (.vector_27) <= (_vector_spacing << 0x5))), function at exception vector 27 too large)

.vector_28      0x9d006580        0x0
 *(.vector_28)
                0x00000001                ASSERT (((_vector_spacing == 0x0) || (SIZEOF (.vector_28) <= (_vector_spacing << 0x5))), function at exception vector 28 too large)

.vector_29      0x9d0065a0        0x0
 *(.vector_29)
                0x00000001                ASSERT (((_vector_spacing == 0x0) || (SIZEOF (.vector_29) <= (_vector_spacing << 0x5))), function at exception vector 29 too large)

.vector_30      0x9d0065c0        0x0
 *(.vector_30)
                0x00000001                ASSERT (((_vector_spacing == 0x0) || (SIZEOF (.vector_30) <= (_vector_spacing << 0x5))), function at exception vector 30 too large)

.vector_31      0x9d0065e0        0x0
 *(.vector_31)
                0x00000001                ASSERT (((_vector_spacing == 0x0) || (SIZEOF (.vector_31) <= (_vector_spacing << 0x5))), function at exception vector 31 too large)

.vector_32      0x9d006600        0x8
 *(.vector_32)
 .vector_32     0x9d006600        0x8 output\serial.o
                0x00000001                ASSERT (((_vector_spacing == 0x0) || (SIZEOF (.vector_32) <= (_vector_spacing << 0x5))), function at exception vector 32 too large)

.vector_33      0x9d006620        0x0
 *(.vector_33)
                0x00000001                ASSERT (((_vector_spacing == 0x0) || (SIZEOF (.vector_33) <= (_vector_spacing << 0x5))), function at exception vector 33 too large)

.vector_34      0x9d006640        0x0
 *(.vector_34)
                0x00000001                ASSERT (((_vector_spacing == 0x0) || (SIZEOF (.vector_34) <= (_vector_spacing << 0x5))), function at exception vector 34 too large)

.vector_35      0x9d006660        0x0
 *(.vector_35)
                0x00000001                ASSERT (((_vector_spacing == 0x0) || (SIZEOF (.vector_35) <= (_vector_spacing << 0x5))), function at exception vector 35 too large)

.vector_36      0x9d006680        0x0
 *(.vector_36)
                0x00000001                ASSERT (((_vector_spacing == 0x0) || (SIZEOF (.vector_36) <= (_vector_spacing << 0x5))), function at exception vector 36 too large)

.vector_37      0x9d0066a0        0x0
 *(.vector_37)
                0x00000001                ASSERT (((_vector_spacing == 0x0) || (SIZEOF (.vector_37) <= (_vector_spacing << 0x5))), function at exception vector 37 too large)

.vector_38      0x9d0066c0        0x0
 *(.vector_38)
                0x00000001                ASSERT (((_vector_spacing == 0x0) || (SIZEOF (.vector_38) <= (_vector_spacing << 0x5))), function at exception vector 38 too large)

.vector_39      0x9d0066e0        0x0
 *(.vector_39)
                0x00000001                ASSERT (((_vector_spacing == 0x0) || (SIZEOF (.vector_39) <= (_vector_spacing << 0x5))), function at exception vector 39 too large)

.vector_40      0x9d006700        0x0
 *(.vector_40)
                0x00000001                ASSERT (((_vector_spacing == 0x0) || (SIZEOF (.vector_40) <= (_vector_spacing << 0x5))), function at exception vector 40 too large)

.vector_41      0x9d006720        0x0
 *(.vector_41)
                0x00000001                ASSERT (((_vector_spacing == 0x0) || (SIZEOF (.vector_41) <= (_vector_spacing << 0x5))), function at exception vector 41 too large)

.vector_42      0x9d006740        0x0
 *(.vector_42)
                0x00000001                ASSERT (((_vector_spacing == 0x0) || (SIZEOF (.vector_42) <= (_vector_spacing << 0x5))), function at exception vector 42 too large)

.vector_43      0x9d006760        0x0
 *(.vector_43)
                0x00000001                ASSERT (((_vector_spacing == 0x0) || (SIZEOF (.vector_43) <= (_vector_spacing << 0x5))), function at exception vector 43 too large)

.vector_44      0x9d006780        0x0
 *(.vector_44)
                0x00000001                ASSERT (((_vector_spacing == 0x0) || (SIZEOF (.vector_44) <= (_vector_spacing << 0x5))), function at exception vector 44 too large)

.vector_45      0x9d0067a0       0x10
 *(.vector_45)
 .vector_45     0x9d0067a0        0x8 output\main.o
 .vector_45     0x9d0067a8        0x8 output\usb_host.o
                0x00000001                ASSERT (((_vector_spacing == 0x0) || (SIZEOF (.vector_45) <= (_vector_spacing << 0x5))), function at exception vector 45 too large)

.vector_46      0x9d0067c0        0x0
 *(.vector_46)
                0x00000001                ASSERT (((_vector_spacing == 0x0) || (SIZEOF (.vector_46) <= (_vector_spacing << 0x5))), function at exception vector 46 too large)

.vector_47      0x9d0067e0        0x0
 *(.vector_47)
                0x00000001                ASSERT (((_vector_spacing == 0x0) || (SIZEOF (.vector_47) <= (_vector_spacing << 0x5))), function at exception vector 47 too large)

.vector_48      0x9d006800        0x0
 *(.vector_48)
                0x00000001                ASSERT (((_vector_spacing == 0x0) || (SIZEOF (.vector_48) <= (_vector_spacing << 0x5))), function at exception vector 48 too large)

.vector_49      0x9d006820        0x0
 *(.vector_49)
                0x00000001                ASSERT (((_vector_spacing == 0x0) || (SIZEOF (.vector_49) <= (_vector_spacing << 0x5))), function at exception vector 49 too large)

.vector_50      0x9d006840        0x0
 *(.vector_50)
                0x00000001                ASSERT (((_vector_spacing == 0x0) || (SIZEOF (.vector_50) <= (_vector_spacing << 0x5))), function at exception vector 50 too large)

.vector_51      0x9d006860        0x0
 *(.vector_51)
                0x00000001                ASSERT (((_vector_spacing == 0x0) || (SIZEOF (.vector_51) <= (_vector_spacing << 0x5))), function at exception vector 51 too large)

.vector_52      0x9d006880        0x0
 *(.vector_52)
                0x00000001                ASSERT (((_vector_spacing == 0x0) || (SIZEOF (.vector_52) <= (_vector_spacing << 0x5))), function at exception vector 52 too large)

.vector_53      0x9d0068a0        0x0
 *(.vector_53)
                0x00000001                ASSERT (((_vector_spacing == 0x0) || (SIZEOF (.vector_53) <= (_vector_spacing << 0x5))), function at exception vector 53 too large)

.vector_54      0x9d0068c0        0x0
 *(.vector_54)
                0x00000001                ASSERT (((_vector_spacing == 0x0) || (SIZEOF (.vector_54) <= (_vector_spacing << 0x5))), function at exception vector 54 too large)

.vector_55      0x9d0068e0        0x0
 *(.vector_55)
                0x00000001                ASSERT (((_vector_spacing == 0x0) || (SIZEOF (.vector_55) <= (_vector_spacing << 0x5))), function at exception vector 55 too large)

.vector_56      0x9d006900        0x0
 *(.vector_56)
                0x00000001                ASSERT (((_vector_spacing == 0x0) || (SIZEOF (.vector_56) <= (_vector_spacing << 0x5))), function at exception vector 56 too large)

.vector_57      0x9d006920        0x0
 *(.vector_57)
                0x00000001                ASSERT (((_vector_spacing == 0x0) || (SIZEOF (.vector_57) <= (_vector_spacing << 0x5))), function at exception vector 57 too large)

.vector_58      0x9d006940        0x0
 *(.vector_58)
                0x00000001                ASSERT (((_vector_spacing == 0x0) || (SIZEOF (.vector_58) <= (_vector_spacing << 0x5))), function at exception vector 58 too large)

.vector_59      0x9d006960        0x0
 *(.vector_59)
                0x00000001                ASSERT (((_vector_spacing == 0x0) || (SIZEOF (.vector_59) <= (_vector_spacing << 0x5))), function at exception vector 59 too large)

.vector_60      0x9d006980        0x0
 *(.vector_60)
                0x00000001                ASSERT (((_vector_spacing == 0x0) || (SIZEOF (.vector_60) <= (_vector_spacing << 0x5))), function at exception vector 60 too large)

.vector_61      0x9d0069a0        0x0
 *(.vector_61)
                0x00000001                ASSERT (((_vector_spacing == 0x0) || (SIZEOF (.vector_61) <= (_vector_spacing << 0x5))), function at exception vector 61 too large)

.vector_62      0x9d0069c0        0x0
 *(.vector_62)
                0x00000001                ASSERT (((_vector_spacing == 0x0) || (SIZEOF (.vector_62) <= (_vector_spacing << 0x5))), function at exception vector 62 too large)

.vector_63      0x9d0069e0        0x0
 *(.vector_63)
                0x00000001                ASSERT (((_vector_spacing == 0x0) || (SIZEOF (.vector_63) <= (_vector_spacing << 0x5))), function at exception vector 63 too large)

.startup
 *(.startup)

.text
 *(.stub .gnu.linkonce.t.*)
 *(.text.*personality*)
 *(.mips16.fn.*)
 *(.mips16.call.*)
 *(.gnu.warning)

.rodata         0x9d007e00       0x48
 *(.rodata.* .gnu.linkonce.r.*)
 .rodata.f5pow  0x9d007e00       0x48 c:/program files/microchip/mplabc32/v2.02/bin/../lib/gcc/pic32mx/4.5.1/../../../../pic32mx/lib/speed\libe.a(_strtod.o)
 *(.rodata1)
                0x9d007e48                . = ALIGN (0x4)

.sdata2         0x9d007e48        0x0
 *(.sdata2 .sdata2.* .gnu.linkonce.s2.*)
                0x9d007e48                . = ALIGN (0x4)

.sbss2          0x9d007e48        0x0
 *(.sbss2 .sbss2.* .gnu.linkonce.sb2.*)
                0x9d007e48                . = ALIGN (0x4)

.eh_frame_hdr
 *(.eh_frame_hdr)

.eh_frame
 *(.eh_frame)

.dbg_data       0xa0000000        0x0
                0xa0000000                . = (. + DEFINED (_DEBUGGER)?0x200:0x0)

.persist        0xa0000000        0x0
                0xa0000000                _persist_begin = .
 *(.persist .persist.*)
                0xa0000000                . = ALIGN (0x4)
                0xa0000000                _persist_end = .

.eh_frame       0xa0000000       0x3c
 *(.eh_frame)
 .eh_frame      0xa0000000       0x28 c:/program files/microchip/mplabc32/v2.02/bin/../lib/gcc/pic32mx/4.5.1/speed\libgcc.a(_udivdi3.o)
 .eh_frame      0xa0000028       0x14 c:/program files/microchip/mplabc32/v2.02/bin/../lib/gcc/pic32mx/4.5.1/speed\libgcc.a(_umoddi3.o)
                                 0x28 (size before relaxing)
                0xa000003c                . = .
                0xa0008030                _gp = (ALIGN (0x10) + 0x7ff0)

.got
 *(.got.plt)
 *(.got)

.sdata          0xa000003c       0xc0
                0xa000003c                _sdata_begin = .
 *(.sdata .sdata.* .gnu.linkonce.s.*)
 .sdata         0xa000003c       0x10 output\main.o
                0xa000003c                HeaderID
                0xa0000040                VoiceID
                0xa0000044                LastFrameID
                0xa0000048                LinkID
 .sdata         0xa000004c        0x4 output\port.o
                0xa000004c                uxInterruptNesting
 .sdata         0xa0000050        0x4 output\tasks.o
 .sdata         0xa0000054        0x4 output\IntQueue.o
 .sdata         0xa0000058        0x4 output\heap_2.o
 .sdata         0xa000005c        0x8 output\usb_config.o
                0xa000005c                usbTPL
 .sdata         0xa0000064        0x4 output\CustomHTTPApp.o
                0xa0000064                RcvAprsSeq
 .sdata         0xa0000068        0xc output\FSIO.o
                0xa0000068                gLastFATSectorRead
                0xa000006c                gLastDataSectorRead
                0xa0000070                cwdptr
 .sdata         0xa0000074        0x2 output\UDP.o
 *fill*         0xa0000076        0x2 00
 .sdata         0xa0000078        0x8 output\DNS.o
 .sdata         0xa0000080       0x38 output\DstaDPlusClientUDP.o
                0xa0000080                RefName
                0xa0000094                ReqDisConnect
                0xa00000ac                Sync
                0xa00000b0                PttOff
                0xa00000b4                ServerSocket
                0xa00000b5                RcvDPlusSocket
                0xa00000b7                DprsSocket
 .sdata         0xa00000b8        0x1 output\FTP.o
 *fill*         0xa00000b9        0x3 00
 .sdata         0xa00000bc        0x4 output\Helpers.o
 .sdata         0xa00000c0        0x1 output\SNTP.o
 .sdata         0xa00000c1        0x2 output\TCP.o
 *fill*         0xa00000c3        0x1 00
 .sdata         0xa00000c4       0x18 output\prvTaskUSB.o
 .sdata         0xa00000dc        0xc output\prvTaskFS.o
 .sdata         0xa00000e8        0x1 output\SMTP.o
 *fill*         0xa00000e9        0x3 00
 .sdata         0xa00000ec        0x4 output\DHCPs.o
                0xa00000ec                bDHCPServerEnabled
 .sdata         0xa00000f0        0x4 c:/program files/microchip/mplabc32/v2.02/bin/../lib/gcc/pic32mx/4.5.1/../../../../pic32mx/lib/speed\libc.a(c32_uart.o)
                0xa00000f0                __C32_UART
 .sdata         0xa00000f4        0x8 c:/program files/microchip/mplabc32/v2.02/bin/../lib/gcc/pic32mx/4.5.1/../../../../pic32mx/lib/speed\libmchp_peripheral_32MX795F512L.a(_rtcc_wait_clock_off_lib.o)
                0xa00000f4                _RtccWaitClkStepSz
                0xa00000f8                _RtccWaitClkSteps
                0xa00000fc                _sdata_end = .

.lit8
 *(.lit8)

.lit4
 *(.lit4)
                0xa00000fc                . = ALIGN (0x4)
                0xa00000fc                _data_end = .
                0xa00000fc                _bss_begin = .

.sbss           0xa00000fc      0x875
                0xa00000fc                _sbss_begin = .
 *(.dynsbss)
 *(.sbss .sbss.* .gnu.linkonce.sb.*)
 .sbss          0xa00000fc        0x4 output\main.o
                0xa00000fc                DebugSW
 .sbss          0xa0000100        0x4 output\port.o
                0xa0000100                uxSavedTaskStackPointer
 .sbss          0xa0000104       0x44 output\tasks.o
                0xa0000104                pxCurrentTCB
 .sbss          0xa0000148       0x40 output\IntQueue.o
                0xa0000168                uxValueForNormallyEmptyQueue
                0xa000016c                uxValueForNormallyFullQueue
 .sbss          0xa0000188        0xc output\QPeek.o
 .sbss          0xa0000194        0xc output\lcd.o
 .sbss          0xa00001a0       0x18 output\prvTaskTCPIP.o
 .sbss          0xa00001b8       0x14 output\heap_2.o
 .sbss          0xa00001cc       0x6c output\usb_host.o
                0xa00001d8                pCurrentConfigurationDescriptor
                0xa00001dc                pDeviceDescriptor
 .sbss          0xa0000238       0xa8 output\CustomHTTPApp.o
                0xa0000238                AccCtlCnt
                0xa000024c                ReqAprsSeq
                0xa0000254                uploadfile
 .sbss          0xa00002e0       0x28 output\FSIO.o
                0xa00002e0                gNeedFATWrite
                0xa00002e4                gBufferOwner
                0xa00002e8                gNeedDataWrite
                0xa00002e9                nextClusterIsLast
                0xa00002ea                gBufferZeroed
                0xa00002eb                recache
                0xa00002ec                utfModeFileName
                0xa00002f0                twoByteMode
 .sbss          0xa0000308       0x14 output\UDP.o
 .sbss          0xa000031c        0x4 output\ARP.o
 .sbss          0xa0000320        0x4 output\DHCP.o
                0xa0000320                DHCPClientInitializedOnce
 .sbss          0xa0000324       0x18 output\DNS.o
 .sbss          0xa000033c      0x134 output\DstaDPlusClientUDP.o
                0xa0000348                AprsMessageSend
                0xa000034c                NodeDPlusState
                0xa0000350                RefSolveState
                0xa000036c                first_pnt
                0xa0000370                last_pnt
                0xa0000380                DprsOpen
 .sbss          0xa0000470       0x40 output\ETHPIC32IntMac.o
                0xa0000484                _CurrWrPtr
                0xa0000488                _CurrRdPtr
                0xa000049c                _stackMgrRxOkPkts
                0xa00004a0                _stackMgrRxBadPkts
                0xa00004a4                _stackMgrInGetHdr
                0xa00004a8                _stackMgrRxDiscarded
                0xa00004ac                _stackMgrTxNotReady
 .sbss          0xa00004b0       0x58 output\FTP.o
 .sbss          0xa0000508       0x4c output\HTTP2.o
 .sbss          0xa0000554        0x4 output\IP.o
 .sbss          0xa0000558        0x8 output\MPFS2.o
 .sbss          0xa0000560       0x20 output\SNTP.o
 .sbss          0xa0000580        0x8 output\StackTsk.o
 .sbss          0xa0000588        0x2 output\TCP.o
 *fill*         0xa000058a        0x2 00
 .sbss          0xa000058c       0x18 output\Tick.o
 .sbss          0xa00005a4       0x1c output\SD-SPI.o
 .sbss          0xa00005c0      0x118 output\prvTaskUSB.o
 .sbss          0xa00006d8       0x5c output\prvTaskFS.o
                0xa00006d8                AprsCallTablePnt
 .sbss          0xa0000734        0x2 output\MACread.o
 *fill*         0xa0000736        0x2 00
 .sbss          0xa0000738       0x34 output\SMTP.o
 .sbss          0xa000076c        0x4 output\DprsSMTP.o
 .sbss          0xa0000770       0x14 output\serial.o
 .sbss          0xa0000784        0xc output\comtest.o
 .sbss          0xa0000790       0x28 output\DHCPs.o
 .sbss          0xa00007b8       0x10 output\NBNS.o
 .sbss          0xa00007c8        0x4 c:/program files/microchip/mplabc32/v2.02/bin/../lib/gcc/pic32mx/4.5.1/../../../../pic32mx/lib/speed\libc.a(ctime.o)
                0xa00007c8                time_zone
 .sbss          0xa00007cc        0x1 c:/program files/microchip/mplabc32/v2.02/bin/../lib/gcc/pic32mx/4.5.1/../../../../pic32mx/lib/speed\libc.a(_iob.o)
                0xa00007cc                _outdone
 *fill*         0xa00007cd        0x3 00
 .sbss          0xa00007d0       0x20 c:/program files/microchip/mplabc32/v2.02/bin/../lib/gcc/pic32mx/4.5.1/../../../../pic32mx/lib/speed\libmchp_peripheral_32MX795F512L.a(eth_descriptors_add_lib.o)
                0xa00007d0                _EthTxFreeList
                0xa00007d8                _EthTxBusyList
                0xa00007e0                _EthRxFreeList
                0xa00007e8                _EthRxBusyList
 .sbss          0xa00007f0        0x4 c:/program files/microchip/mplabc32/v2.02/bin/../lib/gcc/pic32mx/4.5.1/../../../../pic32mx/lib/speed\libc.a(errno.o)
                0xa00007f0                errno
 *(.scommon)
 .scommon       0xa00007f4       0x6c output\main.o
                0xa00007f4                SSN
                0xa00007f8                xDstarHttpQueue
                0xa00007fc                xMessage
                0xa0000804                COS_On
                0xa0000808                PTT_On
                0xa000080c                xDstarDprsMsgQueue
                0xa0000810                FWUpdate
                0xa0000814                PicVer
                0xa0000818                xDstarDprsEmailMsgQueue
                0xa000081c                xDstarRcvQueue
                0xa0000820                xDstarDprsAccQueue
                0xa0000824                xDstarAccQueue
                0xa0000828                xDstarLogQueue
                0xa000082c                voice_pnt
                0xa000082e                left_byte
                0xa0000830                AccessFileReadSW
                0xa0000834                FSHandle
                0xa0000838                ReqConvertLocalRefFile
                0xa000083c                USBHandle
                0xa0000840                ReqRefDomainName
                0xa0000844                xDstarRefQueue
                0xa0000848                MyMACAddr
                0xa0000850                xDstarSndQueue
                0xa0000854                FSInitSW
                0xa0000858                DPRS_SW
                0xa000085c                TCPHandle
 .scommon       0xa0000860       0x10 output\IntQueue.o
                0xa0000860                xHighPriorityNormallyFullTask2
                0xa0000864                xHighPriorityNormallyEmptyTask1
                0xa0000868                xHighPriorityNormallyEmptyTask2
                0xa000086c                xHighPriorityNormallyFullTask1
 .scommon       0xa0000870        0xc output\QPeek.o
                0xa0000870                xHighestPriorityTask
                0xa0000874                xHighPriorityTask
                0xa0000878                xMediumPriorityTask
 .scommon       0xa000087c        0x8 output\lcd.o
                0xa000087c                LCDHandle
                0xa0000880                xLCDQueue
 .scommon       0xa0000884        0x0 output\prvTaskTCPIP.o
 .scommon       0xa0000884       0x10 output\CustomHTTPApp.o
                0xa0000884                CurUser
                0xa000088c                AprsSeq
                0xa0000890                ReqRefList
 .scommon       0xa0000894       0x2c output\FSIO.o
                0xa0000894                utf16Filename
                0xa0000898                recordSearchLength
                0xa000089c                TempClusterCalc
                0xa00008a0                gTimeCrtTime
                0xa00008a4                gFileSlotOpen
                0xa00008a8                gTimeAccDate
                0xa00008aa                gTimeCrtDate
                0xa00008ac                asciiFilename
                0xa00008b0                FSerrno
                0xa00008b2                fileNameLength
                0xa00008b4                dirCleared
                0xa00008b6                gTimeWrtTime
                0xa00008b8                FatRootDirClusterValue
                0xa00008bc                gTimeCrtMS
                0xa00008be                gTimeWrtDate
 .scommon       0xa00008c0        0x6 output\UDP.o
                0xa00008c0                activeUDPSocket
                0xa00008c2                UDPTxCount
                0xa00008c4                UDPRxCount
 *fill*         0xa00008c6        0x2 00
 .scommon       0xa00008c8       0x7c output\DstaDPlusClientUDP.o
                0xa00008c8                Radio_GPS_A_Msg_send
                0xa00008cc                RadioSpeed
                0xa00008d0                RadioDprsSend
                0xa00008d4                Msg
                0xa00008d8                MyCallSign
                0xa00008e0                AprsMsgTX
                0xa00008e3                deviceAddress
                0xa00008e4                RefSkipSW
                0xa00008e8                InetDirection
                0xa00008ec                RadioAtitude
                0xa00008f4                InetAtitude
                0xa00008fc                KeepAliveTimer
                0xa0000900                RadioCall
                0xa0000908                InetCall
                0xa0000910                RefNameSet
                0xa0000914                Inet_GPS_A_Msg_send
                0xa0000918                InetSpeed
                0xa000091c                RefNameTemp
                0xa0000924                InetLat
                0xa000092c                RadioDirection
                0xa0000930                RadioLat
                0xa0000938                InetDprsSend
                0xa000093c                RefNameSave
 .scommon       0xa0000944        0x4 output\ETHPIC32ExtPhy.o
                0xa0000944                _PhyAdd
 .scommon       0xa0000948        0xc output\HTTP2.o
                0xa0000948                curHTTPID
                0xa000094c                httpStubs
 .scommon       0xa0000954        0x8 output\SD-SPI.o
                0xa0000954                gMediaSectorSize
                0xa0000956                gSDMode
                0xa0000958                MDD_SDSPI_finalLBA
 .scommon       0xa000095c        0x8 output\prvTaskUSB.o
                0xa000095c                VoiceMsg
                0xa0000960                headerRead
 .scommon       0xa0000964        0xc output\prvTaskFS.o
                0xa0000964                ReqLoadAprsCallCheck
                0xa0000968                CallCheck_Skip
                0xa000096c                DprsAccessFileReadSW
 .scommon       0xa0000970        0x1 output\MACread.o
                0xa0000970                MACReadWriteSW
 .scommon       0xa0000971        0x0 output\DprsSMTP.o
                0xa0000971                _sbss_end = .

.bss            0xa0000974     0x1db4
 *(.dynbss)
 *(COMMON)
 COMMON         0xa0000974      0x218 output\main.o
                0xa0000974                AdParam
                0xa00009c4                header
                0xa00009f0                Text
                0xa0000a10                DPRS
                0xa0000aa4                rig_buffer
                0xa0000ac4                TimeDate
                0xa0000ad8                AppConfig
                0xa0000b80                voice
 COMMON         0xa0000b8c      0x116 output\CustomHTTPApp.o
                0xa0000b8c                REF_IP_address
                0xa0000b9c                AprsDest
                0xa0000ba8                newAppConfig
                0xa0000c50                AprsSenderCall
                0xa0000c5c                AprsMessage
 *fill*         0xa0000ca2        0x2 00
 COMMON         0xa0000ca4       0x10 output\usb_host_generic.o
                0xa0000ca4                gc_DevData
 COMMON         0xa0000cb4     0x13f2 output\FSIO.o
                0xa0000cb4                tempCWDobj
                0xa0000cf8                fileFoundString
                0xa0000f04                lfnData
                0xa000150c                gDiskData
                0xa0001534                gFATBuffer
                0xa0001734                cwd
                0xa0001778                gDataBuffer
                0xa0001978                recordFoundName
                0xa0001b7c                gFileArray
                0xa0001c48                recordSearchName
                0xa0001e4c                gFileTemp
                0xa0001e90                tempDirectoryString
                0xa000209c                defaultArray
 *fill*         0xa00020a6        0x2 00
 COMMON         0xa00020a8      0x280 output\UDP.o
                0xa00020a8                UDPSocketInfo
 COMMON         0xa0002328      0x273 output\DstaDPlusClientUDP.o
                0xa0002328                RadioLong
                0xa0002334                EmailAddress
                0xa0002364                FirstTable
                0xa0002378                InetLong
                0xa0002384                RDateTime
                0xa0002390                Radio_GPS_A_MSG
                0xa0002408                Inet_GPS_A_MSG
                0xa0002480                RadioMsg
                0xa0002494                CurServerName
                0xa00024a8                DprsMsgDstCallSignSave
                0xa00024b4                RefDomainName
                0xa0002524                InetMsg
                0xa0002538                DCS_recv
 *fill*         0xa000259b        0x1 00
 COMMON         0xa000259c       0x8c output\HTTP2.o
                0xa000259c                curHTTP
 COMMON         0xa0002628        0xa output\StackTsk.o
                0xa0002628                remoteNode
 *fill*         0xa0002632        0x2 00
 COMMON         0xa0002634        0x9 output\prvTaskUSB.o
                0xa0002634                DprsMyCall
 *fill*         0xa000263d        0x3 00
 COMMON         0xa0002640       0x2d output\prvTaskFS.o
                0xa0002640                DprsMsgDstCallSign
                0xa000264c                Radio_Callsign_Check_String
                0xa0002658                DprsMsgSrcCallSign
                0xa0002664                Inet_Callsign_Check_String
 *fill*         0xa000266d        0x3 00
 COMMON         0xa0002670       0x2c output\SMTP.o
                0xa0002670                SMTPClient
 COMMON         0xa000269c       0x8a output\DprsSMTP.o
                0xa000269c                EmailTemp
                0xa0002728                . = ALIGN (0x4)
 *fill*         0xa0002726        0x2 00
                0xa0002728                . = ALIGN (0x4)
                0xa0002728                _end = .
                0xa0002728                _bss_end = .
                0x00020000                _bmxdudba_address = 0x20000
                0x00020000                _bmxdupba_address = 0x20000

/DISCARD/
 *(.pdr)
 *(.reginfo)
 *(.rel.dyn)
 *(.note.GNU-stack)
 *(.note.GNU-stack)
 *(.gnu_debuglink)
 *(.gnu.lto_*)
 *(.discard)

.stab
 *(.stab)

.stabstr
 *(.stabstr)

.stab.excl
 *(.stab.excl)

.stab.exclstr
 *(.stab.exclstr)

.stab.index
 *(.stab.index)

.stab.indexstr
 *(.stab.indexstr)

.comment        0x00000000      0x420
 *(.comment)
 .comment       0x00000000       0x51 output\main.o
                                 0x52 (size before relaxing)
 .comment       0x00000000       0x52 output\IntQueueTimer.o
 .comment       0x00000000       0x52 output\port.o
 .comment       0x00000000       0x52 output\queue.o
 .comment       0x00000000       0x52 output\tasks.o
 .comment       0x00000000       0x52 output\list.o
 .comment       0x00000000       0x52 output\IntQueue.o
 .comment       0x00000000       0x52 output\QPeek.o
 .comment       0x00000000       0x52 output\lcd.o
 .comment       0x00000000       0x52 output\prvTaskTCPIP.o
 .comment       0x00000000       0x52 output\heap_2.o
 .comment       0x00000000       0x52 output\usb_host.o
 .comment       0x00000000       0x52 output\usb_config.o
 .comment       0x00000000       0x52 output\CustomHTTPApp.o
 .comment       0x00000000       0x52 output\usb_host_generic.o
 .comment       0x00000000       0x52 output\FSIO.o
 .comment       0x00000000       0x52 output\UDP.o
 .comment       0x00000000       0x52 output\ARP.o
 .comment       0x00000000       0x52 output\Delay.o
 .comment       0x00000000       0x52 output\DHCP.o
 .comment       0x00000000       0x52 output\DNS.o
 .comment       0x00000000       0x52 output\DstaDPlusClientUDP.o
 .comment       0x00000000       0x52 output\ETHPIC32ExtPhy.o
 .comment       0x00000000       0x52 output\ETHPIC32ExtPhyDP83848.o
 .comment       0x00000000       0x52 output\ETHPIC32IntMac.o
 .comment       0x00000000       0x52 output\FileSystem.o
 .comment       0x00000000       0x52 output\FTP.o
 .comment       0x00000000       0x52 output\Hashes.o
 .comment       0x00000000       0x52 output\Helpers.o
 .comment       0x00000000       0x52 output\HTTP2.o
 .comment       0x00000000       0x52 output\ICMP.o
 .comment       0x00000000       0x52 output\IP.o
 .comment       0x00000000       0x52 output\MPFS2.o
 .comment       0x00000000       0x52 output\Random.o
 .comment       0x00000000       0x52 output\SNTP.o
 .comment       0x00000000       0x52 output\StackTsk.o
 .comment       0x00000000       0x52 output\TCP.o
 .comment       0x00000000       0x52 output\Tick.o
 .comment       0x00000000       0x52 output\MPFSImg2.o
 .comment       0x00000000       0x52 output\SD-SPI.o
 .comment       0x00000000       0x52 output\prvTaskUSB.o
 .comment       0x00000000       0x52 output\prvTaskFS.o
 .comment       0x00000000       0x52 output\MACread.o
 .comment       0x00000000       0x52 output\SMTP.o
 .comment       0x00000000       0x52 output\DprsSMTP.o
 .comment       0x00000000       0x52 output\serial.o
 .comment       0x00000000       0x52 output\comtest.o
 .comment       0x00000000       0x52 output\DHCPs.o
 .comment       0x00000000       0x52 output\NBNS.o
 .comment       0x00000000       0x52 c:/program files/microchip/mplabc32/v2.02/bin/../lib/gcc/pic32mx/4.5.1/speed\libgcc.a(_udivdi3.o)
 .comment       0x00000000       0x52 c:/program files/microchip/mplabc32/v2.02/bin/../lib/gcc/pic32mx/4.5.1/speed\libgcc.a(_umoddi3.o)
 .comment       0x00000000       0x52 c:/program files/microchip/mplabc32/v2.02/bin/../lib/gcc/pic32mx/4.5.1/speed\libgcc.a(floatunsisf.o)
 .comment       0x00000051       0x55 c:/program files/microchip/mplabc32/v2.02/bin/../lib/gcc/pic32mx/4.5.1/../../../../pic32mx/lib/speed\libc.a(memcmp.o)
                                 0x56 (size before relaxing)
 .comment       0x000000a6       0x55 c:/program files/microchip/mplabc32/v2.02/bin/../lib/gcc/pic32mx/4.5.1/../../../../pic32mx/lib/speed\libc.a(memset.o)
                                 0x56 (size before relaxing)
 .comment       0x000000fb       0x55 c:/program files/microchip/mplabc32/v2.02/bin/../lib/gcc/pic32mx/4.5.1/../../../../pic32mx/lib/speed\libc.a(strcmp.o)
                                 0x56 (size before relaxing)
 .comment       0x00000150       0x55 c:/program files/microchip/mplabc32/v2.02/bin/../lib/gcc/pic32mx/4.5.1/../../../../pic32mx/lib/speed\libc.a(strcpy.o)
                                 0x56 (size before relaxing)
 .comment       0x000001a5       0x55 c:/program files/microchip/mplabc32/v2.02/bin/../lib/gcc/pic32mx/4.5.1/../../../../pic32mx/lib/speed\libc.a(strlen.o)
                                 0x56 (size before relaxing)
 .comment       0x00000000       0x52 c:/program files/microchip/mplabc32/v2.02/bin/../lib/gcc/pic32mx/4.5.1/../../../../pic32mx/lib/speed\libc.a(atoi.o)
 .comment       0x00000000       0x52 c:/program files/microchip/mplabc32/v2.02/bin/../lib/gcc/pic32mx/4.5.1/../../../../pic32mx/lib/speed\libc.a(atol.o)
 .comment       0x00000000       0x52 c:/program files/microchip/mplabc32/v2.02/bin/../lib/gcc/pic32mx/4.5.1/../../../../pic32mx/lib/speed\libc.a(ctime.o)
 .comment       0x000001fa       0x4e c:/program files/microchip/mplabc32/v2.02/bin/../lib/gcc/pic32mx/4.5.1/../../../../pic32mx/lib/speed\libc.a(ctype.o)
                                 0xa0 (size before relaxing)
 .comment       0x00000248       0x4f c:/program files/microchip/mplabc32/v2.02/bin/../lib/gcc/pic32mx/4.5.1/../../../../pic32mx/lib/speed\libc.a(ctypef.o)
                                 0xa1 (size before relaxing)
 .comment       0x00000000       0x52 c:/program files/microchip/mplabc32/v2.02/bin/../lib/gcc/pic32mx/4.5.1/../../../../pic32mx/lib/speed\libc.a(strcat.o)
 .comment       0x00000000       0x52 c:/program files/microchip/mplabc32/v2.02/bin/../lib/gcc/pic32mx/4.5.1/../../../../pic32mx/lib/speed\libc.a(strchr.o)
 .comment       0x00000000       0x52 c:/program files/microchip/mplabc32/v2.02/bin/../lib/gcc/pic32mx/4.5.1/../../../../pic32mx/lib/speed\libc.a(strncpy.o)
 .comment       0x00000000       0x52 c:/program files/microchip/mplabc32/v2.02/bin/../lib/gcc/pic32mx/4.5.1/../../../../pic32mx/lib/speed\libc.a(strstr.o)
 .comment       0x00000000       0x52 c:/program files/microchip/mplabc32/v2.02/bin/../lib/gcc/pic32mx/4.5.1/../../../../pic32mx/lib/speed\libc.a(atof.o)
 .comment       0x00000000       0x52 c:/program files/microchip/mplabc32/v2.02/bin/../lib/gcc/pic32mx/4.5.1/../../../../pic32mx/lib/speed\libc.a(sprintf_cdnopsuxX.eo)
 .comment       0x00000000       0x52 c:/program files/microchip/mplabc32/v2.02/bin/../lib/gcc/pic32mx/4.5.1/../../../../pic32mx/lib/speed\libc.a(default-bootstrap-exception-handler.o)
 .comment       0x00000000       0x52 c:/program files/microchip/mplabc32/v2.02/bin/../lib/gcc/pic32mx/4.5.1/../../../../pic32mx/lib/speed\libc.a(default-on-reset.o)
 .comment       0x00000000       0x52 c:/program files/microchip/mplabc32/v2.02/bin/../lib/gcc/pic32mx/4.5.1/../../../../pic32mx/lib/speed\libc.a(default-on-bootstrap.o)
 .comment       0x00000000       0x52 c:/program files/microchip/mplabc32/v2.02/bin/../lib/gcc/pic32mx/4.5.1/../../../../pic32mx/lib/speed\libc.a(strncmp.o)
 .comment       0x00000000       0x52 c:/program files/microchip/mplabc32/v2.02/bin/../lib/gcc/pic32mx/4.5.1/../../../../pic32mx/lib/speed\libc.a(strtod.o)
 .comment       0x00000000       0x52 c:/program files/microchip/mplabc32/v2.02/bin/../lib/gcc/pic32mx/4.5.1/../../../../pic32mx/lib/speed\libc.a(doprnt_cdnopsuxX.eo)
 .comment       0x00000000       0x52 c:/program files/microchip/mplabc32/v2.02/bin/../lib/gcc/pic32mx/4.5.1/../../../../pic32mx/lib/speed\libc.a(_fputc_simple.o)
 .comment       0x00000000       0x52 c:/program files/microchip/mplabc32/v2.02/bin/../lib/gcc/pic32mx/4.5.1/../../../../pic32mx/lib/speed\libc.a(write.o)
 .comment       0x00000000       0x52 c:/program files/microchip/mplabc32/v2.02/bin/../lib/gcc/pic32mx/4.5.1/../../../../pic32mx/lib/speed\libc.a(_iob.o)
 .comment       0x00000000       0x52 c:/program files/microchip/mplabc32/v2.02/bin/../lib/gcc/pic32mx/4.5.1/../../../../pic32mx/lib/speed\libc.a(_flsbuf_simple.o)
 .comment       0x00000000       0x52 c:/program files/microchip/mplabc32/v2.02/bin/../lib/gcc/pic32mx/4.5.1/../../../../pic32mx/lib/speed\libc.a(_mon_putc.o)
 .comment       0x00000000       0x52 c:/program files/microchip/mplabc32/v2.02/bin/../lib/gcc/pic32mx/4.5.1/../../../../pic32mx/lib/speed\libc.a(c32_uart.o)
 .comment       0x00000297       0x9d c:/program files/microchip/mplabc32/v2.02/bin/../lib/gcc/pic32mx/4.5.1/../../../../pic32mx/lib/speed\libe.a(_strtod.o)
                                 0xef (size before relaxing)
 .comment       0x00000334       0x50 c:/program files/microchip/mplabc32/v2.02/bin/../lib/gcc/pic32mx/4.5.1/../../../../pic32mx/lib/speed\libe.a(_ldexp.o)
                                 0xf0 (size before relaxing)
 .comment       0x00000384       0x51 c:/program files/microchip/mplabc32/v2.02/bin/../lib/gcc/pic32mx/4.5.1/../../../../pic32mx/lib/speed\libmchp_peripheral.a(read_core_timer_lib.o)
                                 0x52 (size before relaxing)
 .comment       0x00000000       0x52 c:/program files/microchip/mplabc32/v2.02/bin/../lib/gcc/pic32mx/4.5.1/../../../../pic32mx/lib/speed\libmchp_peripheral.a(write_core_timer_lib.o)
 .comment       0x00000000       0x52 c:/program files/microchip/mplabc32/v2.02/bin/../lib/gcc/pic32mx/4.5.1/../../../../pic32mx/lib/speed\libmchp_peripheral_32MX795F512L.a(eth_ack_packet_lib.o)
 .comment       0x00000000       0x52 c:/program files/microchip/mplabc32/v2.02/bin/../lib/gcc/pic32mx/4.5.1/../../../../pic32mx/lib/speed\libmchp_peripheral_32MX795F512L.a(eth_descriptors_add_lib.o)
 .comment       0x00000000       0x52 c:/program files/microchip/mplabc32/v2.02/bin/../lib/gcc/pic32mx/4.5.1/../../../../pic32mx/lib/speed\libmchp_peripheral_32MX795F512L.a(eth_init_lib.o)
 .comment       0x00000000       0x52 c:/program files/microchip/mplabc32/v2.02/bin/../lib/gcc/pic32mx/4.5.1/../../../../pic32mx/lib/speed\libmchp_peripheral_32MX795F512L.a(eth_mac_open_lib.o)
 .comment       0x00000000       0x52 c:/program files/microchip/mplabc32/v2.02/bin/../lib/gcc/pic32mx/4.5.1/../../../../pic32mx/lib/speed\libmchp_peripheral_32MX795F512L.a(eth_mac_set_address_max_lib.o)
 .comment       0x00000000       0x52 c:/program files/microchip/mplabc32/v2.02/bin/../lib/gcc/pic32mx/4.5.1/../../../../pic32mx/lib/speed\libmchp_peripheral_32MX795F512L.a(eth_rx_buffers_append_lib.o)
 .comment       0x00000000       0x52 c:/program files/microchip/mplabc32/v2.02/bin/../lib/gcc/pic32mx/4.5.1/../../../../pic32mx/lib/speed\libmchp_peripheral_32MX795F512L.a(eth_rx_filters_lib.o)
 .comment       0x00000000       0x52 c:/program files/microchip/mplabc32/v2.02/bin/../lib/gcc/pic32mx/4.5.1/../../../../pic32mx/lib/speed\libmchp_peripheral_32MX795F512L.a(eth_rx_get_packet_lib.o)
 .comment       0x00000000       0x52 c:/program files/microchip/mplabc32/v2.02/bin/../lib/gcc/pic32mx/4.5.1/../../../../pic32mx/lib/speed\libmchp_peripheral_32MX795F512L.a(eth_rx_set_buffer_size_lib.o)
 .comment       0x00000000       0x52 c:/program files/microchip/mplabc32/v2.02/bin/../lib/gcc/pic32mx/4.5.1/../../../../pic32mx/lib/speed\libmchp_peripheral_32MX795F512L.a(eth_tx_packet_lib.o)
 .comment       0x00000000       0x52 c:/program files/microchip/mplabc32/v2.02/bin/../lib/gcc/pic32mx/4.5.1/../../../../pic32mx/lib/speed\libmchp_peripheral_32MX795F512L.a(_eth_append_busy_list_lib.o)
 .comment       0x00000000       0x52 c:/program files/microchip/mplabc32/v2.02/bin/../lib/gcc/pic32mx/4.5.1/../../../../pic32mx/lib/speed\libmchp_peripheral_32MX795F512L.a(eth_miim_access.o)
 .comment       0x00000000       0x52 c:/program files/microchip/mplabc32/v2.02/bin/../lib/gcc/pic32mx/4.5.1/../../../../pic32mx/lib/speed\libmchp_peripheral_32MX795F512L.a(soft_reset_lib.o)
 .comment       0x00000000       0x52 c:/program files/microchip/mplabc32/v2.02/bin/../lib/gcc/pic32mx/4.5.1/../../../../pic32mx/lib/speed\libmchp_peripheral_32MX795F512L.a(pcache.o)
 .comment       0x00000000       0x52 c:/program files/microchip/mplabc32/v2.02/bin/../lib/gcc/pic32mx/4.5.1/../../../../pic32mx/lib/speed\libmchp_peripheral_32MX795F512L.a(set_core_sw0_leg_lib.o)
 .comment       0x00000000       0x52 c:/program files/microchip/mplabc32/v2.02/bin/../lib/gcc/pic32mx/4.5.1/../../../../pic32mx/lib/speed\libmchp_peripheral_32MX795F512L.a(int_disable_interrupts_lib.o)
 .comment       0x00000000       0x52 c:/program files/microchip/mplabc32/v2.02/bin/../lib/gcc/pic32mx/4.5.1/../../../../pic32mx/lib/speed\libmchp_peripheral_32MX795F512L.a(int_restore_interrupts_lib.o)
 .comment       0x00000000       0x52 c:/program files/microchip/mplabc32/v2.02/bin/../lib/gcc/pic32mx/4.5.1/../../../../pic32mx/lib/speed\libmchp_peripheral_32MX795F512L.a(int_enable_mv_int_lib.o)
 .comment       0x00000000       0x52 c:/program files/microchip/mplabc32/v2.02/bin/../lib/gcc/pic32mx/4.5.1/../../../../pic32mx/lib/speed\libmchp_peripheral_32MX795F512L.a(int_tbl_lib.o)
 .comment       0x00000000       0x52 c:/program files/microchip/mplabc32/v2.02/bin/../lib/gcc/pic32mx/4.5.1/../../../../pic32mx/lib/speed\libmchp_peripheral_32MX795F512L.a(rtcc_init_lib.o)
 .comment       0x00000000       0x52 c:/program files/microchip/mplabc32/v2.02/bin/../lib/gcc/pic32mx/4.5.1/../../../../pic32mx/lib/speed\libmchp_peripheral_32MX795F512L.a(rtcc_set_time_date_lib.o)
 .comment       0x00000000       0x52 c:/program files/microchip/mplabc32/v2.02/bin/../lib/gcc/pic32mx/4.5.1/../../../../pic32mx/lib/speed\libmchp_peripheral_32MX795F512L.a(rtcc_open_lib.o)
 .comment       0x00000000       0x52 c:/program files/microchip/mplabc32/v2.02/bin/../lib/gcc/pic32mx/4.5.1/../../../../pic32mx/lib/speed\libmchp_peripheral_32MX795F512L.a(spi_getc_spi1_lib_legacy.o)
 .comment       0x00000000       0x52 c:/program files/microchip/mplabc32/v2.02/bin/../lib/gcc/pic32mx/4.5.1/../../../../pic32mx/lib/speed\libmchp_peripheral_32MX795F512L.a(spi_open_spi1_lib_legacy.o)
 .comment       0x00000000       0x52 c:/program files/microchip/mplabc32/v2.02/bin/../lib/gcc/pic32mx/4.5.1/../../../../pic32mx/lib/speed\libmchp_peripheral_32MX795F512L.a(spi_brg_tbl_lib_legacy.o)
 .comment       0x00000000       0x52 c:/program files/microchip/mplabc32/v2.02/bin/../lib/gcc/pic32mx/4.5.1/../../../../pic32mx/lib/speed\libmchp_peripheral_32MX795F512L.a(port_set_pins_digital_in_lib.o)
 .comment       0x00000000       0x52 c:/program files/microchip/mplabc32/v2.02/bin/../lib/gcc/pic32mx/4.5.1/../../../../pic32mx/lib/speed\libmchp_peripheral_32MX795F512L.a(port_set_pins_digital_out_lib.o)
 .comment       0x00000000       0x52 c:/program files/microchip/mplabc32/v2.02/bin/../lib/gcc/pic32mx/4.5.1/../../../../pic32mx/lib/speed\libmchp_peripheral_32MX795F512L.a(_ports_tbl_libp.o)
 .comment       0x00000000       0x52 c:/program files/microchip/mplabc32/v2.02/bin/../lib/gcc/pic32mx/4.5.1/../../../../pic32mx/lib/speed\libmchp_peripheral_32MX795F512L.a(int_enable_interrupts_lib.o)
 .comment       0x00000000       0x52 c:/program files/microchip/mplabc32/v2.02/bin/../lib/gcc/pic32mx/4.5.1/../../../../pic32mx/lib/speed\libmchp_peripheral_32MX795F512L.a(_rtcc_set_time_and_date_lib.o)
 .comment       0x00000000       0x52 c:/program files/microchip/mplabc32/v2.02/bin/../lib/gcc/pic32mx/4.5.1/../../../../pic32mx/lib/speed\libmchp_peripheral_32MX795F512L.a(_rtcc_wait_clock_off_lib.o)
 .comment       0x00000000       0x52 c:/program files/microchip/mplabc32/v2.02/bin/../lib/gcc/pic32mx/4.5.1/../../../../pic32mx/lib/speed\libc.a(calloc.o)
 .comment       0x00000000       0x52 c:/program files/microchip/mplabc32/v2.02/bin/../lib/gcc/pic32mx/4.5.1/../../../../pic32mx/lib/speed\libc.a(errno.o)
 .comment       0x00000000       0x52 c:/program files/microchip/mplabc32/v2.02/bin/../lib/gcc/pic32mx/4.5.1/../../../../pic32mx/lib/speed\libc.a(malloc.o)
 .comment       0x000003d5       0x4b c:/program files/microchip/mplabc32/v2.02/bin/../lib/gcc/pic32mx/4.5.1/../../../../pic32mx/lib/speed\libc.a(sbrk.o)
                                 0x9d (size before relaxing)
 .comment       0x00000000       0x52 c:/program files/microchip/mplabc32/v2.02/bin/../lib/gcc/pic32mx/4.5.1/speed\libgcc.a(_lshrdi3.o)
 .comment       0x00000000       0x52 c:/program files/microchip/mplabc32/v2.02/bin/../lib/gcc/pic32mx/4.5.1/speed\libgcc.a(_ashldi3.o)

.debug
 *(.debug)

.line
 *(.line)

.debug_srcinfo
 *(.debug_srcinfo)

.debug_sfnames
 *(.debug_sfnames)

.debug_aranges  0x00000000      0x970
 *(.debug_aranges)
 .debug_aranges
                0x00000000       0x20 c:/program files/microchip/mplabc32/v2.02/bin/../lib/gcc/pic32mx/4.5.1/speed\libgcc.a(_udivdi3.o)
 .debug_aranges
                0x00000020       0x20 c:/program files/microchip/mplabc32/v2.02/bin/../lib/gcc/pic32mx/4.5.1/speed\libgcc.a(_umoddi3.o)
 .debug_aranges
                0x00000040       0x20 c:/program files/microchip/mplabc32/v2.02/bin/../lib/gcc/pic32mx/4.5.1/speed\libgcc.a(floatunsisf.o)
 .debug_aranges
                0x00000060       0x20 c:/program files/microchip/mplabc32/v2.02/bin/../lib/gcc/pic32mx/4.5.1/../../../../pic32mx/lib/speed\libc.a(atoi.o)
 .debug_aranges
                0x00000080       0x20 c:/program files/microchip/mplabc32/v2.02/bin/../lib/gcc/pic32mx/4.5.1/../../../../pic32mx/lib/speed\libc.a(atol.o)
 .debug_aranges
                0x000000a0       0x38 c:/program files/microchip/mplabc32/v2.02/bin/../lib/gcc/pic32mx/4.5.1/../../../../pic32mx/lib/speed\libc.a(ctime.o)
 .debug_aranges
                0x000000d8       0xa0 c:/program files/microchip/mplabc32/v2.02/bin/../lib/gcc/pic32mx/4.5.1/../../../../pic32mx/lib/speed\libc.a(ctypef.o)
 .debug_aranges
                0x00000178       0x20 c:/program files/microchip/mplabc32/v2.02/bin/../lib/gcc/pic32mx/4.5.1/../../../../pic32mx/lib/speed\libc.a(strcat.o)
 .debug_aranges
                0x00000198       0x20 c:/program files/microchip/mplabc32/v2.02/bin/../lib/gcc/pic32mx/4.5.1/../../../../pic32mx/lib/speed\libc.a(strchr.o)
 .debug_aranges
                0x000001b8       0x20 c:/program files/microchip/mplabc32/v2.02/bin/../lib/gcc/pic32mx/4.5.1/../../../../pic32mx/lib/speed\libc.a(strncpy.o)
 .debug_aranges
                0x000001d8       0x20 c:/program files/microchip/mplabc32/v2.02/bin/../lib/gcc/pic32mx/4.5.1/../../../../pic32mx/lib/speed\libc.a(strstr.o)
 .debug_aranges
                0x000001f8       0x20 c:/program files/microchip/mplabc32/v2.02/bin/../lib/gcc/pic32mx/4.5.1/../../../../pic32mx/lib/speed\libc.a(atof.o)
 .debug_aranges
                0x00000218       0x20 c:/program files/microchip/mplabc32/v2.02/bin/../lib/gcc/pic32mx/4.5.1/../../../../pic32mx/lib/speed\libc.a(sprintf_cdnopsuxX.eo)
 .debug_aranges
                0x00000238       0x20 c:/program files/microchip/mplabc32/v2.02/bin/../lib/gcc/pic32mx/4.5.1/../../../../pic32mx/lib/speed\libc.a(default-bootstrap-exception-handler.o)
 .debug_aranges
                0x00000258       0x20 c:/program files/microchip/mplabc32/v2.02/bin/../lib/gcc/pic32mx/4.5.1/../../../../pic32mx/lib/speed\libc.a(default-on-reset.o)
 .debug_aranges
                0x00000278       0x20 c:/program files/microchip/mplabc32/v2.02/bin/../lib/gcc/pic32mx/4.5.1/../../../../pic32mx/lib/speed\libc.a(default-on-bootstrap.o)
 .debug_aranges
                0x00000298       0x20 c:/program files/microchip/mplabc32/v2.02/bin/../lib/gcc/pic32mx/4.5.1/../../../../pic32mx/lib/speed\libc.a(strncmp.o)
 .debug_aranges
                0x000002b8       0x28 c:/program files/microchip/mplabc32/v2.02/bin/../lib/gcc/pic32mx/4.5.1/../../../../pic32mx/lib/speed\libc.a(strtod.o)
 .debug_aranges
                0x000002e0       0x20 c:/program files/microchip/mplabc32/v2.02/bin/../lib/gcc/pic32mx/4.5.1/../../../../pic32mx/lib/speed\libc.a(doprnt_cdnopsuxX.eo)
 .debug_aranges
                0x00000300       0x20 c:/program files/microchip/mplabc32/v2.02/bin/../lib/gcc/pic32mx/4.5.1/../../../../pic32mx/lib/speed\libc.a(_fputc_simple.o)
 .debug_aranges
                0x00000320       0x20 c:/program files/microchip/mplabc32/v2.02/bin/../lib/gcc/pic32mx/4.5.1/../../../../pic32mx/lib/speed\libc.a(write.o)
 .debug_aranges
                0x00000340       0x20 c:/program files/microchip/mplabc32/v2.02/bin/../lib/gcc/pic32mx/4.5.1/../../../../pic32mx/lib/speed\libc.a(_flsbuf_simple.o)
 .debug_aranges
                0x00000360       0x20 c:/program files/microchip/mplabc32/v2.02/bin/../lib/gcc/pic32mx/4.5.1/../../../../pic32mx/lib/speed\libc.a(_mon_putc.o)
 .debug_aranges
                0x00000380       0x20 c:/program files/microchip/mplabc32/v2.02/bin/../lib/gcc/pic32mx/4.5.1/../../../../pic32mx/lib/speed\libe.a(_strtod.o)
 .debug_aranges
                0x000003a0       0x20 c:/program files/microchip/mplabc32/v2.02/bin/../lib/gcc/pic32mx/4.5.1/../../../../pic32mx/lib/speed\libe.a(_ldexp.o)
 .debug_aranges
                0x000003c0       0x20 c:/program files/microchip/mplabc32/v2.02/bin/../lib/gcc/pic32mx/4.5.1/../../../../pic32mx/lib/speed\libmchp_peripheral.a(read_core_timer_lib.o)
 .debug_aranges
                0x000003e0       0x20 c:/program files/microchip/mplabc32/v2.02/bin/../lib/gcc/pic32mx/4.5.1/../../../../pic32mx/lib/speed\libmchp_peripheral.a(write_core_timer_lib.o)
 .debug_aranges
                0x00000400       0x48 c:/program files/microchip/mplabc32/v2.02/bin/../lib/gcc/pic32mx/4.5.1/../../../../pic32mx/lib/speed\libmchp_peripheral_32MX795F512L.a(eth_ack_packet_lib.o)
 .debug_aranges
                0x00000448       0x28 c:/program files/microchip/mplabc32/v2.02/bin/../lib/gcc/pic32mx/4.5.1/../../../../pic32mx/lib/speed\libmchp_peripheral_32MX795F512L.a(eth_descriptors_add_lib.o)
 .debug_aranges
                0x00000470       0x20 c:/program files/microchip/mplabc32/v2.02/bin/../lib/gcc/pic32mx/4.5.1/../../../../pic32mx/lib/speed\libmchp_peripheral_32MX795F512L.a(eth_init_lib.o)
 .debug_aranges
                0x00000490       0x20 c:/program files/microchip/mplabc32/v2.02/bin/../lib/gcc/pic32mx/4.5.1/../../../../pic32mx/lib/speed\libmchp_peripheral_32MX795F512L.a(eth_mac_open_lib.o)
 .debug_aranges
                0x000004b0       0x30 c:/program files/microchip/mplabc32/v2.02/bin/../lib/gcc/pic32mx/4.5.1/../../../../pic32mx/lib/speed\libmchp_peripheral_32MX795F512L.a(eth_mac_set_address_max_lib.o)
 .debug_aranges
                0x000004e0       0x20 c:/program files/microchip/mplabc32/v2.02/bin/../lib/gcc/pic32mx/4.5.1/../../../../pic32mx/lib/speed\libmchp_peripheral_32MX795F512L.a(eth_rx_buffers_append_lib.o)
 .debug_aranges
                0x00000500       0x48 c:/program files/microchip/mplabc32/v2.02/bin/../lib/gcc/pic32mx/4.5.1/../../../../pic32mx/lib/speed\libmchp_peripheral_32MX795F512L.a(eth_rx_filters_lib.o)
 .debug_aranges
                0x00000548       0x28 c:/program files/microchip/mplabc32/v2.02/bin/../lib/gcc/pic32mx/4.5.1/../../../../pic32mx/lib/speed\libmchp_peripheral_32MX795F512L.a(eth_rx_get_packet_lib.o)
 .debug_aranges
                0x00000570       0x20 c:/program files/microchip/mplabc32/v2.02/bin/../lib/gcc/pic32mx/4.5.1/../../../../pic32mx/lib/speed\libmchp_peripheral_32MX795F512L.a(eth_rx_set_buffer_size_lib.o)
 .debug_aranges
                0x00000590       0x38 c:/program files/microchip/mplabc32/v2.02/bin/../lib/gcc/pic32mx/4.5.1/../../../../pic32mx/lib/speed\libmchp_peripheral_32MX795F512L.a(eth_tx_packet_lib.o)
 .debug_aranges
                0x000005c8       0x20 c:/program files/microchip/mplabc32/v2.02/bin/../lib/gcc/pic32mx/4.5.1/../../../../pic32mx/lib/speed\libmchp_peripheral_32MX795F512L.a(_eth_append_busy_list_lib.o)
 .debug_aranges
                0x000005e8       0x48 c:/program files/microchip/mplabc32/v2.02/bin/../lib/gcc/pic32mx/4.5.1/../../../../pic32mx/lib/speed\libmchp_peripheral_32MX795F512L.a(eth_miim_access.o)
 .debug_aranges
                0x00000630       0x20 c:/program files/microchip/mplabc32/v2.02/bin/../lib/gcc/pic32mx/4.5.1/../../../../pic32mx/lib/speed\libmchp_peripheral_32MX795F512L.a(soft_reset_lib.o)
 .debug_aranges
                0x00000650       0x28 c:/program files/microchip/mplabc32/v2.02/bin/../lib/gcc/pic32mx/4.5.1/../../../../pic32mx/lib/speed\libmchp_peripheral_32MX795F512L.a(pcache.o)
 .debug_aranges
                0x00000678       0x20 c:/program files/microchip/mplabc32/v2.02/bin/../lib/gcc/pic32mx/4.5.1/../../../../pic32mx/lib/speed\libmchp_peripheral_32MX795F512L.a(set_core_sw0_leg_lib.o)
 .debug_aranges
                0x00000698       0x20 c:/program files/microchip/mplabc32/v2.02/bin/../lib/gcc/pic32mx/4.5.1/../../../../pic32mx/lib/speed\libmchp_peripheral_32MX795F512L.a(int_disable_interrupts_lib.o)
 .debug_aranges
                0x000006b8       0x20 c:/program files/microchip/mplabc32/v2.02/bin/../lib/gcc/pic32mx/4.5.1/../../../../pic32mx/lib/speed\libmchp_peripheral_32MX795F512L.a(int_restore_interrupts_lib.o)
 .debug_aranges
                0x000006d8       0x20 c:/program files/microchip/mplabc32/v2.02/bin/../lib/gcc/pic32mx/4.5.1/../../../../pic32mx/lib/speed\libmchp_peripheral_32MX795F512L.a(int_enable_mv_int_lib.o)
 .debug_aranges
                0x000006f8       0x60 c:/program files/microchip/mplabc32/v2.02/bin/../lib/gcc/pic32mx/4.5.1/../../../../pic32mx/lib/speed\libmchp_peripheral_32MX795F512L.a(int_tbl_lib.o)
 .debug_aranges
                0x00000758       0x20 c:/program files/microchip/mplabc32/v2.02/bin/../lib/gcc/pic32mx/4.5.1/../../../../pic32mx/lib/speed\libmchp_peripheral_32MX795F512L.a(rtcc_init_lib.o)
 .debug_aranges
                0x00000778       0x20 c:/program files/microchip/mplabc32/v2.02/bin/../lib/gcc/pic32mx/4.5.1/../../../../pic32mx/lib/speed\libmchp_peripheral_32MX795F512L.a(rtcc_set_time_date_lib.o)
 .debug_aranges
                0x00000798       0x20 c:/program files/microchip/mplabc32/v2.02/bin/../lib/gcc/pic32mx/4.5.1/../../../../pic32mx/lib/speed\libmchp_peripheral_32MX795F512L.a(rtcc_open_lib.o)
 .debug_aranges
                0x000007b8       0x20 c:/program files/microchip/mplabc32/v2.02/bin/../lib/gcc/pic32mx/4.5.1/../../../../pic32mx/lib/speed\libmchp_peripheral_32MX795F512L.a(spi_getc_spi1_lib_legacy.o)
 .debug_aranges
                0x000007d8       0x20 c:/program files/microchip/mplabc32/v2.02/bin/../lib/gcc/pic32mx/4.5.1/../../../../pic32mx/lib/speed\libmchp_peripheral_32MX795F512L.a(spi_open_spi1_lib_legacy.o)
 .debug_aranges
                0x000007f8       0x20 c:/program files/microchip/mplabc32/v2.02/bin/../lib/gcc/pic32mx/4.5.1/../../../../pic32mx/lib/speed\libmchp_peripheral_32MX795F512L.a(port_set_pins_digital_in_lib.o)
 .debug_aranges
                0x00000818       0x20 c:/program files/microchip/mplabc32/v2.02/bin/../lib/gcc/pic32mx/4.5.1/../../../../pic32mx/lib/speed\libmchp_peripheral_32MX795F512L.a(port_set_pins_digital_out_lib.o)
 .debug_aranges
                0x00000838       0x20 c:/program files/microchip/mplabc32/v2.02/bin/../lib/gcc/pic32mx/4.5.1/../../../../pic32mx/lib/speed\libmchp_peripheral_32MX795F512L.a(int_enable_interrupts_lib.o)
 .debug_aranges
                0x00000858       0x20 c:/program files/microchip/mplabc32/v2.02/bin/../lib/gcc/pic32mx/4.5.1/../../../../pic32mx/lib/speed\libmchp_peripheral_32MX795F512L.a(_rtcc_set_time_and_date_lib.o)
 .debug_aranges
                0x00000878       0x28 c:/program files/microchip/mplabc32/v2.02/bin/../lib/gcc/pic32mx/4.5.1/../../../../pic32mx/lib/speed\libmchp_peripheral_32MX795F512L.a(_rtcc_wait_clock_off_lib.o)
 .debug_aranges
                0x000008a0       0x20 c:/program files/microchip/mplabc32/v2.02/bin/../lib/gcc/pic32mx/4.5.1/../../../../pic32mx/lib/speed\libc.a(calloc.o)
 .debug_aranges
                0x000008c0       0x30 c:/program files/microchip/mplabc32/v2.02/bin/../lib/gcc/pic32mx/4.5.1/../../../../pic32mx/lib/speed\libc.a(malloc.o)
 .debug_aranges
                0x000008f0       0x40 c:/program files/microchip/mplabc32/v2.02/bin/../lib/gcc/pic32mx/4.5.1/../../../../pic32mx/lib/speed\libc.a(sbrk.o)
 .debug_aranges
                0x00000930       0x20 c:/program files/microchip/mplabc32/v2.02/bin/../lib/gcc/pic32mx/4.5.1/speed\libgcc.a(_lshrdi3.o)
 .debug_aranges
                0x00000950       0x20 c:/program files/microchip/mplabc32/v2.02/bin/../lib/gcc/pic32mx/4.5.1/speed\libgcc.a(_ashldi3.o)

.debug_pubnames
                0x00000000      0xc30
 *(.debug_pubnames)
 .debug_pubnames
                0x00000000       0x20 c:/program files/microchip/mplabc32/v2.02/bin/../lib/gcc/pic32mx/4.5.1/speed\libgcc.a(_udivdi3.o)
 .debug_pubnames
                0x00000020       0x20 c:/program files/microchip/mplabc32/v2.02/bin/../lib/gcc/pic32mx/4.5.1/speed\libgcc.a(_umoddi3.o)
 .debug_pubnames
                0x00000040       0x24 c:/program files/microchip/mplabc32/v2.02/bin/../lib/gcc/pic32mx/4.5.1/speed\libgcc.a(floatunsisf.o)
 .debug_pubnames
                0x00000064       0x1b c:/program files/microchip/mplabc32/v2.02/bin/../lib/gcc/pic32mx/4.5.1/../../../../pic32mx/lib/speed\libc.a(atoi.o)
 .debug_pubnames
                0x0000007f       0x1b c:/program files/microchip/mplabc32/v2.02/bin/../lib/gcc/pic32mx/4.5.1/../../../../pic32mx/lib/speed\libc.a(atol.o)
 .debug_pubnames
                0x0000009a       0x41 c:/program files/microchip/mplabc32/v2.02/bin/../lib/gcc/pic32mx/4.5.1/../../../../pic32mx/lib/speed\libc.a(ctime.o)
 .debug_pubnames
                0x000000db       0xe1 c:/program files/microchip/mplabc32/v2.02/bin/../lib/gcc/pic32mx/4.5.1/../../../../pic32mx/lib/speed\libc.a(ctypef.o)
 .debug_pubnames
                0x000001bc       0x1d c:/program files/microchip/mplabc32/v2.02/bin/../lib/gcc/pic32mx/4.5.1/../../../../pic32mx/lib/speed\libc.a(strcat.o)
 .debug_pubnames
                0x000001d9       0x1d c:/program files/microchip/mplabc32/v2.02/bin/../lib/gcc/pic32mx/4.5.1/../../../../pic32mx/lib/speed\libc.a(strchr.o)
 .debug_pubnames
                0x000001f6       0x1e c:/program files/microchip/mplabc32/v2.02/bin/../lib/gcc/pic32mx/4.5.1/../../../../pic32mx/lib/speed\libc.a(strncpy.o)
 .debug_pubnames
                0x00000214       0x1d c:/program files/microchip/mplabc32/v2.02/bin/../lib/gcc/pic32mx/4.5.1/../../../../pic32mx/lib/speed\libc.a(strstr.o)
 .debug_pubnames
                0x00000231       0x1b c:/program files/microchip/mplabc32/v2.02/bin/../lib/gcc/pic32mx/4.5.1/../../../../pic32mx/lib/speed\libc.a(atof.o)
 .debug_pubnames
                0x0000024c       0x29 c:/program files/microchip/mplabc32/v2.02/bin/../lib/gcc/pic32mx/4.5.1/../../../../pic32mx/lib/speed\libc.a(sprintf_cdnopsuxX.eo)
 .debug_pubnames
                0x00000275       0x33 c:/program files/microchip/mplabc32/v2.02/bin/../lib/gcc/pic32mx/4.5.1/../../../../pic32mx/lib/speed\libc.a(default-bootstrap-exception-handler.o)
 .debug_pubnames
                0x000002a8       0x20 c:/program files/microchip/mplabc32/v2.02/bin/../lib/gcc/pic32mx/4.5.1/../../../../pic32mx/lib/speed\libc.a(default-on-reset.o)
 .debug_pubnames
                0x000002c8       0x24 c:/program files/microchip/mplabc32/v2.02/bin/../lib/gcc/pic32mx/4.5.1/../../../../pic32mx/lib/speed\libc.a(default-on-bootstrap.o)
 .debug_pubnames
                0x000002ec       0x1e c:/program files/microchip/mplabc32/v2.02/bin/../lib/gcc/pic32mx/4.5.1/../../../../pic32mx/lib/speed\libc.a(strncmp.o)
 .debug_pubnames
                0x0000030a       0x2a c:/program files/microchip/mplabc32/v2.02/bin/../lib/gcc/pic32mx/4.5.1/../../../../pic32mx/lib/speed\libc.a(strtod.o)
 .debug_pubnames
                0x00000334       0x2a c:/program files/microchip/mplabc32/v2.02/bin/../lib/gcc/pic32mx/4.5.1/../../../../pic32mx/lib/speed\libc.a(doprnt_cdnopsuxX.eo)
 .debug_pubnames
                0x0000035e       0x1c c:/program files/microchip/mplabc32/v2.02/bin/../lib/gcc/pic32mx/4.5.1/../../../../pic32mx/lib/speed\libc.a(_fputc_simple.o)
 .debug_pubnames
                0x0000037a       0x1c c:/program files/microchip/mplabc32/v2.02/bin/../lib/gcc/pic32mx/4.5.1/../../../../pic32mx/lib/speed\libc.a(write.o)
 .debug_pubnames
                0x00000396       0x1e c:/program files/microchip/mplabc32/v2.02/bin/../lib/gcc/pic32mx/4.5.1/../../../../pic32mx/lib/speed\libc.a(_flsbuf_simple.o)
 .debug_pubnames
                0x000003b4       0x20 c:/program files/microchip/mplabc32/v2.02/bin/../lib/gcc/pic32mx/4.5.1/../../../../pic32mx/lib/speed\libc.a(_mon_putc.o)
 .debug_pubnames
                0x000003d4       0x1f c:/program files/microchip/mplabc32/v2.02/bin/../lib/gcc/pic32mx/4.5.1/../../../../pic32mx/lib/speed\libe.a(_strtod.o)
 .debug_pubnames
                0x000003f3       0x1e c:/program files/microchip/mplabc32/v2.02/bin/../lib/gcc/pic32mx/4.5.1/../../../../pic32mx/lib/speed\libe.a(_ldexp.o)
 .debug_pubnames
                0x00000411       0x24 c:/program files/microchip/mplabc32/v2.02/bin/../lib/gcc/pic32mx/4.5.1/../../../../pic32mx/lib/speed\libmchp_peripheral.a(read_core_timer_lib.o)
 .debug_pubnames
                0x00000435       0x25 c:/program files/microchip/mplabc32/v2.02/bin/../lib/gcc/pic32mx/4.5.1/../../../../pic32mx/lib/speed\libmchp_peripheral.a(write_core_timer_lib.o)
 .debug_pubnames
                0x0000045a       0x80 c:/program files/microchip/mplabc32/v2.02/bin/../lib/gcc/pic32mx/4.5.1/../../../../pic32mx/lib/speed\libmchp_peripheral_32MX795F512L.a(eth_ack_packet_lib.o)
 .debug_pubnames
                0x000004da       0x42 c:/program files/microchip/mplabc32/v2.02/bin/../lib/gcc/pic32mx/4.5.1/../../../../pic32mx/lib/speed\libmchp_peripheral_32MX795F512L.a(eth_descriptors_add_lib.o)
 .debug_pubnames
                0x0000051c       0x1e c:/program files/microchip/mplabc32/v2.02/bin/../lib/gcc/pic32mx/4.5.1/../../../../pic32mx/lib/speed\libmchp_peripheral_32MX795F512L.a(eth_init_lib.o)
 .debug_pubnames
                0x0000053a       0x21 c:/program files/microchip/mplabc32/v2.02/bin/../lib/gcc/pic32mx/4.5.1/../../../../pic32mx/lib/speed\libmchp_peripheral_32MX795F512L.a(eth_mac_open_lib.o)
 .debug_pubnames
                0x0000055b       0x52 c:/program files/microchip/mplabc32/v2.02/bin/../lib/gcc/pic32mx/4.5.1/../../../../pic32mx/lib/speed\libmchp_peripheral_32MX795F512L.a(eth_mac_set_address_max_lib.o)
 .debug_pubnames
                0x000005ad       0x29 c:/program files/microchip/mplabc32/v2.02/bin/../lib/gcc/pic32mx/4.5.1/../../../../pic32mx/lib/speed\libmchp_peripheral_32MX795F512L.a(eth_rx_buffers_append_lib.o)
 .debug_pubnames
                0x000005d6       0x92 c:/program files/microchip/mplabc32/v2.02/bin/../lib/gcc/pic32mx/4.5.1/../../../../pic32mx/lib/speed\libmchp_peripheral_32MX795F512L.a(eth_rx_filters_lib.o)
 .debug_pubnames
                0x00000668       0x38 c:/program files/microchip/mplabc32/v2.02/bin/../lib/gcc/pic32mx/4.5.1/../../../../pic32mx/lib/speed\libmchp_peripheral_32MX795F512L.a(eth_rx_get_packet_lib.o)
 .debug_pubnames
                0x000006a0       0x29 c:/program files/microchip/mplabc32/v2.02/bin/../lib/gcc/pic32mx/4.5.1/../../../../pic32mx/lib/speed\libmchp_peripheral_32MX795F512L.a(eth_rx_set_buffer_size_lib.o)
 .debug_pubnames
                0x000006c9       0x66 c:/program files/microchip/mplabc32/v2.02/bin/../lib/gcc/pic32mx/4.5.1/../../../../pic32mx/lib/speed\libmchp_peripheral_32MX795F512L.a(eth_tx_packet_lib.o)
 .debug_pubnames
                0x0000072f       0x29 c:/program files/microchip/mplabc32/v2.02/bin/../lib/gcc/pic32mx/4.5.1/../../../../pic32mx/lib/speed\libmchp_peripheral_32MX795F512L.a(_eth_append_busy_list_lib.o)
 .debug_pubnames
                0x00000758       0x90 c:/program files/microchip/mplabc32/v2.02/bin/../lib/gcc/pic32mx/4.5.1/../../../../pic32mx/lib/speed\libmchp_peripheral_32MX795F512L.a(eth_miim_access.o)
 .debug_pubnames
                0x000007e8       0x20 c:/program files/microchip/mplabc32/v2.02/bin/../lib/gcc/pic32mx/4.5.1/../../../../pic32mx/lib/speed\libmchp_peripheral_32MX795F512L.a(soft_reset_lib.o)
 .debug_pubnames
                0x00000808       0x3b c:/program files/microchip/mplabc32/v2.02/bin/../lib/gcc/pic32mx/4.5.1/../../../../pic32mx/lib/speed\libmchp_peripheral_32MX795F512L.a(pcache.o)
 .debug_pubnames
                0x00000843       0x21 c:/program files/microchip/mplabc32/v2.02/bin/../lib/gcc/pic32mx/4.5.1/../../../../pic32mx/lib/speed\libmchp_peripheral_32MX795F512L.a(set_core_sw0_leg_lib.o)
 .debug_pubnames
                0x00000864       0x2b c:/program files/microchip/mplabc32/v2.02/bin/../lib/gcc/pic32mx/4.5.1/../../../../pic32mx/lib/speed\libmchp_peripheral_32MX795F512L.a(int_disable_interrupts_lib.o)
 .debug_pubnames
                0x0000088f       0x2b c:/program files/microchip/mplabc32/v2.02/bin/../lib/gcc/pic32mx/4.5.1/../../../../pic32mx/lib/speed\libmchp_peripheral_32MX795F512L.a(int_restore_interrupts_lib.o)
 .debug_pubnames
                0x000008ba       0x36 c:/program files/microchip/mplabc32/v2.02/bin/../lib/gcc/pic32mx/4.5.1/../../../../pic32mx/lib/speed\libmchp_peripheral_32MX795F512L.a(int_enable_mv_int_lib.o)
 .debug_pubnames
                0x000008f0       0xca c:/program files/microchip/mplabc32/v2.02/bin/../lib/gcc/pic32mx/4.5.1/../../../../pic32mx/lib/speed\libmchp_peripheral_32MX795F512L.a(int_tbl_lib.o)
 .debug_pubnames
                0x000009ba       0x1f c:/program files/microchip/mplabc32/v2.02/bin/../lib/gcc/pic32mx/4.5.1/../../../../pic32mx/lib/speed\libmchp_peripheral_32MX795F512L.a(rtcc_init_lib.o)
 .debug_pubnames
                0x000009d9       0x26 c:/program files/microchip/mplabc32/v2.02/bin/../lib/gcc/pic32mx/4.5.1/../../../../pic32mx/lib/speed\libmchp_peripheral_32MX795F512L.a(rtcc_set_time_date_lib.o)
 .debug_pubnames
                0x000009ff       0x1f c:/program files/microchip/mplabc32/v2.02/bin/../lib/gcc/pic32mx/4.5.1/../../../../pic32mx/lib/speed\libmchp_peripheral_32MX795F512L.a(rtcc_open_lib.o)
 .debug_pubnames
                0x00000a1e       0x1f c:/program files/microchip/mplabc32/v2.02/bin/../lib/gcc/pic32mx/4.5.1/../../../../pic32mx/lib/speed\libmchp_peripheral_32MX795F512L.a(spi_getc_spi1_lib_legacy.o)
 .debug_pubnames
                0x00000a3d       0x1f c:/program files/microchip/mplabc32/v2.02/bin/../lib/gcc/pic32mx/4.5.1/../../../../pic32mx/lib/speed\libmchp_peripheral_32MX795F512L.a(spi_open_spi1_lib_legacy.o)
 .debug_pubnames
                0x00000a5c       0x2b c:/program files/microchip/mplabc32/v2.02/bin/../lib/gcc/pic32mx/4.5.1/../../../../pic32mx/lib/speed\libmchp_peripheral_32MX795F512L.a(port_set_pins_digital_in_lib.o)
 .debug_pubnames
                0x00000a87       0x2c c:/program files/microchip/mplabc32/v2.02/bin/../lib/gcc/pic32mx/4.5.1/../../../../pic32mx/lib/speed\libmchp_peripheral_32MX795F512L.a(port_set_pins_digital_out_lib.o)
 .debug_pubnames
                0x00000ab3       0x2a c:/program files/microchip/mplabc32/v2.02/bin/../lib/gcc/pic32mx/4.5.1/../../../../pic32mx/lib/speed\libmchp_peripheral_32MX795F512L.a(int_enable_interrupts_lib.o)
 .debug_pubnames
                0x00000add       0x2a c:/program files/microchip/mplabc32/v2.02/bin/../lib/gcc/pic32mx/4.5.1/../../../../pic32mx/lib/speed\libmchp_peripheral_32MX795F512L.a(_rtcc_set_time_and_date_lib.o)
 .debug_pubnames
                0x00000b07       0x3e c:/program files/microchip/mplabc32/v2.02/bin/../lib/gcc/pic32mx/4.5.1/../../../../pic32mx/lib/speed\libmchp_peripheral_32MX795F512L.a(_rtcc_wait_clock_off_lib.o)
 .debug_pubnames
                0x00000b45       0x1d c:/program files/microchip/mplabc32/v2.02/bin/../lib/gcc/pic32mx/4.5.1/../../../../pic32mx/lib/speed\libc.a(calloc.o)
 .debug_pubnames
                0x00000b62       0x32 c:/program files/microchip/mplabc32/v2.02/bin/../lib/gcc/pic32mx/4.5.1/../../../../pic32mx/lib/speed\libc.a(malloc.o)
 .debug_pubnames
                0x00000b94       0x5c c:/program files/microchip/mplabc32/v2.02/bin/../lib/gcc/pic32mx/4.5.1/../../../../pic32mx/lib/speed\libc.a(sbrk.o)
 .debug_pubnames
                0x00000bf0       0x20 c:/program files/microchip/mplabc32/v2.02/bin/../lib/gcc/pic32mx/4.5.1/speed\libgcc.a(_lshrdi3.o)
 .debug_pubnames
                0x00000c10       0x20 c:/program files/microchip/mplabc32/v2.02/bin/../lib/gcc/pic32mx/4.5.1/speed\libgcc.a(_ashldi3.o)

.debug_info     0x00000000     0x4d04
 *(.debug_info .gnu.linkonce.wi.*)
 .debug_info    0x00000000      0x78c c:/program files/microchip/mplabc32/v2.02/bin/../lib/gcc/pic32mx/4.5.1/speed\libgcc.a(_udivdi3.o)
 .debug_info    0x0000078c      0x7c9 c:/program files/microchip/mplabc32/v2.02/bin/../lib/gcc/pic32mx/4.5.1/speed\libgcc.a(_umoddi3.o)
 .debug_info    0x00000f55      0x191 c:/program files/microchip/mplabc32/v2.02/bin/../lib/gcc/pic32mx/4.5.1/speed\libgcc.a(floatunsisf.o)
 .debug_info    0x000010e6       0xcd c:/program files/microchip/mplabc32/v2.02/bin/../lib/gcc/pic32mx/4.5.1/../../../../pic32mx/lib/speed\libc.a(atoi.o)
 .debug_info    0x000011b3       0xcd c:/program files/microchip/mplabc32/v2.02/bin/../lib/gcc/pic32mx/4.5.1/../../../../pic32mx/lib/speed\libc.a(atol.o)
 .debug_info    0x00001280      0x126 c:/program files/microchip/mplabc32/v2.02/bin/../lib/gcc/pic32mx/4.5.1/../../../../pic32mx/lib/speed\libc.a(ctime.o)
 .debug_info    0x000013a6        0x0 c:/program files/microchip/mplabc32/v2.02/bin/../lib/gcc/pic32mx/4.5.1/../../../../pic32mx/lib/speed\libc.a(ctype.o)
 .debug_info    0x000013a6      0x235 c:/program files/microchip/mplabc32/v2.02/bin/../lib/gcc/pic32mx/4.5.1/../../../../pic32mx/lib/speed\libc.a(ctypef.o)
 .debug_info    0x000015db       0xd1 c:/program files/microchip/mplabc32/v2.02/bin/../lib/gcc/pic32mx/4.5.1/../../../../pic32mx/lib/speed\libc.a(strcat.o)
 .debug_info    0x000016ac       0xd1 c:/program files/microchip/mplabc32/v2.02/bin/../lib/gcc/pic32mx/4.5.1/../../../../pic32mx/lib/speed\libc.a(strchr.o)
 .debug_info    0x0000177d       0xd3 c:/program files/microchip/mplabc32/v2.02/bin/../lib/gcc/pic32mx/4.5.1/../../../../pic32mx/lib/speed\libc.a(strncpy.o)
 .debug_info    0x00001850       0xd1 c:/program files/microchip/mplabc32/v2.02/bin/../lib/gcc/pic32mx/4.5.1/../../../../pic32mx/lib/speed\libc.a(strstr.o)
 .debug_info    0x00001921       0xcd c:/program files/microchip/mplabc32/v2.02/bin/../lib/gcc/pic32mx/4.5.1/../../../../pic32mx/lib/speed\libc.a(atof.o)
 .debug_info    0x000019ee       0xe9 c:/program files/microchip/mplabc32/v2.02/bin/../lib/gcc/pic32mx/4.5.1/../../../../pic32mx/lib/speed\libc.a(sprintf_cdnopsuxX.eo)
 .debug_info    0x00001ad7      0x106 c:/program files/microchip/mplabc32/v2.02/bin/../lib/gcc/pic32mx/4.5.1/../../../../pic32mx/lib/speed\libc.a(default-bootstrap-exception-handler.o)
 .debug_info    0x00001bdd       0xe0 c:/program files/microchip/mplabc32/v2.02/bin/../lib/gcc/pic32mx/4.5.1/../../../../pic32mx/lib/speed\libc.a(default-on-reset.o)
 .debug_info    0x00001cbd       0xe8 c:/program files/microchip/mplabc32/v2.02/bin/../lib/gcc/pic32mx/4.5.1/../../../../pic32mx/lib/speed\libc.a(default-on-bootstrap.o)
 .debug_info    0x00001da5       0xd3 c:/program files/microchip/mplabc32/v2.02/bin/../lib/gcc/pic32mx/4.5.1/../../../../pic32mx/lib/speed\libc.a(strncmp.o)
 .debug_info    0x00001e78      0x100 c:/program files/microchip/mplabc32/v2.02/bin/../lib/gcc/pic32mx/4.5.1/../../../../pic32mx/lib/speed\libc.a(strtod.o)
 .debug_info    0x00001f78       0xea c:/program files/microchip/mplabc32/v2.02/bin/../lib/gcc/pic32mx/4.5.1/../../../../pic32mx/lib/speed\libc.a(doprnt_cdnopsuxX.eo)
 .debug_info    0x00002062       0xda c:/program files/microchip/mplabc32/v2.02/bin/../lib/gcc/pic32mx/4.5.1/../../../../pic32mx/lib/speed\libc.a(_fputc_simple.o)
 .debug_info    0x0000213c       0xd1 c:/program files/microchip/mplabc32/v2.02/bin/../lib/gcc/pic32mx/4.5.1/../../../../pic32mx/lib/speed\libc.a(write.o)
 .debug_info    0x0000220d        0x0 c:/program files/microchip/mplabc32/v2.02/bin/../lib/gcc/pic32mx/4.5.1/../../../../pic32mx/lib/speed\libc.a(_iob.o)
 .debug_info    0x0000220d       0xdd c:/program files/microchip/mplabc32/v2.02/bin/../lib/gcc/pic32mx/4.5.1/../../../../pic32mx/lib/speed\libc.a(_flsbuf_simple.o)
 .debug_info    0x000022ea       0xd9 c:/program files/microchip/mplabc32/v2.02/bin/../lib/gcc/pic32mx/4.5.1/../../../../pic32mx/lib/speed\libc.a(_mon_putc.o)
 .debug_info    0x000023c3        0x0 c:/program files/microchip/mplabc32/v2.02/bin/../lib/gcc/pic32mx/4.5.1/../../../../pic32mx/lib/speed\libc.a(c32_uart.o)
 .debug_info    0x000023c3       0xe3 c:/program files/microchip/mplabc32/v2.02/bin/../lib/gcc/pic32mx/4.5.1/../../../../pic32mx/lib/speed\libe.a(_strtod.o)
 .debug_info    0x000024a6       0xef c:/program files/microchip/mplabc32/v2.02/bin/../lib/gcc/pic32mx/4.5.1/../../../../pic32mx/lib/speed\libe.a(_ldexp.o)
 .debug_info    0x00002595       0xbf c:/program files/microchip/mplabc32/v2.02/bin/../lib/gcc/pic32mx/4.5.1/../../../../pic32mx/lib/speed\libmchp_peripheral.a(read_core_timer_lib.o)
 .debug_info    0x00002654       0xc1 c:/program files/microchip/mplabc32/v2.02/bin/../lib/gcc/pic32mx/4.5.1/../../../../pic32mx/lib/speed\libmchp_peripheral.a(write_core_timer_lib.o)
 .debug_info    0x00002715      0x180 c:/program files/microchip/mplabc32/v2.02/bin/../lib/gcc/pic32mx/4.5.1/../../../../pic32mx/lib/speed\libmchp_peripheral_32MX795F512L.a(eth_ack_packet_lib.o)
 .debug_info    0x00002895      0x107 c:/program files/microchip/mplabc32/v2.02/bin/../lib/gcc/pic32mx/4.5.1/../../../../pic32mx/lib/speed\libmchp_peripheral_32MX795F512L.a(eth_descriptors_add_lib.o)
 .debug_info    0x0000299c       0xd3 c:/program files/microchip/mplabc32/v2.02/bin/../lib/gcc/pic32mx/4.5.1/../../../../pic32mx/lib/speed\libmchp_peripheral_32MX795F512L.a(eth_init_lib.o)
 .debug_info    0x00002a6f       0xb7 c:/program files/microchip/mplabc32/v2.02/bin/../lib/gcc/pic32mx/4.5.1/../../../../pic32mx/lib/speed\libmchp_peripheral_32MX795F512L.a(eth_mac_open_lib.o)
 .debug_info    0x00002b26      0x107 c:/program files/microchip/mplabc32/v2.02/bin/../lib/gcc/pic32mx/4.5.1/../../../../pic32mx/lib/speed\libmchp_peripheral_32MX795F512L.a(eth_mac_set_address_max_lib.o)
 .debug_info    0x00002c2d       0xfb c:/program files/microchip/mplabc32/v2.02/bin/../lib/gcc/pic32mx/4.5.1/../../../../pic32mx/lib/speed\libmchp_peripheral_32MX795F512L.a(eth_rx_buffers_append_lib.o)
 .debug_info    0x00002d28      0x15c c:/program files/microchip/mplabc32/v2.02/bin/../lib/gcc/pic32mx/4.5.1/../../../../pic32mx/lib/speed\libmchp_peripheral_32MX795F512L.a(eth_rx_filters_lib.o)
 .debug_info    0x00002e84       0xdd c:/program files/microchip/mplabc32/v2.02/bin/../lib/gcc/pic32mx/4.5.1/../../../../pic32mx/lib/speed\libmchp_peripheral_32MX795F512L.a(eth_rx_get_packet_lib.o)
 .debug_info    0x00002f61       0xc9 c:/program files/microchip/mplabc32/v2.02/bin/../lib/gcc/pic32mx/4.5.1/../../../../pic32mx/lib/speed\libmchp_peripheral_32MX795F512L.a(eth_rx_set_buffer_size_lib.o)
 .debug_info    0x0000302a      0x17f c:/program files/microchip/mplabc32/v2.02/bin/../lib/gcc/pic32mx/4.5.1/../../../../pic32mx/lib/speed\libmchp_peripheral_32MX795F512L.a(eth_tx_packet_lib.o)
 .debug_info    0x000031a9       0xe9 c:/program files/microchip/mplabc32/v2.02/bin/../lib/gcc/pic32mx/4.5.1/../../../../pic32mx/lib/speed\libmchp_peripheral_32MX795F512L.a(_eth_append_busy_list_lib.o)
 .debug_info    0x00003292      0x158 c:/program files/microchip/mplabc32/v2.02/bin/../lib/gcc/pic32mx/4.5.1/../../../../pic32mx/lib/speed\libmchp_peripheral_32MX795F512L.a(eth_miim_access.o)
 .debug_info    0x000033ea       0xc7 c:/program files/microchip/mplabc32/v2.02/bin/../lib/gcc/pic32mx/4.5.1/../../../../pic32mx/lib/speed\libmchp_peripheral_32MX795F512L.a(soft_reset_lib.o)
 .debug_info    0x000034b1       0xd4 c:/program files/microchip/mplabc32/v2.02/bin/../lib/gcc/pic32mx/4.5.1/../../../../pic32mx/lib/speed\libmchp_peripheral_32MX795F512L.a(pcache.o)
 .debug_info    0x00003585       0xbb c:/program files/microchip/mplabc32/v2.02/bin/../lib/gcc/pic32mx/4.5.1/../../../../pic32mx/lib/speed\libmchp_peripheral_32MX795F512L.a(set_core_sw0_leg_lib.o)
 .debug_info    0x00003640       0xcb c:/program files/microchip/mplabc32/v2.02/bin/../lib/gcc/pic32mx/4.5.1/../../../../pic32mx/lib/speed\libmchp_peripheral_32MX795F512L.a(int_disable_interrupts_lib.o)
 .debug_info    0x0000370b       0xcb c:/program files/microchip/mplabc32/v2.02/bin/../lib/gcc/pic32mx/4.5.1/../../../../pic32mx/lib/speed\libmchp_peripheral_32MX795F512L.a(int_restore_interrupts_lib.o)
 .debug_info    0x000037d6       0xd1 c:/program files/microchip/mplabc32/v2.02/bin/../lib/gcc/pic32mx/4.5.1/../../../../pic32mx/lib/speed\libmchp_peripheral_32MX795F512L.a(int_enable_mv_int_lib.o)
 .debug_info    0x000038a7      0x1ab c:/program files/microchip/mplabc32/v2.02/bin/../lib/gcc/pic32mx/4.5.1/../../../../pic32mx/lib/speed\libmchp_peripheral_32MX795F512L.a(int_tbl_lib.o)
 .debug_info    0x00003a52      0x121 c:/program files/microchip/mplabc32/v2.02/bin/../lib/gcc/pic32mx/4.5.1/../../../../pic32mx/lib/speed\libmchp_peripheral_32MX795F512L.a(rtcc_init_lib.o)
 .debug_info    0x00003b73       0xc3 c:/program files/microchip/mplabc32/v2.02/bin/../lib/gcc/pic32mx/4.5.1/../../../../pic32mx/lib/speed\libmchp_peripheral_32MX795F512L.a(rtcc_set_time_date_lib.o)
 .debug_info    0x00003c36      0x121 c:/program files/microchip/mplabc32/v2.02/bin/../lib/gcc/pic32mx/4.5.1/../../../../pic32mx/lib/speed\libmchp_peripheral_32MX795F512L.a(rtcc_open_lib.o)
 .debug_info    0x00003d57       0xbd c:/program files/microchip/mplabc32/v2.02/bin/../lib/gcc/pic32mx/4.5.1/../../../../pic32mx/lib/speed\libmchp_peripheral_32MX795F512L.a(spi_getc_spi1_lib_legacy.o)
 .debug_info    0x00003e14       0xbd c:/program files/microchip/mplabc32/v2.02/bin/../lib/gcc/pic32mx/4.5.1/../../../../pic32mx/lib/speed\libmchp_peripheral_32MX795F512L.a(spi_open_spi1_lib_legacy.o)
 .debug_info    0x00003ed1        0x0 c:/program files/microchip/mplabc32/v2.02/bin/../lib/gcc/pic32mx/4.5.1/../../../../pic32mx/lib/speed\libmchp_peripheral_32MX795F512L.a(spi_brg_tbl_lib_legacy.o)
 .debug_info    0x00003ed1       0xcf c:/program files/microchip/mplabc32/v2.02/bin/../lib/gcc/pic32mx/4.5.1/../../../../pic32mx/lib/speed\libmchp_peripheral_32MX795F512L.a(port_set_pins_digital_in_lib.o)
 .debug_info    0x00003fa0       0xd1 c:/program files/microchip/mplabc32/v2.02/bin/../lib/gcc/pic32mx/4.5.1/../../../../pic32mx/lib/speed\libmchp_peripheral_32MX795F512L.a(port_set_pins_digital_out_lib.o)
 .debug_info    0x00004071        0x0 c:/program files/microchip/mplabc32/v2.02/bin/../lib/gcc/pic32mx/4.5.1/../../../../pic32mx/lib/speed\libmchp_peripheral_32MX795F512L.a(_ports_tbl_libp.o)
 .debug_info    0x00004071       0xc9 c:/program files/microchip/mplabc32/v2.02/bin/../lib/gcc/pic32mx/4.5.1/../../../../pic32mx/lib/speed\libmchp_peripheral_32MX795F512L.a(int_enable_interrupts_lib.o)
 .debug_info    0x0000413a      0x124 c:/program files/microchip/mplabc32/v2.02/bin/../lib/gcc/pic32mx/4.5.1/../../../../pic32mx/lib/speed\libmchp_peripheral_32MX795F512L.a(_rtcc_set_time_and_date_lib.o)
 .debug_info    0x0000425e       0xfc c:/program files/microchip/mplabc32/v2.02/bin/../lib/gcc/pic32mx/4.5.1/../../../../pic32mx/lib/speed\libmchp_peripheral_32MX795F512L.a(_rtcc_wait_clock_off_lib.o)
 .debug_info    0x0000435a       0xd1 c:/program files/microchip/mplabc32/v2.02/bin/../lib/gcc/pic32mx/4.5.1/../../../../pic32mx/lib/speed\libc.a(calloc.o)
 .debug_info    0x0000442b        0x0 c:/program files/microchip/mplabc32/v2.02/bin/../lib/gcc/pic32mx/4.5.1/../../../../pic32mx/lib/speed\libc.a(errno.o)
 .debug_info    0x0000442b      0x100 c:/program files/microchip/mplabc32/v2.02/bin/../lib/gcc/pic32mx/4.5.1/../../../../pic32mx/lib/speed\libc.a(malloc.o)
 .debug_info    0x0000452b      0x139 c:/program files/microchip/mplabc32/v2.02/bin/../lib/gcc/pic32mx/4.5.1/../../../../pic32mx/lib/speed\libc.a(sbrk.o)
 .debug_info    0x00004664      0x352 c:/program files/microchip/mplabc32/v2.02/bin/../lib/gcc/pic32mx/4.5.1/speed\libgcc.a(_lshrdi3.o)
 .debug_info    0x000049b6      0x34e c:/program files/microchip/mplabc32/v2.02/bin/../lib/gcc/pic32mx/4.5.1/speed\libgcc.a(_ashldi3.o)

.debug_abbrev   0x00000000      0xe84
 *(.debug_abbrev)
 .debug_abbrev  0x00000000      0x13d c:/program files/microchip/mplabc32/v2.02/bin/../lib/gcc/pic32mx/4.5.1/speed\libgcc.a(_udivdi3.o)
 .debug_abbrev  0x0000013d      0x15c c:/program files/microchip/mplabc32/v2.02/bin/../lib/gcc/pic32mx/4.5.1/speed\libgcc.a(_umoddi3.o)
 .debug_abbrev  0x00000299       0x61 c:/program files/microchip/mplabc32/v2.02/bin/../lib/gcc/pic32mx/4.5.1/speed\libgcc.a(floatunsisf.o)
 .debug_abbrev  0x000002fa       0x25 c:/program files/microchip/mplabc32/v2.02/bin/../lib/gcc/pic32mx/4.5.1/../../../../pic32mx/lib/speed\libc.a(atoi.o)
 .debug_abbrev  0x0000031f       0x25 c:/program files/microchip/mplabc32/v2.02/bin/../lib/gcc/pic32mx/4.5.1/../../../../pic32mx/lib/speed\libc.a(atol.o)
 .debug_abbrev  0x00000344       0x32 c:/program files/microchip/mplabc32/v2.02/bin/../lib/gcc/pic32mx/4.5.1/../../../../pic32mx/lib/speed\libc.a(ctime.o)
 .debug_abbrev  0x00000376        0x1 c:/program files/microchip/mplabc32/v2.02/bin/../lib/gcc/pic32mx/4.5.1/../../../../pic32mx/lib/speed\libc.a(ctype.o)
 .debug_abbrev  0x00000377       0x25 c:/program files/microchip/mplabc32/v2.02/bin/../lib/gcc/pic32mx/4.5.1/../../../../pic32mx/lib/speed\libc.a(ctypef.o)
 .debug_abbrev  0x0000039c       0x25 c:/program files/microchip/mplabc32/v2.02/bin/../lib/gcc/pic32mx/4.5.1/../../../../pic32mx/lib/speed\libc.a(strcat.o)
 .debug_abbrev  0x000003c1       0x25 c:/program files/microchip/mplabc32/v2.02/bin/../lib/gcc/pic32mx/4.5.1/../../../../pic32mx/lib/speed\libc.a(strchr.o)
 .debug_abbrev  0x000003e6       0x25 c:/program files/microchip/mplabc32/v2.02/bin/../lib/gcc/pic32mx/4.5.1/../../../../pic32mx/lib/speed\libc.a(strncpy.o)
 .debug_abbrev  0x0000040b       0x25 c:/program files/microchip/mplabc32/v2.02/bin/../lib/gcc/pic32mx/4.5.1/../../../../pic32mx/lib/speed\libc.a(strstr.o)
 .debug_abbrev  0x00000430       0x25 c:/program files/microchip/mplabc32/v2.02/bin/../lib/gcc/pic32mx/4.5.1/../../../../pic32mx/lib/speed\libc.a(atof.o)
 .debug_abbrev  0x00000455       0x25 c:/program files/microchip/mplabc32/v2.02/bin/../lib/gcc/pic32mx/4.5.1/../../../../pic32mx/lib/speed\libc.a(sprintf_cdnopsuxX.eo)
 .debug_abbrev  0x0000047a       0x25 c:/program files/microchip/mplabc32/v2.02/bin/../lib/gcc/pic32mx/4.5.1/../../../../pic32mx/lib/speed\libc.a(default-bootstrap-exception-handler.o)
 .debug_abbrev  0x0000049f       0x25 c:/program files/microchip/mplabc32/v2.02/bin/../lib/gcc/pic32mx/4.5.1/../../../../pic32mx/lib/speed\libc.a(default-on-reset.o)
 .debug_abbrev  0x000004c4       0x25 c:/program files/microchip/mplabc32/v2.02/bin/../lib/gcc/pic32mx/4.5.1/../../../../pic32mx/lib/speed\libc.a(default-on-bootstrap.o)
 .debug_abbrev  0x000004e9       0x25 c:/program files/microchip/mplabc32/v2.02/bin/../lib/gcc/pic32mx/4.5.1/../../../../pic32mx/lib/speed\libc.a(strncmp.o)
 .debug_abbrev  0x0000050e       0x49 c:/program files/microchip/mplabc32/v2.02/bin/../lib/gcc/pic32mx/4.5.1/../../../../pic32mx/lib/speed\libc.a(strtod.o)
 .debug_abbrev  0x00000557       0x25 c:/program files/microchip/mplabc32/v2.02/bin/../lib/gcc/pic32mx/4.5.1/../../../../pic32mx/lib/speed\libc.a(doprnt_cdnopsuxX.eo)
 .debug_abbrev  0x0000057c       0x25 c:/program files/microchip/mplabc32/v2.02/bin/../lib/gcc/pic32mx/4.5.1/../../../../pic32mx/lib/speed\libc.a(_fputc_simple.o)
 .debug_abbrev  0x000005a1       0x25 c:/program files/microchip/mplabc32/v2.02/bin/../lib/gcc/pic32mx/4.5.1/../../../../pic32mx/lib/speed\libc.a(write.o)
 .debug_abbrev  0x000005c6        0x1 c:/program files/microchip/mplabc32/v2.02/bin/../lib/gcc/pic32mx/4.5.1/../../../../pic32mx/lib/speed\libc.a(_iob.o)
 .debug_abbrev  0x000005c7       0x25 c:/program files/microchip/mplabc32/v2.02/bin/../lib/gcc/pic32mx/4.5.1/../../../../pic32mx/lib/speed\libc.a(_flsbuf_simple.o)
 .debug_abbrev  0x000005ec       0x25 c:/program files/microchip/mplabc32/v2.02/bin/../lib/gcc/pic32mx/4.5.1/../../../../pic32mx/lib/speed\libc.a(_mon_putc.o)
 .debug_abbrev  0x00000611        0x1 c:/program files/microchip/mplabc32/v2.02/bin/../lib/gcc/pic32mx/4.5.1/../../../../pic32mx/lib/speed\libc.a(c32_uart.o)
 .debug_abbrev  0x00000612       0x32 c:/program files/microchip/mplabc32/v2.02/bin/../lib/gcc/pic32mx/4.5.1/../../../../pic32mx/lib/speed\libe.a(_strtod.o)
 .debug_abbrev  0x00000644       0x32 c:/program files/microchip/mplabc32/v2.02/bin/../lib/gcc/pic32mx/4.5.1/../../../../pic32mx/lib/speed\libe.a(_ldexp.o)
 .debug_abbrev  0x00000676       0x25 c:/program files/microchip/mplabc32/v2.02/bin/../lib/gcc/pic32mx/4.5.1/../../../../pic32mx/lib/speed\libmchp_peripheral.a(read_core_timer_lib.o)
 .debug_abbrev  0x0000069b       0x25 c:/program files/microchip/mplabc32/v2.02/bin/../lib/gcc/pic32mx/4.5.1/../../../../pic32mx/lib/speed\libmchp_peripheral.a(write_core_timer_lib.o)
 .debug_abbrev  0x000006c0       0x58 c:/program files/microchip/mplabc32/v2.02/bin/../lib/gcc/pic32mx/4.5.1/../../../../pic32mx/lib/speed\libmchp_peripheral_32MX795F512L.a(eth_ack_packet_lib.o)
 .debug_abbrev  0x00000718       0x34 c:/program files/microchip/mplabc32/v2.02/bin/../lib/gcc/pic32mx/4.5.1/../../../../pic32mx/lib/speed\libmchp_peripheral_32MX795F512L.a(eth_descriptors_add_lib.o)
 .debug_abbrev  0x0000074c       0x34 c:/program files/microchip/mplabc32/v2.02/bin/../lib/gcc/pic32mx/4.5.1/../../../../pic32mx/lib/speed\libmchp_peripheral_32MX795F512L.a(eth_init_lib.o)
 .debug_abbrev  0x00000780       0x25 c:/program files/microchip/mplabc32/v2.02/bin/../lib/gcc/pic32mx/4.5.1/../../../../pic32mx/lib/speed\libmchp_peripheral_32MX795F512L.a(eth_mac_open_lib.o)
 .debug_abbrev  0x000007a5       0x25 c:/program files/microchip/mplabc32/v2.02/bin/../lib/gcc/pic32mx/4.5.1/../../../../pic32mx/lib/speed\libmchp_peripheral_32MX795F512L.a(eth_mac_set_address_max_lib.o)
 .debug_abbrev  0x000007ca       0x34 c:/program files/microchip/mplabc32/v2.02/bin/../lib/gcc/pic32mx/4.5.1/../../../../pic32mx/lib/speed\libmchp_peripheral_32MX795F512L.a(eth_rx_buffers_append_lib.o)
 .debug_abbrev  0x000007fe       0x25 c:/program files/microchip/mplabc32/v2.02/bin/../lib/gcc/pic32mx/4.5.1/../../../../pic32mx/lib/speed\libmchp_peripheral_32MX795F512L.a(eth_rx_filters_lib.o)
 .debug_abbrev  0x00000823       0x25 c:/program files/microchip/mplabc32/v2.02/bin/../lib/gcc/pic32mx/4.5.1/../../../../pic32mx/lib/speed\libmchp_peripheral_32MX795F512L.a(eth_rx_get_packet_lib.o)
 .debug_abbrev  0x00000848       0x25 c:/program files/microchip/mplabc32/v2.02/bin/../lib/gcc/pic32mx/4.5.1/../../../../pic32mx/lib/speed\libmchp_peripheral_32MX795F512L.a(eth_rx_set_buffer_size_lib.o)
 .debug_abbrev  0x0000086d       0x5d c:/program files/microchip/mplabc32/v2.02/bin/../lib/gcc/pic32mx/4.5.1/../../../../pic32mx/lib/speed\libmchp_peripheral_32MX795F512L.a(eth_tx_packet_lib.o)
 .debug_abbrev  0x000008ca       0x34 c:/program files/microchip/mplabc32/v2.02/bin/../lib/gcc/pic32mx/4.5.1/../../../../pic32mx/lib/speed\libmchp_peripheral_32MX795F512L.a(_eth_append_busy_list_lib.o)
 .debug_abbrev  0x000008fe       0x38 c:/program files/microchip/mplabc32/v2.02/bin/../lib/gcc/pic32mx/4.5.1/../../../../pic32mx/lib/speed\libmchp_peripheral_32MX795F512L.a(eth_miim_access.o)
 .debug_abbrev  0x00000936       0x34 c:/program files/microchip/mplabc32/v2.02/bin/../lib/gcc/pic32mx/4.5.1/../../../../pic32mx/lib/speed\libmchp_peripheral_32MX795F512L.a(soft_reset_lib.o)
 .debug_abbrev  0x0000096a       0x25 c:/program files/microchip/mplabc32/v2.02/bin/../lib/gcc/pic32mx/4.5.1/../../../../pic32mx/lib/speed\libmchp_peripheral_32MX795F512L.a(pcache.o)
 .debug_abbrev  0x0000098f       0x25 c:/program files/microchip/mplabc32/v2.02/bin/../lib/gcc/pic32mx/4.5.1/../../../../pic32mx/lib/speed\libmchp_peripheral_32MX795F512L.a(set_core_sw0_leg_lib.o)
 .debug_abbrev  0x000009b4       0x25 c:/program files/microchip/mplabc32/v2.02/bin/../lib/gcc/pic32mx/4.5.1/../../../../pic32mx/lib/speed\libmchp_peripheral_32MX795F512L.a(int_disable_interrupts_lib.o)
 .debug_abbrev  0x000009d9       0x25 c:/program files/microchip/mplabc32/v2.02/bin/../lib/gcc/pic32mx/4.5.1/../../../../pic32mx/lib/speed\libmchp_peripheral_32MX795F512L.a(int_restore_interrupts_lib.o)
 .debug_abbrev  0x000009fe       0x25 c:/program files/microchip/mplabc32/v2.02/bin/../lib/gcc/pic32mx/4.5.1/../../../../pic32mx/lib/speed\libmchp_peripheral_32MX795F512L.a(int_enable_mv_int_lib.o)
 .debug_abbrev  0x00000a23       0x25 c:/program files/microchip/mplabc32/v2.02/bin/../lib/gcc/pic32mx/4.5.1/../../../../pic32mx/lib/speed\libmchp_peripheral_32MX795F512L.a(int_tbl_lib.o)
 .debug_abbrev  0x00000a48       0x41 c:/program files/microchip/mplabc32/v2.02/bin/../lib/gcc/pic32mx/4.5.1/../../../../pic32mx/lib/speed\libmchp_peripheral_32MX795F512L.a(rtcc_init_lib.o)
 .debug_abbrev  0x00000a89       0x25 c:/program files/microchip/mplabc32/v2.02/bin/../lib/gcc/pic32mx/4.5.1/../../../../pic32mx/lib/speed\libmchp_peripheral_32MX795F512L.a(rtcc_set_time_date_lib.o)
 .debug_abbrev  0x00000aae       0x41 c:/program files/microchip/mplabc32/v2.02/bin/../lib/gcc/pic32mx/4.5.1/../../../../pic32mx/lib/speed\libmchp_peripheral_32MX795F512L.a(rtcc_open_lib.o)
 .debug_abbrev  0x00000aef       0x25 c:/program files/microchip/mplabc32/v2.02/bin/../lib/gcc/pic32mx/4.5.1/../../../../pic32mx/lib/speed\libmchp_peripheral_32MX795F512L.a(spi_getc_spi1_lib_legacy.o)
 .debug_abbrev  0x00000b14       0x25 c:/program files/microchip/mplabc32/v2.02/bin/../lib/gcc/pic32mx/4.5.1/../../../../pic32mx/lib/speed\libmchp_peripheral_32MX795F512L.a(spi_open_spi1_lib_legacy.o)
 .debug_abbrev  0x00000b39        0x1 c:/program files/microchip/mplabc32/v2.02/bin/../lib/gcc/pic32mx/4.5.1/../../../../pic32mx/lib/speed\libmchp_peripheral_32MX795F512L.a(spi_brg_tbl_lib_legacy.o)
 .debug_abbrev  0x00000b3a       0x25 c:/program files/microchip/mplabc32/v2.02/bin/../lib/gcc/pic32mx/4.5.1/../../../../pic32mx/lib/speed\libmchp_peripheral_32MX795F512L.a(port_set_pins_digital_in_lib.o)
 .debug_abbrev  0x00000b5f       0x25 c:/program files/microchip/mplabc32/v2.02/bin/../lib/gcc/pic32mx/4.5.1/../../../../pic32mx/lib/speed\libmchp_peripheral_32MX795F512L.a(port_set_pins_digital_out_lib.o)
 .debug_abbrev  0x00000b84        0x1 c:/program files/microchip/mplabc32/v2.02/bin/../lib/gcc/pic32mx/4.5.1/../../../../pic32mx/lib/speed\libmchp_peripheral_32MX795F512L.a(_ports_tbl_libp.o)
 .debug_abbrev  0x00000b85       0x25 c:/program files/microchip/mplabc32/v2.02/bin/../lib/gcc/pic32mx/4.5.1/../../../../pic32mx/lib/speed\libmchp_peripheral_32MX795F512L.a(int_enable_interrupts_lib.o)
 .debug_abbrev  0x00000baa       0x41 c:/program files/microchip/mplabc32/v2.02/bin/../lib/gcc/pic32mx/4.5.1/../../../../pic32mx/lib/speed\libmchp_peripheral_32MX795F512L.a(_rtcc_set_time_and_date_lib.o)
 .debug_abbrev  0x00000beb       0x34 c:/program files/microchip/mplabc32/v2.02/bin/../lib/gcc/pic32mx/4.5.1/../../../../pic32mx/lib/speed\libmchp_peripheral_32MX795F512L.a(_rtcc_wait_clock_off_lib.o)
 .debug_abbrev  0x00000c1f       0x25 c:/program files/microchip/mplabc32/v2.02/bin/../lib/gcc/pic32mx/4.5.1/../../../../pic32mx/lib/speed\libc.a(calloc.o)
 .debug_abbrev  0x00000c44        0x1 c:/program files/microchip/mplabc32/v2.02/bin/../lib/gcc/pic32mx/4.5.1/../../../../pic32mx/lib/speed\libc.a(errno.o)
 .debug_abbrev  0x00000c45       0x41 c:/program files/microchip/mplabc32/v2.02/bin/../lib/gcc/pic32mx/4.5.1/../../../../pic32mx/lib/speed\libc.a(malloc.o)
 .debug_abbrev  0x00000c86       0x38 c:/program files/microchip/mplabc32/v2.02/bin/../lib/gcc/pic32mx/4.5.1/../../../../pic32mx/lib/speed\libc.a(sbrk.o)
 .debug_abbrev  0x00000cbe       0xe3 c:/program files/microchip/mplabc32/v2.02/bin/../lib/gcc/pic32mx/4.5.1/speed\libgcc.a(_lshrdi3.o)
 .debug_abbrev  0x00000da1       0xe3 c:/program files/microchip/mplabc32/v2.02/bin/../lib/gcc/pic32mx/4.5.1/speed\libgcc.a(_ashldi3.o)

.debug_line     0x00000000     0x21bf
 *(.debug_line)
 .debug_line    0x00000000      0x118 c:/program files/microchip/mplabc32/v2.02/bin/../lib/gcc/pic32mx/4.5.1/speed\libgcc.a(_udivdi3.o)
 .debug_line    0x00000118      0x12e c:/program files/microchip/mplabc32/v2.02/bin/../lib/gcc/pic32mx/4.5.1/speed\libgcc.a(_umoddi3.o)
 .debug_line    0x00000246       0x70 c:/program files/microchip/mplabc32/v2.02/bin/../lib/gcc/pic32mx/4.5.1/speed\libgcc.a(floatunsisf.o)
 .debug_line    0x000002b6       0x85 c:/program files/microchip/mplabc32/v2.02/bin/../lib/gcc/pic32mx/4.5.1/../../../../pic32mx/lib/speed\libc.a(atoi.o)
 .debug_line    0x0000033b       0x85 c:/program files/microchip/mplabc32/v2.02/bin/../lib/gcc/pic32mx/4.5.1/../../../../pic32mx/lib/speed\libc.a(atol.o)
 .debug_line    0x000003c0       0x86 c:/program files/microchip/mplabc32/v2.02/bin/../lib/gcc/pic32mx/4.5.1/../../../../pic32mx/lib/speed\libc.a(ctime.o)
 .debug_line    0x00000446        0x0 c:/program files/microchip/mplabc32/v2.02/bin/../lib/gcc/pic32mx/4.5.1/../../../../pic32mx/lib/speed\libc.a(ctype.o)
 .debug_line    0x00000446       0x87 c:/program files/microchip/mplabc32/v2.02/bin/../lib/gcc/pic32mx/4.5.1/../../../../pic32mx/lib/speed\libc.a(ctypef.o)
 .debug_line    0x000004cd       0x87 c:/program files/microchip/mplabc32/v2.02/bin/../lib/gcc/pic32mx/4.5.1/../../../../pic32mx/lib/speed\libc.a(strcat.o)
 .debug_line    0x00000554       0x87 c:/program files/microchip/mplabc32/v2.02/bin/../lib/gcc/pic32mx/4.5.1/../../../../pic32mx/lib/speed\libc.a(strchr.o)
 .debug_line    0x000005db       0x88 c:/program files/microchip/mplabc32/v2.02/bin/../lib/gcc/pic32mx/4.5.1/../../../../pic32mx/lib/speed\libc.a(strncpy.o)
 .debug_line    0x00000663       0x87 c:/program files/microchip/mplabc32/v2.02/bin/../lib/gcc/pic32mx/4.5.1/../../../../pic32mx/lib/speed\libc.a(strstr.o)
 .debug_line    0x000006ea       0x85 c:/program files/microchip/mplabc32/v2.02/bin/../lib/gcc/pic32mx/4.5.1/../../../../pic32mx/lib/speed\libc.a(atof.o)
 .debug_line    0x0000076f       0x93 c:/program files/microchip/mplabc32/v2.02/bin/../lib/gcc/pic32mx/4.5.1/../../../../pic32mx/lib/speed\libc.a(sprintf_cdnopsuxX.eo)
 .debug_line    0x00000802       0xa6 c:/program files/microchip/mplabc32/v2.02/bin/../lib/gcc/pic32mx/4.5.1/../../../../pic32mx/lib/speed\libc.a(default-bootstrap-exception-handler.o)
 .debug_line    0x000008a8       0x93 c:/program files/microchip/mplabc32/v2.02/bin/../lib/gcc/pic32mx/4.5.1/../../../../pic32mx/lib/speed\libc.a(default-on-reset.o)
 .debug_line    0x0000093b       0x97 c:/program files/microchip/mplabc32/v2.02/bin/../lib/gcc/pic32mx/4.5.1/../../../../pic32mx/lib/speed\libc.a(default-on-bootstrap.o)
 .debug_line    0x000009d2       0x88 c:/program files/microchip/mplabc32/v2.02/bin/../lib/gcc/pic32mx/4.5.1/../../../../pic32mx/lib/speed\libc.a(strncmp.o)
 .debug_line    0x00000a5a       0x87 c:/program files/microchip/mplabc32/v2.02/bin/../lib/gcc/pic32mx/4.5.1/../../../../pic32mx/lib/speed\libc.a(strtod.o)
 .debug_line    0x00000ae1       0x92 c:/program files/microchip/mplabc32/v2.02/bin/../lib/gcc/pic32mx/4.5.1/../../../../pic32mx/lib/speed\libc.a(doprnt_cdnopsuxX.eo)
 .debug_line    0x00000b73       0x91 c:/program files/microchip/mplabc32/v2.02/bin/../lib/gcc/pic32mx/4.5.1/../../../../pic32mx/lib/speed\libc.a(_fputc_simple.o)
 .debug_line    0x00000c04       0x88 c:/program files/microchip/mplabc32/v2.02/bin/../lib/gcc/pic32mx/4.5.1/../../../../pic32mx/lib/speed\libc.a(write.o)
 .debug_line    0x00000c8c        0x0 c:/program files/microchip/mplabc32/v2.02/bin/../lib/gcc/pic32mx/4.5.1/../../../../pic32mx/lib/speed\libc.a(_iob.o)
 .debug_line    0x00000c8c       0x92 c:/program files/microchip/mplabc32/v2.02/bin/../lib/gcc/pic32mx/4.5.1/../../../../pic32mx/lib/speed\libc.a(_flsbuf_simple.o)
 .debug_line    0x00000d1e       0x8c c:/program files/microchip/mplabc32/v2.02/bin/../lib/gcc/pic32mx/4.5.1/../../../../pic32mx/lib/speed\libc.a(_mon_putc.o)
 .debug_line    0x00000daa        0x0 c:/program files/microchip/mplabc32/v2.02/bin/../lib/gcc/pic32mx/4.5.1/../../../../pic32mx/lib/speed\libc.a(c32_uart.o)
 .debug_line    0x00000daa       0x93 c:/program files/microchip/mplabc32/v2.02/bin/../lib/gcc/pic32mx/4.5.1/../../../../pic32mx/lib/speed\libe.a(_strtod.o)
 .debug_line    0x00000e3d       0xa6 c:/program files/microchip/mplabc32/v2.02/bin/../lib/gcc/pic32mx/4.5.1/../../../../pic32mx/lib/speed\libe.a(_ldexp.o)
 .debug_line    0x00000ee3       0x6e c:/program files/microchip/mplabc32/v2.02/bin/../lib/gcc/pic32mx/4.5.1/../../../../pic32mx/lib/speed\libmchp_peripheral.a(read_core_timer_lib.o)
 .debug_line    0x00000f51       0x6f c:/program files/microchip/mplabc32/v2.02/bin/../lib/gcc/pic32mx/4.5.1/../../../../pic32mx/lib/speed\libmchp_peripheral.a(write_core_timer_lib.o)
 .debug_line    0x00000fc0       0x80 c:/program files/microchip/mplabc32/v2.02/bin/../lib/gcc/pic32mx/4.5.1/../../../../pic32mx/lib/speed\libmchp_peripheral_32MX795F512L.a(eth_ack_packet_lib.o)
 .debug_line    0x00001040       0x85 c:/program files/microchip/mplabc32/v2.02/bin/../lib/gcc/pic32mx/4.5.1/../../../../pic32mx/lib/speed\libmchp_peripheral_32MX795F512L.a(eth_descriptors_add_lib.o)
 .debug_line    0x000010c5       0x77 c:/program files/microchip/mplabc32/v2.02/bin/../lib/gcc/pic32mx/4.5.1/../../../../pic32mx/lib/speed\libmchp_peripheral_32MX795F512L.a(eth_init_lib.o)
 .debug_line    0x0000113c       0x69 c:/program files/microchip/mplabc32/v2.02/bin/../lib/gcc/pic32mx/4.5.1/../../../../pic32mx/lib/speed\libmchp_peripheral_32MX795F512L.a(eth_mac_open_lib.o)
 .debug_line    0x000011a5       0x74 c:/program files/microchip/mplabc32/v2.02/bin/../lib/gcc/pic32mx/4.5.1/../../../../pic32mx/lib/speed\libmchp_peripheral_32MX795F512L.a(eth_mac_set_address_max_lib.o)
 .debug_line    0x00001219       0x87 c:/program files/microchip/mplabc32/v2.02/bin/../lib/gcc/pic32mx/4.5.1/../../../../pic32mx/lib/speed\libmchp_peripheral_32MX795F512L.a(eth_rx_buffers_append_lib.o)
 .debug_line    0x000012a0       0x6b c:/program files/microchip/mplabc32/v2.02/bin/../lib/gcc/pic32mx/4.5.1/../../../../pic32mx/lib/speed\libmchp_peripheral_32MX795F512L.a(eth_rx_filters_lib.o)
 .debug_line    0x0000130b       0x6e c:/program files/microchip/mplabc32/v2.02/bin/../lib/gcc/pic32mx/4.5.1/../../../../pic32mx/lib/speed\libmchp_peripheral_32MX795F512L.a(eth_rx_get_packet_lib.o)
 .debug_line    0x00001379       0x73 c:/program files/microchip/mplabc32/v2.02/bin/../lib/gcc/pic32mx/4.5.1/../../../../pic32mx/lib/speed\libmchp_peripheral_32MX795F512L.a(eth_rx_set_buffer_size_lib.o)
 .debug_line    0x000013ec       0x7f c:/program files/microchip/mplabc32/v2.02/bin/../lib/gcc/pic32mx/4.5.1/../../../../pic32mx/lib/speed\libmchp_peripheral_32MX795F512L.a(eth_tx_packet_lib.o)
 .debug_line    0x0000146b       0x87 c:/program files/microchip/mplabc32/v2.02/bin/../lib/gcc/pic32mx/4.5.1/../../../../pic32mx/lib/speed\libmchp_peripheral_32MX795F512L.a(_eth_append_busy_list_lib.o)
 .debug_line    0x000014f2       0x68 c:/program files/microchip/mplabc32/v2.02/bin/../lib/gcc/pic32mx/4.5.1/../../../../pic32mx/lib/speed\libmchp_peripheral_32MX795F512L.a(eth_miim_access.o)
 .debug_line    0x0000155a       0xbf c:/program files/microchip/mplabc32/v2.02/bin/../lib/gcc/pic32mx/4.5.1/../../../../pic32mx/lib/speed\libmchp_peripheral_32MX795F512L.a(soft_reset_lib.o)
 .debug_line    0x00001619       0x62 c:/program files/microchip/mplabc32/v2.02/bin/../lib/gcc/pic32mx/4.5.1/../../../../pic32mx/lib/speed\libmchp_peripheral_32MX795F512L.a(pcache.o)
 .debug_line    0x0000167b       0x6d c:/program files/microchip/mplabc32/v2.02/bin/../lib/gcc/pic32mx/4.5.1/../../../../pic32mx/lib/speed\libmchp_peripheral_32MX795F512L.a(set_core_sw0_leg_lib.o)
 .debug_line    0x000016e8       0x73 c:/program files/microchip/mplabc32/v2.02/bin/../lib/gcc/pic32mx/4.5.1/../../../../pic32mx/lib/speed\libmchp_peripheral_32MX795F512L.a(int_disable_interrupts_lib.o)
 .debug_line    0x0000175b       0x73 c:/program files/microchip/mplabc32/v2.02/bin/../lib/gcc/pic32mx/4.5.1/../../../../pic32mx/lib/speed\libmchp_peripheral_32MX795F512L.a(int_restore_interrupts_lib.o)
 .debug_line    0x000017ce       0x6e c:/program files/microchip/mplabc32/v2.02/bin/../lib/gcc/pic32mx/4.5.1/../../../../pic32mx/lib/speed\libmchp_peripheral_32MX795F512L.a(int_enable_mv_int_lib.o)
 .debug_line    0x0000183c       0x64 c:/program files/microchip/mplabc32/v2.02/bin/../lib/gcc/pic32mx/4.5.1/../../../../pic32mx/lib/speed\libmchp_peripheral_32MX795F512L.a(int_tbl_lib.o)
 .debug_line    0x000018a0       0xda c:/program files/microchip/mplabc32/v2.02/bin/../lib/gcc/pic32mx/4.5.1/../../../../pic32mx/lib/speed\libmchp_peripheral_32MX795F512L.a(rtcc_init_lib.o)
 .debug_line    0x0000197a       0x70 c:/program files/microchip/mplabc32/v2.02/bin/../lib/gcc/pic32mx/4.5.1/../../../../pic32mx/lib/speed\libmchp_peripheral_32MX795F512L.a(rtcc_set_time_date_lib.o)
 .debug_line    0x000019ea       0xda c:/program files/microchip/mplabc32/v2.02/bin/../lib/gcc/pic32mx/4.5.1/../../../../pic32mx/lib/speed\libmchp_peripheral_32MX795F512L.a(rtcc_open_lib.o)
 .debug_line    0x00001ac4       0x71 c:/program files/microchip/mplabc32/v2.02/bin/../lib/gcc/pic32mx/4.5.1/../../../../pic32mx/lib/speed\libmchp_peripheral_32MX795F512L.a(spi_getc_spi1_lib_legacy.o)
 .debug_line    0x00001b35       0x71 c:/program files/microchip/mplabc32/v2.02/bin/../lib/gcc/pic32mx/4.5.1/../../../../pic32mx/lib/speed\libmchp_peripheral_32MX795F512L.a(spi_open_spi1_lib_legacy.o)
 .debug_line    0x00001ba6        0x0 c:/program files/microchip/mplabc32/v2.02/bin/../lib/gcc/pic32mx/4.5.1/../../../../pic32mx/lib/speed\libmchp_peripheral_32MX795F512L.a(spi_brg_tbl_lib_legacy.o)
 .debug_line    0x00001ba6       0x77 c:/program files/microchip/mplabc32/v2.02/bin/../lib/gcc/pic32mx/4.5.1/../../../../pic32mx/lib/speed\libmchp_peripheral_32MX795F512L.a(port_set_pins_digital_in_lib.o)
 .debug_line    0x00001c1d       0x78 c:/program files/microchip/mplabc32/v2.02/bin/../lib/gcc/pic32mx/4.5.1/../../../../pic32mx/lib/speed\libmchp_peripheral_32MX795F512L.a(port_set_pins_digital_out_lib.o)
 .debug_line    0x00001c95        0x0 c:/program files/microchip/mplabc32/v2.02/bin/../lib/gcc/pic32mx/4.5.1/../../../../pic32mx/lib/speed\libmchp_peripheral_32MX795F512L.a(_ports_tbl_libp.o)
 .debug_line    0x00001c95       0x72 c:/program files/microchip/mplabc32/v2.02/bin/../lib/gcc/pic32mx/4.5.1/../../../../pic32mx/lib/speed\libmchp_peripheral_32MX795F512L.a(int_enable_interrupts_lib.o)
 .debug_line    0x00001d07       0xe8 c:/program files/microchip/mplabc32/v2.02/bin/../lib/gcc/pic32mx/4.5.1/../../../../pic32mx/lib/speed\libmchp_peripheral_32MX795F512L.a(_rtcc_set_time_and_date_lib.o)
 .debug_line    0x00001def       0xbd c:/program files/microchip/mplabc32/v2.02/bin/../lib/gcc/pic32mx/4.5.1/../../../../pic32mx/lib/speed\libmchp_peripheral_32MX795F512L.a(_rtcc_wait_clock_off_lib.o)
 .debug_line    0x00001eac       0x87 c:/program files/microchip/mplabc32/v2.02/bin/../lib/gcc/pic32mx/4.5.1/../../../../pic32mx/lib/speed\libc.a(calloc.o)
 .debug_line    0x00001f33        0x0 c:/program files/microchip/mplabc32/v2.02/bin/../lib/gcc/pic32mx/4.5.1/../../../../pic32mx/lib/speed\libc.a(errno.o)
 .debug_line    0x00001f33       0x87 c:/program files/microchip/mplabc32/v2.02/bin/../lib/gcc/pic32mx/4.5.1/../../../../pic32mx/lib/speed\libc.a(malloc.o)
 .debug_line    0x00001fba       0x87 c:/program files/microchip/mplabc32/v2.02/bin/../lib/gcc/pic32mx/4.5.1/../../../../pic32mx/lib/speed\libc.a(sbrk.o)
 .debug_line    0x00002041       0xbe c:/program files/microchip/mplabc32/v2.02/bin/../lib/gcc/pic32mx/4.5.1/speed\libgcc.a(_lshrdi3.o)
 .debug_line    0x000020ff       0xc0 c:/program files/microchip/mplabc32/v2.02/bin/../lib/gcc/pic32mx/4.5.1/speed\libgcc.a(_ashldi3.o)

.debug_frame    0x00000000      0xd10
 *(.debug_frame)
 .debug_frame   0x00000000       0x28 c:/program files/microchip/mplabc32/v2.02/bin/../lib/gcc/pic32mx/4.5.1/speed\libgcc.a(floatunsisf.o)
 .debug_frame   0x00000028       0x20 c:/program files/microchip/mplabc32/v2.02/bin/../lib/gcc/pic32mx/4.5.1/../../../../pic32mx/lib/speed\libc.a(atoi.o)
 .debug_frame   0x00000048       0x20 c:/program files/microchip/mplabc32/v2.02/bin/../lib/gcc/pic32mx/4.5.1/../../../../pic32mx/lib/speed\libc.a(atol.o)
 .debug_frame   0x00000068       0x60 c:/program files/microchip/mplabc32/v2.02/bin/../lib/gcc/pic32mx/4.5.1/../../../../pic32mx/lib/speed\libc.a(ctime.o)
 .debug_frame   0x000000c8      0x120 c:/program files/microchip/mplabc32/v2.02/bin/../lib/gcc/pic32mx/4.5.1/../../../../pic32mx/lib/speed\libc.a(ctypef.o)
 .debug_frame   0x000001e8       0x20 c:/program files/microchip/mplabc32/v2.02/bin/../lib/gcc/pic32mx/4.5.1/../../../../pic32mx/lib/speed\libc.a(strcat.o)
 .debug_frame   0x00000208       0x20 c:/program files/microchip/mplabc32/v2.02/bin/../lib/gcc/pic32mx/4.5.1/../../../../pic32mx/lib/speed\libc.a(strchr.o)
 .debug_frame   0x00000228       0x20 c:/program files/microchip/mplabc32/v2.02/bin/../lib/gcc/pic32mx/4.5.1/../../../../pic32mx/lib/speed\libc.a(strncpy.o)
 .debug_frame   0x00000248       0x2c c:/program files/microchip/mplabc32/v2.02/bin/../lib/gcc/pic32mx/4.5.1/../../../../pic32mx/lib/speed\libc.a(strstr.o)
 .debug_frame   0x00000274       0x28 c:/program files/microchip/mplabc32/v2.02/bin/../lib/gcc/pic32mx/4.5.1/../../../../pic32mx/lib/speed\libc.a(atof.o)
 .debug_frame   0x0000029c       0x2c c:/program files/microchip/mplabc32/v2.02/bin/../lib/gcc/pic32mx/4.5.1/../../../../pic32mx/lib/speed\libc.a(sprintf_cdnopsuxX.eo)
 .debug_frame   0x000002c8       0x20 c:/program files/microchip/mplabc32/v2.02/bin/../lib/gcc/pic32mx/4.5.1/../../../../pic32mx/lib/speed\libc.a(default-bootstrap-exception-handler.o)
 .debug_frame   0x000002e8       0x20 c:/program files/microchip/mplabc32/v2.02/bin/../lib/gcc/pic32mx/4.5.1/../../../../pic32mx/lib/speed\libc.a(default-on-reset.o)
 .debug_frame   0x00000308       0x20 c:/program files/microchip/mplabc32/v2.02/bin/../lib/gcc/pic32mx/4.5.1/../../../../pic32mx/lib/speed\libc.a(default-on-bootstrap.o)
 .debug_frame   0x00000328       0x20 c:/program files/microchip/mplabc32/v2.02/bin/../lib/gcc/pic32mx/4.5.1/../../../../pic32mx/lib/speed\libc.a(strncmp.o)
 .debug_frame   0x00000348       0x40 c:/program files/microchip/mplabc32/v2.02/bin/../lib/gcc/pic32mx/4.5.1/../../../../pic32mx/lib/speed\libc.a(strtod.o)
 .debug_frame   0x00000388       0x38 c:/program files/microchip/mplabc32/v2.02/bin/../lib/gcc/pic32mx/4.5.1/../../../../pic32mx/lib/speed\libc.a(doprnt_cdnopsuxX.eo)
 .debug_frame   0x000003c0       0x2c c:/program files/microchip/mplabc32/v2.02/bin/../lib/gcc/pic32mx/4.5.1/../../../../pic32mx/lib/speed\libc.a(_fputc_simple.o)
 .debug_frame   0x000003ec       0x28 c:/program files/microchip/mplabc32/v2.02/bin/../lib/gcc/pic32mx/4.5.1/../../../../pic32mx/lib/speed\libc.a(write.o)
 .debug_frame   0x00000414       0x28 c:/program files/microchip/mplabc32/v2.02/bin/../lib/gcc/pic32mx/4.5.1/../../../../pic32mx/lib/speed\libc.a(_flsbuf_simple.o)
 .debug_frame   0x0000043c       0x20 c:/program files/microchip/mplabc32/v2.02/bin/../lib/gcc/pic32mx/4.5.1/../../../../pic32mx/lib/speed\libc.a(_mon_putc.o)
 .debug_frame   0x0000045c       0x38 c:/program files/microchip/mplabc32/v2.02/bin/../lib/gcc/pic32mx/4.5.1/../../../../pic32mx/lib/speed\libe.a(_strtod.o)
 .debug_frame   0x00000494       0x34 c:/program files/microchip/mplabc32/v2.02/bin/../lib/gcc/pic32mx/4.5.1/../../../../pic32mx/lib/speed\libe.a(_ldexp.o)
 .debug_frame   0x000004c8       0x20 c:/program files/microchip/mplabc32/v2.02/bin/../lib/gcc/pic32mx/4.5.1/../../../../pic32mx/lib/speed\libmchp_peripheral.a(read_core_timer_lib.o)
 .debug_frame   0x000004e8       0x20 c:/program files/microchip/mplabc32/v2.02/bin/../lib/gcc/pic32mx/4.5.1/../../../../pic32mx/lib/speed\libmchp_peripheral.a(write_core_timer_lib.o)
 .debug_frame   0x00000508       0xb8 c:/program files/microchip/mplabc32/v2.02/bin/../lib/gcc/pic32mx/4.5.1/../../../../pic32mx/lib/speed\libmchp_peripheral_32MX795F512L.a(eth_ack_packet_lib.o)
 .debug_frame   0x000005c0       0x54 c:/program files/microchip/mplabc32/v2.02/bin/../lib/gcc/pic32mx/4.5.1/../../../../pic32mx/lib/speed\libmchp_peripheral_32MX795F512L.a(eth_descriptors_add_lib.o)
 .debug_frame   0x00000614       0x28 c:/program files/microchip/mplabc32/v2.02/bin/../lib/gcc/pic32mx/4.5.1/../../../../pic32mx/lib/speed\libmchp_peripheral_32MX795F512L.a(eth_init_lib.o)
 .debug_frame   0x0000063c       0x20 c:/program files/microchip/mplabc32/v2.02/bin/../lib/gcc/pic32mx/4.5.1/../../../../pic32mx/lib/speed\libmchp_peripheral_32MX795F512L.a(eth_mac_open_lib.o)
 .debug_frame   0x0000065c       0x50 c:/program files/microchip/mplabc32/v2.02/bin/../lib/gcc/pic32mx/4.5.1/../../../../pic32mx/lib/speed\libmchp_peripheral_32MX795F512L.a(eth_mac_set_address_max_lib.o)
 .debug_frame   0x000006ac       0x2c c:/program files/microchip/mplabc32/v2.02/bin/../lib/gcc/pic32mx/4.5.1/../../../../pic32mx/lib/speed\libmchp_peripheral_32MX795F512L.a(eth_rx_buffers_append_lib.o)
 .debug_frame   0x000006d8       0x70 c:/program files/microchip/mplabc32/v2.02/bin/../lib/gcc/pic32mx/4.5.1/../../../../pic32mx/lib/speed\libmchp_peripheral_32MX795F512L.a(eth_rx_filters_lib.o)
 .debug_frame   0x00000748       0x3c c:/program files/microchip/mplabc32/v2.02/bin/../lib/gcc/pic32mx/4.5.1/../../../../pic32mx/lib/speed\libmchp_peripheral_32MX795F512L.a(eth_rx_get_packet_lib.o)
 .debug_frame   0x00000784       0x20 c:/program files/microchip/mplabc32/v2.02/bin/../lib/gcc/pic32mx/4.5.1/../../../../pic32mx/lib/speed\libmchp_peripheral_32MX795F512L.a(eth_rx_set_buffer_size_lib.o)
 .debug_frame   0x000007a4       0x60 c:/program files/microchip/mplabc32/v2.02/bin/../lib/gcc/pic32mx/4.5.1/../../../../pic32mx/lib/speed\libmchp_peripheral_32MX795F512L.a(eth_tx_packet_lib.o)
 .debug_frame   0x00000804       0x20 c:/program files/microchip/mplabc32/v2.02/bin/../lib/gcc/pic32mx/4.5.1/../../../../pic32mx/lib/speed\libmchp_peripheral_32MX795F512L.a(_eth_append_busy_list_lib.o)
 .debug_frame   0x00000824       0x70 c:/program files/microchip/mplabc32/v2.02/bin/../lib/gcc/pic32mx/4.5.1/../../../../pic32mx/lib/speed\libmchp_peripheral_32MX795F512L.a(eth_miim_access.o)
 .debug_frame   0x00000894       0x28 c:/program files/microchip/mplabc32/v2.02/bin/../lib/gcc/pic32mx/4.5.1/../../../../pic32mx/lib/speed\libmchp_peripheral_32MX795F512L.a(soft_reset_lib.o)
 .debug_frame   0x000008bc       0x30 c:/program files/microchip/mplabc32/v2.02/bin/../lib/gcc/pic32mx/4.5.1/../../../../pic32mx/lib/speed\libmchp_peripheral_32MX795F512L.a(pcache.o)
 .debug_frame   0x000008ec       0x20 c:/program files/microchip/mplabc32/v2.02/bin/../lib/gcc/pic32mx/4.5.1/../../../../pic32mx/lib/speed\libmchp_peripheral_32MX795F512L.a(set_core_sw0_leg_lib.o)
 .debug_frame   0x0000090c       0x20 c:/program files/microchip/mplabc32/v2.02/bin/../lib/gcc/pic32mx/4.5.1/../../../../pic32mx/lib/speed\libmchp_peripheral_32MX795F512L.a(int_disable_interrupts_lib.o)
 .debug_frame   0x0000092c       0x20 c:/program files/microchip/mplabc32/v2.02/bin/../lib/gcc/pic32mx/4.5.1/../../../../pic32mx/lib/speed\libmchp_peripheral_32MX795F512L.a(int_restore_interrupts_lib.o)
 .debug_frame   0x0000094c       0x28 c:/program files/microchip/mplabc32/v2.02/bin/../lib/gcc/pic32mx/4.5.1/../../../../pic32mx/lib/speed\libmchp_peripheral_32MX795F512L.a(int_enable_mv_int_lib.o)
 .debug_frame   0x00000974       0xa0 c:/program files/microchip/mplabc32/v2.02/bin/../lib/gcc/pic32mx/4.5.1/../../../../pic32mx/lib/speed\libmchp_peripheral_32MX795F512L.a(int_tbl_lib.o)
 .debug_frame   0x00000a14       0x2c c:/program files/microchip/mplabc32/v2.02/bin/../lib/gcc/pic32mx/4.5.1/../../../../pic32mx/lib/speed\libmchp_peripheral_32MX795F512L.a(rtcc_init_lib.o)
 .debug_frame   0x00000a40       0x28 c:/program files/microchip/mplabc32/v2.02/bin/../lib/gcc/pic32mx/4.5.1/../../../../pic32mx/lib/speed\libmchp_peripheral_32MX795F512L.a(rtcc_set_time_date_lib.o)
 .debug_frame   0x00000a68       0x34 c:/program files/microchip/mplabc32/v2.02/bin/../lib/gcc/pic32mx/4.5.1/../../../../pic32mx/lib/speed\libmchp_peripheral_32MX795F512L.a(rtcc_open_lib.o)
 .debug_frame   0x00000a9c       0x20 c:/program files/microchip/mplabc32/v2.02/bin/../lib/gcc/pic32mx/4.5.1/../../../../pic32mx/lib/speed\libmchp_peripheral_32MX795F512L.a(spi_getc_spi1_lib_legacy.o)
 .debug_frame   0x00000abc       0x20 c:/program files/microchip/mplabc32/v2.02/bin/../lib/gcc/pic32mx/4.5.1/../../../../pic32mx/lib/speed\libmchp_peripheral_32MX795F512L.a(spi_open_spi1_lib_legacy.o)
 .debug_frame   0x00000adc       0x20 c:/program files/microchip/mplabc32/v2.02/bin/../lib/gcc/pic32mx/4.5.1/../../../../pic32mx/lib/speed\libmchp_peripheral_32MX795F512L.a(port_set_pins_digital_in_lib.o)
 .debug_frame   0x00000afc       0x20 c:/program files/microchip/mplabc32/v2.02/bin/../lib/gcc/pic32mx/4.5.1/../../../../pic32mx/lib/speed\libmchp_peripheral_32MX795F512L.a(port_set_pins_digital_out_lib.o)
 .debug_frame   0x00000b1c       0x20 c:/program files/microchip/mplabc32/v2.02/bin/../lib/gcc/pic32mx/4.5.1/../../../../pic32mx/lib/speed\libmchp_peripheral_32MX795F512L.a(int_enable_interrupts_lib.o)
 .debug_frame   0x00000b3c       0x30 c:/program files/microchip/mplabc32/v2.02/bin/../lib/gcc/pic32mx/4.5.1/../../../../pic32mx/lib/speed\libmchp_peripheral_32MX795F512L.a(_rtcc_set_time_and_date_lib.o)
 .debug_frame   0x00000b6c       0x44 c:/program files/microchip/mplabc32/v2.02/bin/../lib/gcc/pic32mx/4.5.1/../../../../pic32mx/lib/speed\libmchp_peripheral_32MX795F512L.a(_rtcc_wait_clock_off_lib.o)
 .debug_frame   0x00000bb0       0x2c c:/program files/microchip/mplabc32/v2.02/bin/../lib/gcc/pic32mx/4.5.1/../../../../pic32mx/lib/speed\libc.a(calloc.o)
 .debug_frame   0x00000bdc       0x68 c:/program files/microchip/mplabc32/v2.02/bin/../lib/gcc/pic32mx/4.5.1/../../../../pic32mx/lib/speed\libc.a(malloc.o)
 .debug_frame   0x00000c44       0x8c c:/program files/microchip/mplabc32/v2.02/bin/../lib/gcc/pic32mx/4.5.1/../../../../pic32mx/lib/speed\libc.a(sbrk.o)
 .debug_frame   0x00000cd0       0x20 c:/program files/microchip/mplabc32/v2.02/bin/../lib/gcc/pic32mx/4.5.1/speed\libgcc.a(_lshrdi3.o)
 .debug_frame   0x00000cf0       0x20 c:/program files/microchip/mplabc32/v2.02/bin/../lib/gcc/pic32mx/4.5.1/speed\libgcc.a(_ashldi3.o)

.debug_str      0x00000000        0x9
 *(.debug_str)
 .debug_str     0x00000000        0x0 c:/program files/microchip/mplabc32/v2.02/bin/../lib/gcc/pic32mx/4.5.1/speed\libgcc.a(_udivdi3.o)
 .debug_str     0x00000000        0x0 c:/program files/microchip/mplabc32/v2.02/bin/../lib/gcc/pic32mx/4.5.1/speed\libgcc.a(_umoddi3.o)
 .debug_str     0x00000000        0x0 c:/program files/microchip/mplabc32/v2.02/bin/../lib/gcc/pic32mx/4.5.1/speed\libgcc.a(floatunsisf.o)
 .debug_str     0x00000000        0x0 c:/program files/microchip/mplabc32/v2.02/bin/../lib/gcc/pic32mx/4.5.1/../../../../pic32mx/lib/speed\libc.a(atoi.o)
 .debug_str     0x00000000        0x0 c:/program files/microchip/mplabc32/v2.02/bin/../lib/gcc/pic32mx/4.5.1/../../../../pic32mx/lib/speed\libc.a(atol.o)
 .debug_str     0x00000000        0x0 c:/program files/microchip/mplabc32/v2.02/bin/../lib/gcc/pic32mx/4.5.1/../../../../pic32mx/lib/speed\libc.a(ctime.o)
 .debug_str     0x00000000        0x0 c:/program files/microchip/mplabc32/v2.02/bin/../lib/gcc/pic32mx/4.5.1/../../../../pic32mx/lib/speed\libc.a(ctype.o)
 .debug_str     0x00000000        0x0 c:/program files/microchip/mplabc32/v2.02/bin/../lib/gcc/pic32mx/4.5.1/../../../../pic32mx/lib/speed\libc.a(ctypef.o)
 .debug_str     0x00000000        0x0 c:/program files/microchip/mplabc32/v2.02/bin/../lib/gcc/pic32mx/4.5.1/../../../../pic32mx/lib/speed\libc.a(strcat.o)
 .debug_str     0x00000000        0x0 c:/program files/microchip/mplabc32/v2.02/bin/../lib/gcc/pic32mx/4.5.1/../../../../pic32mx/lib/speed\libc.a(strchr.o)
 .debug_str     0x00000000        0x0 c:/program files/microchip/mplabc32/v2.02/bin/../lib/gcc/pic32mx/4.5.1/../../../../pic32mx/lib/speed\libc.a(strncpy.o)
 .debug_str     0x00000000        0x0 c:/program files/microchip/mplabc32/v2.02/bin/../lib/gcc/pic32mx/4.5.1/../../../../pic32mx/lib/speed\libc.a(strstr.o)
 .debug_str     0x00000000        0x0 c:/program files/microchip/mplabc32/v2.02/bin/../lib/gcc/pic32mx/4.5.1/../../../../pic32mx/lib/speed\libc.a(atof.o)
 .debug_str     0x00000000        0x0 c:/program files/microchip/mplabc32/v2.02/bin/../lib/gcc/pic32mx/4.5.1/../../../../pic32mx/lib/speed\libc.a(sprintf_cdnopsuxX.eo)
 .debug_str     0x00000000        0x0 c:/program files/microchip/mplabc32/v2.02/bin/../lib/gcc/pic32mx/4.5.1/../../../../pic32mx/lib/speed\libc.a(default-bootstrap-exception-handler.o)
 .debug_str     0x00000000        0x0 c:/program files/microchip/mplabc32/v2.02/bin/../lib/gcc/pic32mx/4.5.1/../../../../pic32mx/lib/speed\libc.a(default-on-reset.o)
 .debug_str     0x00000000        0x0 c:/program files/microchip/mplabc32/v2.02/bin/../lib/gcc/pic32mx/4.5.1/../../../../pic32mx/lib/speed\libc.a(default-on-bootstrap.o)
 .debug_str     0x00000000        0x0 c:/program files/microchip/mplabc32/v2.02/bin/../lib/gcc/pic32mx/4.5.1/../../../../pic32mx/lib/speed\libc.a(strncmp.o)
 .debug_str     0x00000000        0x9 c:/program files/microchip/mplabc32/v2.02/bin/../lib/gcc/pic32mx/4.5.1/../../../../pic32mx/lib/speed\libc.a(strtod.o)
 .debug_str     0x00000009        0x0 c:/program files/microchip/mplabc32/v2.02/bin/../lib/gcc/pic32mx/4.5.1/../../../../pic32mx/lib/speed\libc.a(doprnt_cdnopsuxX.eo)
 .debug_str     0x00000009        0x0 c:/program files/microchip/mplabc32/v2.02/bin/../lib/gcc/pic32mx/4.5.1/../../../../pic32mx/lib/speed\libc.a(_fputc_simple.o)
 .debug_str     0x00000009        0x0 c:/program files/microchip/mplabc32/v2.02/bin/../lib/gcc/pic32mx/4.5.1/../../../../pic32mx/lib/speed\libc.a(write.o)
 .debug_str     0x00000009        0x0 c:/program files/microchip/mplabc32/v2.02/bin/../lib/gcc/pic32mx/4.5.1/../../../../pic32mx/lib/speed\libc.a(_iob.o)
 .debug_str     0x00000009        0x0 c:/program files/microchip/mplabc32/v2.02/bin/../lib/gcc/pic32mx/4.5.1/../../../../pic32mx/lib/speed\libc.a(_flsbuf_simple.o)
 .debug_str     0x00000009        0x0 c:/program files/microchip/mplabc32/v2.02/bin/../lib/gcc/pic32mx/4.5.1/../../../../pic32mx/lib/speed\libc.a(_mon_putc.o)
 .debug_str     0x00000009        0x0 c:/program files/microchip/mplabc32/v2.02/bin/../lib/gcc/pic32mx/4.5.1/../../../../pic32mx/lib/speed\libc.a(c32_uart.o)
 .debug_str     0x00000009        0x0 c:/program files/microchip/mplabc32/v2.02/bin/../lib/gcc/pic32mx/4.5.1/../../../../pic32mx/lib/speed\libe.a(_strtod.o)
 .debug_str     0x00000009        0x0 c:/program files/microchip/mplabc32/v2.02/bin/../lib/gcc/pic32mx/4.5.1/../../../../pic32mx/lib/speed\libe.a(_ldexp.o)
 .debug_str     0x00000009        0x0 c:/program files/microchip/mplabc32/v2.02/bin/../lib/gcc/pic32mx/4.5.1/../../../../pic32mx/lib/speed\libmchp_peripheral.a(read_core_timer_lib.o)
 .debug_str     0x00000009        0x0 c:/program files/microchip/mplabc32/v2.02/bin/../lib/gcc/pic32mx/4.5.1/../../../../pic32mx/lib/speed\libmchp_peripheral.a(write_core_timer_lib.o)
 .debug_str     0x00000009        0x0 c:/program files/microchip/mplabc32/v2.02/bin/../lib/gcc/pic32mx/4.5.1/../../../../pic32mx/lib/speed\libmchp_peripheral_32MX795F512L.a(eth_ack_packet_lib.o)
 .debug_str     0x00000009        0x0 c:/program files/microchip/mplabc32/v2.02/bin/../lib/gcc/pic32mx/4.5.1/../../../../pic32mx/lib/speed\libmchp_peripheral_32MX795F512L.a(eth_descriptors_add_lib.o)
 .debug_str     0x00000009        0x0 c:/program files/microchip/mplabc32/v2.02/bin/../lib/gcc/pic32mx/4.5.1/../../../../pic32mx/lib/speed\libmchp_peripheral_32MX795F512L.a(eth_init_lib.o)
 .debug_str     0x00000009        0x0 c:/program files/microchip/mplabc32/v2.02/bin/../lib/gcc/pic32mx/4.5.1/../../../../pic32mx/lib/speed\libmchp_peripheral_32MX795F512L.a(eth_mac_open_lib.o)
 .debug_str     0x00000009        0x0 c:/program files/microchip/mplabc32/v2.02/bin/../lib/gcc/pic32mx/4.5.1/../../../../pic32mx/lib/speed\libmchp_peripheral_32MX795F512L.a(eth_mac_set_address_max_lib.o)
 .debug_str     0x00000009        0x0 c:/program files/microchip/mplabc32/v2.02/bin/../lib/gcc/pic32mx/4.5.1/../../../../pic32mx/lib/speed\libmchp_peripheral_32MX795F512L.a(eth_rx_buffers_append_lib.o)
 .debug_str     0x00000009        0x0 c:/program files/microchip/mplabc32/v2.02/bin/../lib/gcc/pic32mx/4.5.1/../../../../pic32mx/lib/speed\libmchp_peripheral_32MX795F512L.a(eth_rx_filters_lib.o)
 .debug_str     0x00000009        0x0 c:/program files/microchip/mplabc32/v2.02/bin/../lib/gcc/pic32mx/4.5.1/../../../../pic32mx/lib/speed\libmchp_peripheral_32MX795F512L.a(eth_rx_get_packet_lib.o)
 .debug_str     0x00000009        0x0 c:/program files/microchip/mplabc32/v2.02/bin/../lib/gcc/pic32mx/4.5.1/../../../../pic32mx/lib/speed\libmchp_peripheral_32MX795F512L.a(eth_rx_set_buffer_size_lib.o)
 .debug_str     0x00000009        0x0 c:/program files/microchip/mplabc32/v2.02/bin/../lib/gcc/pic32mx/4.5.1/../../../../pic32mx/lib/speed\libmchp_peripheral_32MX795F512L.a(eth_tx_packet_lib.o)
 .debug_str     0x00000009        0x0 c:/program files/microchip/mplabc32/v2.02/bin/../lib/gcc/pic32mx/4.5.1/../../../../pic32mx/lib/speed\libmchp_peripheral_32MX795F512L.a(_eth_append_busy_list_lib.o)
 .debug_str     0x00000009        0x0 c:/program files/microchip/mplabc32/v2.02/bin/../lib/gcc/pic32mx/4.5.1/../../../../pic32mx/lib/speed\libmchp_peripheral_32MX795F512L.a(eth_miim_access.o)
 .debug_str     0x00000009        0x0 c:/program files/microchip/mplabc32/v2.02/bin/../lib/gcc/pic32mx/4.5.1/../../../../pic32mx/lib/speed\libmchp_peripheral_32MX795F512L.a(soft_reset_lib.o)
 .debug_str     0x00000009        0x0 c:/program files/microchip/mplabc32/v2.02/bin/../lib/gcc/pic32mx/4.5.1/../../../../pic32mx/lib/speed\libmchp_peripheral_32MX795F512L.a(pcache.o)
 .debug_str     0x00000009        0x0 c:/program files/microchip/mplabc32/v2.02/bin/../lib/gcc/pic32mx/4.5.1/../../../../pic32mx/lib/speed\libmchp_peripheral_32MX795F512L.a(set_core_sw0_leg_lib.o)
 .debug_str     0x00000009        0x0 c:/program files/microchip/mplabc32/v2.02/bin/../lib/gcc/pic32mx/4.5.1/../../../../pic32mx/lib/speed\libmchp_peripheral_32MX795F512L.a(int_disable_interrupts_lib.o)
 .debug_str     0x00000009        0x0 c:/program files/microchip/mplabc32/v2.02/bin/../lib/gcc/pic32mx/4.5.1/../../../../pic32mx/lib/speed\libmchp_peripheral_32MX795F512L.a(int_restore_interrupts_lib.o)
 .debug_str     0x00000009        0x0 c:/program files/microchip/mplabc32/v2.02/bin/../lib/gcc/pic32mx/4.5.1/../../../../pic32mx/lib/speed\libmchp_peripheral_32MX795F512L.a(int_enable_mv_int_lib.o)
 .debug_str     0x00000009        0x0 c:/program files/microchip/mplabc32/v2.02/bin/../lib/gcc/pic32mx/4.5.1/../../../../pic32mx/lib/speed\libmchp_peripheral_32MX795F512L.a(int_tbl_lib.o)
 .debug_str     0x00000009        0x0 c:/program files/microchip/mplabc32/v2.02/bin/../lib/gcc/pic32mx/4.5.1/../../../../pic32mx/lib/speed\libmchp_peripheral_32MX795F512L.a(rtcc_init_lib.o)
 .debug_str     0x00000009        0x0 c:/program files/microchip/mplabc32/v2.02/bin/../lib/gcc/pic32mx/4.5.1/../../../../pic32mx/lib/speed\libmchp_peripheral_32MX795F512L.a(rtcc_set_time_date_lib.o)
 .debug_str     0x00000009        0x0 c:/program files/microchip/mplabc32/v2.02/bin/../lib/gcc/pic32mx/4.5.1/../../../../pic32mx/lib/speed\libmchp_peripheral_32MX795F512L.a(rtcc_open_lib.o)
 .debug_str     0x00000009        0x0 c:/program files/microchip/mplabc32/v2.02/bin/../lib/gcc/pic32mx/4.5.1/../../../../pic32mx/lib/speed\libmchp_peripheral_32MX795F512L.a(spi_getc_spi1_lib_legacy.o)
 .debug_str     0x00000009        0x0 c:/program files/microchip/mplabc32/v2.02/bin/../lib/gcc/pic32mx/4.5.1/../../../../pic32mx/lib/speed\libmchp_peripheral_32MX795F512L.a(spi_open_spi1_lib_legacy.o)
 .debug_str     0x00000009        0x0 c:/program files/microchip/mplabc32/v2.02/bin/../lib/gcc/pic32mx/4.5.1/../../../../pic32mx/lib/speed\libmchp_peripheral_32MX795F512L.a(spi_brg_tbl_lib_legacy.o)
 .debug_str     0x00000009        0x0 c:/program files/microchip/mplabc32/v2.02/bin/../lib/gcc/pic32mx/4.5.1/../../../../pic32mx/lib/speed\libmchp_peripheral_32MX795F512L.a(port_set_pins_digital_in_lib.o)
 .debug_str     0x00000009        0x0 c:/program files/microchip/mplabc32/v2.02/bin/../lib/gcc/pic32mx/4.5.1/../../../../pic32mx/lib/speed\libmchp_peripheral_32MX795F512L.a(port_set_pins_digital_out_lib.o)
 .debug_str     0x00000009        0x0 c:/program files/microchip/mplabc32/v2.02/bin/../lib/gcc/pic32mx/4.5.1/../../../../pic32mx/lib/speed\libmchp_peripheral_32MX795F512L.a(_ports_tbl_libp.o)
 .debug_str     0x00000009        0x0 c:/program files/microchip/mplabc32/v2.02/bin/../lib/gcc/pic32mx/4.5.1/../../../../pic32mx/lib/speed\libmchp_peripheral_32MX795F512L.a(int_enable_interrupts_lib.o)
 .debug_str     0x00000009        0x0 c:/program files/microchip/mplabc32/v2.02/bin/../lib/gcc/pic32mx/4.5.1/../../../../pic32mx/lib/speed\libmchp_peripheral_32MX795F512L.a(_rtcc_set_time_and_date_lib.o)
 .debug_str     0x00000009        0x0 c:/program files/microchip/mplabc32/v2.02/bin/../lib/gcc/pic32mx/4.5.1/../../../../pic32mx/lib/speed\libmchp_peripheral_32MX795F512L.a(_rtcc_wait_clock_off_lib.o)
 .debug_str     0x00000009        0x0 c:/program files/microchip/mplabc32/v2.02/bin/../lib/gcc/pic32mx/4.5.1/../../../../pic32mx/lib/speed\libc.a(calloc.o)
 .debug_str     0x00000009        0x0 c:/program files/microchip/mplabc32/v2.02/bin/../lib/gcc/pic32mx/4.5.1/../../../../pic32mx/lib/speed\libc.a(errno.o)
 .debug_str     0x00000009        0x0 c:/program files/microchip/mplabc32/v2.02/bin/../lib/gcc/pic32mx/4.5.1/../../../../pic32mx/lib/speed\libc.a(malloc.o)
 .debug_str     0x00000009        0x0 c:/program files/microchip/mplabc32/v2.02/bin/../lib/gcc/pic32mx/4.5.1/../../../../pic32mx/lib/speed\libc.a(sbrk.o)
 .debug_str     0x00000009        0x0 c:/program files/microchip/mplabc32/v2.02/bin/../lib/gcc/pic32mx/4.5.1/speed\libgcc.a(_lshrdi3.o)
 .debug_str     0x00000009        0x0 c:/program files/microchip/mplabc32/v2.02/bin/../lib/gcc/pic32mx/4.5.1/speed\libgcc.a(_ashldi3.o)

.debug_loc      0x00000000     0x1567
 *(.debug_loc)
 .debug_loc     0x00000000      0xa47 c:/program files/microchip/mplabc32/v2.02/bin/../lib/gcc/pic32mx/4.5.1/speed\libgcc.a(_udivdi3.o)
 .debug_loc     0x00000a47      0xa1d c:/program files/microchip/mplabc32/v2.02/bin/../lib/gcc/pic32mx/4.5.1/speed\libgcc.a(_umoddi3.o)
 .debug_loc     0x00001464       0x68 c:/program files/microchip/mplabc32/v2.02/bin/../lib/gcc/pic32mx/4.5.1/speed\libgcc.a(floatunsisf.o)
 .debug_loc     0x000014cc       0x5f c:/program files/microchip/mplabc32/v2.02/bin/../lib/gcc/pic32mx/4.5.1/speed\libgcc.a(_lshrdi3.o)
 .debug_loc     0x0000152b       0x3c c:/program files/microchip/mplabc32/v2.02/bin/../lib/gcc/pic32mx/4.5.1/speed\libgcc.a(_ashldi3.o)

.debug_macinfo
 *(.debug_macinfo)

.debug_weaknames
 *(.debug_weaknames)

.debug_funcnames
 *(.debug_funcnames)

.debug_typenames
 *(.debug_typenames)

.debug_varnames
 *(.debug_varnames)

.debug_pubtypes
                0x00000000      0x1aa
 *(.debug_pubtypes)
 .debug_pubtypes
                0x00000000       0x59 c:/program files/microchip/mplabc32/v2.02/bin/../lib/gcc/pic32mx/4.5.1/speed\libgcc.a(_udivdi3.o)
 .debug_pubtypes
                0x00000059       0x59 c:/program files/microchip/mplabc32/v2.02/bin/../lib/gcc/pic32mx/4.5.1/speed\libgcc.a(_umoddi3.o)
 .debug_pubtypes
                0x000000b2       0x34 c:/program files/microchip/mplabc32/v2.02/bin/../lib/gcc/pic32mx/4.5.1/speed\libgcc.a(floatunsisf.o)
 .debug_pubtypes
                0x000000e6       0x62 c:/program files/microchip/mplabc32/v2.02/bin/../lib/gcc/pic32mx/4.5.1/speed\libgcc.a(_lshrdi3.o)
 .debug_pubtypes
                0x00000148       0x62 c:/program files/microchip/mplabc32/v2.02/bin/../lib/gcc/pic32mx/4.5.1/speed\libgcc.a(_ashldi3.o)

.debug_ranges   0x00000000      0x708
 *(.debug_ranges)
 .debug_ranges  0x00000000       0xc0 c:/program files/microchip/mplabc32/v2.02/bin/../lib/gcc/pic32mx/4.5.1/speed\libgcc.a(_udivdi3.o)
 .debug_ranges  0x000000c0       0xf8 c:/program files/microchip/mplabc32/v2.02/bin/../lib/gcc/pic32mx/4.5.1/speed\libgcc.a(_umoddi3.o)
 .debug_ranges  0x000001b8       0x10 c:/program files/microchip/mplabc32/v2.02/bin/../lib/gcc/pic32mx/4.5.1/../../../../pic32mx/lib/speed\libc.a(atoi.o)
 .debug_ranges  0x000001c8       0x10 c:/program files/microchip/mplabc32/v2.02/bin/../lib/gcc/pic32mx/4.5.1/../../../../pic32mx/lib/speed\libc.a(atol.o)
 .debug_ranges  0x000001d8       0x28 c:/program files/microchip/mplabc32/v2.02/bin/../lib/gcc/pic32mx/4.5.1/../../../../pic32mx/lib/speed\libc.a(ctime.o)
 .debug_ranges  0x00000200       0x90 c:/program files/microchip/mplabc32/v2.02/bin/../lib/gcc/pic32mx/4.5.1/../../../../pic32mx/lib/speed\libc.a(ctypef.o)
 .debug_ranges  0x00000290       0x10 c:/program files/microchip/mplabc32/v2.02/bin/../lib/gcc/pic32mx/4.5.1/../../../../pic32mx/lib/speed\libc.a(strcat.o)
 .debug_ranges  0x000002a0       0x10 c:/program files/microchip/mplabc32/v2.02/bin/../lib/gcc/pic32mx/4.5.1/../../../../pic32mx/lib/speed\libc.a(strchr.o)
 .debug_ranges  0x000002b0       0x10 c:/program files/microchip/mplabc32/v2.02/bin/../lib/gcc/pic32mx/4.5.1/../../../../pic32mx/lib/speed\libc.a(strncpy.o)
 .debug_ranges  0x000002c0       0x10 c:/program files/microchip/mplabc32/v2.02/bin/../lib/gcc/pic32mx/4.5.1/../../../../pic32mx/lib/speed\libc.a(strstr.o)
 .debug_ranges  0x000002d0       0x10 c:/program files/microchip/mplabc32/v2.02/bin/../lib/gcc/pic32mx/4.5.1/../../../../pic32mx/lib/speed\libc.a(atof.o)
 .debug_ranges  0x000002e0       0x10 c:/program files/microchip/mplabc32/v2.02/bin/../lib/gcc/pic32mx/4.5.1/../../../../pic32mx/lib/speed\libc.a(sprintf_cdnopsuxX.eo)
 .debug_ranges  0x000002f0       0x10 c:/program files/microchip/mplabc32/v2.02/bin/../lib/gcc/pic32mx/4.5.1/../../../../pic32mx/lib/speed\libc.a(default-bootstrap-exception-handler.o)
 .debug_ranges  0x00000300       0x10 c:/program files/microchip/mplabc32/v2.02/bin/../lib/gcc/pic32mx/4.5.1/../../../../pic32mx/lib/speed\libc.a(default-on-reset.o)
 .debug_ranges  0x00000310       0x10 c:/program files/microchip/mplabc32/v2.02/bin/../lib/gcc/pic32mx/4.5.1/../../../../pic32mx/lib/speed\libc.a(default-on-bootstrap.o)
 .debug_ranges  0x00000320       0x10 c:/program files/microchip/mplabc32/v2.02/bin/../lib/gcc/pic32mx/4.5.1/../../../../pic32mx/lib/speed\libc.a(strncmp.o)
 .debug_ranges  0x00000330       0x18 c:/program files/microchip/mplabc32/v2.02/bin/../lib/gcc/pic32mx/4.5.1/../../../../pic32mx/lib/speed\libc.a(strtod.o)
 .debug_ranges  0x00000348       0x10 c:/program files/microchip/mplabc32/v2.02/bin/../lib/gcc/pic32mx/4.5.1/../../../../pic32mx/lib/speed\libc.a(doprnt_cdnopsuxX.eo)
 .debug_ranges  0x00000358       0x10 c:/program files/microchip/mplabc32/v2.02/bin/../lib/gcc/pic32mx/4.5.1/../../../../pic32mx/lib/speed\libc.a(_fputc_simple.o)
 .debug_ranges  0x00000368       0x10 c:/program files/microchip/mplabc32/v2.02/bin/../lib/gcc/pic32mx/4.5.1/../../../../pic32mx/lib/speed\libc.a(write.o)
 .debug_ranges  0x00000378       0x10 c:/program files/microchip/mplabc32/v2.02/bin/../lib/gcc/pic32mx/4.5.1/../../../../pic32mx/lib/speed\libc.a(_flsbuf_simple.o)
 .debug_ranges  0x00000388       0x10 c:/program files/microchip/mplabc32/v2.02/bin/../lib/gcc/pic32mx/4.5.1/../../../../pic32mx/lib/speed\libc.a(_mon_putc.o)
 .debug_ranges  0x00000398       0x10 c:/program files/microchip/mplabc32/v2.02/bin/../lib/gcc/pic32mx/4.5.1/../../../../pic32mx/lib/speed\libe.a(_strtod.o)
 .debug_ranges  0x000003a8       0x10 c:/program files/microchip/mplabc32/v2.02/bin/../lib/gcc/pic32mx/4.5.1/../../../../pic32mx/lib/speed\libe.a(_ldexp.o)
 .debug_ranges  0x000003b8       0x10 c:/program files/microchip/mplabc32/v2.02/bin/../lib/gcc/pic32mx/4.5.1/../../../../pic32mx/lib/speed\libmchp_peripheral.a(read_core_timer_lib.o)
 .debug_ranges  0x000003c8       0x10 c:/program files/microchip/mplabc32/v2.02/bin/../lib/gcc/pic32mx/4.5.1/../../../../pic32mx/lib/speed\libmchp_peripheral.a(write_core_timer_lib.o)
 .debug_ranges  0x000003d8       0x38 c:/program files/microchip/mplabc32/v2.02/bin/../lib/gcc/pic32mx/4.5.1/../../../../pic32mx/lib/speed\libmchp_peripheral_32MX795F512L.a(eth_ack_packet_lib.o)
 .debug_ranges  0x00000410       0x18 c:/program files/microchip/mplabc32/v2.02/bin/../lib/gcc/pic32mx/4.5.1/../../../../pic32mx/lib/speed\libmchp_peripheral_32MX795F512L.a(eth_descriptors_add_lib.o)
 .debug_ranges  0x00000428       0x10 c:/program files/microchip/mplabc32/v2.02/bin/../lib/gcc/pic32mx/4.5.1/../../../../pic32mx/lib/speed\libmchp_peripheral_32MX795F512L.a(eth_init_lib.o)
 .debug_ranges  0x00000438       0x10 c:/program files/microchip/mplabc32/v2.02/bin/../lib/gcc/pic32mx/4.5.1/../../../../pic32mx/lib/speed\libmchp_peripheral_32MX795F512L.a(eth_mac_open_lib.o)
 .debug_ranges  0x00000448       0x20 c:/program files/microchip/mplabc32/v2.02/bin/../lib/gcc/pic32mx/4.5.1/../../../../pic32mx/lib/speed\libmchp_peripheral_32MX795F512L.a(eth_mac_set_address_max_lib.o)
 .debug_ranges  0x00000468       0x10 c:/program files/microchip/mplabc32/v2.02/bin/../lib/gcc/pic32mx/4.5.1/../../../../pic32mx/lib/speed\libmchp_peripheral_32MX795F512L.a(eth_rx_buffers_append_lib.o)
 .debug_ranges  0x00000478       0x38 c:/program files/microchip/mplabc32/v2.02/bin/../lib/gcc/pic32mx/4.5.1/../../../../pic32mx/lib/speed\libmchp_peripheral_32MX795F512L.a(eth_rx_filters_lib.o)
 .debug_ranges  0x000004b0       0x18 c:/program files/microchip/mplabc32/v2.02/bin/../lib/gcc/pic32mx/4.5.1/../../../../pic32mx/lib/speed\libmchp_peripheral_32MX795F512L.a(eth_rx_get_packet_lib.o)
 .debug_ranges  0x000004c8       0x10 c:/program files/microchip/mplabc32/v2.02/bin/../lib/gcc/pic32mx/4.5.1/../../../../pic32mx/lib/speed\libmchp_peripheral_32MX795F512L.a(eth_rx_set_buffer_size_lib.o)
 .debug_ranges  0x000004d8       0x28 c:/program files/microchip/mplabc32/v2.02/bin/../lib/gcc/pic32mx/4.5.1/../../../../pic32mx/lib/speed\libmchp_peripheral_32MX795F512L.a(eth_tx_packet_lib.o)
 .debug_ranges  0x00000500       0x10 c:/program files/microchip/mplabc32/v2.02/bin/../lib/gcc/pic32mx/4.5.1/../../../../pic32mx/lib/speed\libmchp_peripheral_32MX795F512L.a(_eth_append_busy_list_lib.o)
 .debug_ranges  0x00000510       0x38 c:/program files/microchip/mplabc32/v2.02/bin/../lib/gcc/pic32mx/4.5.1/../../../../pic32mx/lib/speed\libmchp_peripheral_32MX795F512L.a(eth_miim_access.o)
 .debug_ranges  0x00000548       0x10 c:/program files/microchip/mplabc32/v2.02/bin/../lib/gcc/pic32mx/4.5.1/../../../../pic32mx/lib/speed\libmchp_peripheral_32MX795F512L.a(soft_reset_lib.o)
 .debug_ranges  0x00000558       0x18 c:/program files/microchip/mplabc32/v2.02/bin/../lib/gcc/pic32mx/4.5.1/../../../../pic32mx/lib/speed\libmchp_peripheral_32MX795F512L.a(pcache.o)
 .debug_ranges  0x00000570       0x10 c:/program files/microchip/mplabc32/v2.02/bin/../lib/gcc/pic32mx/4.5.1/../../../../pic32mx/lib/speed\libmchp_peripheral_32MX795F512L.a(set_core_sw0_leg_lib.o)
 .debug_ranges  0x00000580       0x10 c:/program files/microchip/mplabc32/v2.02/bin/../lib/gcc/pic32mx/4.5.1/../../../../pic32mx/lib/speed\libmchp_peripheral_32MX795F512L.a(int_disable_interrupts_lib.o)
 .debug_ranges  0x00000590       0x10 c:/program files/microchip/mplabc32/v2.02/bin/../lib/gcc/pic32mx/4.5.1/../../../../pic32mx/lib/speed\libmchp_peripheral_32MX795F512L.a(int_restore_interrupts_lib.o)
 .debug_ranges  0x000005a0       0x10 c:/program files/microchip/mplabc32/v2.02/bin/../lib/gcc/pic32mx/4.5.1/../../../../pic32mx/lib/speed\libmchp_peripheral_32MX795F512L.a(int_enable_mv_int_lib.o)
 .debug_ranges  0x000005b0       0x50 c:/program files/microchip/mplabc32/v2.02/bin/../lib/gcc/pic32mx/4.5.1/../../../../pic32mx/lib/speed\libmchp_peripheral_32MX795F512L.a(int_tbl_lib.o)
 .debug_ranges  0x00000600       0x10 c:/program files/microchip/mplabc32/v2.02/bin/../lib/gcc/pic32mx/4.5.1/../../../../pic32mx/lib/speed\libmchp_peripheral_32MX795F512L.a(rtcc_init_lib.o)
 .debug_ranges  0x00000610       0x10 c:/program files/microchip/mplabc32/v2.02/bin/../lib/gcc/pic32mx/4.5.1/../../../../pic32mx/lib/speed\libmchp_peripheral_32MX795F512L.a(rtcc_set_time_date_lib.o)
 .debug_ranges  0x00000620       0x10 c:/program files/microchip/mplabc32/v2.02/bin/../lib/gcc/pic32mx/4.5.1/../../../../pic32mx/lib/speed\libmchp_peripheral_32MX795F512L.a(rtcc_open_lib.o)
 .debug_ranges  0x00000630       0x10 c:/program files/microchip/mplabc32/v2.02/bin/../lib/gcc/pic32mx/4.5.1/../../../../pic32mx/lib/speed\libmchp_peripheral_32MX795F512L.a(spi_getc_spi1_lib_legacy.o)
 .debug_ranges  0x00000640       0x10 c:/program files/microchip/mplabc32/v2.02/bin/../lib/gcc/pic32mx/4.5.1/../../../../pic32mx/lib/speed\libmchp_peripheral_32MX795F512L.a(spi_open_spi1_lib_legacy.o)
 .debug_ranges  0x00000650       0x10 c:/program files/microchip/mplabc32/v2.02/bin/../lib/gcc/pic32mx/4.5.1/../../../../pic32mx/lib/speed\libmchp_peripheral_32MX795F512L.a(port_set_pins_digital_in_lib.o)
 .debug_ranges  0x00000660       0x10 c:/program files/microchip/mplabc32/v2.02/bin/../lib/gcc/pic32mx/4.5.1/../../../../pic32mx/lib/speed\libmchp_peripheral_32MX795F512L.a(port_set_pins_digital_out_lib.o)
 .debug_ranges  0x00000670       0x10 c:/program files/microchip/mplabc32/v2.02/bin/../lib/gcc/pic32mx/4.5.1/../../../../pic32mx/lib/speed\libmchp_peripheral_32MX795F512L.a(int_enable_interrupts_lib.o)
 .debug_ranges  0x00000680       0x10 c:/program files/microchip/mplabc32/v2.02/bin/../lib/gcc/pic32mx/4.5.1/../../../../pic32mx/lib/speed\libmchp_peripheral_32MX795F512L.a(_rtcc_set_time_and_date_lib.o)
 .debug_ranges  0x00000690       0x18 c:/program files/microchip/mplabc32/v2.02/bin/../lib/gcc/pic32mx/4.5.1/../../../../pic32mx/lib/speed\libmchp_peripheral_32MX795F512L.a(_rtcc_wait_clock_off_lib.o)
 .debug_ranges  0x000006a8       0x10 c:/program files/microchip/mplabc32/v2.02/bin/../lib/gcc/pic32mx/4.5.1/../../../../pic32mx/lib/speed\libc.a(calloc.o)
 .debug_ranges  0x000006b8       0x20 c:/program files/microchip/mplabc32/v2.02/bin/../lib/gcc/pic32mx/4.5.1/../../../../pic32mx/lib/speed\libc.a(malloc.o)
 .debug_ranges  0x000006d8       0x30 c:/program files/microchip/mplabc32/v2.02/bin/../lib/gcc/pic32mx/4.5.1/../../../../pic32mx/lib/speed\libc.a(sbrk.o)

.gnu.attributes
                0x00000000       0x10
 *(.gnu.attributes)
 .gnu.attributes
                0x00000000       0x10 output\main.o
 .gnu.attributes
                0x00000010       0x10 output\IntQueueTimer.o
 .gnu.attributes
                0x00000020       0x10 output\port.o
 .gnu.attributes
                0x00000030       0x10 output\queue.o
 .gnu.attributes
                0x00000040       0x10 output\tasks.o
 .gnu.attributes
                0x00000050       0x10 output\list.o
 .gnu.attributes
                0x00000060       0x10 output\IntQueue.o
 .gnu.attributes
                0x00000070       0x10 output\QPeek.o
 .gnu.attributes
                0x00000080       0x10 output\lcd.o
 .gnu.attributes
                0x00000090       0x10 output\prvTaskTCPIP.o
 .gnu.attributes
                0x000000a0       0x10 output\heap_2.o
 .gnu.attributes
                0x000000b0       0x10 output\usb_host.o
 .gnu.attributes
                0x000000c0       0x10 output\usb_config.o
 .gnu.attributes
                0x000000d0       0x10 output\CustomHTTPApp.o
 .gnu.attributes
                0x000000e0       0x10 output\usb_host_generic.o
 .gnu.attributes
                0x000000f0       0x10 output\FSIO.o
 .gnu.attributes
                0x00000100       0x10 output\UDP.o
 .gnu.attributes
                0x00000110       0x10 output\ARP.o
 .gnu.attributes
                0x00000120       0x10 output\Delay.o
 .gnu.attributes
                0x00000130       0x10 output\DHCP.o
 .gnu.attributes
                0x00000140       0x10 output\DNS.o
 .gnu.attributes
                0x00000150       0x10 output\DstaDPlusClientUDP.o
 .gnu.attributes
                0x00000160       0x10 output\ETHPIC32ExtPhy.o
 .gnu.attributes
                0x00000170       0x10 output\ETHPIC32ExtPhyDP83848.o
 .gnu.attributes
                0x00000180       0x10 output\ETHPIC32IntMac.o
 .gnu.attributes
                0x00000190       0x10 output\FileSystem.o
 .gnu.attributes
                0x000001a0       0x10 output\FTP.o
 .gnu.attributes
                0x000001b0       0x10 output\Hashes.o
 .gnu.attributes
                0x000001c0       0x10 output\Helpers.o
 .gnu.attributes
                0x000001d0       0x10 output\HTTP2.o
 .gnu.attributes
                0x000001e0       0x10 output\ICMP.o
 .gnu.attributes
                0x000001f0       0x10 output\IP.o
 .gnu.attributes
                0x00000200       0x10 output\MPFS2.o
 .gnu.attributes
                0x00000210       0x10 output\Random.o
 .gnu.attributes
                0x00000220       0x10 output\SNTP.o
 .gnu.attributes
                0x00000230       0x10 output\StackTsk.o
 .gnu.attributes
                0x00000240       0x10 output\TCP.o
 .gnu.attributes
                0x00000250       0x10 output\Tick.o
 .gnu.attributes
                0x00000260       0x10 output\MPFSImg2.o
 .gnu.attributes
                0x00000270       0x10 output\SD-SPI.o
 .gnu.attributes
                0x00000280       0x10 output\prvTaskUSB.o
 .gnu.attributes
                0x00000290       0x10 output\prvTaskFS.o
 .gnu.attributes
                0x000002a0       0x10 output\MACread.o
 .gnu.attributes
                0x000002b0       0x10 output\SMTP.o
 .gnu.attributes
                0x000002c0       0x10 output\DprsSMTP.o
 .gnu.attributes
                0x000002d0       0x10 output\serial.o
 .gnu.attributes
                0x000002e0       0x10 output\comtest.o
 .gnu.attributes
                0x000002f0       0x10 output\DHCPs.o
 .gnu.attributes
                0x00000300       0x10 output\NBNS.o
 .gnu.attributes
                0x00000310       0x10 c:/program files/microchip/mplabc32/v2.02/bin/../lib/gcc/pic32mx/4.5.1/speed\libgcc.a(_udivdi3.o)
 .gnu.attributes
                0x00000320       0x10 c:/program files/microchip/mplabc32/v2.02/bin/../lib/gcc/pic32mx/4.5.1/speed\libgcc.a(_umoddi3.o)
 .gnu.attributes
                0x00000330       0x10 c:/program files/microchip/mplabc32/v2.02/bin/../lib/gcc/pic32mx/4.5.1/speed\libgcc.a(floatunsisf.o)
 .gnu.attributes
                0x00000340       0x10 c:/program files/microchip/mplabc32/v2.02/bin/../lib/gcc/pic32mx/4.5.1/../../../../pic32mx/lib/speed\libc.a(atoi.o)
 .gnu.attributes
                0x00000350       0x10 c:/program files/microchip/mplabc32/v2.02/bin/../lib/gcc/pic32mx/4.5.1/../../../../pic32mx/lib/speed\libc.a(atol.o)
 .gnu.attributes
                0x00000360       0x10 c:/program files/microchip/mplabc32/v2.02/bin/../lib/gcc/pic32mx/4.5.1/../../../../pic32mx/lib/speed\libc.a(ctime.o)
 .gnu.attributes
                0x00000370       0x10 c:/program files/microchip/mplabc32/v2.02/bin/../lib/gcc/pic32mx/4.5.1/../../../../pic32mx/lib/speed\libc.a(ctype.o)
 .gnu.attributes
                0x00000380       0x10 c:/program files/microchip/mplabc32/v2.02/bin/../lib/gcc/pic32mx/4.5.1/../../../../pic32mx/lib/speed\libc.a(ctypef.o)
 .gnu.attributes
                0x00000390       0x10 c:/program files/microchip/mplabc32/v2.02/bin/../lib/gcc/pic32mx/4.5.1/../../../../pic32mx/lib/speed\libc.a(strcat.o)
 .gnu.attributes
                0x000003a0       0x10 c:/program files/microchip/mplabc32/v2.02/bin/../lib/gcc/pic32mx/4.5.1/../../../../pic32mx/lib/speed\libc.a(strchr.o)
 .gnu.attributes
                0x000003b0       0x10 c:/program files/microchip/mplabc32/v2.02/bin/../lib/gcc/pic32mx/4.5.1/../../../../pic32mx/lib/speed\libc.a(strncpy.o)
 .gnu.attributes
                0x000003c0       0x10 c:/program files/microchip/mplabc32/v2.02/bin/../lib/gcc/pic32mx/4.5.1/../../../../pic32mx/lib/speed\libc.a(strstr.o)
 .gnu.attributes
                0x000003d0       0x10 c:/program files/microchip/mplabc32/v2.02/bin/../lib/gcc/pic32mx/4.5.1/../../../../pic32mx/lib/speed\libc.a(atof.o)
 .gnu.attributes
                0x000003e0       0x10 c:/program files/microchip/mplabc32/v2.02/bin/../lib/gcc/pic32mx/4.5.1/../../../../pic32mx/lib/speed\libc.a(sprintf_cdnopsuxX.eo)
 .gnu.attributes
                0x000003f0       0x10 c:/program files/microchip/mplabc32/v2.02/bin/../lib/gcc/pic32mx/4.5.1/../../../../pic32mx/lib/speed\libc.a(default-bootstrap-exception-handler.o)
 .gnu.attributes
                0x00000400       0x10 c:/program files/microchip/mplabc32/v2.02/bin/../lib/gcc/pic32mx/4.5.1/../../../../pic32mx/lib/speed\libc.a(default-on-reset.o)
 .gnu.attributes
                0x00000410       0x10 c:/program files/microchip/mplabc32/v2.02/bin/../lib/gcc/pic32mx/4.5.1/../../../../pic32mx/lib/speed\libc.a(default-on-bootstrap.o)
 .gnu.attributes
                0x00000420       0x10 c:/program files/microchip/mplabc32/v2.02/bin/../lib/gcc/pic32mx/4.5.1/../../../../pic32mx/lib/speed\libc.a(strncmp.o)
 .gnu.attributes
                0x00000430       0x10 c:/program files/microchip/mplabc32/v2.02/bin/../lib/gcc/pic32mx/4.5.1/../../../../pic32mx/lib/speed\libc.a(strtod.o)
 .gnu.attributes
                0x00000440       0x10 c:/program files/microchip/mplabc32/v2.02/bin/../lib/gcc/pic32mx/4.5.1/../../../../pic32mx/lib/speed\libc.a(doprnt_cdnopsuxX.eo)
 .gnu.attributes
                0x00000450       0x10 c:/program files/microchip/mplabc32/v2.02/bin/../lib/gcc/pic32mx/4.5.1/../../../../pic32mx/lib/speed\libc.a(_fputc_simple.o)
 .gnu.attributes
                0x00000460       0x10 c:/program files/microchip/mplabc32/v2.02/bin/../lib/gcc/pic32mx/4.5.1/../../../../pic32mx/lib/speed\libc.a(write.o)
 .gnu.attributes
                0x00000470       0x10 c:/program files/microchip/mplabc32/v2.02/bin/../lib/gcc/pic32mx/4.5.1/../../../../pic32mx/lib/speed\libc.a(_iob.o)
 .gnu.attributes
                0x00000480       0x10 c:/program files/microchip/mplabc32/v2.02/bin/../lib/gcc/pic32mx/4.5.1/../../../../pic32mx/lib/speed\libc.a(_flsbuf_simple.o)
 .gnu.attributes
                0x00000490       0x10 c:/program files/microchip/mplabc32/v2.02/bin/../lib/gcc/pic32mx/4.5.1/../../../../pic32mx/lib/speed\libc.a(_mon_putc.o)
 .gnu.attributes
                0x000004a0       0x10 c:/program files/microchip/mplabc32/v2.02/bin/../lib/gcc/pic32mx/4.5.1/../../../../pic32mx/lib/speed\libc.a(c32_uart.o)
 .gnu.attributes
                0x000004b0       0x10 c:/program files/microchip/mplabc32/v2.02/bin/../lib/gcc/pic32mx/4.5.1/../../../../pic32mx/lib/speed\libe.a(_strtod.o)
 .gnu.attributes
                0x000004c0       0x10 c:/program files/microchip/mplabc32/v2.02/bin/../lib/gcc/pic32mx/4.5.1/../../../../pic32mx/lib/speed\libe.a(_ldexp.o)
 .gnu.attributes
                0x000004d0       0x10 c:/program files/microchip/mplabc32/v2.02/bin/../lib/gcc/pic32mx/4.5.1/../../../../pic32mx/lib/speed\libmchp_peripheral.a(read_core_timer_lib.o)
 .gnu.attributes
                0x000004e0       0x10 c:/program files/microchip/mplabc32/v2.02/bin/../lib/gcc/pic32mx/4.5.1/../../../../pic32mx/lib/speed\libmchp_peripheral.a(write_core_timer_lib.o)
 .gnu.attributes
                0x000004f0       0x10 c:/program files/microchip/mplabc32/v2.02/bin/../lib/gcc/pic32mx/4.5.1/../../../../pic32mx/lib/speed\libmchp_peripheral_32MX795F512L.a(eth_ack_packet_lib.o)
 .gnu.attributes
                0x00000500       0x10 c:/program files/microchip/mplabc32/v2.02/bin/../lib/gcc/pic32mx/4.5.1/../../../../pic32mx/lib/speed\libmchp_peripheral_32MX795F512L.a(eth_descriptors_add_lib.o)
 .gnu.attributes
                0x00000510       0x10 c:/program files/microchip/mplabc32/v2.02/bin/../lib/gcc/pic32mx/4.5.1/../../../../pic32mx/lib/speed\libmchp_peripheral_32MX795F512L.a(eth_init_lib.o)
 .gnu.attributes
                0x00000520       0x10 c:/program files/microchip/mplabc32/v2.02/bin/../lib/gcc/pic32mx/4.5.1/../../../../pic32mx/lib/speed\libmchp_peripheral_32MX795F512L.a(eth_mac_open_lib.o)
 .gnu.attributes
                0x00000530       0x10 c:/program files/microchip/mplabc32/v2.02/bin/../lib/gcc/pic32mx/4.5.1/../../../../pic32mx/lib/speed\libmchp_peripheral_32MX795F512L.a(eth_mac_set_address_max_lib.o)
 .gnu.attributes
                0x00000540       0x10 c:/program files/microchip/mplabc32/v2.02/bin/../lib/gcc/pic32mx/4.5.1/../../../../pic32mx/lib/speed\libmchp_peripheral_32MX795F512L.a(eth_rx_buffers_append_lib.o)
 .gnu.attributes
                0x00000550       0x10 c:/program files/microchip/mplabc32/v2.02/bin/../lib/gcc/pic32mx/4.5.1/../../../../pic32mx/lib/speed\libmchp_peripheral_32MX795F512L.a(eth_rx_filters_lib.o)
 .gnu.attributes
                0x00000560       0x10 c:/program files/microchip/mplabc32/v2.02/bin/../lib/gcc/pic32mx/4.5.1/../../../../pic32mx/lib/speed\libmchp_peripheral_32MX795F512L.a(eth_rx_get_packet_lib.o)
 .gnu.attributes
                0x00000570       0x10 c:/program files/microchip/mplabc32/v2.02/bin/../lib/gcc/pic32mx/4.5.1/../../../../pic32mx/lib/speed\libmchp_peripheral_32MX795F512L.a(eth_rx_set_buffer_size_lib.o)
 .gnu.attributes
                0x00000580       0x10 c:/program files/microchip/mplabc32/v2.02/bin/../lib/gcc/pic32mx/4.5.1/../../../../pic32mx/lib/speed\libmchp_peripheral_32MX795F512L.a(eth_tx_packet_lib.o)
 .gnu.attributes
                0x00000590       0x10 c:/program files/microchip/mplabc32/v2.02/bin/../lib/gcc/pic32mx/4.5.1/../../../../pic32mx/lib/speed\libmchp_peripheral_32MX795F512L.a(_eth_append_busy_list_lib.o)
 .gnu.attributes
                0x000005a0       0x10 c:/program files/microchip/mplabc32/v2.02/bin/../lib/gcc/pic32mx/4.5.1/../../../../pic32mx/lib/speed\libmchp_peripheral_32MX795F512L.a(eth_miim_access.o)
 .gnu.attributes
                0x000005b0       0x10 c:/program files/microchip/mplabc32/v2.02/bin/../lib/gcc/pic32mx/4.5.1/../../../../pic32mx/lib/speed\libmchp_peripheral_32MX795F512L.a(soft_reset_lib.o)
 .gnu.attributes
                0x000005c0       0x10 c:/program files/microchip/mplabc32/v2.02/bin/../lib/gcc/pic32mx/4.5.1/../../../../pic32mx/lib/speed\libmchp_peripheral_32MX795F512L.a(pcache.o)
 .gnu.attributes
                0x000005d0       0x10 c:/program files/microchip/mplabc32/v2.02/bin/../lib/gcc/pic32mx/4.5.1/../../../../pic32mx/lib/speed\libmchp_peripheral_32MX795F512L.a(set_core_sw0_leg_lib.o)
 .gnu.attributes
                0x000005e0       0x10 c:/program files/microchip/mplabc32/v2.02/bin/../lib/gcc/pic32mx/4.5.1/../../../../pic32mx/lib/speed\libmchp_peripheral_32MX795F512L.a(int_disable_interrupts_lib.o)
 .gnu.attributes
                0x000005f0       0x10 c:/program files/microchip/mplabc32/v2.02/bin/../lib/gcc/pic32mx/4.5.1/../../../../pic32mx/lib/speed\libmchp_peripheral_32MX795F512L.a(int_restore_interrupts_lib.o)
 .gnu.attributes
                0x00000600       0x10 c:/program files/microchip/mplabc32/v2.02/bin/../lib/gcc/pic32mx/4.5.1/../../../../pic32mx/lib/speed\libmchp_peripheral_32MX795F512L.a(int_enable_mv_int_lib.o)
 .gnu.attributes
                0x00000610       0x10 c:/program files/microchip/mplabc32/v2.02/bin/../lib/gcc/pic32mx/4.5.1/../../../../pic32mx/lib/speed\libmchp_peripheral_32MX795F512L.a(int_tbl_lib.o)
 .gnu.attributes
                0x00000620       0x10 c:/program files/microchip/mplabc32/v2.02/bin/../lib/gcc/pic32mx/4.5.1/../../../../pic32mx/lib/speed\libmchp_peripheral_32MX795F512L.a(rtcc_init_lib.o)
 .gnu.attributes
                0x00000630       0x10 c:/program files/microchip/mplabc32/v2.02/bin/../lib/gcc/pic32mx/4.5.1/../../../../pic32mx/lib/speed\libmchp_peripheral_32MX795F512L.a(rtcc_set_time_date_lib.o)
 .gnu.attributes
                0x00000640       0x10 c:/program files/microchip/mplabc32/v2.02/bin/../lib/gcc/pic32mx/4.5.1/../../../../pic32mx/lib/speed\libmchp_peripheral_32MX795F512L.a(rtcc_open_lib.o)
 .gnu.attributes
                0x00000650       0x10 c:/program files/microchip/mplabc32/v2.02/bin/../lib/gcc/pic32mx/4.5.1/../../../../pic32mx/lib/speed\libmchp_peripheral_32MX795F512L.a(spi_getc_spi1_lib_legacy.o)
 .gnu.attributes
                0x00000660       0x10 c:/program files/microchip/mplabc32/v2.02/bin/../lib/gcc/pic32mx/4.5.1/../../../../pic32mx/lib/speed\libmchp_peripheral_32MX795F512L.a(spi_open_spi1_lib_legacy.o)
 .gnu.attributes
                0x00000670       0x10 c:/program files/microchip/mplabc32/v2.02/bin/../lib/gcc/pic32mx/4.5.1/../../../../pic32mx/lib/speed\libmchp_peripheral_32MX795F512L.a(spi_brg_tbl_lib_legacy.o)
 .gnu.attributes
                0x00000680       0x10 c:/program files/microchip/mplabc32/v2.02/bin/../lib/gcc/pic32mx/4.5.1/../../../../pic32mx/lib/speed\libmchp_peripheral_32MX795F512L.a(port_set_pins_digital_in_lib.o)
 .gnu.attributes
                0x00000690       0x10 c:/program files/microchip/mplabc32/v2.02/bin/../lib/gcc/pic32mx/4.5.1/../../../../pic32mx/lib/speed\libmchp_peripheral_32MX795F512L.a(port_set_pins_digital_out_lib.o)
 .gnu.attributes
                0x000006a0       0x10 c:/program files/microchip/mplabc32/v2.02/bin/../lib/gcc/pic32mx/4.5.1/../../../../pic32mx/lib/speed\libmchp_peripheral_32MX795F512L.a(_ports_tbl_libp.o)
 .gnu.attributes
                0x000006b0       0x10 c:/program files/microchip/mplabc32/v2.02/bin/../lib/gcc/pic32mx/4.5.1/../../../../pic32mx/lib/speed\libmchp_peripheral_32MX795F512L.a(int_enable_interrupts_lib.o)
 .gnu.attributes
                0x000006c0       0x10 c:/program files/microchip/mplabc32/v2.02/bin/../lib/gcc/pic32mx/4.5.1/../../../../pic32mx/lib/speed\libmchp_peripheral_32MX795F512L.a(_rtcc_set_time_and_date_lib.o)
 .gnu.attributes
                0x000006d0       0x10 c:/program files/microchip/mplabc32/v2.02/bin/../lib/gcc/pic32mx/4.5.1/../../../../pic32mx/lib/speed\libmchp_peripheral_32MX795F512L.a(_rtcc_wait_clock_off_lib.o)
 .gnu.attributes
                0x000006e0       0x10 c:/program files/microchip/mplabc32/v2.02/bin/../lib/gcc/pic32mx/4.5.1/../../../../pic32mx/lib/speed\libc.a(calloc.o)
 .gnu.attributes
                0x000006f0       0x10 c:/program files/microchip/mplabc32/v2.02/bin/../lib/gcc/pic32mx/4.5.1/../../../../pic32mx/lib/speed\libc.a(errno.o)
 .gnu.attributes
                0x00000700       0x10 c:/program files/microchip/mplabc32/v2.02/bin/../lib/gcc/pic32mx/4.5.1/../../../../pic32mx/lib/speed\libc.a(malloc.o)
 .gnu.attributes
                0x00000710       0x10 c:/program files/microchip/mplabc32/v2.02/bin/../lib/gcc/pic32mx/4.5.1/../../../../pic32mx/lib/speed\libc.a(sbrk.o)
 .gnu.attributes
                0x00000720       0x10 c:/program files/microchip/mplabc32/v2.02/bin/../lib/gcc/pic32mx/4.5.1/speed\libgcc.a(_lshrdi3.o)
 .gnu.attributes
                0x00000730       0x10 c:/program files/microchip/mplabc32/v2.02/bin/../lib/gcc/pic32mx/4.5.1/speed\libgcc.a(_ashldi3.o)
                0x00000001                __MPLAB_BUILD = 0x1
                0x00000000                _min_heap_size = 0x0
LOAD c:/program files/microchip/mplabc32/v2.02/bin/../lib/gcc/pic32mx/4.5.1/speed\libgcc.a
START GROUP
LOAD c:/program files/microchip/mplabc32/v2.02/bin/../lib/gcc/pic32mx/4.5.1/../../../../pic32mx/lib/speed\libdebug.a
LOAD c:/program files/microchip/mplabc32/v2.02/bin/../lib/gcc/pic32mx/4.5.1/../../../../pic32mx/lib/speed\libc.a
LOAD c:/program files/microchip/mplabc32/v2.02/bin/../lib/gcc/pic32mx/4.5.1/../../../../pic32mx/lib/speed\libm.a
LOAD c:/program files/microchip/mplabc32/v2.02/bin/../lib/gcc/pic32mx/4.5.1/../../../../pic32mx/lib/speed\libe.a
LOAD c:/program files/microchip/mplabc32/v2.02/bin/../lib/gcc/pic32mx/4.5.1/../../../../pic32mx/lib/speed\libdsp.a
LOAD c:/program files/microchip/mplabc32/v2.02/bin/../lib/gcc/pic32mx/4.5.1/../../../../pic32mx/lib/speed\libmchp_peripheral.a
LOAD c:/program files/microchip/mplabc32/v2.02/bin/../lib/gcc/pic32mx/4.5.1/../../../../pic32mx/lib/speed\libmchp_peripheral_32MX795F512L.a
END GROUP
LOAD c:/program files/microchip/mplabc32/v2.02/bin/../lib/gcc/pic32mx/4.5.1/speed\libgcc.a
OUTPUT(./output\Node.elf elf32-tradlittlemips)
LOAD stack
LOAD data_init

.stack          0xa001cd18      0x400
 .stack         0xa001cd18      0x400 stack

.bss            0xa000273c    0x17cf4
 .bss           0xa000273c     0xe290 output\heap_2.o
 .bss           0xa00109cc     0x5df8 output\TCP.o
 .bss           0xa00167c4     0x3c6c output\ETHPIC32IntMac.o

.data           0xa001a430      0x85c
 .data          0xa001a430      0x85c output\DstaDPlusClientUDP.o
                0xa001a430                aprs_symbol
                0xa001aa18                crc_tabccitt

.bss            0xa001ac8c     0x1298
 .bss           0xa001ac8c      0x7d0 output\port.o
                0xa001ac8c                xISRStack
 .bss           0xa001b45c      0x4bc output\DstaDPlusClientUDP.o
 .bss           0xa001b918      0x320 output\prvTaskUSB.o
 .bss           0xa001bc38      0x2ec output\CustomHTTPApp.o

.bss            0xa001c000      0x754
 .bss           0xa001c000      0x200 output\usb_host.o
 .bss           0xa001c200      0x190 output\IntQueue.o
 .bss           0xa001c390      0x174 output\FTP.o
 .bss           0xa001c504      0x15c output\prvTaskFS.o
 .bss           0xa001c660       0xf4 output\DprsSMTP.o

.data           0xa001bf24       0xcc
 .data          0xa001bf24       0xcc output\prvTaskUSB.o
                0xa001bf30                NullVoice0
                0xa001bf3c                NullVoice1
                0xa001bf48                NullVoice_ID31
                0xa001bf54                ConnectedMsg

.bss            0xa001c754      0x18c
 .bss           0xa001c754       0xc8 output\tasks.o
 .bss           0xa001c81c       0xc4 output\HTTP2.o

.data           0xa001c8e0       0x98
 .data          0xa001c8e0       0x98 output\FTP.o
                0xa001c8e0                _ftpCommandString
                0xa001c928                _ftpResponseString

.bss            0xa001c978      0x214
 .bss           0xa001c978       0x80 output\DHCP.o
 .bss           0xa001c9f8       0x78 output\main.o
 .bss           0xa001ca70       0x6c output\SNTP.o
 .bss           0xa001cadc       0x60 output\MPFS2.o
 .bss           0xa001cb3c       0x50 output\ARP.o

.bss            0xa001cb90       0xac
 .bss           0xa001cb90       0x40 c:/program files/microchip/mplabc32/v2.02/bin/../lib/gcc/pic32mx/4.5.1/../../../../pic32mx/lib/speed\libc.a(ctime.o)
 .bss           0xa001cbd0       0x40 c:/program files/microchip/mplabc32/v2.02/bin/../lib/gcc/pic32mx/4.5.1/../../../../pic32mx/lib/speed\libc.a(_iob.o)
                0xa001cbd0                _sibuf
                0xa001cbf0                _sobuf
 .bss           0xa001cc10       0x2c output\NBNS.o

.data           0xa001cc3c       0x28
 .data          0xa001cc3c       0x28 output\CustomHTTPApp.o

.bss            0xa001cc64       0x6c
 .bss           0xa001cc64       0x28 output\SD-SPI.o
 .bss           0xa001cc8c       0x24 output\DHCPs.o
 .bss           0xa001ccb0       0x20 output\prvTaskTCPIP.o

.data           0xa001bff0       0x10
 .data          0xa001bff0       0x10 output\usb_config.o
                0xa001bff0                usbClientDrvTable

.data           0xa001ccd0       0x10
 .data          0xa001ccd0       0x10 output\prvTaskFS.o

.bss            0xa001cce0       0x1c
 .bss           0xa001cce0       0x10 output\MACread.o
 .bss           0xa001ccf0        0xc output\DNS.o

.text           0x9d007e50    0x102ec
 .text          0x9d007e50    0x102ec output\FSIO.o
                0x9d007e50                FSInit
                0x9d007fac                FILEfind
                0x9d0096ec                FILEopen
                0x9d00999c                FILEget_next_cluster
                0x9d009af0                DISKmount
                0x9d009c04                LoadMBR
                0x9d00a014                LoadBootSector
                0x9d00a800                GetFullClusterNumber
                0x9d00a848                Write_File_Entry
                0x9d00a998                FAT_erase_cluster_chain
                0x9d00ab48                Cache_File_Entry
                0x9d00aee4                CreateFileEntry
                0x9d00b530                CreateFirstCluster
                0x9d00b600                FindEmptyEntries
                0x9d00b934                PopulateEntries
                0x9d00badc                Alias_LFN_Object
                0x9d00c51c                CacheTime
                0x9d00c848                FILEallocate_new_cluster
                0x9d00c98c                FATfindEmptyCluster
                0x9d00cb20                FSfclose
                0x9d00cd44                Fill_File_Object
                0x9d00d024                Fill_LFN_Object
                0x9d00d180                LoadDirAttrib
                0x9d00d2a0                FILEerase
                0x9d00d50c                FSrename
                0x9d00d71c                wFSrename
                0x9d00d764                wFSfopen
                0x9d00d7ac                FSfopen
                0x9d00e10c                FSftell
                0x9d00e124                FSremove
                0x9d00e37c                wFSremove
                0x9d00e3bc                FSrewind
                0x9d00e418                FSerror
                0x9d00e424                FileObjectCopy
                0x9d00e4a0                FILECreateHeadCluster
                0x9d00e61c                EraseCluster
                0x9d00e748                ReadByte
                0x9d00e76c                ReadWord
                0x9d00e7e0                ReadDWord
                0x9d00e868                Cluster2Sector
                0x9d00e944                FSattrib
                0x9d00ea84                FSfwrite
                0x9d00ef1c                flushData
                0x9d00efbc                FSfeof
                0x9d00efe4                FSfread
                0x9d00f3c0                FormatFileName
                0x9d00fc4c                FormatDirName
                0x9d0105f8                ValidateChars
                0x9d010c6c                FSfseek
                0x9d011024                ReadFAT
                0x9d0114e4                WriteFAT
                0x9d011ab4                FSchdir
                0x9d011ae4                wFSchdir
                0x9d011b2c                chdirhelper
                0x9d012524                FSgetcwd
                0x9d013354                wFSgetcwd
                0x9d01339c                GetPreviousEntry
                0x9d013a68                FSmkdir
                0x9d013a98                wFSmkdir
                0x9d013ae0                mkdirhelper
                0x9d01471c                CreateDIR
                0x9d0148e8                writeDotEntries
                0x9d014b28                FSrmdir
                0x9d014b68                wFSrmdir
                0x9d014bbc                rmdirhelper
                0x9d015fc8                eraseDir
                0x9d0160fc                FindFirst
                0x9d0165fc                FindNext
                0x9d016a54                wFindFirst
                0x9d016aa4                FSputc
                0x9d016b00                str_put_n_chars
                0x9d016b88                FSfprintf
                0x9d016bd8                FSvfprintf

.rodata         0x9d01813c     0xb764
 .rodata        0x9d01813c     0xb764 output\MPFSImg2.o
                0x9d01813c                MPFS_Start

.text           0x9d0238a0    0x40be0
 .text          0x9d0238a0     0xa264 output\CustomHTTPApp.o
                0x9d0238a0                HTTPNeedsAuth
                0x9d023918                HTTPCheckAuth
                0x9d023990                HTTPExecuteGet
                0x9d0239d0                HTTPExecutePost
                0x9d0292f0                HTTPPrint_hellomsg
                0x9d029388                HTTPPrintIP
                0x9d029444                HTTPPrint_config_dhcpchecked
                0x9d0294a4                HTTPPrint_config_ip
                0x9d0294cc                HTTPPrint_config_gw
                0x9d0294f8                HTTPPrint_config_subnet
                0x9d029524                HTTPPrint_config_dns1
                0x9d029550                HTTPPrint_config_dns2
                0x9d02957c                HTTPPrint_config_mac
                0x9d0296d0                HTTPPrint_reboot
                0x9d0296e0                HTTPPrint_rebootaddr
                0x9d029708                HTTPPrint_status_ok
                0x9d029790                HTTPPrint_status_fail
                0x9d029818                HTTPPrint_server_name
                0x9d029858                HTTPPrint_JitterSize
                0x9d0298c4                HTTPPrint_TimeZone
                0x9d029930                HTTPPrint_TimeZoneMinutes
                0x9d02999c                HTTPPrint_CurTime
                0x9d029a08                HTTPPrint_CurDate
                0x9d029a70                HTTPPrint_CurPTT
                0x9d029af4                HTTPPrint_CurCOS
                0x9d029b78                HTTPPrint_CurUser
                0x9d029c74                HTTPPrint_CurSSN
                0x9d029d04                HTTPPrint_RefName
                0x9d029db0                HTTPPrint_auth_call
                0x9d029e14                HTTPPrint_pin
                0x9d029e78                HTTPPrint_NodeName
                0x9d029edc                HTTPPrint_NtpName
                0x9d029f1c                HTTPPrint_delay_time
                0x9d029f88                HTTPPrint_time_out
                0x9d029ff4                HTTPPrint_keep_alive
                0x9d02a060                HTTPPrint_jittter_size
                0x9d02a0cc                HTTPPrint_RX_AutoPolarity
                0x9d02a15c                HTTPPrint_RX_Polarity
                0x9d02a1ec                HTTPPrint_TX_Polarity
                0x9d02a280                HTTPPrint_COS_Check
                0x9d02a310                HTTPPrint_SN_Squelch
                0x9d02a37c                HTTPPrint_CRC_Check
                0x9d02a40c                HTTPPrint_LastFrame
                0x9d02a49c                HTTPPrint_HeaderGen
                0x9d02a530                HTTPPrint_HeaderGenType
                0x9d02a5c0                HTTPPrint_HeaderRep
                0x9d02a650                HTTPPrint_HalfFull
                0x9d02a6e0                HTTPPrint_user_id
                0x9d02a720                HTTPPrint_user_pass
                0x9d02a760                HTTPPrint_user_passC
                0x9d02a7a0                HTTPPrint_BeaconM
                0x9d02a804                HTTPPrint_BeaconCall
                0x9d02a868                HTTPPrint_BeaconIntv
                0x9d02a8e4                HTTPPrint_alt_mycall
                0x9d02a948                HTTPPrint_alt_mycall2
                0x9d02a9ac                HTTPPrint_alt_yourcall
                0x9d02aa10                HTTPPrint_alt_rpt1call
                0x9d02aa74                HTTPPrint_alt_rpt2call
                0x9d02aad8                HTTPPrint_flag0
                0x9d02ab6c                HTTPPrint_flag1
                0x9d02abfc                HTTPPrint_flag2
                0x9d02ac8c                HTTPPrint_flag3
                0x9d02ad1c                HTTPPrint_flag4
                0x9d02adac                HTTPPrint_flag5
                0x9d02ae3c                HTTPPrint_flag6
                0x9d02aecc                HTTPPrint_flag7
                0x9d02af5c                HTTPPrint_Aflag
                0x9d02aff0                HTTPPrint_a_mycall
                0x9d02b080                HTTPPrint_a_mycall2
                0x9d02b110                HTTPPrint_a_yourcall
                0x9d02b1a0                HTTPPrint_a_rpt1call
                0x9d02b230                HTTPPrint_a_rpt2call
                0x9d02b2c0                HTTPPrint_ircDDB
                0x9d02b354                HTTPPrint_ircDDBtype
                0x9d02b460                HTTPPrint_RefSelectFirst
                0x9d02b5a4                HTTPPrint_RefSelect
                0x9d02b850                HTTPPrint_Band
                0x9d02b8b0                HTTPPrint_BandSelect
                0x9d02bdd4                HTTPPrint_ReConnect
                0x9d02be34                HTTPPrint_ConnectUser
                0x9d02bf60                HTTPPrint_AutConnect
                0x9d02bfc0                HTTPPrint_Repeater
                0x9d02c020                HTTPPrint_DisableRFcmd
                0x9d02c080                HTTPPrint_VoiceMsg
                0x9d02c0e0                HTTPPrint_CurRef
                0x9d02c1ac                HTTPPrint_Notice
                0x9d02c1ec                HTTPPrint_DPRS_checked
                0x9d02c248                HTTPPrint_dprsRadio
                0x9d02c2a4                HTTPPrint_dprsInet
                0x9d02c300                HTTPPrint_dprsip
                0x9d02c340                HTTPPrint_dprsport
                0x9d02c3ac                HTTPPrint_dprscall
                0x9d02c404                HTTPPrint_dstarid
                0x9d02c44c                HTTPPrint_altdstarid
                0x9d02c4c4                HTTPPrint_dprsvalid
                0x9d02c51c                HTTPPrint_plat
                0x9d02c5ec                HTTPPrint_plong
                0x9d02c6c4                HTTPPrint_pcomment
                0x9d02c728                HTTPPrint_pinterval
                0x9d02c78c                HTTPPrint_clientID
                0x9d02c7e8                HTTPPrint_dprsAutoLink
                0x9d02c844                HTTPPrint_dprsAutoReLink
                0x9d02c8a0                HTTPPrint_DateTime
                0x9d02c968                HTTPPrint_http
                0x9d02cba0                HTTPPrint_EmailAccessFirst
                0x9d02cbbc                HTTPPrint_EmailAccess
                0x9d02ce08                HTTPPrint_accessFirst
                0x9d02ce24                HTTPPrint_access
                0x9d02d008                HTTPPrint_uploaded
                0x9d02d0e8                HTTPPrint_smtpserver
                0x9d02d168                HTTPPrint_smtpport
                0x9d02d1d0                HTTPPrint_CurAPRS
                0x9d02d254                HTTPPrint_smtpuser
                0x9d02d294                HTTPPrint_smtppass
                0x9d02d2d4                HTTPPrint_smtp_auth
                0x9d02d364                HTTPPrint_ack
                0x9d02d3ec                HTTPPrint_DebugSwitch
                0x9d02d470                HTTPPrint_destination
                0x9d02d4b0                HTTPPrint_mesgBody
                0x9d02d4f0                HTTPPrint_orgSSID
                0x9d02d6a8                HTTPPrint_altSSID
                0x9d02d924                HTTPPrint_sendercall
                0x9d02d964                HTTPPrint_LastMsg
                0x9d02d9a4                NVMemOperation
                0x9d02da88                delay_us
 .text          0x9d02db04     0x8bd8 output\DstaDPlusClientUDP.o
                0x9d02db04                DstarDPlusClientUDP
                0x9d032504                KeepAliveSend
                0x9d032f28                ReLoadMsg
                0x9d032f88                InetHeaderLog
 .text          0x9d0366dc     0x81a4 output\TCP.o
                0x9d0367f0                TCPInit
                0x9d036ad8                TCPOpen
                0x9d036f40                TCPWasReset
                0x9d036fc4                TCPIsConnected
                0x9d037004                TCPDisconnect
                0x9d037274                TCPClose
                0x9d0372d0                TCPGetRemoteInfo
                0x9d03733c                TCPFlush
                0x9d0373b0                TCPIsPutReady
                0x9d03757c                TCPPut
                0x9d0378c0                TCPPutArray
                0x9d037ccc                TCPPutString
                0x9d037d24                TCPGetTxFIFOFull
                0x9d037dc8                TCPDiscard
                0x9d037e58                TCPIsGetReady
                0x9d037fc4                TCPGet
                0x9d038248                TCPGetArray
                0x9d0385f4                TCPGetRxFIFOFree
                0x9d038690                TCPPeekArray
                0x9d038920                TCPPeek
                0x9d03896c                TCPFindArrayEx
                0x9d038f78                TCPFindEx
                0x9d038fd8                TCPTick
                0x9d03a070                TCPProcess
                0x9d03dff4                TCPAdjustFIFOSize
 .text          0x9d03e880     0x752c output\usb_host.o
                0x9d03e880                USBHostClearEndpointErrors
                0x9d03e91c                USBHostDeviceSpecificClientDriver
                0x9d03e940                USBHostDeviceStatus
                0x9d03e9e8                USBHostInit
                0x9d03eaec                USBHostIssueDeviceRequest
                0x9d03ee5c                USBHostRead
                0x9d03efc4                USBHostResetDevice
                0x9d03f020                USBHostResumeDevice
                0x9d03f08c                USBHostSetDeviceConfiguration
                0x9d03f148                USBHostSetNAKTimeout
                0x9d03f20c                USBHostShutdown
                0x9d03f2a0                USBHostSuspendDevice
                0x9d03f310                USBHostTasks
                0x9d0413f8                USBHostTerminateTransfer
                0x9d041488                USBHostTransferIsComplete
                0x9d0415d8                USBHostVbusEvent
                0x9d041680                USBHostWrite
                0x9d0417ec                _USB_CheckCommandAndEnumerationAttempts
                0x9d041894                _USB_FindClassDriver
                0x9d041a2c                _USB_FindDeviceLevelClientDriver
                0x9d041ca4                _USB_FindEndpoint
                0x9d041d68                _USB_FindNextToken
                0x9d043678                _USB_FindServiceEndpoint
                0x9d043900                _USB_FreeConfigMemory
                0x9d043a90                _USB_FreeMemory
                0x9d043b80                _USB_InitControlRead
                0x9d043c68                _USB_InitControlWrite
                0x9d043d70                _USB_InitRead
                0x9d043e78                _USB_InitWrite
                0x9d043f80                _USB_NotifyClients
                0x9d04408c                _USB_NotifyDataClients
                0x9d044120                _USB_ParseConfigurationDescriptor
                0x9d044a3c                _USB_ResetDATA0
                0x9d044b38                _USB_SendToken
                0x9d044c30                _USB_SetBDT
                0x9d044fb4                _USB_TransferInProgress
                0x9d045098                _USB1Interrupt
 .text          0x9d045dac     0x6354 output\prvTaskUSB.o
                0x9d045dac                CheckForNewAttach
                0x9d0461b4                USB_ApplicationEventHandler
                0x9d046358                prvTaskUSB
                0x9d046860                Ptt_Off
                0x9d048fbc                JitterBufferInit
                0x9d0490c4                JitterBufferSave
                0x9d049160                JitterBufferSend
                0x9d049494                BeepSend
                0x9d049c38                DisConnectedMsgSend
                0x9d04a1dc                NotFoundMsgSend
                0x9d04a77c                swaps_usb
                0x9d04b380                update_crc_dstar
                0x9d04b3f4                result_crc_dstar
 .text          0x9d04c100     0x4a10 output\prvTaskFS.o
                0x9d04c100                prvTaskFS
                0x9d04cd58                GetRefDateTime
                0x9d04cf20                callsign_check
                0x9d04d6a8                ConnectMSG
                0x9d04d8a0                CallSignPlay
                0x9d04dd5c                MsgPlay
                0x9d04e0cc                SendConnectMsg
                0x9d04e40c                GetTimeDate
 .text          0x9d050b10     0x3b70 output\HTTP2.o
                0x9d050b10                HTTPPrint
                0x9d05163c                HTTPPrint_
                0x9d051678                HTTPInit
                0x9d05178c                HTTPServer
                0x9d053f88                HTTPGetArg
                0x9d054048                HTTPReadPostName
                0x9d0540b8                HTTPReadPostValue
                0x9d054490                HTTPIncFile
 .text          0x9d054680     0x27c4 output\SMTP.o
                0x9d054680                SMTPBeginUsage
                0x9d054710                SMTPEndUsage
                0x9d0547bc                SMTPTask
                0x9d056798                SMTPSendMail
                0x9d0567b0                SMTPIsBusy
                0x9d0567c0                SMTPIsPutReady
                0x9d056804                SMTPPut
                0x9d05698c                SMTPPutArray
                0x9d056a30                SMTPPutString
                0x9d056abc                SMTPFlush
                0x9d056ae4                SMTPPutDone
 .text          0x9d056e44     0x1ee0 output\FTP.o
                0x9d056e44                FTPInit
                0x9d056ed8                FTPServer
                0x9d0572a4                FTPGetUser
                0x9d057364                FTPGetStage
                0x9d058ca8                FTPVerify
 .text          0x9d058d24     0x186c output\SD-SPI.o
                0x9d058d24                MDD_SDSPI_MediaDetect
                0x9d058d40                MDD_SDSPI_ReadSectorSize
                0x9d058d4c                MDD_SDSPI_ReadCapacity
                0x9d058d58                MDD_SDSPI_InitIO
                0x9d058da4                MDD_SDSPI_ShutdownMedia
                0x9d058de0                SendMMCCmd
                0x9d0590a4                MDD_SDSPI_SectorRead
                0x9d059134                MDD_SDSPI_AsyncReadTasks
                0x9d0595c4                MDD_SDSPI_AsyncWriteTasks
                0x9d059b2c                MDD_SDSPI_SectorWrite
                0x9d059c0c                Delayms
                0x9d059c74                CloseSPIM
                0x9d059c90                WriteSPIM
                0x9d059ce4                MDD_SDSPI_ReadMedia
                0x9d059d28                OpenSPIM
                0x9d059e58                InitSPISlowMode
                0x9d059f24                MDD_SDSPI_MediaInitialize
 .text          0x9d05a590     0x1850 output\DHCP.o
                0x9d05a590                DHCPInit
                0x9d05a674                DHCPDisable
                0x9d05a6d0                DHCPEnable
                0x9d05a718                DHCPIsEnabled
                0x9d05a738                DHCPIsBound
                0x9d05a75c                DHCPStateChanged
                0x9d05a7ac                DHCPIsServerDetected
                0x9d05a7d0                DHCPTask
 .text          0x9d05bde0     0x17a4 output\tasks.o
                0x9d05bde0                xTaskGenericCreate
                0x9d05c02c                vTaskDelete
                0x9d05c130                vTaskDelay
                0x9d05c1cc                vTaskPrioritySet
                0x9d05c398                vTaskSuspend
                0x9d05c4b4                xTaskIsTaskSuspended
                0x9d05c520                vTaskResume
                0x9d05c638                xTaskResumeFromISR
                0x9d05c738                vTaskStartScheduler
                0x9d05c7d4                vTaskEndScheduler
                0x9d05c824                vTaskSuspendAll
                0x9d05c838                xTaskResumeAll
                0x9d05c9d8                xTaskGetTickCount
                0x9d05ca0c                xTaskGetTickCountFromISR
                0x9d05ca48                uxTaskGetNumberOfTasks
                0x9d05ca54                vTaskIncrementTick
                0x9d05cc0c                vTaskSwitchContext
                0x9d05cce4                vTaskPlaceOnEventList
                0x9d05cd80                xTaskRemoveFromEventList
                0x9d05ce94                vTaskSetTimeOutState
                0x9d05ceb8                xTaskCheckForTimeOut
                0x9d05cfb0                vTaskMissedYield
                0x9d05d41c                uxTaskGetStackHighWaterMark
                0x9d05d4b8                vTaskEnterCritical
                0x9d05d510                vTaskExitCritical
 .text          0x9d05d584     0x1560 output\MPFS2.o
                0x9d05d584                MPFSInit
                0x9d05d5f8                MPFSOpen
                0x9d05d8f8                MPFSOpenID
                0x9d05da54                MPFSClose
                0x9d05daa4                MPFSGet
                0x9d05dcb8                MPFSGetArray
                0x9d05df38                MPFSGetLong
                0x9d05df80                MPFSSeek
                0x9d05e434                MPFSGetTimestamp
                0x9d05e4e0                MPFSGetMicrotime
                0x9d05e58c                MPFSGetFlags
                0x9d05e638                MPFSGetSize
                0x9d05e6e4                MPFSGetBytesRem
                0x9d05e768                MPFSGetStartAddr
                0x9d05e814                MPFSGetEndAddr
                0x9d05e8d0                MPFSGetFilename
                0x9d05e9bc                MPFSGetPosition
                0x9d05ea18                MPFSGetID
 .text          0x9d05eae4     0x1420 output\Helpers.o
                0x9d05eae4                LFSRSeedRand
                0x9d05eb58                LFSRRand
                0x9d05ebc0                GenerateRandomDWORD
                0x9d05ee08                StringToIPAddress
                0x9d05f1a0                Base64Decode
                0x9d05f4ac                Base64Encode
                0x9d05f750                uitoa
                0x9d05f86c                hexatob
                0x9d05f948                btohexa_high
                0x9d05f994                btohexa_low
                0x9d05f9e0                stricmppgm2ram
                0x9d05fb3c                swaps
                0x9d05fb78                swapl
                0x9d05fc48                CalcIPChecksum
                0x9d05fd1c                strupr
                0x9d05fda8                FormatNetBIOSName
                0x9d05fe60                strnchr
 .text          0x9d05ff04     0x1244 output\ETHPIC32ExtPhy.o
                0x9d05ff04                EthPhyRestartNegotiation
                0x9d05ff88                EthPhyGetHwConfigFlags
                0x9d05ffe8                EthPhyInit
                0x9d0604bc                EthPhyNegotiationComplete
                0x9d060710                EthPhyGetNegotiationResult
                0x9d060a44                EthPhyGetLinkStatus
                0x9d060b0c                EthPhyReset
                0x9d060c08                EthPhyScanLinkStart
                0x9d060c34                EthPhyScanLinkRead
                0x9d060c90                EthPhyScanLinkStop
 .text          0x9d061148     0x11d0 output\UDP.o
                0x9d061148                UDPInit
                0x9d0611ac                UDPOpenEx
                0x9d0613dc                UDPTask
                0x9d06190c                UDPIsOpened
                0x9d061944                UDPClose
                0x9d0619d0                UDPSetTxBuffer
                0x9d061a20                UDPSetRxBuffer
                0x9d061a60                UDPIsPutReady
                0x9d061adc                UDPPut
                0x9d061b58                UDPPutArray
                0x9d061bf0                UDPPutString
                0x9d061c38                UDPFlush
                0x9d061e08                UDPIsGetReady
                0x9d061e88                UDPGet
                0x9d061efc                UDPGetArray
                0x9d061fac                UDPDiscard
                0x9d061ffc                UDPProcess
 .text          0x9d062318     0x1128 c:/program files/microchip/mplabc32/v2.02/bin/../lib/gcc/pic32mx/4.5.1/../../../../pic32mx/lib/speed\libm.a(dp32.o)
                0x9d062318                __subdf3
                0x9d062318                dpsub
                0x9d062320                dpadd
                0x9d062320                __adddf3
                0x9d062744                dpmul
                0x9d062744                __muldf3
                0x9d062a6c                dpdiv
                0x9d062a6c                __divdf3
                0x9d062f20                __floatsidf
                0x9d062f20                litodp
                0x9d062f94                ultodp
                0x9d062fe4                fptodp
                0x9d062fe4                __extendsfdf2
                0x9d063088                __truncdfsf2
                0x9d063088                dptofp
                0x9d063180                dptoli
                0x9d063180                __fixdfsi
                0x9d063208                __fixunsdfsi
                0x9d063208                dptoul
                0x9d06328c                __nedf2
                0x9d06328c                __gtdf2
                0x9d06328c                __ledf2
                0x9d06328c                __ltdf2
                0x9d06328c                __gedf2
                0x9d06328c                dpcmp
                0x9d06328c                __eqdf2
                0x9d0633b0                __negdf2
                0x9d0633c8                fabs
                0x9d0633c8                dpfabs
                0x9d0633e4                nan
                0x9d0633e4                dpnan
 .text          0x9d063440     0x1040 output\IntQueue.o
                0x9d063440                vStartInterruptQueueTasks
                0x9d063e60                xFirstTimerHandler
                0x9d06407c                xSecondTimerHandler
                0x9d0643d4                xAreIntQueueTasksStillRunning

.dinit          0x9d064480     0x1024
 .dinit         0x9d064480     0x1024 data_init

.text           0x9d0654a4     0x2920
 .text          0x9d0654a4      0xe68 output\DNS.o
                0x9d0654a4                DNSBeginUsage
                0x9d0654e4                DNSEndUsage
                0x9d065544                DNSResolve
                0x9d0655c8                DNSIsResolved
 .text          0x9d06630c      0xdf0 output\ETHPIC32IntMac.o
                0x9d06630c                MACInit
                0x9d066740                MACIsLinked
                0x9d066750                MACGetTxBaseAddr
                0x9d066778                MACGetHttpBaseAddr
                0x9d066788                MACGetSslBaseAddr
                0x9d066798                MACSetWritePtr
                0x9d0667c0                MACIsTxReady
                0x9d06696c                MACPut
                0x9d066990                MACPutArray
                0x9d0669e0                MACPutHeader
                0x9d066ab0                MACFlush
                0x9d066b10                MACDiscardRx
                0x9d066b60                MACGetHeader
                0x9d066d78                MACSetReadPtrInRx
                0x9d066d9c                MACSetReadPtr
                0x9d066dc4                MACGet
                0x9d066de0                MACGetArray
                0x9d066e40                MACGetFreeRxSize
                0x9d066e84                MACMemCopyAsync
                0x9d066f18                MACIsMemCopyDone
                0x9d066f24                CalcIPBufferChecksum
                0x9d066f5c                MACCalcRxChecksum
 .text          0x9d0670fc      0xcc8 output\queue.o
                0x9d0670fc                xQueueCreate
                0x9d06726c                xQueueGenericSend
                0x9d0674a4                xQueueGenericSendFromISR
                0x9d067594                xQueueGenericReceive
                0x9d067848                xQueueReceiveFromISR
                0x9d067938                uxQueueMessagesWaiting
                0x9d067974                uxQueueMessagesWaitingFromISR
                0x9d067998                vQueueDelete
                0x9d067d1c                xQueueIsQueueEmptyFromISR
                0x9d067d90                xQueueIsQueueFullFromISR

.text._vfprintf_cdnopsuxX
                0x9d067dc4      0xc7c
 .text._vfprintf_cdnopsuxX
                0x9d067dc4      0xc7c c:/program files/microchip/mplabc32/v2.02/bin/../lib/gcc/pic32mx/4.5.1/../../../../pic32mx/lib/speed\libc.a(doprnt_cdnopsuxX.eo)
                0x9d067dc4                _vfprintf_s
                0x9d067dc4                _vfprintf_0
                0x9d067dc4                _vfprintf_cdnopuxX
                0x9d067dc4                _vfprintf_cdnopsuxX

.rodata         0x9d068a40      0xbcc
 .rodata        0x9d068a40      0xbcc output\CustomHTTPApp.o
                0x9d069604                countPerMicroSec

.text           0x9d06960c      0xb90
 .text          0x9d06960c      0xb90 output\DHCPs.o
                0x9d06960c                DHCPServerTask

.rodata         0x9d06a19c      0xa58
 .rodata        0x9d06a19c      0xa58 output\DstaDPlusClientUDP.o

.text           0x9d06abf4     0x21d4
 .text          0x9d06abf4      0x8ec c:/program files/microchip/mplabc32/v2.02/bin/../lib/gcc/pic32mx/4.5.1/../../../../pic32mx/lib/speed\libm.a(fp32.o)
                0x9d06abf4                __subsf3
                0x9d06abf4                fpsub
                0x9d06abfc                fpadd
                0x9d06abfc                __addsf3
                0x9d06ae68                fpmul
                0x9d06ae68                __mulsf3
                0x9d06b020                fpdiv
                0x9d06b020                __divsf3
                0x9d06b24c                litofp
                0x9d06b24c                sitofp
                0x9d06b24c                __floatsisf
                0x9d06b2a8                uitofp
                0x9d06b2a8                ultofp
                0x9d06b2f4                fptosi
                0x9d06b2f4                fptoli
                0x9d06b2f4                __fixsfsi
                0x9d06b36c                __fixunssfsi
                0x9d06b36c                fptoul
                0x9d06b36c                fptoui
                0x9d06b3e0                __eqsf2
                0x9d06b3e0                __nesf2
                0x9d06b3e0                __lesf2
                0x9d06b3e0                __ltsf2
                0x9d06b3e0                fpcmp
                0x9d06b3e0                __gtsf2
                0x9d06b3e0                __gesf2
                0x9d06b474                fpfabs
                0x9d06b474                fabsf
                0x9d06b484                __negsf2
                0x9d06b494                fpnan
                0x9d06b494                nanf
 .text          0x9d06b4e0      0x874 output\prvTaskTCPIP.o
                0x9d06b4e0                prvTaskTCPIP
                0x9d06b8c4                DisplayIPValue
 .text          0x9d06bd54      0x864 output\SNTP.o
                0x9d06bd54                SNTPClient
                0x9d06c530                SNTPGetUTCSeconds
 .text          0x9d06c5b8      0x810 output\MACread.o
                0x9d06c5b8                MACreadInit
                0x9d06c5e8                MACBeginRead
                0x9d06c608                MACRead
                0x9d06c690                MACreadEndRead
                0x9d06c69c                MACReadArray
                0x9d06c88c                MACBeginWrite
                0x9d06c8ac                MACWrite
                0x9d06c938                MACWriteArray
                0x9d06c9c0                MACEndWrite
                0x9d06cc4c                MACreadIsBusy
                0x9d06cd98                ReadMacFromEEPROM

.rodata         0x9d06cdc8      0x7d4
 .rodata        0x9d06cdc8      0x7d4 c:/program files/microchip/mplabc32/v2.02/bin/../lib/gcc/pic32mx/4.5.1/../../../../pic32mx/lib/speed\libmchp_peripheral_32MX795F512L.a(int_tbl_lib.o)
                0x9d06cdc8                __IntSrcTbl
                0x9d06d2e4                __IntVectorTbl

.text           0x9d06d59c     0x1fe8
 .text          0x9d06d59c      0x780 output\main.o
                0x9d06d59c                main
                0x9d06dd04                vApplicationStackOverflowHook
                0x9d06dd0c                _general_exception_handler
 .text          0x9d06dd1c      0x6e0 output\NBNS.o
                0x9d06dd1c                NBNSTask
 .text          0x9d06e3fc      0x658 output\QPeek.o
                0x9d06e3fc                vStartQueuePeekTasks
                0x9d06ea24                xAreQueuePeekTasksStillRunning
 .text          0x9d06ea54      0x5a4 output\usb_host_generic.o
                0x9d06ea54                USBHostGenericInit
                0x9d06ebc4                USBHostGenericEventHandler
                0x9d06ed84                USBHostGenericGetDeviceAddress
                0x9d06ee2c                USBHostGenericRead
                0x9d06ef18                USBHostGenericWrite
 .text          0x9d06eff8      0x58c output\ARP.o
                0x9d06f0dc                ARPInit
                0x9d06f14c                ARPProcess
                0x9d06f358                ARPResolve
                0x9d06f45c                ARPIsResolved
                0x9d06f508                SwapARPPacket

.rodata         0x9d06f584      0x9c4
 .rodata        0x9d06f584      0x548 output\HTTP2.o
 .rodata        0x9d06facc      0x47c output\prvTaskFS.o

.text           0x9d06ff48      0xd20
 .text          0x9d06ff48      0x46c output\lcd.o
                0x9d06ff48                xStartLCDTask
 .text          0x9d0703b4      0x46c c:/program files/microchip/mplabc32/v2.02/bin/../lib/gcc/pic32mx/4.5.1/speed\libgcc.a(_umoddi3.o)
                0x9d0703b4                __umoddi3
 .text          0x9d070820      0x448 c:/program files/microchip/mplabc32/v2.02/bin/../lib/gcc/pic32mx/4.5.1/speed\libgcc.a(_udivdi3.o)
                0x9d070820                __udivdi3

.text.EthRxBuffersAppend
                0x9d070c68      0x448
 .text.EthRxBuffersAppend
                0x9d070c68      0x448 c:/program files/microchip/mplabc32/v2.02/bin/../lib/gcc/pic32mx/4.5.1/../../../../pic32mx/lib/speed\libmchp_peripheral_32MX795F512L.a(eth_rx_buffers_append_lib.o)
                0x9d070c68                EthRxBuffersAppend

.text           0x9d0710b0      0x850
 .text          0x9d0710b0      0x440 output\port_asm.o
                0x9d0710b0                vT5InterruptHandler
                0x9d071258                vPortStartFirstTask
                0x9d07131c                vPortYieldISR
 .text          0x9d0714f0      0x410 output\StackTsk.o
                0x9d0714f0                StackInit
                0x9d07159c                StackTask
                0x9d071828                StackTaskUDP

.text.__strtod  0x9d071900      0x3f0
 .text.__strtod
                0x9d071900      0x3f0 c:/program files/microchip/mplabc32/v2.02/bin/../lib/gcc/pic32mx/4.5.1/../../../../pic32mx/lib/speed\libe.a(_strtod.o)
                0x9d071900                __strtod

.text           0x9d071cf0      0xa68
 .text          0x9d071cf0      0x390 output\DprsSMTP.o
                0x9d071cf0                DprsSMTP
 .text          0x9d072080      0x388 output\serial.o
                0x9d072080                xSerialPortInitMinimal
                0x9d0721bc                xSerialGetChar
                0x9d072214                xSerialPutChar
                0x9d0722b4                vSerialClose
                0x9d0722c0                vU2InterruptHandler
 .text          0x9d072408      0x350 output\IntQueueTimer_isr.o
                0x9d072408                vT3InterruptWrapper
                0x9d0725b0                vT4InterruptWrapper

.rodata         0x9d072758      0x338
 .rodata        0x9d072758      0x338 output\prvTaskUSB.o

.text           0x9d072a90      0x330
 .text          0x9d072a90      0x330 output\heap_2.o
                0x9d072a90                pvPortMalloc
                0x9d072cd8                vPortFree
                0x9d072dac                xPortGetFreeHeapSize
                0x9d072db8                vPortInitialiseBlocks

.rodata         0x9d072dc0      0x2f0
 .rodata        0x9d072dc0      0x2f0 output\FTP.o

.text           0x9d0730b0      0xb14
 .text          0x9d0730b0      0x2dc output\IP.o
                0x9d0730b0                IPGetHeader
                0x9d0731cc                IPPutHeader
                0x9d0732d4                IPSetRxBuffer
 .text          0x9d07338c      0x2d8 output\port.o
                0x9d07338c                pxPortInitialiseStack
                0x9d073470                prvSetupTimerInterrupt
                0x9d073534                vPortEndScheduler
                0x9d07353c                xPortStartScheduler
                0x9d0735c4                vPortIncrementTick
                0x9d073610                uxPortSetInterruptMaskFromISR
                0x9d07364c                vPortClearInterruptMaskFromISR
 .text          0x9d073664      0x2bc output\Tick.o
                0x9d073664                TickInit
                0x9d073768                TickGet
                0x9d073790                TickGetDiv256
                0x9d0737f0                TickGetDiv64K
                0x9d073850                TickConvertToMilliseconds
                0x9d0738a8                _T1Interrupt
 .text          0x9d073920      0x2a4 output\comtest.o
                0x9d073920                vStartComTasks
                0x9d073b8c                xAreComTestTasksStillRunning

.text.gmtime    0x9d073bc4      0x2a4
 .text.gmtime   0x9d073bc4      0x2a4 c:/program files/microchip/mplabc32/v2.02/bin/../lib/gcc/pic32mx/4.5.1/../../../../pic32mx/lib/speed\libc.a(ctime.o)
                0x9d073bc4                gmtime

.text           0x9d073e68      0x254
 .text          0x9d073e68      0x254 output\list.o
                0x9d073e68                vListInitialise
                0x9d073eb8                vListInitialiseItem
                0x9d073ecc                vListInsertEnd
                0x9d073f58                vListInsert
                0x9d074034                vListRemove

.text._RtccSetTimeAndDate
                0x9d0740bc      0x23c
 .text._RtccSetTimeAndDate
                0x9d0740bc      0x23c c:/program files/microchip/mplabc32/v2.02/bin/../lib/gcc/pic32mx/4.5.1/../../../../pic32mx/lib/speed\libmchp_peripheral_32MX795F512L.a(_rtcc_set_time_and_date_lib.o)
                0x9d0740bc                _RtccSetTimeAndDate

.text           0x9d0742f8      0x230
 .text          0x9d0742f8      0x230 output\IntQueueTimer.o
                0x9d0742f8                vInitialiseTimerForIntQueueTest
                0x9d074478                vT3InterruptHandler
                0x9d0744d0                vT4InterruptHandler

.text.RtccOpen  0x9d074528      0x1ec
 .text.RtccOpen
                0x9d074528      0x1ec c:/program files/microchip/mplabc32/v2.02/bin/../lib/gcc/pic32mx/4.5.1/../../../../pic32mx/lib/speed\libmchp_peripheral_32MX795F512L.a(rtcc_open_lib.o)
                0x9d074528                RtccOpen

.text._EthAckPacket
                0x9d074714      0x1dc
 .text._EthAckPacket
                0x9d074714      0x1dc c:/program files/microchip/mplabc32/v2.02/bin/../lib/gcc/pic32mx/4.5.1/../../../../pic32mx/lib/speed\libmchp_peripheral_32MX795F512L.a(eth_ack_packet_lib.o)
                0x9d074714                _EthAckPacket

.text.__ldexp   0x9d0748f0      0x1d4
 .text.__ldexp  0x9d0748f0      0x1d4 c:/program files/microchip/mplabc32/v2.02/bin/../lib/gcc/pic32mx/4.5.1/../../../../pic32mx/lib/speed\libe.a(_ldexp.o)
                0x9d0748f0                __ldexp

.text.RtccInit  0x9d074ac4      0x1ac
 .text.RtccInit
                0x9d074ac4      0x1ac c:/program files/microchip/mplabc32/v2.02/bin/../lib/gcc/pic32mx/4.5.1/../../../../pic32mx/lib/speed\libmchp_peripheral_32MX795F512L.a(rtcc_init_lib.o)
                0x9d074ac4                RtccInit

.text           0x9d074c70      0x1a8
 .text          0x9d074c70      0x1a8 output\serial_isr.o
                0x9d074c70                vU2InterruptWrapper

.text.EthTxSendBuffer
                0x9d074e18      0x1a4
 .text.EthTxSendBuffer
                0x9d074e18      0x1a4 c:/program files/microchip/mplabc32/v2.02/bin/../lib/gcc/pic32mx/4.5.1/../../../../pic32mx/lib/speed\libmchp_peripheral_32MX795F512L.a(eth_tx_packet_lib.o)
                0x9d074e18                EthTxSendBuffer

.text           0x9d074fbc      0x1a0
 .text          0x9d074fbc      0x1a0 c:/program files/microchip/mplabc32/v2.02/bin/../lib/gcc/pic32mx/4.5.1/../../../../pic32mx/lib/speed\libc.a(strcpy.o)
                0x9d074fbc                strcpy

.text._EthAppendBusyList
                0x9d07515c      0x19c
 .text._EthAppendBusyList
                0x9d07515c      0x19c c:/program files/microchip/mplabc32/v2.02/bin/../lib/gcc/pic32mx/4.5.1/../../../../pic32mx/lib/speed\libmchp_peripheral_32MX795F512L.a(_eth_append_busy_list_lib.o)
                0x9d07515c                _EthAppendBusyList

.text._EthRxAckBuffer
                0x9d0752f8      0x184
 .text._EthRxAckBuffer
                0x9d0752f8      0x184 c:/program files/microchip/mplabc32/v2.02/bin/../lib/gcc/pic32mx/4.5.1/../../../../pic32mx/lib/speed\libmchp_peripheral_32MX795F512L.a(eth_ack_packet_lib.o)

.text.EthRxGetPacket
                0x9d07547c      0x180
 .text.EthRxGetPacket
                0x9d07547c      0x180 c:/program files/microchip/mplabc32/v2.02/bin/../lib/gcc/pic32mx/4.5.1/../../../../pic32mx/lib/speed\libmchp_peripheral_32MX795F512L.a(eth_rx_get_packet_lib.o)
                0x9d07547c                EthRxGetPacket

.text           0x9d0755fc      0x5a4
 .text          0x9d0755fc      0x17c output\ETHPIC32ExtPhyDP83848.o
                0x9d0755fc                EthPhyConfigureMII
                0x9d07569c                EthPhyConfigureMdix
                0x9d07575c                EthPhyMIIMAddress
                0x9d075768                EthPhyMIIMClock
 .text          0x9d075778      0x168 c:/program files/microchip/mplabc32/v2.02/bin/../lib/gcc/pic32mx/4.5.1/../../../../pic32mx/lib/speed\libc.a(memcpy.o)
                0x9d075778                memcpy
 .text          0x9d0758e0      0x168 c:/program files/microchip/mplabc32/v2.02/bin/../lib/gcc/pic32mx/4.5.1/../../../../pic32mx/lib/speed\libc.a(strlen.o)
                0x9d0758e0                strlen
 .text          0x9d075a48      0x158 output\ICMP.o
                0x9d075a48                ICMPProcess

.text.fputc     0x9d075ba0      0x140
 .text.fputc    0x9d075ba0      0x140 c:/program files/microchip/mplabc32/v2.02/bin/../lib/gcc/pic32mx/4.5.1/../../../../pic32mx/lib/speed\libc.a(_fputc_simple.o)
                0x9d075ba0                fputc

.text.EthMIIMConfig
                0x9d075ce0      0x13c
 .text.EthMIIMConfig
                0x9d075ce0      0x13c c:/program files/microchip/mplabc32/v2.02/bin/../lib/gcc/pic32mx/4.5.1/../../../../pic32mx/lib/speed\libmchp_peripheral_32MX795F512L.a(eth_miim_access.o)
                0x9d075ce0                EthMIIMConfig

.text.EthDescriptorsPoolAdd
                0x9d075e1c      0x134
 .text.EthDescriptorsPoolAdd
                0x9d075e1c      0x134 c:/program files/microchip/mplabc32/v2.02/bin/../lib/gcc/pic32mx/4.5.1/../../../../pic32mx/lib/speed\libmchp_peripheral_32MX795F512L.a(eth_descriptors_add_lib.o)
                0x9d075e1c                EthDescriptorsPoolAdd

.text._flsbuf   0x9d075f50      0x12c
 .text._flsbuf  0x9d075f50      0x12c c:/program files/microchip/mplabc32/v2.02/bin/../lib/gcc/pic32mx/4.5.1/../../../../pic32mx/lib/speed\libc.a(_flsbuf_simple.o)
                0x9d075f50                _flsbuf

.text           0x9d07607c      0x120
 .text          0x9d07607c      0x120 c:/program files/microchip/mplabc32/v2.02/bin/../lib/gcc/pic32mx/4.5.1/../../../../pic32mx/lib/speed\libc.a(strcmp.o)
                0x9d07607c                strcmp

.rodata         0x9d07619c      0x104
 .rodata        0x9d07619c      0x104 c:/program files/microchip/mplabc32/v2.02/bin/../lib/gcc/pic32mx/4.5.1/../../../../pic32mx/lib/speed\libc.a(ctype.o)
                0x9d07619c                _ctype

.text._RtccWaitClockOff
                0x9d0762a0       0xf8
 .text._RtccWaitClockOff
                0x9d0762a0       0xf8 c:/program files/microchip/mplabc32/v2.02/bin/../lib/gcc/pic32mx/4.5.1/../../../../pic32mx/lib/speed\libmchp_peripheral_32MX795F512L.a(_rtcc_wait_clock_off_lib.o)
                0x9d0762a0                _RtccWaitClockOff

.rodata         0x9d076398       0xf0
 .rodata        0x9d076398       0xf0 output\SD-SPI.o
                0x9d076398                sdmmc_cmdtable

.text.strncpy   0x9d076488       0xe8
 .text.strncpy  0x9d076488       0xe8 c:/program files/microchip/mplabc32/v2.02/bin/../lib/gcc/pic32mx/4.5.1/../../../../pic32mx/lib/speed\libc.a(strncpy.o)
                0x9d076488                strncpy

.rodata         0x9d076570       0xe0
 .rodata        0x9d076570       0xe0 output\DHCP.o

.text           0x9d076650       0xd4
 .text          0x9d076650       0xd4 output\Delay.o
                0x9d076650                DelayMs
                0x9d0766d4                Delay10us

.text.general_exception
                0x9d076724       0xd0
 .text.general_exception
                0x9d076724       0xd0 c:/program files/microchip/mplabc32/v2.02/bin/../lib/gcc/pic32mx/4.5.1/../../../../pic32mx/lib/speed\libc.a(general-exception.o)
                0x9d076724                _general_exception_context

.rodata         0x9d0767f8      0x188
 .rodata        0x9d0767f8       0xd0 c:/program files/microchip/mplabc32/v2.02/bin/../lib/gcc/pic32mx/4.5.1/../../../../pic32mx/lib/speed\libc.a(doprnt_cdnopsuxX.eo)
 .rodata        0x9d0768c8       0xb8 output\DprsSMTP.o

.text._mon_putc
                0x9d076980       0xb4
 .text._mon_putc
                0x9d076980       0xb4 c:/program files/microchip/mplabc32/v2.02/bin/../lib/gcc/pic32mx/4.5.1/../../../../pic32mx/lib/speed\libc.a(_mon_putc.o)
                0x9d076980                _mon_putc

.text.EthInit   0x9d076a34       0xb4
 .text.EthInit  0x9d076a34       0xb4 c:/program files/microchip/mplabc32/v2.02/bin/../lib/gcc/pic32mx/4.5.1/../../../../pic32mx/lib/speed\libmchp_peripheral_32MX795F512L.a(eth_init_lib.o)
                0x9d076a34                EthInit

.text.EthMACOpen
                0x9d076ae8       0xb4
 .text.EthMACOpen
                0x9d076ae8       0xb4 c:/program files/microchip/mplabc32/v2.02/bin/../lib/gcc/pic32mx/4.5.1/../../../../pic32mx/lib/speed\libmchp_peripheral_32MX795F512L.a(eth_mac_open_lib.o)
                0x9d076ae8                EthMACOpen

.text           0x9d076b9c       0xa8
 .text          0x9d076b9c       0xa8 c:/program files/microchip/mplabc32/v2.02/bin/../lib/gcc/pic32mx/4.5.1/../../../../pic32mx/lib/speed\libc.a(memset.o)
                0x9d076b9c                memset

.text.atoi      0x9d076c44       0xa4
 .text.atoi     0x9d076c44       0xa4 c:/program files/microchip/mplabc32/v2.02/bin/../lib/gcc/pic32mx/4.5.1/../../../../pic32mx/lib/speed\libc.a(atoi.o)
                0x9d076c44                atoi

.text.atol      0x9d076ce8       0xa4
 .text.atol     0x9d076ce8       0xa4 c:/program files/microchip/mplabc32/v2.02/bin/../lib/gcc/pic32mx/4.5.1/../../../../pic32mx/lib/speed\libc.a(atol.o)
                0x9d076ce8                atol

.text.strstr    0x9d076d8c       0xa4
 .text.strstr   0x9d076d8c       0xa4 c:/program files/microchip/mplabc32/v2.02/bin/../lib/gcc/pic32mx/4.5.1/../../../../pic32mx/lib/speed\libc.a(strstr.o)
                0x9d076d8c                strstr

.rodata         0x9d076e30       0x98
 .rodata        0x9d076e30       0x98 output\prvTaskTCPIP.o

.text           0x9d076ec8       0x98
 .text          0x9d076ec8       0x98 c:/program files/microchip/mplabc32/v2.02/bin/../lib/gcc/pic32mx/4.5.1/../../../../pic32mx/lib/speed\libc.a(memcmp.o)
                0x9d076ec8                memcmp

.rodata         0x9d076f60       0x90
 .rodata        0x9d076f60       0x90 output\SMTP.o

.text.write     0x9d076ff0       0x88
 .text.write    0x9d076ff0       0x88 c:/program files/microchip/mplabc32/v2.02/bin/../lib/gcc/pic32mx/4.5.1/../../../../pic32mx/lib/speed\libc.a(write.o)
                0x9d076ff0                write

.rodata         0x9d077078       0x80
 .rodata        0x9d077078       0x80 c:/program files/microchip/mplabc32/v2.02/bin/../lib/gcc/pic32mx/4.5.1/../../../../pic32mx/lib/speed\libmchp_peripheral_32MX795F512L.a(spi_brg_tbl_lib_legacy.o)
                0x9d077078                _SpiBrgConvTbl

.text.SoftReset
                0x9d0770f8       0x78
 .text.SoftReset
                0x9d0770f8       0x78 c:/program files/microchip/mplabc32/v2.02/bin/../lib/gcc/pic32mx/4.5.1/../../../../pic32mx/lib/speed\libmchp_peripheral_32MX795F512L.a(soft_reset_lib.o)
                0x9d0770f8                SoftReset

.text.strncmp   0x9d077170       0x70
 .text.strncmp  0x9d077170       0x70 c:/program files/microchip/mplabc32/v2.02/bin/../lib/gcc/pic32mx/4.5.1/../../../../pic32mx/lib/speed\libc.a(strncmp.o)
                0x9d077170                strncmp

.text._sprintf_cdnopsuxX
                0x9d0771e0       0x68
 .text._sprintf_cdnopsuxX
                0x9d0771e0       0x68 c:/program files/microchip/mplabc32/v2.02/bin/../lib/gcc/pic32mx/4.5.1/../../../../pic32mx/lib/speed\libc.a(sprintf_cdnopsuxX.eo)
                0x9d0771e0                _sprintf_s
                0x9d0771e0                _sprintf_cdnopuxX
                0x9d0771e0                _sprintf_0
                0x9d0771e0                _sprintf_cdnopsuxX

.rodata         0x9d077248       0x60
 .rodata        0x9d077248       0x60 output\main.o

.text.OpenSPI1  0x9d0772a8       0x60
 .text.OpenSPI1
                0x9d0772a8       0x60 c:/program files/microchip/mplabc32/v2.02/bin/../lib/gcc/pic32mx/4.5.1/../../../../pic32mx/lib/speed\libmchp_peripheral_32MX795F512L.a(spi_open_spi1_lib_legacy.o)
                0x9d0772a8                OpenSPI1

.text.INTEnable
                0x9d077308       0x58
 .text.INTEnable
                0x9d077308       0x58 c:/program files/microchip/mplabc32/v2.02/bin/../lib/gcc/pic32mx/4.5.1/../../../../pic32mx/lib/speed\libmchp_peripheral_32MX795F512L.a(int_tbl_lib.o)
                0x9d077308                INTEnable

.rodata         0x9d077360       0x54
 .rodata        0x9d077360       0x54 c:/program files/microchip/mplabc32/v2.02/bin/../lib/gcc/pic32mx/4.5.1/../../../../pic32mx/lib/speed\libmchp_peripheral_32MX795F512L.a(_ports_tbl_libp.o)
                0x9d077360                PortRegTbl

.text           0x9d0773b4       0x4c
 .text          0x9d0773b4       0x4c c:/program files/microchip/mplabc32/v2.02/bin/../lib/gcc/pic32mx/4.5.1/speed\libgcc.a(floatunsisf.o)
                0x9d0773b4                __floatunsisf

.rodata         0x9d077400       0x4c
 .rodata        0x9d077400       0x4c c:/program files/microchip/mplabc32/v2.02/bin/../lib/gcc/pic32mx/4.5.1/../../../../pic32mx/lib/speed\libc.a(ctime.o)

.text.EthMACSetAddress
                0x9d07744c       0x48
 .text.EthMACSetAddress
                0x9d07744c       0x48 c:/program files/microchip/mplabc32/v2.02/bin/../lib/gcc/pic32mx/4.5.1/../../../../pic32mx/lib/speed\libmchp_peripheral_32MX795F512L.a(eth_mac_set_address_max_lib.o)
                0x9d07744c                EthMACSetAddress

.text           0x9d077494       0x88
 .text          0x9d077494       0x44 c:/program files/microchip/mplabc32/v2.02/bin/../lib/gcc/pic32mx/4.5.1/speed\libgcc.a(_lshrdi3.o)
                0x9d077494                __lshrdi3
 .text          0x9d0774d8       0x44 c:/program files/microchip/mplabc32/v2.02/bin/../lib/gcc/pic32mx/4.5.1/speed\libgcc.a(_ashldi3.o)
                0x9d0774d8                __ashldi3

.text.EthMIIMReadStart
                0x9d07751c       0x40
 .text.EthMIIMReadStart
                0x9d07751c       0x40 c:/program files/microchip/mplabc32/v2.02/bin/../lib/gcc/pic32mx/4.5.1/../../../../pic32mx/lib/speed\libmchp_peripheral_32MX795F512L.a(eth_miim_access.o)
                0x9d07751c                EthMIIMReadStart

.text.PORTSetPinsDigitalIn
                0x9d07755c       0x40
 .text.PORTSetPinsDigitalIn
                0x9d07755c       0x40 c:/program files/microchip/mplabc32/v2.02/bin/../lib/gcc/pic32mx/4.5.1/../../../../pic32mx/lib/speed\libmchp_peripheral_32MX795F512L.a(port_set_pins_digital_in_lib.o)
                0x9d07755c                PORTSetPinsDigitalIn

.text.PORTSetPinsDigitalOut
                0x9d07759c       0x40
 .text.PORTSetPinsDigitalOut
                0x9d07759c       0x40 c:/program files/microchip/mplabc32/v2.02/bin/../lib/gcc/pic32mx/4.5.1/../../../../pic32mx/lib/speed\libmchp_peripheral_32MX795F512L.a(port_set_pins_digital_out_lib.o)
                0x9d07759c                PORTSetPinsDigitalOut

.text.localtime
                0x9d0775dc       0x3c
 .text.localtime
                0x9d0775dc       0x3c c:/program files/microchip/mplabc32/v2.02/bin/../lib/gcc/pic32mx/4.5.1/../../../../pic32mx/lib/speed\libc.a(ctime.o)
                0x9d0775dc                localtime

.text.EthRxGetBuffer
                0x9d077618       0x3c
 .text.EthRxGetBuffer
                0x9d077618       0x3c c:/program files/microchip/mplabc32/v2.02/bin/../lib/gcc/pic32mx/4.5.1/../../../../pic32mx/lib/speed\libmchp_peripheral_32MX795F512L.a(eth_rx_get_packet_lib.o)
                0x9d077618                EthRxGetBuffer

.text.strcat    0x9d077654       0x38
 .text.strcat   0x9d077654       0x38 c:/program files/microchip/mplabc32/v2.02/bin/../lib/gcc/pic32mx/4.5.1/../../../../pic32mx/lib/speed\libc.a(strcat.o)
                0x9d077654                strcat

.text.EthMIIMWriteStart
                0x9d07768c       0x38
 .text.EthMIIMWriteStart
                0x9d07768c       0x38 c:/program files/microchip/mplabc32/v2.02/bin/../lib/gcc/pic32mx/4.5.1/../../../../pic32mx/lib/speed\libmchp_peripheral_32MX795F512L.a(eth_miim_access.o)
                0x9d07768c                EthMIIMWriteStart

.text.EthMIIMScanStart
                0x9d0776c4       0x34
 .text.EthMIIMScanStart
                0x9d0776c4       0x34 c:/program files/microchip/mplabc32/v2.02/bin/../lib/gcc/pic32mx/4.5.1/../../../../pic32mx/lib/speed\libmchp_peripheral_32MX795F512L.a(eth_miim_access.o)
                0x9d0776c4                EthMIIMScanStart

.text.INTEnableSystemMultiVectoredInt
                0x9d0776f8       0x34
 .text.INTEnableSystemMultiVectoredInt
                0x9d0776f8       0x34 c:/program files/microchip/mplabc32/v2.02/bin/../lib/gcc/pic32mx/4.5.1/../../../../pic32mx/lib/speed\libmchp_peripheral_32MX795F512L.a(int_enable_mv_int_lib.o)
                0x9d0776f8                INTEnableSystemMultiVectoredInt

.text.EthTxAcknowledgeBuffer
                0x9d07772c       0x30
 .text.EthTxAcknowledgeBuffer
                0x9d07772c       0x30 c:/program files/microchip/mplabc32/v2.02/bin/../lib/gcc/pic32mx/4.5.1/../../../../pic32mx/lib/speed\libmchp_peripheral_32MX795F512L.a(eth_ack_packet_lib.o)
                0x9d07772c                EthTxAcknowledgeBuffer

.text.EthRxSetBufferSize
                0x9d07775c       0x30
 .text.EthRxSetBufferSize
                0x9d07775c       0x30 c:/program files/microchip/mplabc32/v2.02/bin/../lib/gcc/pic32mx/4.5.1/../../../../pic32mx/lib/speed\libmchp_peripheral_32MX795F512L.a(eth_rx_set_buffer_size_lib.o)
                0x9d07775c                EthRxSetBufferSize

.text.INTClearFlag
                0x9d07778c       0x2c
 .text.INTClearFlag
                0x9d07778c       0x2c c:/program files/microchip/mplabc32/v2.02/bin/../lib/gcc/pic32mx/4.5.1/../../../../pic32mx/lib/speed\libmchp_peripheral_32MX795F512L.a(int_tbl_lib.o)
                0x9d07778c                INTClearFlag

.rodata         0x9d0777b8       0x28
 .rodata        0x9d0777b8       0x28 output\lcd.o

.text.strchr    0x9d0777e0       0x28
 .text.strchr   0x9d0777e0       0x28 c:/program files/microchip/mplabc32/v2.02/bin/../lib/gcc/pic32mx/4.5.1/../../../../pic32mx/lib/speed\libc.a(strchr.o)
                0x9d0777e0                strchr

.text.atof      0x9d077808       0x28
 .text.atof     0x9d077808       0x28 c:/program files/microchip/mplabc32/v2.02/bin/../lib/gcc/pic32mx/4.5.1/../../../../pic32mx/lib/speed\libc.a(atof.o)
                0x9d077808                atof

.text.EthMIIMReadResult
                0x9d077830       0x28
 .text.EthMIIMReadResult
                0x9d077830       0x28 c:/program files/microchip/mplabc32/v2.02/bin/../lib/gcc/pic32mx/4.5.1/../../../../pic32mx/lib/speed\libmchp_peripheral_32MX795F512L.a(eth_miim_access.o)
                0x9d077830                EthMIIMReadResult

.text.RtccSetTimeDate
                0x9d077858       0x28
 .text.RtccSetTimeDate
                0x9d077858       0x28 c:/program files/microchip/mplabc32/v2.02/bin/../lib/gcc/pic32mx/4.5.1/../../../../pic32mx/lib/speed\libmchp_peripheral_32MX795F512L.a(rtcc_set_time_date_lib.o)
                0x9d077858                RtccSetTimeDate

.rodata         0x9d077880       0x24
 .rodata        0x9d077880       0x24 output\TCP.o
                0x9d077880                TCPSocketInitializer

.text.tolower   0x9d0778a4       0x24
 .text.tolower  0x9d0778a4       0x24 c:/program files/microchip/mplabc32/v2.02/bin/../lib/gcc/pic32mx/4.5.1/../../../../pic32mx/lib/speed\libc.a(ctypef.o)
                0x9d0778a4                tolower

.text.toupper   0x9d0778c8       0x24
 .text.toupper  0x9d0778c8       0x24 c:/program files/microchip/mplabc32/v2.02/bin/../lib/gcc/pic32mx/4.5.1/../../../../pic32mx/lib/speed\libc.a(ctypef.o)
                0x9d0778c8                toupper

.rodata         0x9d0778ec       0x60
 .rodata        0x9d0778ec       0x20 output\IntQueue.o
 .rodata        0x9d07790c       0x20 output\QPeek.o
 .rodata        0x9d07792c       0x20 output\FSIO.o

.text.EthMIIMScanResult
                0x9d07794c       0x20
 .text.EthMIIMScanResult
                0x9d07794c       0x20 c:/program files/microchip/mplabc32/v2.02/bin/../lib/gcc/pic32mx/4.5.1/../../../../pic32mx/lib/speed\libmchp_peripheral_32MX795F512L.a(eth_miim_access.o)
                0x9d07794c                EthMIIMScanResult

.text.getcSPI1  0x9d07796c       0x20
 .text.getcSPI1
                0x9d07796c       0x20 c:/program files/microchip/mplabc32/v2.02/bin/../lib/gcc/pic32mx/4.5.1/../../../../pic32mx/lib/speed\libmchp_peripheral_32MX795F512L.a(spi_getc_spi1_lib_legacy.o)
                0x9d07796c                getcSPI1

.text._dstrtod  0x9d07798c       0x1c
 .text._dstrtod
                0x9d07798c       0x1c c:/program files/microchip/mplabc32/v2.02/bin/../lib/gcc/pic32mx/4.5.1/../../../../pic32mx/lib/speed\libc.a(strtod.o)
                0x9d07798c                _dstrtod

.text.EthRxAcknowledgeBuffer
                0x9d0779a8       0x1c
 .text.EthRxAcknowledgeBuffer
                0x9d0779a8       0x1c c:/program files/microchip/mplabc32/v2.02/bin/../lib/gcc/pic32mx/4.5.1/../../../../pic32mx/lib/speed\libmchp_peripheral_32MX795F512L.a(eth_ack_packet_lib.o)
                0x9d0779a8                EthRxAcknowledgeBuffer

.text.INTRestoreInterrupts
                0x9d0779c4       0x1c
 .text.INTRestoreInterrupts
                0x9d0779c4       0x1c c:/program files/microchip/mplabc32/v2.02/bin/../lib/gcc/pic32mx/4.5.1/../../../../pic32mx/lib/speed\libmchp_peripheral_32MX795F512L.a(int_restore_interrupts_lib.o)
                0x9d0779c4                INTRestoreInterrupts

.text           0x9d0779e0       0x18
 .text          0x9d0779e0       0x18 c:/program files/microchip/mplabc32/v2.02/bin/../lib/gcc/pic32mx/4.5.1/../../../../pic32mx/lib/speed\libc.a(default-nmi-handler.o)
                0x9d0779e0                _nmi_handler

.text.CheKseg0CacheOn
                0x9d0779f8       0x18
 .text.CheKseg0CacheOn
                0x9d0779f8       0x18 c:/program files/microchip/mplabc32/v2.02/bin/../lib/gcc/pic32mx/4.5.1/../../../../pic32mx/lib/speed\libmchp_peripheral_32MX795F512L.a(pcache.o)
                0x9d0779f8                CheKseg0CacheOn

.text           0x9d077a10       0x10
 .text          0x9d077a10       0x10 c:/program files/microchip/mplabc32/v2.02/bin/../lib/gcc/pic32mx/4.5.1/../../../../pic32mx/lib/speed/crt0.o
                0x9d077a18                __crt0_exit

.rodata         0x9d077a20       0x40
 .rodata        0x9d077a20       0x10 output\SNTP.o
 .rodata        0x9d077a30       0x10 output\comtest.o
 .rodata        0x9d077a40       0x10 output\NBNS.o
 .rodata        0x9d077a50       0x10 c:/program files/microchip/mplabc32/v2.02/bin/../lib/gcc/pic32mx/4.5.1/../../../../pic32mx/lib/speed\libe.a(_strtod.o)

.text.EthRxFiltersSet
                0x9d077a60       0x10
 .text.EthRxFiltersSet
                0x9d077a60       0x10 c:/program files/microchip/mplabc32/v2.02/bin/../lib/gcc/pic32mx/4.5.1/../../../../pic32mx/lib/speed\libmchp_peripheral_32MX795F512L.a(eth_rx_filters_lib.o)
                0x9d077a60                EthRxFiltersSet

.text.EthRxFiltersClr
                0x9d077a70       0x10
 .text.EthRxFiltersClr
                0x9d077a70       0x10 c:/program files/microchip/mplabc32/v2.02/bin/../lib/gcc/pic32mx/4.5.1/../../../../pic32mx/lib/speed\libmchp_peripheral_32MX795F512L.a(eth_rx_filters_lib.o)
                0x9d077a70                EthRxFiltersClr

.text.SetCoreSW0
                0x9d077a80       0x10
 .text.SetCoreSW0
                0x9d077a80       0x10 c:/program files/microchip/mplabc32/v2.02/bin/../lib/gcc/pic32mx/4.5.1/../../../../pic32mx/lib/speed\libmchp_peripheral_32MX795F512L.a(set_core_sw0_leg_lib.o)
                0x9d077a80                SetCoreSW0

.rodata         0x9d077a90        0xc
 .rodata        0x9d077a90        0xc output\serial.o

.text._bootstrap_exception_handler
                0x9d077a9c        0xc
 .text._bootstrap_exception_handler
                0x9d077a9c        0xc c:/program files/microchip/mplabc32/v2.02/bin/../lib/gcc/pic32mx/4.5.1/../../../../pic32mx/lib/speed\libc.a(default-bootstrap-exception-handler.o)
                0x9d077a9c                _bootstrap_exception_handler

.rodata         0x9d077aa8       0x18
 .rodata        0x9d077aa8        0x8 output\tasks.o
 .rodata        0x9d077ab0        0x8 output\ETHPIC32IntMac.o
 .rodata        0x9d077ab8        0x8 output\MPFS2.o

.text._on_reset
                0x9d077ac0        0x8
 .text._on_reset
                0x9d077ac0        0x8 c:/program files/microchip/mplabc32/v2.02/bin/../lib/gcc/pic32mx/4.5.1/../../../../pic32mx/lib/speed\libc.a(default-on-reset.o)
                0x9d077ac0                _on_reset

.text._on_bootstrap
                0x9d077ac8        0x8
 .text._on_bootstrap
                0x9d077ac8        0x8 c:/program files/microchip/mplabc32/v2.02/bin/../lib/gcc/pic32mx/4.5.1/../../../../pic32mx/lib/speed\libc.a(default-on-bootstrap.o)
                0x9d077ac8                _on_bootstrap

.text.ReadCoreTimer
                0x9d077ad0        0x8
 .text.ReadCoreTimer
                0x9d077ad0        0x8 c:/program files/microchip/mplabc32/v2.02/bin/../lib/gcc/pic32mx/4.5.1/../../../../pic32mx/lib/speed\libmchp_peripheral.a(read_core_timer_lib.o)
                0x9d077ad0                ReadCoreTimer

.text.WriteCoreTimer
                0x9d077ad8        0x8
 .text.WriteCoreTimer
                0x9d077ad8        0x8 c:/program files/microchip/mplabc32/v2.02/bin/../lib/gcc/pic32mx/4.5.1/../../../../pic32mx/lib/speed\libmchp_peripheral.a(write_core_timer_lib.o)
                0x9d077ad8                WriteCoreTimer

.text.INTDisableInterrupts
                0x9d077ae0        0x8
 .text.INTDisableInterrupts
                0x9d077ae0        0x8 c:/program files/microchip/mplabc32/v2.02/bin/../lib/gcc/pic32mx/4.5.1/../../../../pic32mx/lib/speed\libmchp_peripheral_32MX795F512L.a(int_disable_interrupts_lib.o)
                0x9d077ae0                INTDisableInterrupts

.text.INTEnableInterrupts
                0x9d077ae8        0x8
 .text.INTEnableInterrupts
                0x9d077ae8        0x8 c:/program files/microchip/mplabc32/v2.02/bin/../lib/gcc/pic32mx/4.5.1/../../../../pic32mx/lib/speed\libmchp_peripheral_32MX795F512L.a(int_enable_interrupts_lib.o)
                0x9d077ae8                INTEnableInterrupts

.rodata         0x9d0767f4        0x4
 .rodata        0x9d0767f4        0x4 output\port.o
                0x9d0767f4                xISRStackTop

.rodata         0x9d077af0        0x2
 .rodata        0x9d077af0        0x2 output\heap_2.o
